Archive member included to satisfy reference by file (symbol)

/usr/lib/gcc/arm-none-eabi/13.2.1/../../../arm-none-eabi/lib/thumb/v7e-m+dp/hard/libc_nano.a(libc_a-sprintf.o)
                              build/File_Handling.o (sprintf)
/usr/lib/gcc/arm-none-eabi/13.2.1/../../../arm-none-eabi/lib/thumb/v7e-m+dp/hard/libc_nano.a(libc_a-strcpy.o)
                              build/File_Handling.o (strcpy)
/usr/lib/gcc/arm-none-eabi/13.2.1/../../../arm-none-eabi/lib/thumb/v7e-m+dp/hard/libc_nano.a(libc_a-impure.o)
                              /usr/lib/gcc/arm-none-eabi/13.2.1/../../../arm-none-eabi/lib/thumb/v7e-m+dp/hard/libc_nano.a(libc_a-sprintf.o) (_impure_ptr)
/usr/lib/gcc/arm-none-eabi/13.2.1/../../../arm-none-eabi/lib/thumb/v7e-m+dp/hard/libc_nano.a(libc_a-nano-svfprintf.o)
                              /usr/lib/gcc/arm-none-eabi/13.2.1/../../../arm-none-eabi/lib/thumb/v7e-m+dp/hard/libc_nano.a(libc_a-sprintf.o) (_svfprintf_r)
/usr/lib/gcc/arm-none-eabi/13.2.1/../../../arm-none-eabi/lib/thumb/v7e-m+dp/hard/libc_nano.a(libc_a-init.o)
                              /usr/lib/gcc/arm-none-eabi/13.2.1/../../../arm-none-eabi/lib/thumb/v7e-m+dp/hard/crt0.o (__libc_init_array)
/usr/lib/gcc/arm-none-eabi/13.2.1/../../../arm-none-eabi/lib/thumb/v7e-m+dp/hard/libc_nano.a(libc_a-strlen.o)
                              build/File_Handling.o (strlen)
/usr/lib/gcc/arm-none-eabi/13.2.1/../../../arm-none-eabi/lib/thumb/v7e-m+dp/hard/libc_nano.a(libc_a-memset.o)
                              /usr/lib/gcc/arm-none-eabi/13.2.1/../../../arm-none-eabi/lib/thumb/v7e-m+dp/hard/crt0.o (memset)
/usr/lib/gcc/arm-none-eabi/13.2.1/../../../arm-none-eabi/lib/thumb/v7e-m+dp/hard/libc_nano.a(libc_a-errno.o)
                              build/sysmem.o (__errno)
/usr/lib/gcc/arm-none-eabi/13.2.1/../../../arm-none-eabi/lib/thumb/v7e-m+dp/hard/libc_nano.a(libc_a-mallocr.o)
                              /usr/lib/gcc/arm-none-eabi/13.2.1/../../../arm-none-eabi/lib/thumb/v7e-m+dp/hard/libc_nano.a(libc_a-nano-svfprintf.o) (_malloc_r)
/usr/lib/gcc/arm-none-eabi/13.2.1/../../../arm-none-eabi/lib/thumb/v7e-m+dp/hard/libc_nano.a(libc_a-freer.o)
                              /usr/lib/gcc/arm-none-eabi/13.2.1/../../../arm-none-eabi/lib/thumb/v7e-m+dp/hard/libc_nano.a(libc_a-nano-svfprintf.o) (_free_r)
/usr/lib/gcc/arm-none-eabi/13.2.1/../../../arm-none-eabi/lib/thumb/v7e-m+dp/hard/libc_nano.a(libc_a-memmove.o)
                              /usr/lib/gcc/arm-none-eabi/13.2.1/../../../arm-none-eabi/lib/thumb/v7e-m+dp/hard/libc_nano.a(libc_a-nano-svfprintf.o) (memmove)
/usr/lib/gcc/arm-none-eabi/13.2.1/../../../arm-none-eabi/lib/thumb/v7e-m+dp/hard/libc_nano.a(libc_a-memchr.o)
                              /usr/lib/gcc/arm-none-eabi/13.2.1/../../../arm-none-eabi/lib/thumb/v7e-m+dp/hard/libc_nano.a(libc_a-nano-svfprintf.o) (memchr)
/usr/lib/gcc/arm-none-eabi/13.2.1/../../../arm-none-eabi/lib/thumb/v7e-m+dp/hard/libc_nano.a(libc_a-memcpy.o)
                              /usr/lib/gcc/arm-none-eabi/13.2.1/../../../arm-none-eabi/lib/thumb/v7e-m+dp/hard/libc_nano.a(libc_a-nano-svfprintf.o) (memcpy)
/usr/lib/gcc/arm-none-eabi/13.2.1/../../../arm-none-eabi/lib/thumb/v7e-m+dp/hard/libc_nano.a(libc_a-malloc.o)
                              build/File_Handling.o (malloc)
/usr/lib/gcc/arm-none-eabi/13.2.1/../../../arm-none-eabi/lib/thumb/v7e-m+dp/hard/libc_nano.a(libc_a-reallocr.o)
                              /usr/lib/gcc/arm-none-eabi/13.2.1/../../../arm-none-eabi/lib/thumb/v7e-m+dp/hard/libc_nano.a(libc_a-nano-svfprintf.o) (_realloc_r)
/usr/lib/gcc/arm-none-eabi/13.2.1/../../../arm-none-eabi/lib/thumb/v7e-m+dp/hard/libc_nano.a(libc_a-nano-vfprintf_i.o)
                              /usr/lib/gcc/arm-none-eabi/13.2.1/../../../arm-none-eabi/lib/thumb/v7e-m+dp/hard/libc_nano.a(libc_a-nano-svfprintf.o) (_printf_i)
/usr/lib/gcc/arm-none-eabi/13.2.1/../../../arm-none-eabi/lib/thumb/v7e-m+dp/hard/libc_nano.a(libc_a-mlock.o)
                              /usr/lib/gcc/arm-none-eabi/13.2.1/../../../arm-none-eabi/lib/thumb/v7e-m+dp/hard/libc_nano.a(libc_a-mallocr.o) (__malloc_lock)
/usr/lib/gcc/arm-none-eabi/13.2.1/../../../arm-none-eabi/lib/thumb/v7e-m+dp/hard/libc_nano.a(libc_a-strcmp.o)
                              build/File_Handling.o (strcmp)
/usr/lib/gcc/arm-none-eabi/13.2.1/../../../arm-none-eabi/lib/thumb/v7e-m+dp/hard/libc_nano.a(libc_a-exit.o)
                              /usr/lib/gcc/arm-none-eabi/13.2.1/../../../arm-none-eabi/lib/thumb/v7e-m+dp/hard/crt0.o (exit)
/usr/lib/gcc/arm-none-eabi/13.2.1/../../../arm-none-eabi/lib/thumb/v7e-m+dp/hard/libc_nano.a(libc_a-atexit.o)
                              /usr/lib/gcc/arm-none-eabi/13.2.1/../../../arm-none-eabi/lib/thumb/v7e-m+dp/hard/crt0.o (atexit)
/usr/lib/gcc/arm-none-eabi/13.2.1/../../../arm-none-eabi/lib/thumb/v7e-m+dp/hard/libc_nano.a(libc_a-fini.o)
                              /usr/lib/gcc/arm-none-eabi/13.2.1/../../../arm-none-eabi/lib/thumb/v7e-m+dp/hard/crt0.o (__libc_fini_array)
/usr/lib/gcc/arm-none-eabi/13.2.1/../../../arm-none-eabi/lib/thumb/v7e-m+dp/hard/libc_nano.a(libc_a-sbrkr.o)
                              /usr/lib/gcc/arm-none-eabi/13.2.1/../../../arm-none-eabi/lib/thumb/v7e-m+dp/hard/libc_nano.a(libc_a-mallocr.o) (_sbrk_r)
/usr/lib/gcc/arm-none-eabi/13.2.1/../../../arm-none-eabi/lib/thumb/v7e-m+dp/hard/libc_nano.a(libc_a-msizer.o)
                              /usr/lib/gcc/arm-none-eabi/13.2.1/../../../arm-none-eabi/lib/thumb/v7e-m+dp/hard/libc_nano.a(libc_a-reallocr.o) (_malloc_usable_size_r)
/usr/lib/gcc/arm-none-eabi/13.2.1/../../../arm-none-eabi/lib/thumb/v7e-m+dp/hard/libc_nano.a(libc_a-findfp.o)
                              /usr/lib/gcc/arm-none-eabi/13.2.1/../../../arm-none-eabi/lib/thumb/v7e-m+dp/hard/libc_nano.a(libc_a-exit.o) (__stdio_exit_handler)
/usr/lib/gcc/arm-none-eabi/13.2.1/../../../arm-none-eabi/lib/thumb/v7e-m+dp/hard/libc_nano.a(libc_a-fflush.o)
                              /usr/lib/gcc/arm-none-eabi/13.2.1/../../../arm-none-eabi/lib/thumb/v7e-m+dp/hard/libc_nano.a(libc_a-findfp.o) (_fflush_r)
/usr/lib/gcc/arm-none-eabi/13.2.1/../../../arm-none-eabi/lib/thumb/v7e-m+dp/hard/libc_nano.a(libc_a-fwalk.o)
                              /usr/lib/gcc/arm-none-eabi/13.2.1/../../../arm-none-eabi/lib/thumb/v7e-m+dp/hard/libc_nano.a(libc_a-findfp.o) (_fwalk_sglue)
/usr/lib/gcc/arm-none-eabi/13.2.1/../../../arm-none-eabi/lib/thumb/v7e-m+dp/hard/libc_nano.a(libc_a-__atexit.o)
                              /usr/lib/gcc/arm-none-eabi/13.2.1/../../../arm-none-eabi/lib/thumb/v7e-m+dp/hard/libc_nano.a(libc_a-atexit.o) (__register_exitproc)
/usr/lib/gcc/arm-none-eabi/13.2.1/../../../arm-none-eabi/lib/thumb/v7e-m+dp/hard/libc_nano.a(libc_a-reent.o)
                              /usr/lib/gcc/arm-none-eabi/13.2.1/../../../arm-none-eabi/lib/thumb/v7e-m+dp/hard/libc_nano.a(libc_a-sbrkr.o) (errno)
/usr/lib/gcc/arm-none-eabi/13.2.1/../../../arm-none-eabi/lib/thumb/v7e-m+dp/hard/libc_nano.a(libc_a-stdio.o)
                              /usr/lib/gcc/arm-none-eabi/13.2.1/../../../arm-none-eabi/lib/thumb/v7e-m+dp/hard/libc_nano.a(libc_a-findfp.o) (__sread)
/usr/lib/gcc/arm-none-eabi/13.2.1/../../../arm-none-eabi/lib/thumb/v7e-m+dp/hard/libc_nano.a(libc_a-closer.o)
                              /usr/lib/gcc/arm-none-eabi/13.2.1/../../../arm-none-eabi/lib/thumb/v7e-m+dp/hard/libc_nano.a(libc_a-stdio.o) (_close_r)
/usr/lib/gcc/arm-none-eabi/13.2.1/../../../arm-none-eabi/lib/thumb/v7e-m+dp/hard/libc_nano.a(libc_a-__call_atexit.o)
                              /usr/lib/gcc/arm-none-eabi/13.2.1/../../../arm-none-eabi/lib/thumb/v7e-m+dp/hard/libc_nano.a(libc_a-__atexit.o) (__call_exitprocs)
/usr/lib/gcc/arm-none-eabi/13.2.1/../../../arm-none-eabi/lib/thumb/v7e-m+dp/hard/libc_nano.a(libc_a-readr.o)
                              /usr/lib/gcc/arm-none-eabi/13.2.1/../../../arm-none-eabi/lib/thumb/v7e-m+dp/hard/libc_nano.a(libc_a-stdio.o) (_read_r)
/usr/lib/gcc/arm-none-eabi/13.2.1/../../../arm-none-eabi/lib/thumb/v7e-m+dp/hard/libc_nano.a(libc_a-lseekr.o)
                              /usr/lib/gcc/arm-none-eabi/13.2.1/../../../arm-none-eabi/lib/thumb/v7e-m+dp/hard/libc_nano.a(libc_a-stdio.o) (_lseek_r)
/usr/lib/gcc/arm-none-eabi/13.2.1/../../../arm-none-eabi/lib/thumb/v7e-m+dp/hard/libc_nano.a(libc_a-writer.o)
                              /usr/lib/gcc/arm-none-eabi/13.2.1/../../../arm-none-eabi/lib/thumb/v7e-m+dp/hard/libc_nano.a(libc_a-stdio.o) (_write_r)
/usr/lib/gcc/arm-none-eabi/13.2.1/thumb/v7e-m+dp/hard/libgcc.a(_aeabi_uldivmod.o)
                              build/stm32f7xx_hal_rcc.o (__aeabi_uldivmod)
/usr/lib/gcc/arm-none-eabi/13.2.1/thumb/v7e-m+dp/hard/libgcc.a(_udivmoddi4.o)
                              /usr/lib/gcc/arm-none-eabi/13.2.1/thumb/v7e-m+dp/hard/libgcc.a(_aeabi_uldivmod.o) (__udivmoddi4)
/usr/lib/gcc/arm-none-eabi/13.2.1/thumb/v7e-m+dp/hard/libgcc.a(_dvmd_tls.o)
                              /usr/lib/gcc/arm-none-eabi/13.2.1/thumb/v7e-m+dp/hard/libgcc.a(_aeabi_uldivmod.o) (__aeabi_ldiv0)

Discarded input sections

 .text          0x00000000        0x0 /usr/lib/gcc/arm-none-eabi/13.2.1/thumb/v7e-m+dp/hard/crti.o
 .data          0x00000000        0x0 /usr/lib/gcc/arm-none-eabi/13.2.1/thumb/v7e-m+dp/hard/crti.o
 .bss           0x00000000        0x0 /usr/lib/gcc/arm-none-eabi/13.2.1/thumb/v7e-m+dp/hard/crti.o
 .data          0x00000000        0x4 /usr/lib/gcc/arm-none-eabi/13.2.1/thumb/v7e-m+dp/hard/crtbegin.o
 .rodata        0x00000000       0x24 /usr/lib/gcc/arm-none-eabi/13.2.1/thumb/v7e-m+dp/hard/crtbegin.o
 .text          0x00000000       0x70 /usr/lib/gcc/arm-none-eabi/13.2.1/../../../arm-none-eabi/lib/thumb/v7e-m+dp/hard/crt0.o
 .data          0x00000000        0x0 /usr/lib/gcc/arm-none-eabi/13.2.1/../../../arm-none-eabi/lib/thumb/v7e-m+dp/hard/crt0.o
 .bss           0x00000000        0x0 /usr/lib/gcc/arm-none-eabi/13.2.1/../../../arm-none-eabi/lib/thumb/v7e-m+dp/hard/crt0.o
 .ARM.extab     0x00000000        0x0 /usr/lib/gcc/arm-none-eabi/13.2.1/../../../arm-none-eabi/lib/thumb/v7e-m+dp/hard/crt0.o
 .ARM.exidx     0x00000000       0x10 /usr/lib/gcc/arm-none-eabi/13.2.1/../../../arm-none-eabi/lib/thumb/v7e-m+dp/hard/crt0.o
 .debug_line    0x00000000       0x75 /usr/lib/gcc/arm-none-eabi/13.2.1/../../../arm-none-eabi/lib/thumb/v7e-m+dp/hard/crt0.o
 .debug_line_str
                0x00000000       0x82 /usr/lib/gcc/arm-none-eabi/13.2.1/../../../arm-none-eabi/lib/thumb/v7e-m+dp/hard/crt0.o
 .debug_info    0x00000000       0x24 /usr/lib/gcc/arm-none-eabi/13.2.1/../../../arm-none-eabi/lib/thumb/v7e-m+dp/hard/crt0.o
 .debug_abbrev  0x00000000       0x14 /usr/lib/gcc/arm-none-eabi/13.2.1/../../../arm-none-eabi/lib/thumb/v7e-m+dp/hard/crt0.o
 .debug_aranges
                0x00000000       0x20 /usr/lib/gcc/arm-none-eabi/13.2.1/../../../arm-none-eabi/lib/thumb/v7e-m+dp/hard/crt0.o
 .debug_str     0x00000000       0x8e /usr/lib/gcc/arm-none-eabi/13.2.1/../../../arm-none-eabi/lib/thumb/v7e-m+dp/hard/crt0.o
 .ARM.attributes
                0x00000000       0x1e /usr/lib/gcc/arm-none-eabi/13.2.1/../../../arm-none-eabi/lib/thumb/v7e-m+dp/hard/crt0.o
 .text          0x00000000        0x0 build/main.o
 .data          0x00000000        0x0 build/main.o
 .bss           0x00000000        0x0 build/main.o
 .text.Advanced_Controller_Temp
                0x00000000       0xe4 build/main.o
 .bss.temp32    0x00000000        0x4 build/main.o
 .text          0x00000000        0x0 build/bsp_driver_sd.o
 .data          0x00000000        0x0 build/bsp_driver_sd.o
 .bss           0x00000000        0x0 build/bsp_driver_sd.o
 .text.BSP_SD_ITConfig
                0x00000000        0x4 build/bsp_driver_sd.o
 .text.BSP_SD_ReadBlocks_DMA
                0x00000000       0x18 build/bsp_driver_sd.o
 .text.BSP_SD_WriteBlocks_DMA
                0x00000000       0x18 build/bsp_driver_sd.o
 .text.BSP_SD_Erase
                0x00000000       0x18 build/bsp_driver_sd.o
 .text.BSP_SD_AbortCallback
                0x00000000        0x2 build/bsp_driver_sd.o
 .text.HAL_SD_AbortCallback
                0x00000000        0x8 build/bsp_driver_sd.o
 .text.BSP_SD_WriteCpltCallback
                0x00000000        0x2 build/bsp_driver_sd.o
 .text.HAL_SD_TxCpltCallback
                0x00000000        0x8 build/bsp_driver_sd.o
 .text.BSP_SD_ReadCpltCallback
                0x00000000        0x2 build/bsp_driver_sd.o
 .text.HAL_SD_RxCpltCallback
                0x00000000        0x8 build/bsp_driver_sd.o
 .text          0x00000000        0x0 build/sd_diskio.o
 .data          0x00000000        0x0 build/sd_diskio.o
 .bss           0x00000000        0x0 build/sd_diskio.o
 .text          0x00000000        0x0 build/fatfs.o
 .data          0x00000000        0x0 build/fatfs.o
 .bss           0x00000000        0x0 build/fatfs.o
 .bss.SDFile    0x00000000     0x1030 build/fatfs.o
 .bss.SDFatFS   0x00000000     0x1034 build/fatfs.o
 .text          0x00000000        0x0 build/fatfs_platform.o
 .data          0x00000000        0x0 build/fatfs_platform.o
 .bss           0x00000000        0x0 build/fatfs_platform.o
 .text          0x00000000        0x0 build/stm32f7xx_it.o
 .data          0x00000000        0x0 build/stm32f7xx_it.o
 .bss           0x00000000        0x0 build/stm32f7xx_it.o
 .text          0x00000000        0x0 build/stm32f7xx_hal_msp.o
 .data          0x00000000        0x0 build/stm32f7xx_hal_msp.o
 .bss           0x00000000        0x0 build/stm32f7xx_hal_msp.o
 .text.HAL_ADC_MspDeInit
                0x00000000       0x68 build/stm32f7xx_hal_msp.o
 .text.HAL_SD_MspDeInit
                0x00000000       0x3c build/stm32f7xx_hal_msp.o
 .text.HAL_TIM_Base_MspDeInit
                0x00000000       0x78 build/stm32f7xx_hal_msp.o
 .text.HAL_UART_MspDeInit
                0x00000000       0x2c build/stm32f7xx_hal_msp.o
 .text          0x00000000        0x0 build/stm32f7xx_hal_adc.o
 .data          0x00000000        0x0 build/stm32f7xx_hal_adc.o
 .bss           0x00000000        0x0 build/stm32f7xx_hal_adc.o
 .text.HAL_ADC_MspInit
                0x00000000        0x2 build/stm32f7xx_hal_adc.o
 .text.HAL_ADC_MspDeInit
                0x00000000        0x2 build/stm32f7xx_hal_adc.o
 .text.HAL_ADC_DeInit
                0x00000000       0x3a build/stm32f7xx_hal_adc.o
 .text.HAL_ADC_PollForEvent
                0x00000000       0x7e build/stm32f7xx_hal_adc.o
 .text.HAL_ADC_Start_IT
                0x00000000      0x144 build/stm32f7xx_hal_adc.o
 .text.HAL_ADC_Stop_IT
                0x00000000       0x4c build/stm32f7xx_hal_adc.o
 .text.HAL_ADC_Start_DMA
                0x00000000      0x180 build/stm32f7xx_hal_adc.o
 .text.HAL_ADC_Stop_DMA
                0x00000000       0x78 build/stm32f7xx_hal_adc.o
 .text.HAL_ADC_ConvHalfCpltCallback
                0x00000000        0x2 build/stm32f7xx_hal_adc.o
 .text.ADC_DMAHalfConvCplt
                0x00000000        0xa build/stm32f7xx_hal_adc.o
 .text.ADC_DMAError
                0x00000000       0x16 build/stm32f7xx_hal_adc.o
 .text.ADC_DMAConvCplt
                0x00000000       0x72 build/stm32f7xx_hal_adc.o
 .text.HAL_ADC_AnalogWDGConfig
                0x00000000       0x78 build/stm32f7xx_hal_adc.o
 .text.HAL_ADC_GetState
                0x00000000        0x4 build/stm32f7xx_hal_adc.o
 .text.HAL_ADC_GetError
                0x00000000        0x4 build/stm32f7xx_hal_adc.o
 .text          0x00000000        0x0 build/stm32f7xx_hal_adc_ex.o
 .data          0x00000000        0x0 build/stm32f7xx_hal_adc_ex.o
 .bss           0x00000000        0x0 build/stm32f7xx_hal_adc_ex.o
 .text.ADC_MultiModeDMAError
                0x00000000       0x16 build/stm32f7xx_hal_adc_ex.o
 .text.ADC_MultiModeDMAHalfConvCplt
                0x00000000        0xa build/stm32f7xx_hal_adc_ex.o
 .text.ADC_MultiModeDMAConvCplt
                0x00000000       0x62 build/stm32f7xx_hal_adc_ex.o
 .text.HAL_ADCEx_InjectedStart
                0x00000000       0xfc build/stm32f7xx_hal_adc_ex.o
 .text.HAL_ADCEx_InjectedStart_IT
                0x00000000      0x104 build/stm32f7xx_hal_adc_ex.o
 .text.HAL_ADCEx_InjectedStop
                0x00000000       0x64 build/stm32f7xx_hal_adc_ex.o
 .text.HAL_ADCEx_InjectedPollForConversion
                0x00000000       0xb2 build/stm32f7xx_hal_adc_ex.o
 .text.HAL_ADCEx_InjectedStop_IT
                0x00000000       0x6c build/stm32f7xx_hal_adc_ex.o
 .text.HAL_ADCEx_InjectedGetValue
                0x00000000       0x40 build/stm32f7xx_hal_adc_ex.o
 .text.HAL_ADCEx_MultiModeStart_DMA
                0x00000000      0x130 build/stm32f7xx_hal_adc_ex.o
 .text.HAL_ADCEx_MultiModeStop_DMA
                0x00000000       0x64 build/stm32f7xx_hal_adc_ex.o
 .text.HAL_ADCEx_MultiModeGetValue
                0x00000000        0xc build/stm32f7xx_hal_adc_ex.o
 .text.HAL_ADCEx_InjectedConfigChannel
                0x00000000      0x208 build/stm32f7xx_hal_adc_ex.o
 .text.HAL_ADCEx_MultiModeConfigChannel
                0x00000000       0x58 build/stm32f7xx_hal_adc_ex.o
 .text          0x00000000        0x0 build/stm32f7xx_hal_rcc.o
 .data          0x00000000        0x0 build/stm32f7xx_hal_rcc.o
 .bss           0x00000000        0x0 build/stm32f7xx_hal_rcc.o
 .text.HAL_RCC_DeInit
                0x00000000      0x158 build/stm32f7xx_hal_rcc.o
 .text.HAL_RCC_MCOConfig
                0x00000000       0x98 build/stm32f7xx_hal_rcc.o
 .text.HAL_RCC_EnableCSS
                0x00000000       0x10 build/stm32f7xx_hal_rcc.o
 .text.HAL_RCC_DisableCSS
                0x00000000       0x10 build/stm32f7xx_hal_rcc.o
 .text.HAL_RCC_GetOscConfig
                0x00000000       0xe0 build/stm32f7xx_hal_rcc.o
 .text.HAL_RCC_GetClockConfig
                0x00000000       0x3c build/stm32f7xx_hal_rcc.o
 .text.HAL_RCC_CSSCallback
                0x00000000        0x2 build/stm32f7xx_hal_rcc.o
 .text.HAL_RCC_NMI_IRQHandler
                0x00000000       0x20 build/stm32f7xx_hal_rcc.o
 .text          0x00000000        0x0 build/stm32f7xx_hal_rcc_ex.o
 .data          0x00000000        0x0 build/stm32f7xx_hal_rcc_ex.o
 .bss           0x00000000        0x0 build/stm32f7xx_hal_rcc_ex.o
 .text.HAL_RCCEx_GetPeriphCLKConfig
                0x00000000      0x188 build/stm32f7xx_hal_rcc_ex.o
 .text.HAL_RCCEx_GetPeriphCLKFreq
                0x00000000      0x1e4 build/stm32f7xx_hal_rcc_ex.o
 .text.HAL_RCCEx_EnablePLLI2S
                0x00000000       0x78 build/stm32f7xx_hal_rcc_ex.o
 .text.HAL_RCCEx_DisablePLLI2S
                0x00000000       0x34 build/stm32f7xx_hal_rcc_ex.o
 .text.HAL_RCCEx_EnablePLLSAI
                0x00000000       0x78 build/stm32f7xx_hal_rcc_ex.o
 .text.HAL_RCCEx_DisablePLLSAI
                0x00000000       0x34 build/stm32f7xx_hal_rcc_ex.o
 .text          0x00000000        0x0 build/stm32f7xx_hal_flash.o
 .data          0x00000000        0x0 build/stm32f7xx_hal_flash.o
 .bss           0x00000000        0x0 build/stm32f7xx_hal_flash.o
 .text.FLASH_Program_DoubleWord
                0x00000000       0x34 build/stm32f7xx_hal_flash.o
 .text.FLASH_Program_Word
                0x00000000       0x28 build/stm32f7xx_hal_flash.o
 .text.FLASH_Program_HalfWord
                0x00000000       0x28 build/stm32f7xx_hal_flash.o
 .text.FLASH_Program_Byte
                0x00000000       0x24 build/stm32f7xx_hal_flash.o
 .text.FLASH_SetErrorCode
                0x00000000       0x74 build/stm32f7xx_hal_flash.o
 .text.HAL_FLASH_Program_IT
                0x00000000       0x74 build/stm32f7xx_hal_flash.o
 .text.HAL_FLASH_EndOfOperationCallback
                0x00000000        0x2 build/stm32f7xx_hal_flash.o
 .text.HAL_FLASH_OperationErrorCallback
                0x00000000        0x2 build/stm32f7xx_hal_flash.o
 .text.HAL_FLASH_IRQHandler
                0x00000000      0x108 build/stm32f7xx_hal_flash.o
 .text.HAL_FLASH_Unlock
                0x00000000       0x30 build/stm32f7xx_hal_flash.o
 .text.HAL_FLASH_Lock
                0x00000000       0x14 build/stm32f7xx_hal_flash.o
 .text.HAL_FLASH_OB_Unlock
                0x00000000       0x28 build/stm32f7xx_hal_flash.o
 .text.HAL_FLASH_OB_Lock
                0x00000000       0x14 build/stm32f7xx_hal_flash.o
 .text.HAL_FLASH_GetError
                0x00000000        0xc build/stm32f7xx_hal_flash.o
 .text.FLASH_WaitForLastOperation
                0x00000000       0x64 build/stm32f7xx_hal_flash.o
 .text.HAL_FLASH_Program
                0x00000000       0x7c build/stm32f7xx_hal_flash.o
 .text.HAL_FLASH_OB_Launch
                0x00000000       0x1c build/stm32f7xx_hal_flash.o
 .bss.pFlash    0x00000000       0x1c build/stm32f7xx_hal_flash.o
 .debug_info    0x00000000      0x7d4 build/stm32f7xx_hal_flash.o
 .debug_abbrev  0x00000000      0x2cd build/stm32f7xx_hal_flash.o
 .debug_loc     0x00000000      0x556 build/stm32f7xx_hal_flash.o
 .debug_aranges
                0x00000000       0xa0 build/stm32f7xx_hal_flash.o
 .debug_ranges  0x00000000       0x90 build/stm32f7xx_hal_flash.o
 .debug_line    0x00000000      0x770 build/stm32f7xx_hal_flash.o
 .debug_str     0x00000000      0x510 build/stm32f7xx_hal_flash.o
 .comment       0x00000000       0x27 build/stm32f7xx_hal_flash.o
 .debug_frame   0x00000000      0x168 build/stm32f7xx_hal_flash.o
 .ARM.attributes
                0x00000000       0x32 build/stm32f7xx_hal_flash.o
 .text          0x00000000        0x0 build/stm32f7xx_hal_flash_ex.o
 .data          0x00000000        0x0 build/stm32f7xx_hal_flash_ex.o
 .bss           0x00000000        0x0 build/stm32f7xx_hal_flash_ex.o
 .text.FLASH_MassErase
                0x00000000       0x50 build/stm32f7xx_hal_flash_ex.o
 .text.FLASH_OB_GetWRP
                0x00000000       0x14 build/stm32f7xx_hal_flash_ex.o
 .text.FLASH_OB_GetUser
                0x00000000       0x14 build/stm32f7xx_hal_flash_ex.o
 .text.FLASH_OB_BOR_LevelConfig
                0x00000000       0x14 build/stm32f7xx_hal_flash_ex.o
 .text.FLASH_OB_GetRDP
                0x00000000       0x1c build/stm32f7xx_hal_flash_ex.o
 .text.FLASH_OB_GetBOR
                0x00000000       0x10 build/stm32f7xx_hal_flash_ex.o
 .text.FLASH_OB_GetBootAddress
                0x00000000       0x18 build/stm32f7xx_hal_flash_ex.o
 .text.FLASH_OB_EnableWRP
                0x00000000       0x20 build/stm32f7xx_hal_flash_ex.o
 .text.FLASH_OB_DisableWRP
                0x00000000       0x1c build/stm32f7xx_hal_flash_ex.o
 .text.FLASH_OB_RDP_LevelConfig
                0x00000000       0x18 build/stm32f7xx_hal_flash_ex.o
 .text.FLASH_OB_UserConfig
                0x00000000       0x48 build/stm32f7xx_hal_flash_ex.o
 .text.FLASH_OB_BootAddressConfig
                0x00000000       0x34 build/stm32f7xx_hal_flash_ex.o
 .text.HAL_FLASHEx_OBProgram
                0x00000000       0xc4 build/stm32f7xx_hal_flash_ex.o
 .text.HAL_FLASHEx_OBGetConfig
                0x00000000       0x32 build/stm32f7xx_hal_flash_ex.o
 .text.FLASH_Erase_Sector
                0x00000000       0x58 build/stm32f7xx_hal_flash_ex.o
 .text.HAL_FLASHEx_Erase
                0x00000000       0x98 build/stm32f7xx_hal_flash_ex.o
 .text.HAL_FLASHEx_Erase_IT
                0x00000000       0x68 build/stm32f7xx_hal_flash_ex.o
 .debug_info    0x00000000      0x9f6 build/stm32f7xx_hal_flash_ex.o
 .debug_abbrev  0x00000000      0x28f build/stm32f7xx_hal_flash_ex.o
 .debug_loc     0x00000000      0x97c build/stm32f7xx_hal_flash_ex.o
 .debug_aranges
                0x00000000       0xa0 build/stm32f7xx_hal_flash_ex.o
 .debug_ranges  0x00000000       0x90 build/stm32f7xx_hal_flash_ex.o
 .debug_line    0x00000000      0x72c build/stm32f7xx_hal_flash_ex.o
 .debug_str     0x00000000      0x5ef build/stm32f7xx_hal_flash_ex.o
 .comment       0x00000000       0x27 build/stm32f7xx_hal_flash_ex.o
 .debug_frame   0x00000000      0x190 build/stm32f7xx_hal_flash_ex.o
 .ARM.attributes
                0x00000000       0x32 build/stm32f7xx_hal_flash_ex.o
 .text          0x00000000        0x0 build/stm32f7xx_hal_gpio.o
 .data          0x00000000        0x0 build/stm32f7xx_hal_gpio.o
 .bss           0x00000000        0x0 build/stm32f7xx_hal_gpio.o
 .text.HAL_GPIO_DeInit
                0x00000000      0x14c build/stm32f7xx_hal_gpio.o
 .text.HAL_GPIO_LockPin
                0x00000000       0x2e build/stm32f7xx_hal_gpio.o
 .text.HAL_GPIO_EXTI_Callback
                0x00000000        0x2 build/stm32f7xx_hal_gpio.o
 .text.HAL_GPIO_EXTI_IRQHandler
                0x00000000       0x1c build/stm32f7xx_hal_gpio.o
 .text          0x00000000        0x0 build/stm32f7xx_hal_dma.o
 .data          0x00000000        0x0 build/stm32f7xx_hal_dma.o
 .bss           0x00000000        0x0 build/stm32f7xx_hal_dma.o
 .text.DMA_SetConfig
                0x00000000       0x2c build/stm32f7xx_hal_dma.o
 .text.DMA_CalcBaseAndBitshift
                0x00000000       0x3c build/stm32f7xx_hal_dma.o
 .text.DMA_CheckFifoParam
                0x00000000       0x8e build/stm32f7xx_hal_dma.o
 .text.HAL_DMA_Init
                0x00000000       0xd0 build/stm32f7xx_hal_dma.o
 .text.HAL_DMA_DeInit
                0x00000000       0x64 build/stm32f7xx_hal_dma.o
 .text.HAL_DMA_Start
                0x00000000       0x48 build/stm32f7xx_hal_dma.o
 .text.HAL_DMA_Start_IT
                0x00000000       0x74 build/stm32f7xx_hal_dma.o
 .text.HAL_DMA_Abort
                0x00000000       0x94 build/stm32f7xx_hal_dma.o
 .text.HAL_DMA_Abort_IT
                0x00000000       0x26 build/stm32f7xx_hal_dma.o
 .text.HAL_DMA_PollForTransfer
                0x00000000      0x128 build/stm32f7xx_hal_dma.o
 .text.HAL_DMA_IRQHandler
                0x00000000      0x1dc build/stm32f7xx_hal_dma.o
 .text.HAL_DMA_RegisterCallback
                0x00000000       0x5a build/stm32f7xx_hal_dma.o
 .text.HAL_DMA_UnRegisterCallback
                0x00000000       0x6e build/stm32f7xx_hal_dma.o
 .text.HAL_DMA_GetState
                0x00000000        0x6 build/stm32f7xx_hal_dma.o
 .text.HAL_DMA_GetError
                0x00000000        0x4 build/stm32f7xx_hal_dma.o
 .rodata.flagBitshiftOffset.0
                0x00000000        0x8 build/stm32f7xx_hal_dma.o
 .debug_info    0x00000000      0xbb6 build/stm32f7xx_hal_dma.o
 .debug_abbrev  0x00000000      0x2fe build/stm32f7xx_hal_dma.o
 .debug_loc     0x00000000      0xe9a build/stm32f7xx_hal_dma.o
 .debug_aranges
                0x00000000       0x90 build/stm32f7xx_hal_dma.o
 .debug_ranges  0x00000000       0x80 build/stm32f7xx_hal_dma.o
 .debug_line    0x00000000      0xdbe build/stm32f7xx_hal_dma.o
 .debug_str     0x00000000      0x769 build/stm32f7xx_hal_dma.o
 .comment       0x00000000       0x27 build/stm32f7xx_hal_dma.o
 .debug_frame   0x00000000      0x188 build/stm32f7xx_hal_dma.o
 .ARM.attributes
                0x00000000       0x32 build/stm32f7xx_hal_dma.o
 .text          0x00000000        0x0 build/stm32f7xx_hal_dma_ex.o
 .data          0x00000000        0x0 build/stm32f7xx_hal_dma_ex.o
 .bss           0x00000000        0x0 build/stm32f7xx_hal_dma_ex.o
 .text.DMA_MultiBufferSetConfig
                0x00000000       0x24 build/stm32f7xx_hal_dma_ex.o
 .text.HAL_DMAEx_MultiBufferStart
                0x00000000       0x5e build/stm32f7xx_hal_dma_ex.o
 .text.HAL_DMAEx_MultiBufferStart_IT
                0x00000000      0xeec build/stm32f7xx_hal_dma_ex.o
 .text.HAL_DMAEx_ChangeMemory
                0x00000000       0x10 build/stm32f7xx_hal_dma_ex.o
 .debug_info    0x00000000      0x5ff build/stm32f7xx_hal_dma_ex.o
 .debug_abbrev  0x00000000      0x1d6 build/stm32f7xx_hal_dma_ex.o
 .debug_loc     0x00000000      0x4d5 build/stm32f7xx_hal_dma_ex.o
 .debug_aranges
                0x00000000       0x38 build/stm32f7xx_hal_dma_ex.o
 .debug_ranges  0x00000000       0x28 build/stm32f7xx_hal_dma_ex.o
 .debug_line    0x00000000      0xe2e build/stm32f7xx_hal_dma_ex.o
 .debug_str     0x00000000      0x546 build/stm32f7xx_hal_dma_ex.o
 .comment       0x00000000       0x27 build/stm32f7xx_hal_dma_ex.o
 .debug_frame   0x00000000       0x74 build/stm32f7xx_hal_dma_ex.o
 .ARM.attributes
                0x00000000       0x32 build/stm32f7xx_hal_dma_ex.o
 .text          0x00000000        0x0 build/stm32f7xx_hal_pwr.o
 .data          0x00000000        0x0 build/stm32f7xx_hal_pwr.o
 .bss           0x00000000        0x0 build/stm32f7xx_hal_pwr.o
 .text.HAL_PWR_DeInit
                0x00000000       0x18 build/stm32f7xx_hal_pwr.o
 .text.HAL_PWR_EnableBkUpAccess
                0x00000000       0x10 build/stm32f7xx_hal_pwr.o
 .text.HAL_PWR_DisableBkUpAccess
                0x00000000       0x10 build/stm32f7xx_hal_pwr.o
 .text.HAL_PWR_ConfigPVD
                0x00000000       0x84 build/stm32f7xx_hal_pwr.o
 .text.HAL_PWR_EnablePVD
                0x00000000       0x10 build/stm32f7xx_hal_pwr.o
 .text.HAL_PWR_DisablePVD
                0x00000000       0x10 build/stm32f7xx_hal_pwr.o
 .text.HAL_PWR_EnableWakeUpPin
                0x00000000       0x20 build/stm32f7xx_hal_pwr.o
 .text.HAL_PWR_DisableWakeUpPin
                0x00000000       0x10 build/stm32f7xx_hal_pwr.o
 .text.HAL_PWR_EnterSLEEPMode
                0x00000000       0x28 build/stm32f7xx_hal_pwr.o
 .text.HAL_PWR_EnterSTOPMode
                0x00000000       0x40 build/stm32f7xx_hal_pwr.o
 .text.HAL_PWR_EnterSTANDBYMode
                0x00000000       0x20 build/stm32f7xx_hal_pwr.o
 .text.HAL_PWR_PVDCallback
                0x00000000        0x2 build/stm32f7xx_hal_pwr.o
 .text.HAL_PWR_PVD_IRQHandler
                0x00000000       0x20 build/stm32f7xx_hal_pwr.o
 .text.HAL_PWR_EnableSleepOnExit
                0x00000000       0x10 build/stm32f7xx_hal_pwr.o
 .text.HAL_PWR_DisableSleepOnExit
                0x00000000       0x10 build/stm32f7xx_hal_pwr.o
 .text.HAL_PWR_EnableSEVOnPend
                0x00000000       0x10 build/stm32f7xx_hal_pwr.o
 .text.HAL_PWR_DisableSEVOnPend
                0x00000000       0x10 build/stm32f7xx_hal_pwr.o
 .debug_info    0x00000000      0xa94 build/stm32f7xx_hal_pwr.o
 .debug_abbrev  0x00000000      0x1cf build/stm32f7xx_hal_pwr.o
 .debug_loc     0x00000000       0x7f build/stm32f7xx_hal_pwr.o
 .debug_aranges
                0x00000000       0xa0 build/stm32f7xx_hal_pwr.o
 .debug_ranges  0x00000000       0x90 build/stm32f7xx_hal_pwr.o
 .debug_line    0x00000000      0x3dc build/stm32f7xx_hal_pwr.o
 .debug_str     0x00000000      0x630 build/stm32f7xx_hal_pwr.o
 .comment       0x00000000       0x27 build/stm32f7xx_hal_pwr.o
 .debug_frame   0x00000000      0x128 build/stm32f7xx_hal_pwr.o
 .ARM.attributes
                0x00000000       0x32 build/stm32f7xx_hal_pwr.o
 .text          0x00000000        0x0 build/stm32f7xx_hal_pwr_ex.o
 .data          0x00000000        0x0 build/stm32f7xx_hal_pwr_ex.o
 .bss           0x00000000        0x0 build/stm32f7xx_hal_pwr_ex.o
 .text.HAL_PWREx_EnableBkUpReg
                0x00000000       0x3c build/stm32f7xx_hal_pwr_ex.o
 .text.HAL_PWREx_DisableBkUpReg
                0x00000000       0x3c build/stm32f7xx_hal_pwr_ex.o
 .text.HAL_PWREx_EnableFlashPowerDown
                0x00000000       0x10 build/stm32f7xx_hal_pwr_ex.o
 .text.HAL_PWREx_DisableFlashPowerDown
                0x00000000       0x10 build/stm32f7xx_hal_pwr_ex.o
 .text.HAL_PWREx_EnableMainRegulatorLowVoltage
                0x00000000       0x10 build/stm32f7xx_hal_pwr_ex.o
 .text.HAL_PWREx_DisableMainRegulatorLowVoltage
                0x00000000       0x10 build/stm32f7xx_hal_pwr_ex.o
 .text.HAL_PWREx_EnableLowRegulatorLowVoltage
                0x00000000       0x10 build/stm32f7xx_hal_pwr_ex.o
 .text.HAL_PWREx_DisableLowRegulatorLowVoltage
                0x00000000       0x10 build/stm32f7xx_hal_pwr_ex.o
 .text.HAL_PWREx_DisableOverDrive
                0x00000000       0x7c build/stm32f7xx_hal_pwr_ex.o
 .text.HAL_PWREx_EnterUnderDriveSTOPMode
                0x00000000       0x98 build/stm32f7xx_hal_pwr_ex.o
 .text.HAL_PWREx_GetVoltageRange
                0x00000000       0x10 build/stm32f7xx_hal_pwr_ex.o
 .text.HAL_PWREx_ControlVoltageScaling
                0x00000000       0xc0 build/stm32f7xx_hal_pwr_ex.o
 .text          0x00000000        0x0 build/stm32f7xx_hal_cortex.o
 .data          0x00000000        0x0 build/stm32f7xx_hal_cortex.o
 .bss           0x00000000        0x0 build/stm32f7xx_hal_cortex.o
 .text.__NVIC_DisableIRQ
                0x00000000       0x24 build/stm32f7xx_hal_cortex.o
 .text.__NVIC_GetPriority
                0x00000000       0x20 build/stm32f7xx_hal_cortex.o
 .text.NVIC_DecodePriority
                0x00000000       0x3e build/stm32f7xx_hal_cortex.o
 .text.__NVIC_SystemReset
                0x00000000       0x24 build/stm32f7xx_hal_cortex.o
 .text.HAL_NVIC_DisableIRQ
                0x00000000        0x8 build/stm32f7xx_hal_cortex.o
 .text.HAL_NVIC_SystemReset
                0x00000000        0x6 build/stm32f7xx_hal_cortex.o
 .text.HAL_MPU_Disable
                0x00000000       0x1c build/stm32f7xx_hal_cortex.o
 .text.HAL_MPU_Enable
                0x00000000       0x20 build/stm32f7xx_hal_cortex.o
 .text.HAL_MPU_EnableRegion
                0x00000000       0x18 build/stm32f7xx_hal_cortex.o
 .text.HAL_MPU_DisableRegion
                0x00000000       0x18 build/stm32f7xx_hal_cortex.o
 .text.HAL_MPU_ConfigRegion
                0x00000000       0x58 build/stm32f7xx_hal_cortex.o
 .text.HAL_NVIC_GetPriorityGrouping
                0x00000000       0x10 build/stm32f7xx_hal_cortex.o
 .text.HAL_NVIC_GetPriority
                0x00000000       0x18 build/stm32f7xx_hal_cortex.o
 .text.HAL_NVIC_SetPendingIRQ
                0x00000000       0x1c build/stm32f7xx_hal_cortex.o
 .text.HAL_NVIC_GetPendingIRQ
                0x00000000       0x24 build/stm32f7xx_hal_cortex.o
 .text.HAL_NVIC_ClearPendingIRQ
                0x00000000       0x1c build/stm32f7xx_hal_cortex.o
 .text.HAL_NVIC_GetActive
                0x00000000       0x24 build/stm32f7xx_hal_cortex.o
 .text.HAL_SYSTICK_CLKSourceConfig
                0x00000000       0x20 build/stm32f7xx_hal_cortex.o
 .text.HAL_SYSTICK_Callback
                0x00000000        0x2 build/stm32f7xx_hal_cortex.o
 .text.HAL_SYSTICK_IRQHandler
                0x00000000        0x8 build/stm32f7xx_hal_cortex.o
 .text          0x00000000        0x0 build/stm32f7xx_hal.o
 .data          0x00000000        0x0 build/stm32f7xx_hal.o
 .bss           0x00000000        0x0 build/stm32f7xx_hal.o
 .text.HAL_MspInit
                0x00000000        0x2 build/stm32f7xx_hal.o
 .text.HAL_MspDeInit
                0x00000000        0x2 build/stm32f7xx_hal.o
 .text.HAL_DeInit
                0x00000000       0x2c build/stm32f7xx_hal.o
 .text.HAL_GetTickPrio
                0x00000000        0xc build/stm32f7xx_hal.o
 .text.HAL_SetTickFreq
                0x00000000       0x2c build/stm32f7xx_hal.o
 .text.HAL_GetTickFreq
                0x00000000        0xc build/stm32f7xx_hal.o
 .text.HAL_SuspendTick
                0x00000000        0xe build/stm32f7xx_hal.o
 .text.HAL_ResumeTick
                0x00000000        0xe build/stm32f7xx_hal.o
 .text.HAL_GetHalVersion
                0x00000000        0x8 build/stm32f7xx_hal.o
 .text.HAL_GetREVID
                0x00000000        0xc build/stm32f7xx_hal.o
 .text.HAL_GetDEVID
                0x00000000       0x10 build/stm32f7xx_hal.o
 .text.HAL_GetUIDw0
                0x00000000        0xc build/stm32f7xx_hal.o
 .text.HAL_GetUIDw1
                0x00000000        0xc build/stm32f7xx_hal.o
 .text.HAL_GetUIDw2
                0x00000000        0xc build/stm32f7xx_hal.o
 .text.HAL_DBGMCU_EnableDBGSleepMode
                0x00000000       0x10 build/stm32f7xx_hal.o
 .text.HAL_DBGMCU_DisableDBGSleepMode
                0x00000000       0x10 build/stm32f7xx_hal.o
 .text.HAL_DBGMCU_EnableDBGStopMode
                0x00000000       0x10 build/stm32f7xx_hal.o
 .text.HAL_DBGMCU_DisableDBGStopMode
                0x00000000       0x10 build/stm32f7xx_hal.o
 .text.HAL_DBGMCU_EnableDBGStandbyMode
                0x00000000       0x10 build/stm32f7xx_hal.o
 .text.HAL_DBGMCU_DisableDBGStandbyMode
                0x00000000       0x10 build/stm32f7xx_hal.o
 .text.HAL_EnableCompensationCell
                0x00000000       0x10 build/stm32f7xx_hal.o
 .text.HAL_DisableCompensationCell
                0x00000000       0x10 build/stm32f7xx_hal.o
 .text.HAL_EnableFMCMemorySwapping
                0x00000000       0x10 build/stm32f7xx_hal.o
 .text.HAL_DisableFMCMemorySwapping
                0x00000000       0x10 build/stm32f7xx_hal.o
 .text.HAL_EnableMemorySwappingBank
                0x00000000       0x10 build/stm32f7xx_hal.o
 .text.HAL_DisableMemorySwappingBank
                0x00000000       0x10 build/stm32f7xx_hal.o
 .text          0x00000000        0x0 build/stm32f7xx_hal_i2c.o
 .data          0x00000000        0x0 build/stm32f7xx_hal_i2c.o
 .bss           0x00000000        0x0 build/stm32f7xx_hal_i2c.o
 .text.I2C_Flush_TXDR
                0x00000000       0x22 build/stm32f7xx_hal_i2c.o
 .text.I2C_TransferConfig
                0x00000000       0x3c build/stm32f7xx_hal_i2c.o
 .text.I2C_Enable_IRQ
                0x00000000       0x9c build/stm32f7xx_hal_i2c.o
 .text.I2C_Disable_IRQ
                0x00000000       0x70 build/stm32f7xx_hal_i2c.o
 .text.I2C_ConvertOtherXferOptions
                0x00000000       0x1e build/stm32f7xx_hal_i2c.o
 .text.I2C_IsErrorOccurred
                0x00000000      0x118 build/stm32f7xx_hal_i2c.o
 .text.I2C_WaitOnTXISFlagUntilTimeout
                0x00000000       0x60 build/stm32f7xx_hal_i2c.o
 .text.I2C_WaitOnFlagUntilTimeout
                0x00000000       0x7c build/stm32f7xx_hal_i2c.o
 .text.I2C_RequestMemoryWrite
                0x00000000       0x7c build/stm32f7xx_hal_i2c.o
 .text.I2C_RequestMemoryRead
                0x00000000       0x78 build/stm32f7xx_hal_i2c.o
 .text.I2C_WaitOnSTOPFlagUntilTimeout
                0x00000000       0x5e build/stm32f7xx_hal_i2c.o
 .text.I2C_WaitOnRXNEFlagUntilTimeout
                0x00000000       0xaa build/stm32f7xx_hal_i2c.o
 .text.HAL_I2C_MspInit
                0x00000000        0x2 build/stm32f7xx_hal_i2c.o
 .text.HAL_I2C_Init
                0x00000000       0xc8 build/stm32f7xx_hal_i2c.o
 .text.HAL_I2C_MspDeInit
                0x00000000        0x2 build/stm32f7xx_hal_i2c.o
 .text.HAL_I2C_DeInit
                0x00000000       0x32 build/stm32f7xx_hal_i2c.o
 .text.HAL_I2C_Master_Transmit
                0x00000000      0x1a4 build/stm32f7xx_hal_i2c.o
 .text.HAL_I2C_Master_Receive
                0x00000000      0x17c build/stm32f7xx_hal_i2c.o
 .text.HAL_I2C_Slave_Transmit
                0x00000000      0x1f4 build/stm32f7xx_hal_i2c.o
 .text.HAL_I2C_Slave_Receive
                0x00000000      0x184 build/stm32f7xx_hal_i2c.o
 .text.HAL_I2C_Master_Transmit_IT
                0x00000000       0xc8 build/stm32f7xx_hal_i2c.o
 .text.HAL_I2C_Master_Receive_IT
                0x00000000       0x98 build/stm32f7xx_hal_i2c.o
 .text.HAL_I2C_Slave_Transmit_IT
                0x00000000       0x8c build/stm32f7xx_hal_i2c.o
 .text.HAL_I2C_Slave_Receive_IT
                0x00000000       0x64 build/stm32f7xx_hal_i2c.o
 .text.HAL_I2C_Master_Transmit_DMA
                0x00000000      0x174 build/stm32f7xx_hal_i2c.o
 .text.HAL_I2C_Master_Receive_DMA
                0x00000000      0x150 build/stm32f7xx_hal_i2c.o
 .text.HAL_I2C_Slave_Transmit_DMA
                0x00000000      0x140 build/stm32f7xx_hal_i2c.o
 .text.HAL_I2C_Slave_Receive_DMA
                0x00000000       0xf4 build/stm32f7xx_hal_i2c.o
 .text.HAL_I2C_Mem_Write
                0x00000000      0x1aa build/stm32f7xx_hal_i2c.o
 .text.HAL_I2C_Mem_Read
                0x00000000      0x1b0 build/stm32f7xx_hal_i2c.o
 .text.HAL_I2C_Mem_Write_IT
                0x00000000       0xb8 build/stm32f7xx_hal_i2c.o
 .text.HAL_I2C_Mem_Read_IT
                0x00000000       0xb4 build/stm32f7xx_hal_i2c.o
 .text.HAL_I2C_Mem_Write_DMA
                0x00000000      0x134 build/stm32f7xx_hal_i2c.o
 .text.HAL_I2C_Mem_Read_DMA
                0x00000000      0x134 build/stm32f7xx_hal_i2c.o
 .text.HAL_I2C_IsDeviceReady
                0x00000000      0x13c build/stm32f7xx_hal_i2c.o
 .text.HAL_I2C_Master_Seq_Transmit_IT
                0x00000000      0x10c build/stm32f7xx_hal_i2c.o
 .text.HAL_I2C_Master_Seq_Transmit_DMA
                0x00000000      0x1e4 build/stm32f7xx_hal_i2c.o
 .text.HAL_I2C_Master_Seq_Receive_IT
                0x00000000       0xb4 build/stm32f7xx_hal_i2c.o
 .text.HAL_I2C_Master_Seq_Receive_DMA
                0x00000000      0x174 build/stm32f7xx_hal_i2c.o
 .text.HAL_I2C_Slave_Seq_Transmit_IT
                0x00000000       0xe4 build/stm32f7xx_hal_i2c.o
 .text.HAL_I2C_Slave_Seq_Transmit_DMA
                0x00000000      0x1ac build/stm32f7xx_hal_i2c.o
 .text.HAL_I2C_Slave_Seq_Receive_IT
                0x00000000       0xe4 build/stm32f7xx_hal_i2c.o
 .text.HAL_I2C_Slave_Seq_Receive_DMA
                0x00000000      0x1ac build/stm32f7xx_hal_i2c.o
 .text.HAL_I2C_EnableListen_IT
                0x00000000       0x2c build/stm32f7xx_hal_i2c.o
 .text.HAL_I2C_DisableListen_IT
                0x00000000       0x3a build/stm32f7xx_hal_i2c.o
 .text.HAL_I2C_Master_Abort_IT
                0x00000000       0x88 build/stm32f7xx_hal_i2c.o
 .text.HAL_I2C_EV_IRQHandler
                0x00000000       0x10 build/stm32f7xx_hal_i2c.o
 .text.HAL_I2C_MasterTxCpltCallback
                0x00000000        0x2 build/stm32f7xx_hal_i2c.o
 .text.HAL_I2C_MasterRxCpltCallback
                0x00000000        0x2 build/stm32f7xx_hal_i2c.o
 .text.I2C_ITMasterSeqCplt
                0x00000000       0x54 build/stm32f7xx_hal_i2c.o
 .text.HAL_I2C_SlaveTxCpltCallback
                0x00000000        0x2 build/stm32f7xx_hal_i2c.o
 .text.HAL_I2C_SlaveRxCpltCallback
                0x00000000        0x2 build/stm32f7xx_hal_i2c.o
 .text.I2C_ITSlaveSeqCplt
                0x00000000       0x82 build/stm32f7xx_hal_i2c.o
 .text.I2C_DMASlaveTransmitCplt
                0x00000000       0x22 build/stm32f7xx_hal_i2c.o
 .text.I2C_DMASlaveReceiveCplt
                0x00000000       0x26 build/stm32f7xx_hal_i2c.o
 .text.HAL_I2C_AddrCallback
                0x00000000        0x2 build/stm32f7xx_hal_i2c.o
 .text.I2C_ITAddrCplt
                0x00000000       0xa0 build/stm32f7xx_hal_i2c.o
 .text.HAL_I2C_ListenCpltCallback
                0x00000000        0x2 build/stm32f7xx_hal_i2c.o
 .text.I2C_ITListenCplt
                0x00000000       0x68 build/stm32f7xx_hal_i2c.o
 .text.HAL_I2C_MemTxCpltCallback
                0x00000000        0x2 build/stm32f7xx_hal_i2c.o
 .text.HAL_I2C_MemRxCpltCallback
                0x00000000        0x2 build/stm32f7xx_hal_i2c.o
 .text.HAL_I2C_ErrorCallback
                0x00000000        0x2 build/stm32f7xx_hal_i2c.o
 .text.HAL_I2C_AbortCpltCallback
                0x00000000        0x2 build/stm32f7xx_hal_i2c.o
 .text.I2C_TreatErrorCallback
                0x00000000       0x2e build/stm32f7xx_hal_i2c.o
 .text.I2C_ITError
                0x00000000      0x130 build/stm32f7xx_hal_i2c.o
 .text.I2C_ITSlaveCplt
                0x00000000      0x1f0 build/stm32f7xx_hal_i2c.o
 .text.I2C_Slave_ISR_IT
                0x00000000      0x14a build/stm32f7xx_hal_i2c.o
 .text.I2C_ITMasterCplt
                0x00000000      0x12e build/stm32f7xx_hal_i2c.o
 .text.I2C_Master_ISR_IT
                0x00000000      0x1ac build/stm32f7xx_hal_i2c.o
 .text.I2C_Mem_ISR_DMA
                0x00000000      0x1d0 build/stm32f7xx_hal_i2c.o
 .text.I2C_Slave_ISR_DMA
                0x00000000      0x124 build/stm32f7xx_hal_i2c.o
 .text.I2C_Master_ISR_DMA
                0x00000000      0x154 build/stm32f7xx_hal_i2c.o
 .text.I2C_DMAError
                0x00000000       0x44 build/stm32f7xx_hal_i2c.o
 .text.I2C_DMAMasterTransmitCplt
                0x00000000       0x5a build/stm32f7xx_hal_i2c.o
 .text.I2C_DMAMasterReceiveCplt
                0x00000000       0x6a build/stm32f7xx_hal_i2c.o
 .text.I2C_Mem_ISR_IT
                0x00000000      0x1c0 build/stm32f7xx_hal_i2c.o
 .text.HAL_I2C_ER_IRQHandler
                0x00000000       0x6a build/stm32f7xx_hal_i2c.o
 .text.I2C_DMAAbort
                0x00000000       0x1a build/stm32f7xx_hal_i2c.o
 .text.HAL_I2C_GetState
                0x00000000        0x6 build/stm32f7xx_hal_i2c.o
 .text.HAL_I2C_GetMode
                0x00000000        0x6 build/stm32f7xx_hal_i2c.o
 .text.HAL_I2C_GetError
                0x00000000        0x4 build/stm32f7xx_hal_i2c.o
 .debug_info    0x00000000     0x471d build/stm32f7xx_hal_i2c.o
 .debug_abbrev  0x00000000      0x2e4 build/stm32f7xx_hal_i2c.o
 .debug_loc     0x00000000     0x655b build/stm32f7xx_hal_i2c.o
 .debug_aranges
                0x00000000      0x2a0 build/stm32f7xx_hal_i2c.o
 .debug_ranges  0x00000000      0x290 build/stm32f7xx_hal_i2c.o
 .debug_line    0x00000000     0x4da9 build/stm32f7xx_hal_i2c.o
 .debug_str     0x00000000     0x1055 build/stm32f7xx_hal_i2c.o
 .comment       0x00000000       0x27 build/stm32f7xx_hal_i2c.o
 .debug_frame   0x00000000      0x988 build/stm32f7xx_hal_i2c.o
 .ARM.attributes
                0x00000000       0x32 build/stm32f7xx_hal_i2c.o
 .text          0x00000000        0x0 build/stm32f7xx_hal_i2c_ex.o
 .data          0x00000000        0x0 build/stm32f7xx_hal_i2c_ex.o
 .bss           0x00000000        0x0 build/stm32f7xx_hal_i2c_ex.o
 .text.HAL_I2CEx_ConfigAnalogFilter
                0x00000000       0x5c build/stm32f7xx_hal_i2c_ex.o
 .text.HAL_I2CEx_ConfigDigitalFilter
                0x00000000       0x58 build/stm32f7xx_hal_i2c_ex.o
 .text.HAL_I2CEx_EnableFastModePlus
                0x00000000       0x2c build/stm32f7xx_hal_i2c_ex.o
 .text.HAL_I2CEx_DisableFastModePlus
                0x00000000       0x2c build/stm32f7xx_hal_i2c_ex.o
 .debug_info    0x00000000      0xab8 build/stm32f7xx_hal_i2c_ex.o
 .debug_abbrev  0x00000000      0x1b5 build/stm32f7xx_hal_i2c_ex.o
 .debug_loc     0x00000000      0x197 build/stm32f7xx_hal_i2c_ex.o
 .debug_aranges
                0x00000000       0x38 build/stm32f7xx_hal_i2c_ex.o
 .debug_ranges  0x00000000       0x28 build/stm32f7xx_hal_i2c_ex.o
 .debug_line    0x00000000      0x274 build/stm32f7xx_hal_i2c_ex.o
 .debug_str     0x00000000      0x8d5 build/stm32f7xx_hal_i2c_ex.o
 .comment       0x00000000       0x27 build/stm32f7xx_hal_i2c_ex.o
 .debug_frame   0x00000000       0x60 build/stm32f7xx_hal_i2c_ex.o
 .ARM.attributes
                0x00000000       0x32 build/stm32f7xx_hal_i2c_ex.o
 .text          0x00000000        0x0 build/stm32f7xx_hal_exti.o
 .data          0x00000000        0x0 build/stm32f7xx_hal_exti.o
 .bss           0x00000000        0x0 build/stm32f7xx_hal_exti.o
 .text.HAL_EXTI_SetConfigLine
                0x00000000       0xd4 build/stm32f7xx_hal_exti.o
 .text.HAL_EXTI_GetConfigLine
                0x00000000       0xa8 build/stm32f7xx_hal_exti.o
 .text.HAL_EXTI_ClearConfigLine
                0x00000000       0x84 build/stm32f7xx_hal_exti.o
 .text.HAL_EXTI_RegisterCallback
                0x00000000        0xe build/stm32f7xx_hal_exti.o
 .text.HAL_EXTI_GetHandle
                0x00000000        0xc build/stm32f7xx_hal_exti.o
 .text.HAL_EXTI_IRQHandler
                0x00000000       0x24 build/stm32f7xx_hal_exti.o
 .text.HAL_EXTI_GetPending
                0x00000000       0x18 build/stm32f7xx_hal_exti.o
 .text.HAL_EXTI_ClearPending
                0x00000000       0x14 build/stm32f7xx_hal_exti.o
 .text.HAL_EXTI_GenerateSWI
                0x00000000       0x14 build/stm32f7xx_hal_exti.o
 .debug_info    0x00000000      0x613 build/stm32f7xx_hal_exti.o
 .debug_abbrev  0x00000000      0x1ef build/stm32f7xx_hal_exti.o
 .debug_loc     0x00000000      0x5f6 build/stm32f7xx_hal_exti.o
 .debug_aranges
                0x00000000       0x60 build/stm32f7xx_hal_exti.o
 .debug_ranges  0x00000000       0x50 build/stm32f7xx_hal_exti.o
 .debug_line    0x00000000      0x55d build/stm32f7xx_hal_exti.o
 .debug_str     0x00000000      0x3de build/stm32f7xx_hal_exti.o
 .comment       0x00000000       0x27 build/stm32f7xx_hal_exti.o
 .debug_frame   0x00000000       0xe8 build/stm32f7xx_hal_exti.o
 .ARM.attributes
                0x00000000       0x32 build/stm32f7xx_hal_exti.o
 .text          0x00000000        0x0 build/stm32f7xx_ll_rcc.o
 .data          0x00000000        0x0 build/stm32f7xx_ll_rcc.o
 .bss           0x00000000        0x0 build/stm32f7xx_ll_rcc.o
 .text.LL_RCC_DeInit
                0x00000000       0x98 build/stm32f7xx_ll_rcc.o
 .text.LL_RCC_GetCECClockFreq
                0x00000000       0x30 build/stm32f7xx_ll_rcc.o
 .text.LL_RCC_GetSystemClocksFreq
                0x00000000       0x20 build/stm32f7xx_ll_rcc.o
 .text.LL_RCC_GetI2CClockFreq
                0x00000000      0x120 build/stm32f7xx_ll_rcc.o
 .text.LL_RCC_GetLPTIMClockFreq
                0x00000000       0x6c build/stm32f7xx_ll_rcc.o
 .text.LL_RCC_GetDFSDMClockFreq
                0x00000000       0x28 build/stm32f7xx_ll_rcc.o
 .text.RCC_PLL_GetFreqDomain_48M
                0x00000000       0x40 build/stm32f7xx_ll_rcc.o
 .text.RCC_PLLSAI_GetFreqDomain_SAI
                0x00000000       0x50 build/stm32f7xx_ll_rcc.o
 .text.RCC_PLLSAI_GetFreqDomain_48M
                0x00000000       0x48 build/stm32f7xx_ll_rcc.o
 .text.LL_RCC_GetSDMMCClockFreq
                0x00000000       0x94 build/stm32f7xx_ll_rcc.o
 .text.LL_RCC_GetRNGClockFreq
                0x00000000       0x34 build/stm32f7xx_ll_rcc.o
 .text.LL_RCC_GetUSBClockFreq
                0x00000000       0x34 build/stm32f7xx_ll_rcc.o
 .text.RCC_PLLSAI_GetFreqDomain_LTDC
                0x00000000       0x58 build/stm32f7xx_ll_rcc.o
 .text.LL_RCC_GetLTDCClockFreq
                0x00000000       0x18 build/stm32f7xx_ll_rcc.o
 .text.RCC_PLLI2S_GetFreqDomain_SAI
                0x00000000       0x50 build/stm32f7xx_ll_rcc.o
 .text.LL_RCC_GetSAIClockFreq
                0x00000000      0x11c build/stm32f7xx_ll_rcc.o
 .text.LL_RCC_GetDFSDMAudioClockFreq
                0x00000000       0x24 build/stm32f7xx_ll_rcc.o
 .text.RCC_PLLI2S_GetFreqDomain_SPDIFRX
                0x00000000       0x48 build/stm32f7xx_ll_rcc.o
 .text.LL_RCC_GetSPDIFRXClockFreq
                0x00000000       0x18 build/stm32f7xx_ll_rcc.o
 .text.RCC_PLLI2S_GetFreqDomain_I2S
                0x00000000       0x44 build/stm32f7xx_ll_rcc.o
 .text.LL_RCC_GetI2SClockFreq
                0x00000000       0x34 build/stm32f7xx_ll_rcc.o
 .rodata.aRCC_PLLSAIDIVRPrescTable
                0x00000000        0x4 build/stm32f7xx_ll_rcc.o
 .text          0x00000000        0x0 build/stm32f7xx_ll_utils.o
 .data          0x00000000        0x0 build/stm32f7xx_ll_utils.o
 .bss           0x00000000        0x0 build/stm32f7xx_ll_utils.o
 .text.UTILS_GetPLLOutputFrequency
                0x00000000       0x20 build/stm32f7xx_ll_utils.o
 .text.UTILS_PLL_IsBusy
                0x00000000       0x30 build/stm32f7xx_ll_utils.o
 .text.LL_Init1msTick
                0x00000000       0x20 build/stm32f7xx_ll_utils.o
 .text.LL_mDelay
                0x00000000       0x2a build/stm32f7xx_ll_utils.o
 .text.LL_SetSystemCoreClock
                0x00000000        0xc build/stm32f7xx_ll_utils.o
 .text.LL_SetFlashLatency
                0x00000000      0x160 build/stm32f7xx_ll_utils.o
 .text.UTILS_EnablePLLAndSwitchSystem
                0x00000000       0xac build/stm32f7xx_ll_utils.o
 .text.LL_PLL_ConfigSystemClock_HSI
                0x00000000       0x64 build/stm32f7xx_ll_utils.o
 .text.LL_PLL_ConfigSystemClock_HSE
                0x00000000       0x84 build/stm32f7xx_ll_utils.o
 .debug_info    0x00000000      0xdcd build/stm32f7xx_ll_utils.o
 .debug_abbrev  0x00000000      0x2f3 build/stm32f7xx_ll_utils.o
 .debug_loc     0x00000000      0x93f build/stm32f7xx_ll_utils.o
 .debug_aranges
                0x00000000       0x60 build/stm32f7xx_ll_utils.o
 .debug_ranges  0x00000000       0x50 build/stm32f7xx_ll_utils.o
 .debug_line    0x00000000      0x7ae build/stm32f7xx_ll_utils.o
 .debug_str     0x00000000      0x76e build/stm32f7xx_ll_utils.o
 .comment       0x00000000       0x27 build/stm32f7xx_ll_utils.o
 .debug_frame   0x00000000       0xec build/stm32f7xx_ll_utils.o
 .ARM.attributes
                0x00000000       0x32 build/stm32f7xx_ll_utils.o
 .text          0x00000000        0x0 build/stm32f7xx_ll_exti.o
 .data          0x00000000        0x0 build/stm32f7xx_ll_exti.o
 .bss           0x00000000        0x0 build/stm32f7xx_ll_exti.o
 .text.LL_EXTI_DeInit
                0x00000000       0x1c build/stm32f7xx_ll_exti.o
 .text.LL_EXTI_Init
                0x00000000       0xd8 build/stm32f7xx_ll_exti.o
 .text.LL_EXTI_StructInit
                0x00000000        0xe build/stm32f7xx_ll_exti.o
 .debug_info    0x00000000      0x52a build/stm32f7xx_ll_exti.o
 .debug_abbrev  0x00000000      0x1d9 build/stm32f7xx_ll_exti.o
 .debug_loc     0x00000000      0x322 build/stm32f7xx_ll_exti.o
 .debug_aranges
                0x00000000       0x30 build/stm32f7xx_ll_exti.o
 .debug_ranges  0x00000000       0x98 build/stm32f7xx_ll_exti.o
 .debug_line    0x00000000      0x36c build/stm32f7xx_ll_exti.o
 .debug_str     0x00000000      0x381 build/stm32f7xx_ll_exti.o
 .comment       0x00000000       0x27 build/stm32f7xx_ll_exti.o
 .debug_frame   0x00000000       0x50 build/stm32f7xx_ll_exti.o
 .ARM.attributes
                0x00000000       0x32 build/stm32f7xx_ll_exti.o
 .text          0x00000000        0x0 build/stm32f7xx_ll_gpio.o
 .data          0x00000000        0x0 build/stm32f7xx_ll_gpio.o
 .bss           0x00000000        0x0 build/stm32f7xx_ll_gpio.o
 .text.LL_GPIO_DeInit
                0x00000000      0x17c build/stm32f7xx_ll_gpio.o
 .text.LL_GPIO_StructInit
                0x00000000       0x16 build/stm32f7xx_ll_gpio.o
 .text          0x00000000        0x0 build/stm32f7xx_ll_dma.o
 .data          0x00000000        0x0 build/stm32f7xx_ll_dma.o
 .bss           0x00000000        0x0 build/stm32f7xx_ll_dma.o
 .text.LL_DMA_DeInit
                0x00000000      0x1f8 build/stm32f7xx_ll_dma.o
 .text.LL_DMA_Init
                0x00000000       0x9c build/stm32f7xx_ll_dma.o
 .text.LL_DMA_StructInit
                0x00000000       0x22 build/stm32f7xx_ll_dma.o
 .rodata.STREAM_OFFSET_TAB
                0x00000000        0x8 build/stm32f7xx_ll_dma.o
 .debug_info    0x00000000      0xb2f build/stm32f7xx_ll_dma.o
 .debug_abbrev  0x00000000      0x26a build/stm32f7xx_ll_dma.o
 .debug_loc     0x00000000      0x6ad build/stm32f7xx_ll_dma.o
 .debug_aranges
                0x00000000       0x30 build/stm32f7xx_ll_dma.o
 .debug_ranges  0x00000000       0x68 build/stm32f7xx_ll_dma.o
 .debug_line    0x00000000      0x502 build/stm32f7xx_ll_dma.o
 .debug_str     0x00000000      0x5e5 build/stm32f7xx_ll_dma.o
 .comment       0x00000000       0x27 build/stm32f7xx_ll_dma.o
 .debug_frame   0x00000000       0x60 build/stm32f7xx_ll_dma.o
 .ARM.attributes
                0x00000000       0x32 build/stm32f7xx_ll_dma.o
 .text          0x00000000        0x0 build/stm32f7xx_ll_sdmmc.o
 .data          0x00000000        0x0 build/stm32f7xx_ll_sdmmc.o
 .bss           0x00000000        0x0 build/stm32f7xx_ll_sdmmc.o
 .text.SDMMC_PowerState_OFF
                0x00000000        0x8 build/stm32f7xx_ll_sdmmc.o
 .text.SDMMC_GetDataCounter
                0x00000000        0x4 build/stm32f7xx_ll_sdmmc.o
 .text.SDMMC_GetFIFOCount
                0x00000000        0x6 build/stm32f7xx_ll_sdmmc.o
 .text.SDMMC_SetSDMMCReadWaitMode
                0x00000000        0xe build/stm32f7xx_ll_sdmmc.o
 .text.SDMMC_CmdSDEraseStartAdd
                0x00000000       0x30 build/stm32f7xx_ll_sdmmc.o
 .text.SDMMC_CmdSDEraseEndAdd
                0x00000000       0x30 build/stm32f7xx_ll_sdmmc.o
 .text.SDMMC_CmdEraseStartAdd
                0x00000000       0x30 build/stm32f7xx_ll_sdmmc.o
 .text.SDMMC_CmdEraseEndAdd
                0x00000000       0x30 build/stm32f7xx_ll_sdmmc.o
 .text.SDMMC_CmdErase
                0x00000000       0x30 build/stm32f7xx_ll_sdmmc.o
 .text.SDMMC_CmdSetRelAddMmc
                0x00000000       0x32 build/stm32f7xx_ll_sdmmc.o
 .text.SDMMC_CmdStatusRegister
                0x00000000       0x30 build/stm32f7xx_ll_sdmmc.o
 .text.SDMMC_CmdSwitch
                0x00000000       0x30 build/stm32f7xx_ll_sdmmc.o
 .text.SDMMC_CmdSendEXTCSD
                0x00000000       0x30 build/stm32f7xx_ll_sdmmc.o
 .text.SDMMC_CmdOpCondition
                0x00000000       0x2a build/stm32f7xx_ll_sdmmc.o
 .text          0x00000000        0x0 build/stm32f7xx_hal_sd.o
 .data          0x00000000        0x0 build/stm32f7xx_hal_sd.o
 .bss           0x00000000        0x0 build/stm32f7xx_hal_sd.o
 .text.SD_DMATransmitCplt
                0x00000000        0xe build/stm32f7xx_hal_sd.o
 .text.SD_PowerOFF
                0x00000000        0xa build/stm32f7xx_hal_sd.o
 .text.SD_Read_IT
                0x00000000       0x38 build/stm32f7xx_hal_sd.o
 .text.SD_Write_IT
                0x00000000       0x48 build/stm32f7xx_hal_sd.o
 .text.SD_SendSDStatus
                0x00000000      0x106 build/stm32f7xx_hal_sd.o
 .text.HAL_SD_MspInit
                0x00000000        0x2 build/stm32f7xx_hal_sd.o
 .text.HAL_SD_MspDeInit
                0x00000000        0x2 build/stm32f7xx_hal_sd.o
 .text.HAL_SD_DeInit
                0x00000000       0x24 build/stm32f7xx_hal_sd.o
 .text.HAL_SD_ReadBlocks_IT
                0x00000000       0xcc build/stm32f7xx_hal_sd.o
 .text.HAL_SD_WriteBlocks_IT
                0x00000000       0xc4 build/stm32f7xx_hal_sd.o
 .text.HAL_SD_ReadBlocks_DMA
                0x00000000      0x134 build/stm32f7xx_hal_sd.o
 .text.HAL_SD_WriteBlocks_DMA
                0x00000000      0x130 build/stm32f7xx_hal_sd.o
 .text.HAL_SD_Erase
                0x00000000       0xf8 build/stm32f7xx_hal_sd.o
 .text.HAL_SD_GetState
                0x00000000        0x6 build/stm32f7xx_hal_sd.o
 .text.HAL_SD_GetError
                0x00000000        0x4 build/stm32f7xx_hal_sd.o
 .text.HAL_SD_TxCpltCallback
                0x00000000        0x2 build/stm32f7xx_hal_sd.o
 .text.HAL_SD_RxCpltCallback
                0x00000000        0x2 build/stm32f7xx_hal_sd.o
 .text.HAL_SD_ErrorCallback
                0x00000000        0x2 build/stm32f7xx_hal_sd.o
 .text.SD_DMAReceiveCplt
                0x00000000       0x48 build/stm32f7xx_hal_sd.o
 .text.HAL_SD_AbortCallback
                0x00000000        0x2 build/stm32f7xx_hal_sd.o
 .text.HAL_SD_GetCardCID
                0x00000000       0x58 build/stm32f7xx_hal_sd.o
 .text.HAL_SD_GetCardStatus
                0x00000000       0xac build/stm32f7xx_hal_sd.o
 .text.SD_DMAError
                0x00000000       0x68 build/stm32f7xx_hal_sd.o
 .text.SD_DMATxAbort
                0x00000000       0x44 build/stm32f7xx_hal_sd.o
 .text.SD_DMARxAbort
                0x00000000       0x44 build/stm32f7xx_hal_sd.o
 .text.HAL_SD_IRQHandler
                0x00000000      0x1c8 build/stm32f7xx_hal_sd.o
 .text.HAL_SD_Abort
                0x00000000       0x92 build/stm32f7xx_hal_sd.o
 .text.HAL_SD_Abort_IT
                0x00000000       0xa8 build/stm32f7xx_hal_sd.o
 .text          0x00000000        0x0 build/stm32f7xx_ll_spi.o
 .data          0x00000000        0x0 build/stm32f7xx_ll_spi.o
 .bss           0x00000000        0x0 build/stm32f7xx_ll_spi.o
 .text.LL_SPI_DeInit
                0x00000000       0xd4 build/stm32f7xx_ll_spi.o
 .text.LL_SPI_StructInit
                0x00000000       0x1e build/stm32f7xx_ll_spi.o
 .text.LL_I2S_DeInit
                0x00000000        0x8 build/stm32f7xx_ll_spi.o
 .text.LL_I2S_Init
                0x00000000       0xac build/stm32f7xx_ll_spi.o
 .text.LL_I2S_StructInit
                0x00000000       0x12 build/stm32f7xx_ll_spi.o
 .text.LL_I2S_ConfigPrescaler
                0x00000000       0x10 build/stm32f7xx_ll_spi.o
 .text          0x00000000        0x0 build/stm32f7xx_hal_tim.o
 .data          0x00000000        0x0 build/stm32f7xx_hal_tim.o
 .bss           0x00000000        0x0 build/stm32f7xx_hal_tim.o
 .text.TIM_TI2_SetConfig
                0x00000000       0x36 build/stm32f7xx_hal_tim.o
 .text.TIM_TI3_SetConfig
                0x00000000       0x36 build/stm32f7xx_hal_tim.o
 .text.TIM_TI4_SetConfig
                0x00000000       0x36 build/stm32f7xx_hal_tim.o
 .text.HAL_TIM_Base_MspInit
                0x00000000        0x2 build/stm32f7xx_hal_tim.o
 .text.HAL_TIM_Base_MspDeInit
                0x00000000        0x2 build/stm32f7xx_hal_tim.o
 .text.HAL_TIM_Base_DeInit
                0x00000000       0x66 build/stm32f7xx_hal_tim.o
 .text.HAL_TIM_Base_Start
                0x00000000       0x88 build/stm32f7xx_hal_tim.o
 .text.HAL_TIM_Base_Start_DMA
                0x00000000       0xdc build/stm32f7xx_hal_tim.o
 .text.HAL_TIM_Base_Stop_DMA
                0x00000000       0x3c build/stm32f7xx_hal_tim.o
 .text.HAL_TIM_OC_MspInit
                0x00000000        0x2 build/stm32f7xx_hal_tim.o
 .text.HAL_TIM_OC_MspDeInit
                0x00000000        0x2 build/stm32f7xx_hal_tim.o
 .text.HAL_TIM_OC_DeInit
                0x00000000       0x66 build/stm32f7xx_hal_tim.o
 .text.HAL_TIM_PWM_MspDeInit
                0x00000000        0x2 build/stm32f7xx_hal_tim.o
 .text.HAL_TIM_PWM_DeInit
                0x00000000       0x66 build/stm32f7xx_hal_tim.o
 .text.HAL_TIM_IC_MspInit
                0x00000000        0x2 build/stm32f7xx_hal_tim.o
 .text.HAL_TIM_IC_MspDeInit
                0x00000000        0x2 build/stm32f7xx_hal_tim.o
 .text.HAL_TIM_IC_DeInit
                0x00000000       0x66 build/stm32f7xx_hal_tim.o
 .text.HAL_TIM_OnePulse_MspInit
                0x00000000        0x2 build/stm32f7xx_hal_tim.o
 .text.HAL_TIM_OnePulse_MspDeInit
                0x00000000        0x2 build/stm32f7xx_hal_tim.o
 .text.HAL_TIM_OnePulse_DeInit
                0x00000000       0x4e build/stm32f7xx_hal_tim.o
 .text.HAL_TIM_Encoder_MspInit
                0x00000000        0x2 build/stm32f7xx_hal_tim.o
 .text.HAL_TIM_Encoder_MspDeInit
                0x00000000        0x2 build/stm32f7xx_hal_tim.o
 .text.HAL_TIM_Encoder_DeInit
                0x00000000       0x4e build/stm32f7xx_hal_tim.o
 .text.HAL_TIM_DMABurst_MultiWriteStart
                0x00000000      0x1b4 build/stm32f7xx_hal_tim.o
 .text.HAL_TIM_DMABurst_WriteStart
                0x00000000       0x16 build/stm32f7xx_hal_tim.o
 .text.HAL_TIM_DMABurst_WriteStop
                0x00000000       0x84 build/stm32f7xx_hal_tim.o
 .text.HAL_TIM_DMABurst_MultiReadStart
                0x00000000      0x1b4 build/stm32f7xx_hal_tim.o
 .text.HAL_TIM_DMABurst_ReadStart
                0x00000000       0x16 build/stm32f7xx_hal_tim.o
 .text.HAL_TIM_DMABurst_ReadStop
                0x00000000       0x84 build/stm32f7xx_hal_tim.o
 .text.HAL_TIM_GenerateEvent
                0x00000000       0x2a build/stm32f7xx_hal_tim.o
 .text.HAL_TIM_ConfigTI1Input
                0x00000000       0x10 build/stm32f7xx_hal_tim.o
 .text.HAL_TIM_ReadCapturedValue
                0x00000000       0x32 build/stm32f7xx_hal_tim.o
 .text.TIM_DMAPeriodElapsedCplt
                0x00000000       0x16 build/stm32f7xx_hal_tim.o
 .text.HAL_TIM_PeriodElapsedHalfCpltCallback
                0x00000000        0x2 build/stm32f7xx_hal_tim.o
 .text.TIM_DMAPeriodElapsedHalfCplt
                0x00000000        0xa build/stm32f7xx_hal_tim.o
 .text.TIM_DMACaptureCplt
                0x00000000       0x80 build/stm32f7xx_hal_tim.o
 .text.HAL_TIM_IC_CaptureHalfCpltCallback
                0x00000000        0x2 build/stm32f7xx_hal_tim.o
 .text.TIM_DMACaptureHalfCplt
                0x00000000       0x3e build/stm32f7xx_hal_tim.o
 .text.TIM_DMADelayPulseCplt
                0x00000000       0x70 build/stm32f7xx_hal_tim.o
 .text.HAL_TIM_PWM_PulseFinishedHalfCpltCallback
                0x00000000        0x2 build/stm32f7xx_hal_tim.o
 .text.TIM_DMADelayPulseHalfCplt
                0x00000000       0x3e build/stm32f7xx_hal_tim.o
 .text.TIM_DMATriggerCplt
                0x00000000       0x16 build/stm32f7xx_hal_tim.o
 .text.HAL_TIM_TriggerHalfCpltCallback
                0x00000000        0x2 build/stm32f7xx_hal_tim.o
 .text.TIM_DMATriggerHalfCplt
                0x00000000        0xa build/stm32f7xx_hal_tim.o
 .text.HAL_TIM_ErrorCallback
                0x00000000        0x2 build/stm32f7xx_hal_tim.o
 .text.TIM_DMAError
                0x00000000       0x5c build/stm32f7xx_hal_tim.o
 .text.HAL_TIM_Base_GetState
                0x00000000        0x6 build/stm32f7xx_hal_tim.o
 .text.HAL_TIM_OC_GetState
                0x00000000        0x6 build/stm32f7xx_hal_tim.o
 .text.HAL_TIM_PWM_GetState
                0x00000000        0x6 build/stm32f7xx_hal_tim.o
 .text.HAL_TIM_IC_GetState
                0x00000000        0x6 build/stm32f7xx_hal_tim.o
 .text.HAL_TIM_OnePulse_GetState
                0x00000000        0x6 build/stm32f7xx_hal_tim.o
 .text.HAL_TIM_Encoder_GetState
                0x00000000        0x6 build/stm32f7xx_hal_tim.o
 .text.HAL_TIM_GetActiveChannel
                0x00000000        0x4 build/stm32f7xx_hal_tim.o
 .text.HAL_TIM_GetChannelState
                0x00000000       0x4a build/stm32f7xx_hal_tim.o
 .text.HAL_TIM_DMABurstState
                0x00000000        0x6 build/stm32f7xx_hal_tim.o
 .text.HAL_TIM_OC_Init
                0x00000000       0x60 build/stm32f7xx_hal_tim.o
 .text.HAL_TIM_IC_Init
                0x00000000       0x60 build/stm32f7xx_hal_tim.o
 .text.HAL_TIM_OnePulse_Init
                0x00000000       0x5c build/stm32f7xx_hal_tim.o
 .text.HAL_TIM_Encoder_Init
                0x00000000       0xb0 build/stm32f7xx_hal_tim.o
 .text.HAL_TIM_OC_ConfigChannel
                0x00000000       0x7a build/stm32f7xx_hal_tim.o
 .text.TIM_TI1_SetConfig
                0x00000000       0x94 build/stm32f7xx_hal_tim.o
 .text.HAL_TIM_IC_ConfigChannel
                0x00000000       0xcc build/stm32f7xx_hal_tim.o
 .text.HAL_TIM_OnePulse_ConfigChannel
                0x00000000      0x100 build/stm32f7xx_hal_tim.o
 .text.HAL_TIM_ConfigOCrefClear
                0x00000000      0x144 build/stm32f7xx_hal_tim.o
 .text.TIM_SlaveTimer_SetConfig
                0x00000000       0xbc build/stm32f7xx_hal_tim.o
 .text.HAL_TIM_SlaveConfigSynchro
                0x00000000       0x52 build/stm32f7xx_hal_tim.o
 .text.HAL_TIM_SlaveConfigSynchro_IT
                0x00000000       0x52 build/stm32f7xx_hal_tim.o
 .text.HAL_TIM_OC_Start
                0x00000000      0x158 build/stm32f7xx_hal_tim.o
 .text.HAL_TIM_OC_Stop
                0x00000000       0xac build/stm32f7xx_hal_tim.o
 .text.HAL_TIM_OC_Start_IT
                0x00000000      0x1c4 build/stm32f7xx_hal_tim.o
 .text.HAL_TIM_OC_Stop_IT
                0x00000000      0x100 build/stm32f7xx_hal_tim.o
 .text.HAL_TIM_OC_Start_DMA
                0x00000000      0x31c build/stm32f7xx_hal_tim.o
 .text.HAL_TIM_OC_Stop_DMA
                0x00000000      0x118 build/stm32f7xx_hal_tim.o
 .text.HAL_TIM_PWM_Start_IT
                0x00000000      0x1c4 build/stm32f7xx_hal_tim.o
 .text.HAL_TIM_PWM_Stop_IT
                0x00000000      0x100 build/stm32f7xx_hal_tim.o
 .text.HAL_TIM_PWM_Start_DMA
                0x00000000      0x31c build/stm32f7xx_hal_tim.o
 .text.HAL_TIM_PWM_Stop_DMA
                0x00000000      0x118 build/stm32f7xx_hal_tim.o
 .text.HAL_TIM_IC_Start
                0x00000000      0x168 build/stm32f7xx_hal_tim.o
 .text.HAL_TIM_IC_Stop
                0x00000000       0x9a build/stm32f7xx_hal_tim.o
 .text.HAL_TIM_IC_Start_IT
                0x00000000      0x1ac build/stm32f7xx_hal_tim.o
 .text.HAL_TIM_IC_Stop_IT
                0x00000000       0xea build/stm32f7xx_hal_tim.o
 .text.HAL_TIM_IC_Start_DMA
                0x00000000      0x27c build/stm32f7xx_hal_tim.o
 .text.HAL_TIM_IC_Stop_DMA
                0x00000000      0x100 build/stm32f7xx_hal_tim.o
 .text.HAL_TIM_OnePulse_Start
                0x00000000       0x84 build/stm32f7xx_hal_tim.o
 .text.HAL_TIM_OnePulse_Stop
                0x00000000       0x80 build/stm32f7xx_hal_tim.o
 .text.HAL_TIM_OnePulse_Start_IT
                0x00000000       0x98 build/stm32f7xx_hal_tim.o
 .text.HAL_TIM_OnePulse_Stop_IT
                0x00000000       0x94 build/stm32f7xx_hal_tim.o
 .text.HAL_TIM_Encoder_Start
                0x00000000       0xc8 build/stm32f7xx_hal_tim.o
 .text.HAL_TIM_Encoder_Stop
                0x00000000       0xe6 build/stm32f7xx_hal_tim.o
 .text.HAL_TIM_Encoder_Start_IT
                0x00000000       0xf4 build/stm32f7xx_hal_tim.o
 .text.HAL_TIM_Encoder_Stop_IT
                0x00000000      0x110 build/stm32f7xx_hal_tim.o
 .text.HAL_TIM_Encoder_Start_DMA
                0x00000000      0x24c build/stm32f7xx_hal_tim.o
 .text.HAL_TIM_Encoder_Stop_DMA
                0x00000000      0x128 build/stm32f7xx_hal_tim.o
 .text          0x00000000        0x0 build/stm32f7xx_hal_tim_ex.o
 .data          0x00000000        0x0 build/stm32f7xx_hal_tim_ex.o
 .bss           0x00000000        0x0 build/stm32f7xx_hal_tim_ex.o
 .text.TIM_CCxNChannelCmd
                0x00000000       0x1e build/stm32f7xx_hal_tim_ex.o
 .text.TIM_DMAErrorCCxN
                0x00000000       0x44 build/stm32f7xx_hal_tim_ex.o
 .text.TIM_DMADelayPulseNCplt
                0x00000000       0x58 build/stm32f7xx_hal_tim_ex.o
 .text.HAL_TIMEx_HallSensor_MspInit
                0x00000000        0x2 build/stm32f7xx_hal_tim_ex.o
 .text.HAL_TIMEx_HallSensor_Init
                0x00000000       0xd8 build/stm32f7xx_hal_tim_ex.o
 .text.HAL_TIMEx_HallSensor_MspDeInit
                0x00000000        0x2 build/stm32f7xx_hal_tim_ex.o
 .text.HAL_TIMEx_HallSensor_DeInit
                0x00000000       0x4e build/stm32f7xx_hal_tim_ex.o
 .text.HAL_TIMEx_HallSensor_Start
                0x00000000       0xc8 build/stm32f7xx_hal_tim_ex.o
 .text.HAL_TIMEx_HallSensor_Stop
                0x00000000       0x42 build/stm32f7xx_hal_tim_ex.o
 .text.HAL_TIMEx_HallSensor_Start_IT
                0x00000000       0xd4 build/stm32f7xx_hal_tim_ex.o
 .text.HAL_TIMEx_HallSensor_Stop_IT
                0x00000000       0x4c build/stm32f7xx_hal_tim_ex.o
 .text.HAL_TIMEx_HallSensor_Start_DMA
                0x00000000       0xfc build/stm32f7xx_hal_tim_ex.o
 .text.HAL_TIMEx_HallSensor_Stop_DMA
                0x00000000       0x4a build/stm32f7xx_hal_tim_ex.o
 .text.HAL_TIMEx_OCN_Start
                0x00000000      0x100 build/stm32f7xx_hal_tim_ex.o
 .text.HAL_TIMEx_OCN_Stop
                0x00000000       0x76 build/stm32f7xx_hal_tim_ex.o
 .text.HAL_TIMEx_OCN_Start_IT
                0x00000000      0x138 build/stm32f7xx_hal_tim_ex.o
 .text.HAL_TIMEx_OCN_Stop_IT
                0x00000000       0xc4 build/stm32f7xx_hal_tim_ex.o
 .text.HAL_TIMEx_OCN_Start_DMA
                0x00000000      0x22c build/stm32f7xx_hal_tim_ex.o
 .text.HAL_TIMEx_OCN_Stop_DMA
                0x00000000       0xc2 build/stm32f7xx_hal_tim_ex.o
 .text.HAL_TIMEx_PWMN_Start
                0x00000000      0x100 build/stm32f7xx_hal_tim_ex.o
 .text.HAL_TIMEx_PWMN_Stop
                0x00000000       0x76 build/stm32f7xx_hal_tim_ex.o
 .text.HAL_TIMEx_PWMN_Start_IT
                0x00000000      0x138 build/stm32f7xx_hal_tim_ex.o
 .text.HAL_TIMEx_PWMN_Stop_IT
                0x00000000       0xc4 build/stm32f7xx_hal_tim_ex.o
 .text.HAL_TIMEx_PWMN_Start_DMA
                0x00000000      0x22c build/stm32f7xx_hal_tim_ex.o
 .text.HAL_TIMEx_PWMN_Stop_DMA
                0x00000000       0xc2 build/stm32f7xx_hal_tim_ex.o
 .text.HAL_TIMEx_OnePulseN_Start
                0x00000000       0x7a build/stm32f7xx_hal_tim_ex.o
 .text.HAL_TIMEx_OnePulseN_Stop
                0x00000000       0x72 build/stm32f7xx_hal_tim_ex.o
 .text.HAL_TIMEx_OnePulseN_Start_IT
                0x00000000       0x90 build/stm32f7xx_hal_tim_ex.o
 .text.HAL_TIMEx_OnePulseN_Stop_IT
                0x00000000       0x86 build/stm32f7xx_hal_tim_ex.o
 .text.HAL_TIMEx_ConfigCommutEvent
                0x00000000       0x76 build/stm32f7xx_hal_tim_ex.o
 .text.HAL_TIMEx_ConfigCommutEvent_IT
                0x00000000       0x76 build/stm32f7xx_hal_tim_ex.o
 .text.HAL_TIMEx_ConfigCommutEvent_DMA
                0x00000000       0x94 build/stm32f7xx_hal_tim_ex.o
 .text.HAL_TIMEx_ConfigBreakDeadTime
                0x00000000       0x90 build/stm32f7xx_hal_tim_ex.o
 .text.HAL_TIMEx_ConfigBreakInput
                0x00000000       0xa4 build/stm32f7xx_hal_tim_ex.o
 .text.HAL_TIMEx_RemapConfig
                0x00000000       0x24 build/stm32f7xx_hal_tim_ex.o
 .text.HAL_TIMEx_GroupChannel5
                0x00000000       0x3e build/stm32f7xx_hal_tim_ex.o
 .text.TIMEx_DMACommutationCplt
                0x00000000       0x10 build/stm32f7xx_hal_tim_ex.o
 .text.HAL_TIMEx_CommutHalfCpltCallback
                0x00000000        0x2 build/stm32f7xx_hal_tim_ex.o
 .text.TIMEx_DMACommutationHalfCplt
                0x00000000       0x10 build/stm32f7xx_hal_tim_ex.o
 .text.HAL_TIMEx_HallSensor_GetState
                0x00000000        0x6 build/stm32f7xx_hal_tim_ex.o
 .text.HAL_TIMEx_GetChannelNState
                0x00000000       0x2a build/stm32f7xx_hal_tim_ex.o
 .text          0x00000000        0x0 build/stm32f7xx_ll_tim.o
 .data          0x00000000        0x0 build/stm32f7xx_ll_tim.o
 .bss           0x00000000        0x0 build/stm32f7xx_ll_tim.o
 .text.OC1Config
                0x00000000       0x78 build/stm32f7xx_ll_tim.o
 .text.OC2Config
                0x00000000       0x80 build/stm32f7xx_ll_tim.o
 .text.OC3Config
                0x00000000       0x7c build/stm32f7xx_ll_tim.o
 .text.OC4Config
                0x00000000       0x60 build/stm32f7xx_ll_tim.o
 .text.OC5Config
                0x00000000       0x60 build/stm32f7xx_ll_tim.o
 .text.OC6Config
                0x00000000       0x60 build/stm32f7xx_ll_tim.o
 .text.IC1Config
                0x00000000       0x38 build/stm32f7xx_ll_tim.o
 .text.IC2Config
                0x00000000       0x3a build/stm32f7xx_ll_tim.o
 .text.IC3Config
                0x00000000       0x3a build/stm32f7xx_ll_tim.o
 .text.IC4Config
                0x00000000       0x3a build/stm32f7xx_ll_tim.o
 .text.LL_TIM_DeInit
                0x00000000      0x1e8 build/stm32f7xx_ll_tim.o
 .text.LL_TIM_StructInit
                0x00000000       0x12 build/stm32f7xx_ll_tim.o
 .text.LL_TIM_OC_StructInit
                0x00000000       0x14 build/stm32f7xx_ll_tim.o
 .text.LL_TIM_OC_Init
                0x00000000       0x54 build/stm32f7xx_ll_tim.o
 .text.LL_TIM_IC_StructInit
                0x00000000       0x10 build/stm32f7xx_ll_tim.o
 .text.LL_TIM_IC_Init
                0x00000000       0x3c build/stm32f7xx_ll_tim.o
 .text.LL_TIM_ENCODER_StructInit
                0x00000000       0x1c build/stm32f7xx_ll_tim.o
 .text.LL_TIM_ENCODER_Init
                0x00000000       0x60 build/stm32f7xx_ll_tim.o
 .text.LL_TIM_HALLSENSOR_StructInit
                0x00000000        0xc build/stm32f7xx_ll_tim.o
 .text.LL_TIM_HALLSENSOR_Init
                0x00000000       0x60 build/stm32f7xx_ll_tim.o
 .text.LL_TIM_BDTR_StructInit
                0x00000000       0x1a build/stm32f7xx_ll_tim.o
 .text.LL_TIM_BDTR_Init
                0x00000000       0x70 build/stm32f7xx_ll_tim.o
 .text          0x00000000        0x0 build/stm32f7xx_ll_usart.o
 .data          0x00000000        0x0 build/stm32f7xx_ll_usart.o
 .bss           0x00000000        0x0 build/stm32f7xx_ll_usart.o
 .text.LL_USART_DeInit
                0x00000000      0x114 build/stm32f7xx_ll_usart.o
 .text.LL_USART_StructInit
                0x00000000       0x18 build/stm32f7xx_ll_usart.o
 .text.LL_USART_ClockInit
                0x00000000       0x3e build/stm32f7xx_ll_usart.o
 .text.LL_USART_ClockStructInit
                0x00000000        0xc build/stm32f7xx_ll_usart.o
 .text          0x00000000        0x0 build/system_stm32f7xx.o
 .data          0x00000000        0x0 build/system_stm32f7xx.o
 .bss           0x00000000        0x0 build/system_stm32f7xx.o
 .text.SystemCoreClockUpdate
                0x00000000       0xa0 build/system_stm32f7xx.o
 .text          0x00000000        0x0 build/File_Handling.o
 .data          0x00000000        0x0 build/File_Handling.o
 .bss           0x00000000        0x0 build/File_Handling.o
 .text.Send_Uart
                0x00000000        0x2 build/File_Handling.o
 .rodata.Scan_SD.str1.4
                0x00000000       0x29 build/File_Handling.o
 .text.Scan_SD  0x00000000       0xd4 build/File_Handling.o
 .rodata.Format_SD.str1.4
                0x00000000        0x2 build/File_Handling.o
 .text.Format_SD
                0x00000000       0x8c build/File_Handling.o
 .text.Write_File
                0x00000000       0x60 build/File_Handling.o
 .text.Read_File
                0x00000000      0x108 build/File_Handling.o
 .text.Update_File
                0x00000000       0x60 build/File_Handling.o
 .rodata.Create_Dir.str1.4
                0x00000000       0x4e build/File_Handling.o
 .text.Create_Dir
                0x00000000       0x54 build/File_Handling.o
 .rodata.Check_SD_Space.str1.4
                0x00000000       0x3a build/File_Handling.o
 .text.Check_SD_Space
                0x00000000       0xb0 build/File_Handling.o
 .text.Update_File_float
                0x00000000       0x5c build/File_Handling.o
 .bss.free_space
                0x00000000        0x4 build/File_Handling.o
 .bss.total     0x00000000        0x4 build/File_Handling.o
 .bss.fre_clust
                0x00000000        0x4 build/File_Handling.o
 .bss.pfs       0x00000000        0x4 build/File_Handling.o
 .text          0x00000000        0x0 build/diskio.o
 .data          0x00000000        0x0 build/diskio.o
 .bss           0x00000000        0x0 build/diskio.o
 .text.get_fattime
                0x00000000        0x4 build/diskio.o
 .text          0x00000000        0x0 build/ff.o
 .data          0x00000000        0x0 build/ff.o
 .bss           0x00000000        0x0 build/ff.o
 .text.putc_init
                0x00000000        0xa build/ff.o
 .text.putc_bfd
                0x00000000       0x4e build/ff.o
 .text.putc_flush
                0x00000000       0x3a build/ff.o
 .text.f_opendir
                0x00000000       0x8e build/ff.o
 .text.f_closedir
                0x00000000       0x24 build/ff.o
 .text.f_readdir
                0x00000000       0x4e build/ff.o
 .text.f_getfree
                0x00000000       0xde build/ff.o
 .text.f_truncate
                0x00000000       0xac build/ff.o
 .text.f_mkdir  0x00000000      0x162 build/ff.o
 .text.f_rename
                0x00000000      0x126 build/ff.o
 .rodata.f_mkfs.str1.4
                0x00000000       0x34 build/ff.o
 .text.f_mkfs   0x00000000      0x690 build/ff.o
 .text.f_gets   0x00000000       0x56 build/ff.o
 .text.f_putc   0x00000000       0x1e build/ff.o
 .text.f_puts   0x00000000       0x26 build/ff.o
 .text.f_printf
                0x00000000      0x244 build/ff.o
 .rodata.cst.0  0x00000000        0xe build/ff.o
 .rodata.cst32.1
                0x00000000        0xe build/ff.o
 .text          0x00000000        0x0 build/ff_gen_drv.o
 .data          0x00000000        0x0 build/ff_gen_drv.o
 .bss           0x00000000        0x0 build/ff_gen_drv.o
 .text.FATFS_UnLinkDriverEx
                0x00000000       0x3c build/ff_gen_drv.o
 .text.FATFS_UnLinkDriver
                0x00000000        0xa build/ff_gen_drv.o
 .text.FATFS_GetAttachedDriversNbr
                0x00000000        0xc build/ff_gen_drv.o
 .text          0x00000000        0x0 build/syscall.o
 .data          0x00000000        0x0 build/syscall.o
 .bss           0x00000000        0x0 build/syscall.o
 .debug_info    0x00000000      0x15d build/syscall.o
 .debug_abbrev  0x00000000       0x5f build/syscall.o
 .debug_aranges
                0x00000000       0x18 build/syscall.o
 .debug_line    0x00000000       0xec build/syscall.o
 .debug_str     0x00000000      0x242 build/syscall.o
 .comment       0x00000000       0x27 build/syscall.o
 .ARM.attributes
                0x00000000       0x32 build/syscall.o
 .text          0x00000000        0x0 build/sysmem.o
 .data          0x00000000        0x0 build/sysmem.o
 .bss           0x00000000        0x0 build/sysmem.o
 .text          0x00000000        0x0 build/syscalls.o
 .data          0x00000000        0x0 build/syscalls.o
 .bss           0x00000000        0x0 build/syscalls.o
 .text.initialise_monitor_handles
                0x00000000        0x2 build/syscalls.o
 .text._getpid  0x00000000        0x4 build/syscalls.o
 .text._kill    0x00000000       0x10 build/syscalls.o
 .text._exit    0x00000000        0xc build/syscalls.o
 .text._read    0x00000000       0x20 build/syscalls.o
 .text._write   0x00000000       0x1c build/syscalls.o
 .text._close   0x00000000        0x6 build/syscalls.o
 .text._fstat   0x00000000        0xa build/syscalls.o
 .text._isatty  0x00000000        0x4 build/syscalls.o
 .text._lseek   0x00000000        0x4 build/syscalls.o
 .text._open    0x00000000        0xa build/syscalls.o
 .text._wait    0x00000000       0x10 build/syscalls.o
 .text._unlink  0x00000000       0x10 build/syscalls.o
 .text._times   0x00000000        0x6 build/syscalls.o
 .text._stat    0x00000000        0xa build/syscalls.o
 .text._link    0x00000000       0x10 build/syscalls.o
 .text._fork    0x00000000       0x10 build/syscalls.o
 .text._execve  0x00000000       0x10 build/syscalls.o
 .data.environ  0x00000000        0x4 build/syscalls.o
 .bss.__env     0x00000000        0x4 build/syscalls.o
 .debug_info    0x00000000      0x848 build/syscalls.o
 .debug_abbrev  0x00000000      0x1e3 build/syscalls.o
 .debug_loc     0x00000000      0x583 build/syscalls.o
 .debug_aranges
                0x00000000       0xa8 build/syscalls.o
 .debug_ranges  0x00000000       0x98 build/syscalls.o
 .debug_line    0x00000000      0x36d build/syscalls.o
 .debug_str     0x00000000      0x3fc build/syscalls.o
 .comment       0x00000000       0x27 build/syscalls.o
 .debug_frame   0x00000000      0x190 build/syscalls.o
 .ARM.attributes
                0x00000000       0x32 build/syscalls.o
 .text          0x00000000        0x0 build/stm32f7xx_hal_uart.o
 .data          0x00000000        0x0 build/stm32f7xx_hal_uart.o
 .bss           0x00000000        0x0 build/stm32f7xx_hal_uart.o
 .text.UART_EndTxTransfer
                0x00000000       0x18 build/stm32f7xx_hal_uart.o
 .text.UART_TxISR_8BIT
                0x00000000       0x54 build/stm32f7xx_hal_uart.o
 .text.UART_TxISR_16BIT
                0x00000000       0x58 build/stm32f7xx_hal_uart.o
 .text.HAL_UART_MspInit
                0x00000000        0x2 build/stm32f7xx_hal_uart.o
 .text.HAL_UART_MspDeInit
                0x00000000        0x2 build/stm32f7xx_hal_uart.o
 .text.HAL_UART_DeInit
                0x00000000       0x40 build/stm32f7xx_hal_uart.o
 .text.HAL_UART_Transmit_IT
                0x00000000       0x64 build/stm32f7xx_hal_uart.o
 .text.HAL_UART_Transmit_DMA
                0x00000000       0x94 build/stm32f7xx_hal_uart.o
 .text.HAL_UART_DMAPause
                0x00000000       0x8a build/stm32f7xx_hal_uart.o
 .text.HAL_UART_DMAResume
                0x00000000       0x7a build/stm32f7xx_hal_uart.o
 .text.HAL_UART_DMAStop
                0x00000000       0xac build/stm32f7xx_hal_uart.o
 .text.HAL_UART_Abort
                0x00000000      0x100 build/stm32f7xx_hal_uart.o
 .text.HAL_UART_AbortTransmit
                0x00000000       0x68 build/stm32f7xx_hal_uart.o
 .text.HAL_UART_AbortReceive
                0x00000000       0xae build/stm32f7xx_hal_uart.o
 .text.HAL_UART_TxCpltCallback
                0x00000000        0x2 build/stm32f7xx_hal_uart.o
 .text.UART_DMATransmitCplt
                0x00000000       0x46 build/stm32f7xx_hal_uart.o
 .text.UART_EndTransmit_IT
                0x00000000       0x22 build/stm32f7xx_hal_uart.o
 .text.HAL_UART_TxHalfCpltCallback
                0x00000000        0x2 build/stm32f7xx_hal_uart.o
 .text.UART_DMATxHalfCplt
                0x00000000        0xa build/stm32f7xx_hal_uart.o
 .text.HAL_UART_RxCpltCallback
                0x00000000        0x2 build/stm32f7xx_hal_uart.o
 .text.HAL_UART_RxHalfCpltCallback
                0x00000000        0x2 build/stm32f7xx_hal_uart.o
 .text.HAL_UART_ErrorCallback
                0x00000000        0x2 build/stm32f7xx_hal_uart.o
 .text.UART_DMAError
                0x00000000       0x56 build/stm32f7xx_hal_uart.o
 .text.UART_DMAAbortOnError
                0x00000000       0x14 build/stm32f7xx_hal_uart.o
 .text.HAL_UART_AbortCpltCallback
                0x00000000        0x2 build/stm32f7xx_hal_uart.o
 .text.HAL_UART_Abort_IT
                0x00000000      0x130 build/stm32f7xx_hal_uart.o
 .text.UART_DMARxAbortCallback
                0x00000000       0x40 build/stm32f7xx_hal_uart.o
 .text.UART_DMATxAbortCallback
                0x00000000       0x36 build/stm32f7xx_hal_uart.o
 .text.HAL_UART_AbortTransmitCpltCallback
                0x00000000        0x2 build/stm32f7xx_hal_uart.o
 .text.HAL_UART_AbortTransmit_IT
                0x00000000       0x80 build/stm32f7xx_hal_uart.o
 .text.UART_DMATxOnlyAbortCallback
                0x00000000       0x14 build/stm32f7xx_hal_uart.o
 .text.HAL_UART_AbortReceiveCpltCallback
                0x00000000        0x2 build/stm32f7xx_hal_uart.o
 .text.HAL_UART_AbortReceive_IT
                0x00000000       0xcc build/stm32f7xx_hal_uart.o
 .text.UART_DMARxOnlyAbortCallback
                0x00000000       0x28 build/stm32f7xx_hal_uart.o
 .text.HAL_UARTEx_RxEventCallback
                0x00000000        0x2 build/stm32f7xx_hal_uart.o
 .text.UART_RxISR_8BIT
                0x00000000       0xd0 build/stm32f7xx_hal_uart.o
 .text.UART_RxISR_16BIT
                0x00000000       0xce build/stm32f7xx_hal_uart.o
 .text.UART_DMARxHalfCplt
                0x00000000       0x20 build/stm32f7xx_hal_uart.o
 .text.UART_DMAReceiveCplt
                0x00000000       0x90 build/stm32f7xx_hal_uart.o
 .text.HAL_UARTEx_WakeupCallback
                0x00000000        0x2 build/stm32f7xx_hal_uart.o
 .text.HAL_UART_IRQHandler
                0x00000000      0x2e8 build/stm32f7xx_hal_uart.o
 .text.HAL_UART_ReceiverTimeout_Config
                0x00000000        0xe build/stm32f7xx_hal_uart.o
 .text.HAL_UART_EnableReceiverTimeout
                0x00000000       0x38 build/stm32f7xx_hal_uart.o
 .text.HAL_UART_DisableReceiverTimeout
                0x00000000       0x38 build/stm32f7xx_hal_uart.o
 .text.HAL_MultiProcessor_EnterMuteMode
                0x00000000        0xc build/stm32f7xx_hal_uart.o
 .text.HAL_HalfDuplex_EnableTransmitter
                0x00000000       0x48 build/stm32f7xx_hal_uart.o
 .text.HAL_HalfDuplex_EnableReceiver
                0x00000000       0x48 build/stm32f7xx_hal_uart.o
 .text.HAL_LIN_SendBreak
                0x00000000       0x2e build/stm32f7xx_hal_uart.o
 .text.HAL_UART_GetState
                0x00000000        0xa build/stm32f7xx_hal_uart.o
 .text.HAL_UART_GetError
                0x00000000        0x6 build/stm32f7xx_hal_uart.o
 .text.HAL_UART_Transmit
                0x00000000       0xc6 build/stm32f7xx_hal_uart.o
 .text.HAL_UART_Receive
                0x00000000      0x116 build/stm32f7xx_hal_uart.o
 .text.HAL_HalfDuplex_Init
                0x00000000       0x6e build/stm32f7xx_hal_uart.o
 .text.HAL_LIN_Init
                0x00000000       0x92 build/stm32f7xx_hal_uart.o
 .text.HAL_MultiProcessor_Init
                0x00000000       0x8a build/stm32f7xx_hal_uart.o
 .text.HAL_MultiProcessor_EnableMuteMode
                0x00000000       0x34 build/stm32f7xx_hal_uart.o
 .text.HAL_MultiProcessor_DisableMuteMode
                0x00000000       0x34 build/stm32f7xx_hal_uart.o
 .text.UART_Start_Receive_IT
                0x00000000       0xd4 build/stm32f7xx_hal_uart.o
 .text.HAL_UART_Receive_IT
                0x00000000       0x40 build/stm32f7xx_hal_uart.o
 .text.UART_Start_Receive_DMA
                0x00000000       0xa8 build/stm32f7xx_hal_uart.o
 .text.HAL_UART_Receive_DMA
                0x00000000       0x40 build/stm32f7xx_hal_uart.o
 .text          0x00000000        0x0 build/stm32f7xx_hal_uart_ex.o
 .data          0x00000000        0x0 build/stm32f7xx_hal_uart_ex.o
 .bss           0x00000000        0x0 build/stm32f7xx_hal_uart_ex.o
 .text.UARTEx_Wakeup_AddressConfig
                0x00000000       0x2e build/stm32f7xx_hal_uart_ex.o
 .text.HAL_RS485Ex_Init
                0x00000000       0x7e build/stm32f7xx_hal_uart_ex.o
 .text.HAL_UARTEx_EnableClockStopMode
                0x00000000       0x34 build/stm32f7xx_hal_uart_ex.o
 .text.HAL_UARTEx_DisableClockStopMode
                0x00000000       0x34 build/stm32f7xx_hal_uart_ex.o
 .text.HAL_MultiProcessorEx_AddressLength_Set
                0x00000000       0x36 build/stm32f7xx_hal_uart_ex.o
 .text.HAL_UARTEx_StopModeWakeUpSourceConfig
                0x00000000       0x7e build/stm32f7xx_hal_uart_ex.o
 .text.HAL_UARTEx_EnableStopMode
                0x00000000       0x2e build/stm32f7xx_hal_uart_ex.o
 .text.HAL_UARTEx_DisableStopMode
                0x00000000       0x2e build/stm32f7xx_hal_uart_ex.o
 .text.HAL_UARTEx_ReceiveToIdle
                0x00000000      0x15e build/stm32f7xx_hal_uart_ex.o
 .text.HAL_UARTEx_ReceiveToIdle_IT
                0x00000000       0x4e build/stm32f7xx_hal_uart_ex.o
 .text.HAL_UARTEx_ReceiveToIdle_DMA
                0x00000000       0x50 build/stm32f7xx_hal_uart_ex.o
 .text.HAL_UARTEx_GetRxEventType
                0x00000000        0x4 build/stm32f7xx_hal_uart_ex.o
 .debug_info    0x00000000     0x119b build/stm32f7xx_hal_uart_ex.o
 .debug_abbrev  0x00000000      0x301 build/stm32f7xx_hal_uart_ex.o
 .debug_loc     0x00000000      0xd8a build/stm32f7xx_hal_uart_ex.o
 .debug_aranges
                0x00000000       0x78 build/stm32f7xx_hal_uart_ex.o
 .debug_ranges  0x00000000       0x80 build/stm32f7xx_hal_uart_ex.o
 .debug_line    0x00000000      0x8e1 build/stm32f7xx_hal_uart_ex.o
 .debug_str     0x00000000      0x970 build/stm32f7xx_hal_uart_ex.o
 .comment       0x00000000       0x27 build/stm32f7xx_hal_uart_ex.o
 .debug_frame   0x00000000      0x138 build/stm32f7xx_hal_uart_ex.o
 .ARM.attributes
                0x00000000       0x32 build/stm32f7xx_hal_uart_ex.o
 .text          0x00000000       0x14 build/startup_stm32f767xx.o
 .data          0x00000000        0x0 build/startup_stm32f767xx.o
 .bss           0x00000000        0x0 build/startup_stm32f767xx.o
 .data          0x00000000        0x0 /usr/lib/gcc/arm-none-eabi/13.2.1/../../../arm-none-eabi/lib/thumb/v7e-m+dp/hard/libc_nano.a(libc_a-sprintf.o)
 .bss           0x00000000        0x0 /usr/lib/gcc/arm-none-eabi/13.2.1/../../../arm-none-eabi/lib/thumb/v7e-m+dp/hard/libc_nano.a(libc_a-sprintf.o)
 .text          0x00000000       0xbc /usr/lib/gcc/arm-none-eabi/13.2.1/../../../arm-none-eabi/lib/thumb/v7e-m+dp/hard/libc_nano.a(libc_a-strcpy.o)
 .data          0x00000000        0x0 /usr/lib/gcc/arm-none-eabi/13.2.1/../../../arm-none-eabi/lib/thumb/v7e-m+dp/hard/libc_nano.a(libc_a-strcpy.o)
 .bss           0x00000000        0x0 /usr/lib/gcc/arm-none-eabi/13.2.1/../../../arm-none-eabi/lib/thumb/v7e-m+dp/hard/libc_nano.a(libc_a-strcpy.o)
 .debug_info    0x00000000       0xc3 /usr/lib/gcc/arm-none-eabi/13.2.1/../../../arm-none-eabi/lib/thumb/v7e-m+dp/hard/libc_nano.a(libc_a-strcpy.o)
 .debug_abbrev  0x00000000       0x7b /usr/lib/gcc/arm-none-eabi/13.2.1/../../../arm-none-eabi/lib/thumb/v7e-m+dp/hard/libc_nano.a(libc_a-strcpy.o)
 .debug_loclists
                0x00000000       0x2c /usr/lib/gcc/arm-none-eabi/13.2.1/../../../arm-none-eabi/lib/thumb/v7e-m+dp/hard/libc_nano.a(libc_a-strcpy.o)
 .debug_aranges
                0x00000000       0x20 /usr/lib/gcc/arm-none-eabi/13.2.1/../../../arm-none-eabi/lib/thumb/v7e-m+dp/hard/libc_nano.a(libc_a-strcpy.o)
 .debug_rnglists
                0x00000000       0x14 /usr/lib/gcc/arm-none-eabi/13.2.1/../../../arm-none-eabi/lib/thumb/v7e-m+dp/hard/libc_nano.a(libc_a-strcpy.o)
 .debug_line    0x00000000       0xb9 /usr/lib/gcc/arm-none-eabi/13.2.1/../../../arm-none-eabi/lib/thumb/v7e-m+dp/hard/libc_nano.a(libc_a-strcpy.o)
 .debug_str     0x00000000      0x19a /usr/lib/gcc/arm-none-eabi/13.2.1/../../../arm-none-eabi/lib/thumb/v7e-m+dp/hard/libc_nano.a(libc_a-strcpy.o)
 .comment       0x00000000       0x27 /usr/lib/gcc/arm-none-eabi/13.2.1/../../../arm-none-eabi/lib/thumb/v7e-m+dp/hard/libc_nano.a(libc_a-strcpy.o)
 .debug_frame   0x00000000       0x20 /usr/lib/gcc/arm-none-eabi/13.2.1/../../../arm-none-eabi/lib/thumb/v7e-m+dp/hard/libc_nano.a(libc_a-strcpy.o)
 .ARM.attributes
                0x00000000       0x32 /usr/lib/gcc/arm-none-eabi/13.2.1/../../../arm-none-eabi/lib/thumb/v7e-m+dp/hard/libc_nano.a(libc_a-strcpy.o)
 .text          0x00000000        0x0 /usr/lib/gcc/arm-none-eabi/13.2.1/../../../arm-none-eabi/lib/thumb/v7e-m+dp/hard/libc_nano.a(libc_a-impure.o)
 .bss           0x00000000        0x0 /usr/lib/gcc/arm-none-eabi/13.2.1/../../../arm-none-eabi/lib/thumb/v7e-m+dp/hard/libc_nano.a(libc_a-impure.o)
 .data          0x00000000        0x0 /usr/lib/gcc/arm-none-eabi/13.2.1/../../../arm-none-eabi/lib/thumb/v7e-m+dp/hard/libc_nano.a(libc_a-nano-svfprintf.o)
 .bss           0x00000000        0x0 /usr/lib/gcc/arm-none-eabi/13.2.1/../../../arm-none-eabi/lib/thumb/v7e-m+dp/hard/libc_nano.a(libc_a-nano-svfprintf.o)
 .data          0x00000000        0x0 /usr/lib/gcc/arm-none-eabi/13.2.1/../../../arm-none-eabi/lib/thumb/v7e-m+dp/hard/libc_nano.a(libc_a-init.o)
 .bss           0x00000000        0x0 /usr/lib/gcc/arm-none-eabi/13.2.1/../../../arm-none-eabi/lib/thumb/v7e-m+dp/hard/libc_nano.a(libc_a-init.o)
 .text          0x00000000       0xd8 /usr/lib/gcc/arm-none-eabi/13.2.1/../../../arm-none-eabi/lib/thumb/v7e-m+dp/hard/libc_nano.a(libc_a-strlen.o)
 .data          0x00000000        0x0 /usr/lib/gcc/arm-none-eabi/13.2.1/../../../arm-none-eabi/lib/thumb/v7e-m+dp/hard/libc_nano.a(libc_a-strlen.o)
 .bss           0x00000000        0x0 /usr/lib/gcc/arm-none-eabi/13.2.1/../../../arm-none-eabi/lib/thumb/v7e-m+dp/hard/libc_nano.a(libc_a-strlen.o)
 .ARM.extab     0x00000000        0x0 /usr/lib/gcc/arm-none-eabi/13.2.1/../../../arm-none-eabi/lib/thumb/v7e-m+dp/hard/libc_nano.a(libc_a-strlen.o)
 .ARM.exidx     0x00000000        0x8 /usr/lib/gcc/arm-none-eabi/13.2.1/../../../arm-none-eabi/lib/thumb/v7e-m+dp/hard/libc_nano.a(libc_a-strlen.o)
 .debug_line    0x00000000       0x86 /usr/lib/gcc/arm-none-eabi/13.2.1/../../../arm-none-eabi/lib/thumb/v7e-m+dp/hard/libc_nano.a(libc_a-strlen.o)
 .debug_line_str
                0x00000000       0x98 /usr/lib/gcc/arm-none-eabi/13.2.1/../../../arm-none-eabi/lib/thumb/v7e-m+dp/hard/libc_nano.a(libc_a-strlen.o)
 .debug_info    0x00000000       0x33 /usr/lib/gcc/arm-none-eabi/13.2.1/../../../arm-none-eabi/lib/thumb/v7e-m+dp/hard/libc_nano.a(libc_a-strlen.o)
 .debug_abbrev  0x00000000       0x28 /usr/lib/gcc/arm-none-eabi/13.2.1/../../../arm-none-eabi/lib/thumb/v7e-m+dp/hard/libc_nano.a(libc_a-strlen.o)
 .debug_aranges
                0x00000000       0x20 /usr/lib/gcc/arm-none-eabi/13.2.1/../../../arm-none-eabi/lib/thumb/v7e-m+dp/hard/libc_nano.a(libc_a-strlen.o)
 .debug_str     0x00000000       0xab /usr/lib/gcc/arm-none-eabi/13.2.1/../../../arm-none-eabi/lib/thumb/v7e-m+dp/hard/libc_nano.a(libc_a-strlen.o)
 .eh_frame      0x00000000       0x34 /usr/lib/gcc/arm-none-eabi/13.2.1/../../../arm-none-eabi/lib/thumb/v7e-m+dp/hard/libc_nano.a(libc_a-strlen.o)
 .ARM.attributes
                0x00000000       0x1c /usr/lib/gcc/arm-none-eabi/13.2.1/../../../arm-none-eabi/lib/thumb/v7e-m+dp/hard/libc_nano.a(libc_a-strlen.o)
 .data          0x00000000        0x0 /usr/lib/gcc/arm-none-eabi/13.2.1/../../../arm-none-eabi/lib/thumb/v7e-m+dp/hard/libc_nano.a(libc_a-memset.o)
 .bss           0x00000000        0x0 /usr/lib/gcc/arm-none-eabi/13.2.1/../../../arm-none-eabi/lib/thumb/v7e-m+dp/hard/libc_nano.a(libc_a-memset.o)
 .data          0x00000000        0x0 /usr/lib/gcc/arm-none-eabi/13.2.1/../../../arm-none-eabi/lib/thumb/v7e-m+dp/hard/libc_nano.a(libc_a-errno.o)
 .bss           0x00000000        0x0 /usr/lib/gcc/arm-none-eabi/13.2.1/../../../arm-none-eabi/lib/thumb/v7e-m+dp/hard/libc_nano.a(libc_a-errno.o)
 .data          0x00000000        0x0 /usr/lib/gcc/arm-none-eabi/13.2.1/../../../arm-none-eabi/lib/thumb/v7e-m+dp/hard/libc_nano.a(libc_a-mallocr.o)
 .data          0x00000000        0x0 /usr/lib/gcc/arm-none-eabi/13.2.1/../../../arm-none-eabi/lib/thumb/v7e-m+dp/hard/libc_nano.a(libc_a-freer.o)
 .bss           0x00000000        0x0 /usr/lib/gcc/arm-none-eabi/13.2.1/../../../arm-none-eabi/lib/thumb/v7e-m+dp/hard/libc_nano.a(libc_a-freer.o)
 .data          0x00000000        0x0 /usr/lib/gcc/arm-none-eabi/13.2.1/../../../arm-none-eabi/lib/thumb/v7e-m+dp/hard/libc_nano.a(libc_a-memmove.o)
 .bss           0x00000000        0x0 /usr/lib/gcc/arm-none-eabi/13.2.1/../../../arm-none-eabi/lib/thumb/v7e-m+dp/hard/libc_nano.a(libc_a-memmove.o)
 .data          0x00000000        0x0 /usr/lib/gcc/arm-none-eabi/13.2.1/../../../arm-none-eabi/lib/thumb/v7e-m+dp/hard/libc_nano.a(libc_a-memchr.o)
 .bss           0x00000000        0x0 /usr/lib/gcc/arm-none-eabi/13.2.1/../../../arm-none-eabi/lib/thumb/v7e-m+dp/hard/libc_nano.a(libc_a-memchr.o)
 .ARM.extab     0x00000000        0x0 /usr/lib/gcc/arm-none-eabi/13.2.1/../../../arm-none-eabi/lib/thumb/v7e-m+dp/hard/libc_nano.a(libc_a-memchr.o)
 .eh_frame      0x00000000       0x50 /usr/lib/gcc/arm-none-eabi/13.2.1/../../../arm-none-eabi/lib/thumb/v7e-m+dp/hard/libc_nano.a(libc_a-memchr.o)
 .data          0x00000000        0x0 /usr/lib/gcc/arm-none-eabi/13.2.1/../../../arm-none-eabi/lib/thumb/v7e-m+dp/hard/libc_nano.a(libc_a-memcpy.o)
 .bss           0x00000000        0x0 /usr/lib/gcc/arm-none-eabi/13.2.1/../../../arm-none-eabi/lib/thumb/v7e-m+dp/hard/libc_nano.a(libc_a-memcpy.o)
 .ARM.extab     0x00000000        0x0 /usr/lib/gcc/arm-none-eabi/13.2.1/../../../arm-none-eabi/lib/thumb/v7e-m+dp/hard/libc_nano.a(libc_a-memcpy.o)
 .eh_frame      0x00000000       0x2c /usr/lib/gcc/arm-none-eabi/13.2.1/../../../arm-none-eabi/lib/thumb/v7e-m+dp/hard/libc_nano.a(libc_a-memcpy.o)
 .data          0x00000000        0x0 /usr/lib/gcc/arm-none-eabi/13.2.1/../../../arm-none-eabi/lib/thumb/v7e-m+dp/hard/libc_nano.a(libc_a-malloc.o)
 .bss           0x00000000        0x0 /usr/lib/gcc/arm-none-eabi/13.2.1/../../../arm-none-eabi/lib/thumb/v7e-m+dp/hard/libc_nano.a(libc_a-malloc.o)
 .data          0x00000000        0x0 /usr/lib/gcc/arm-none-eabi/13.2.1/../../../arm-none-eabi/lib/thumb/v7e-m+dp/hard/libc_nano.a(libc_a-reallocr.o)
 .bss           0x00000000        0x0 /usr/lib/gcc/arm-none-eabi/13.2.1/../../../arm-none-eabi/lib/thumb/v7e-m+dp/hard/libc_nano.a(libc_a-reallocr.o)
 .data          0x00000000        0x0 /usr/lib/gcc/arm-none-eabi/13.2.1/../../../arm-none-eabi/lib/thumb/v7e-m+dp/hard/libc_nano.a(libc_a-nano-vfprintf_i.o)
 .bss           0x00000000        0x0 /usr/lib/gcc/arm-none-eabi/13.2.1/../../../arm-none-eabi/lib/thumb/v7e-m+dp/hard/libc_nano.a(libc_a-nano-vfprintf_i.o)
 .data          0x00000000        0x0 /usr/lib/gcc/arm-none-eabi/13.2.1/../../../arm-none-eabi/lib/thumb/v7e-m+dp/hard/libc_nano.a(libc_a-mlock.o)
 .bss           0x00000000        0x0 /usr/lib/gcc/arm-none-eabi/13.2.1/../../../arm-none-eabi/lib/thumb/v7e-m+dp/hard/libc_nano.a(libc_a-mlock.o)
 .text          0x00000000      0x2e0 /usr/lib/gcc/arm-none-eabi/13.2.1/../../../arm-none-eabi/lib/thumb/v7e-m+dp/hard/libc_nano.a(libc_a-strcmp.o)
 .data          0x00000000        0x0 /usr/lib/gcc/arm-none-eabi/13.2.1/../../../arm-none-eabi/lib/thumb/v7e-m+dp/hard/libc_nano.a(libc_a-strcmp.o)
 .bss           0x00000000        0x0 /usr/lib/gcc/arm-none-eabi/13.2.1/../../../arm-none-eabi/lib/thumb/v7e-m+dp/hard/libc_nano.a(libc_a-strcmp.o)
 .ARM.extab     0x00000000        0x0 /usr/lib/gcc/arm-none-eabi/13.2.1/../../../arm-none-eabi/lib/thumb/v7e-m+dp/hard/libc_nano.a(libc_a-strcmp.o)
 .ARM.exidx     0x00000000        0x8 /usr/lib/gcc/arm-none-eabi/13.2.1/../../../arm-none-eabi/lib/thumb/v7e-m+dp/hard/libc_nano.a(libc_a-strcmp.o)
 .debug_line    0x00000000      0x10e /usr/lib/gcc/arm-none-eabi/13.2.1/../../../arm-none-eabi/lib/thumb/v7e-m+dp/hard/libc_nano.a(libc_a-strcmp.o)
 .debug_line_str
                0x00000000       0x98 /usr/lib/gcc/arm-none-eabi/13.2.1/../../../arm-none-eabi/lib/thumb/v7e-m+dp/hard/libc_nano.a(libc_a-strcmp.o)
 .debug_info    0x00000000       0x33 /usr/lib/gcc/arm-none-eabi/13.2.1/../../../arm-none-eabi/lib/thumb/v7e-m+dp/hard/libc_nano.a(libc_a-strcmp.o)
 .debug_abbrev  0x00000000       0x28 /usr/lib/gcc/arm-none-eabi/13.2.1/../../../arm-none-eabi/lib/thumb/v7e-m+dp/hard/libc_nano.a(libc_a-strcmp.o)
 .debug_aranges
                0x00000000       0x20 /usr/lib/gcc/arm-none-eabi/13.2.1/../../../arm-none-eabi/lib/thumb/v7e-m+dp/hard/libc_nano.a(libc_a-strcmp.o)
 .debug_str     0x00000000       0xab /usr/lib/gcc/arm-none-eabi/13.2.1/../../../arm-none-eabi/lib/thumb/v7e-m+dp/hard/libc_nano.a(libc_a-strcmp.o)
 .debug_frame   0x00000000       0x7c /usr/lib/gcc/arm-none-eabi/13.2.1/../../../arm-none-eabi/lib/thumb/v7e-m+dp/hard/libc_nano.a(libc_a-strcmp.o)
 .ARM.attributes
                0x00000000       0x1e /usr/lib/gcc/arm-none-eabi/13.2.1/../../../arm-none-eabi/lib/thumb/v7e-m+dp/hard/libc_nano.a(libc_a-strcmp.o)
 .text          0x00000000       0x24 /usr/lib/gcc/arm-none-eabi/13.2.1/../../../arm-none-eabi/lib/thumb/v7e-m+dp/hard/libc_nano.a(libc_a-exit.o)
 .data          0x00000000        0x0 /usr/lib/gcc/arm-none-eabi/13.2.1/../../../arm-none-eabi/lib/thumb/v7e-m+dp/hard/libc_nano.a(libc_a-exit.o)
 .bss           0x00000000        0x0 /usr/lib/gcc/arm-none-eabi/13.2.1/../../../arm-none-eabi/lib/thumb/v7e-m+dp/hard/libc_nano.a(libc_a-exit.o)
 .debug_info    0x00000000      0x11b /usr/lib/gcc/arm-none-eabi/13.2.1/../../../arm-none-eabi/lib/thumb/v7e-m+dp/hard/libc_nano.a(libc_a-exit.o)
 .debug_abbrev  0x00000000       0xd8 /usr/lib/gcc/arm-none-eabi/13.2.1/../../../arm-none-eabi/lib/thumb/v7e-m+dp/hard/libc_nano.a(libc_a-exit.o)
 .debug_loclists
                0x00000000       0x1b /usr/lib/gcc/arm-none-eabi/13.2.1/../../../arm-none-eabi/lib/thumb/v7e-m+dp/hard/libc_nano.a(libc_a-exit.o)
 .debug_aranges
                0x00000000       0x20 /usr/lib/gcc/arm-none-eabi/13.2.1/../../../arm-none-eabi/lib/thumb/v7e-m+dp/hard/libc_nano.a(libc_a-exit.o)
 .debug_line    0x00000000      0x12d /usr/lib/gcc/arm-none-eabi/13.2.1/../../../arm-none-eabi/lib/thumb/v7e-m+dp/hard/libc_nano.a(libc_a-exit.o)
 .debug_str     0x00000000      0x1c2 /usr/lib/gcc/arm-none-eabi/13.2.1/../../../arm-none-eabi/lib/thumb/v7e-m+dp/hard/libc_nano.a(libc_a-exit.o)
 .comment       0x00000000       0x27 /usr/lib/gcc/arm-none-eabi/13.2.1/../../../arm-none-eabi/lib/thumb/v7e-m+dp/hard/libc_nano.a(libc_a-exit.o)
 .debug_frame   0x00000000       0x28 /usr/lib/gcc/arm-none-eabi/13.2.1/../../../arm-none-eabi/lib/thumb/v7e-m+dp/hard/libc_nano.a(libc_a-exit.o)
 .ARM.attributes
                0x00000000       0x32 /usr/lib/gcc/arm-none-eabi/13.2.1/../../../arm-none-eabi/lib/thumb/v7e-m+dp/hard/libc_nano.a(libc_a-exit.o)
 .text          0x00000000        0xc /usr/lib/gcc/arm-none-eabi/13.2.1/../../../arm-none-eabi/lib/thumb/v7e-m+dp/hard/libc_nano.a(libc_a-atexit.o)
 .data          0x00000000        0x0 /usr/lib/gcc/arm-none-eabi/13.2.1/../../../arm-none-eabi/lib/thumb/v7e-m+dp/hard/libc_nano.a(libc_a-atexit.o)
 .bss           0x00000000        0x0 /usr/lib/gcc/arm-none-eabi/13.2.1/../../../arm-none-eabi/lib/thumb/v7e-m+dp/hard/libc_nano.a(libc_a-atexit.o)
 .debug_info    0x00000000      0x11e /usr/lib/gcc/arm-none-eabi/13.2.1/../../../arm-none-eabi/lib/thumb/v7e-m+dp/hard/libc_nano.a(libc_a-atexit.o)
 .debug_abbrev  0x00000000       0xc1 /usr/lib/gcc/arm-none-eabi/13.2.1/../../../arm-none-eabi/lib/thumb/v7e-m+dp/hard/libc_nano.a(libc_a-atexit.o)
 .debug_loclists
                0x00000000       0x2b /usr/lib/gcc/arm-none-eabi/13.2.1/../../../arm-none-eabi/lib/thumb/v7e-m+dp/hard/libc_nano.a(libc_a-atexit.o)
 .debug_aranges
                0x00000000       0x20 /usr/lib/gcc/arm-none-eabi/13.2.1/../../../arm-none-eabi/lib/thumb/v7e-m+dp/hard/libc_nano.a(libc_a-atexit.o)
 .debug_line    0x00000000       0xc3 /usr/lib/gcc/arm-none-eabi/13.2.1/../../../arm-none-eabi/lib/thumb/v7e-m+dp/hard/libc_nano.a(libc_a-atexit.o)
 .debug_str     0x00000000      0x1d9 /usr/lib/gcc/arm-none-eabi/13.2.1/../../../arm-none-eabi/lib/thumb/v7e-m+dp/hard/libc_nano.a(libc_a-atexit.o)
 .comment       0x00000000       0x27 /usr/lib/gcc/arm-none-eabi/13.2.1/../../../arm-none-eabi/lib/thumb/v7e-m+dp/hard/libc_nano.a(libc_a-atexit.o)
 .debug_frame   0x00000000       0x20 /usr/lib/gcc/arm-none-eabi/13.2.1/../../../arm-none-eabi/lib/thumb/v7e-m+dp/hard/libc_nano.a(libc_a-atexit.o)
 .ARM.attributes
                0x00000000       0x32 /usr/lib/gcc/arm-none-eabi/13.2.1/../../../arm-none-eabi/lib/thumb/v7e-m+dp/hard/libc_nano.a(libc_a-atexit.o)
 .text          0x00000000       0x28 /usr/lib/gcc/arm-none-eabi/13.2.1/../../../arm-none-eabi/lib/thumb/v7e-m+dp/hard/libc_nano.a(libc_a-fini.o)
 .data          0x00000000        0x0 /usr/lib/gcc/arm-none-eabi/13.2.1/../../../arm-none-eabi/lib/thumb/v7e-m+dp/hard/libc_nano.a(libc_a-fini.o)
 .bss           0x00000000        0x0 /usr/lib/gcc/arm-none-eabi/13.2.1/../../../arm-none-eabi/lib/thumb/v7e-m+dp/hard/libc_nano.a(libc_a-fini.o)
 .debug_info    0x00000000       0xf7 /usr/lib/gcc/arm-none-eabi/13.2.1/../../../arm-none-eabi/lib/thumb/v7e-m+dp/hard/libc_nano.a(libc_a-fini.o)
 .debug_abbrev  0x00000000       0xcc /usr/lib/gcc/arm-none-eabi/13.2.1/../../../arm-none-eabi/lib/thumb/v7e-m+dp/hard/libc_nano.a(libc_a-fini.o)
 .debug_loclists
                0x00000000       0x42 /usr/lib/gcc/arm-none-eabi/13.2.1/../../../arm-none-eabi/lib/thumb/v7e-m+dp/hard/libc_nano.a(libc_a-fini.o)
 .debug_aranges
                0x00000000       0x20 /usr/lib/gcc/arm-none-eabi/13.2.1/../../../arm-none-eabi/lib/thumb/v7e-m+dp/hard/libc_nano.a(libc_a-fini.o)
 .debug_line    0x00000000       0xd2 /usr/lib/gcc/arm-none-eabi/13.2.1/../../../arm-none-eabi/lib/thumb/v7e-m+dp/hard/libc_nano.a(libc_a-fini.o)
 .debug_str     0x00000000      0x1d3 /usr/lib/gcc/arm-none-eabi/13.2.1/../../../arm-none-eabi/lib/thumb/v7e-m+dp/hard/libc_nano.a(libc_a-fini.o)
 .comment       0x00000000       0x27 /usr/lib/gcc/arm-none-eabi/13.2.1/../../../arm-none-eabi/lib/thumb/v7e-m+dp/hard/libc_nano.a(libc_a-fini.o)
 .debug_frame   0x00000000       0x34 /usr/lib/gcc/arm-none-eabi/13.2.1/../../../arm-none-eabi/lib/thumb/v7e-m+dp/hard/libc_nano.a(libc_a-fini.o)
 .ARM.attributes
                0x00000000       0x32 /usr/lib/gcc/arm-none-eabi/13.2.1/../../../arm-none-eabi/lib/thumb/v7e-m+dp/hard/libc_nano.a(libc_a-fini.o)
 .data          0x00000000        0x0 /usr/lib/gcc/arm-none-eabi/13.2.1/../../../arm-none-eabi/lib/thumb/v7e-m+dp/hard/libc_nano.a(libc_a-sbrkr.o)
 .bss           0x00000000        0x0 /usr/lib/gcc/arm-none-eabi/13.2.1/../../../arm-none-eabi/lib/thumb/v7e-m+dp/hard/libc_nano.a(libc_a-sbrkr.o)
 .data          0x00000000        0x0 /usr/lib/gcc/arm-none-eabi/13.2.1/../../../arm-none-eabi/lib/thumb/v7e-m+dp/hard/libc_nano.a(libc_a-msizer.o)
 .bss           0x00000000        0x0 /usr/lib/gcc/arm-none-eabi/13.2.1/../../../arm-none-eabi/lib/thumb/v7e-m+dp/hard/libc_nano.a(libc_a-msizer.o)
 .text          0x00000000      0x224 /usr/lib/gcc/arm-none-eabi/13.2.1/../../../arm-none-eabi/lib/thumb/v7e-m+dp/hard/libc_nano.a(libc_a-findfp.o)
 .data          0x00000000        0xc /usr/lib/gcc/arm-none-eabi/13.2.1/../../../arm-none-eabi/lib/thumb/v7e-m+dp/hard/libc_nano.a(libc_a-findfp.o)
 .text          0x00000000      0x1a8 /usr/lib/gcc/arm-none-eabi/13.2.1/../../../arm-none-eabi/lib/thumb/v7e-m+dp/hard/libc_nano.a(libc_a-fflush.o)
 .data          0x00000000        0x0 /usr/lib/gcc/arm-none-eabi/13.2.1/../../../arm-none-eabi/lib/thumb/v7e-m+dp/hard/libc_nano.a(libc_a-fflush.o)
 .bss           0x00000000        0x0 /usr/lib/gcc/arm-none-eabi/13.2.1/../../../arm-none-eabi/lib/thumb/v7e-m+dp/hard/libc_nano.a(libc_a-fflush.o)
 .debug_info    0x00000000      0xa33 /usr/lib/gcc/arm-none-eabi/13.2.1/../../../arm-none-eabi/lib/thumb/v7e-m+dp/hard/libc_nano.a(libc_a-fflush.o)
 .debug_abbrev  0x00000000      0x2e4 /usr/lib/gcc/arm-none-eabi/13.2.1/../../../arm-none-eabi/lib/thumb/v7e-m+dp/hard/libc_nano.a(libc_a-fflush.o)
 .debug_loclists
                0x00000000      0x2f3 /usr/lib/gcc/arm-none-eabi/13.2.1/../../../arm-none-eabi/lib/thumb/v7e-m+dp/hard/libc_nano.a(libc_a-fflush.o)
 .debug_aranges
                0x00000000       0x20 /usr/lib/gcc/arm-none-eabi/13.2.1/../../../arm-none-eabi/lib/thumb/v7e-m+dp/hard/libc_nano.a(libc_a-fflush.o)
 .debug_rnglists
                0x00000000       0x59 /usr/lib/gcc/arm-none-eabi/13.2.1/../../../arm-none-eabi/lib/thumb/v7e-m+dp/hard/libc_nano.a(libc_a-fflush.o)
 .debug_line    0x00000000      0x446 /usr/lib/gcc/arm-none-eabi/13.2.1/../../../arm-none-eabi/lib/thumb/v7e-m+dp/hard/libc_nano.a(libc_a-fflush.o)
 .debug_str     0x00000000      0x546 /usr/lib/gcc/arm-none-eabi/13.2.1/../../../arm-none-eabi/lib/thumb/v7e-m+dp/hard/libc_nano.a(libc_a-fflush.o)
 .comment       0x00000000       0x27 /usr/lib/gcc/arm-none-eabi/13.2.1/../../../arm-none-eabi/lib/thumb/v7e-m+dp/hard/libc_nano.a(libc_a-fflush.o)
 .debug_frame   0x00000000       0x8c /usr/lib/gcc/arm-none-eabi/13.2.1/../../../arm-none-eabi/lib/thumb/v7e-m+dp/hard/libc_nano.a(libc_a-fflush.o)
 .ARM.attributes
                0x00000000       0x32 /usr/lib/gcc/arm-none-eabi/13.2.1/../../../arm-none-eabi/lib/thumb/v7e-m+dp/hard/libc_nano.a(libc_a-fflush.o)
 .text          0x00000000       0x44 /usr/lib/gcc/arm-none-eabi/13.2.1/../../../arm-none-eabi/lib/thumb/v7e-m+dp/hard/libc_nano.a(libc_a-fwalk.o)
 .data          0x00000000        0x0 /usr/lib/gcc/arm-none-eabi/13.2.1/../../../arm-none-eabi/lib/thumb/v7e-m+dp/hard/libc_nano.a(libc_a-fwalk.o)
 .bss           0x00000000        0x0 /usr/lib/gcc/arm-none-eabi/13.2.1/../../../arm-none-eabi/lib/thumb/v7e-m+dp/hard/libc_nano.a(libc_a-fwalk.o)
 .debug_info    0x00000000      0x7c8 /usr/lib/gcc/arm-none-eabi/13.2.1/../../../arm-none-eabi/lib/thumb/v7e-m+dp/hard/libc_nano.a(libc_a-fwalk.o)
 .debug_abbrev  0x00000000      0x19b /usr/lib/gcc/arm-none-eabi/13.2.1/../../../arm-none-eabi/lib/thumb/v7e-m+dp/hard/libc_nano.a(libc_a-fwalk.o)
 .debug_loclists
                0x00000000       0x87 /usr/lib/gcc/arm-none-eabi/13.2.1/../../../arm-none-eabi/lib/thumb/v7e-m+dp/hard/libc_nano.a(libc_a-fwalk.o)
 .debug_aranges
                0x00000000       0x20 /usr/lib/gcc/arm-none-eabi/13.2.1/../../../arm-none-eabi/lib/thumb/v7e-m+dp/hard/libc_nano.a(libc_a-fwalk.o)
 .debug_line    0x00000000      0x1d1 /usr/lib/gcc/arm-none-eabi/13.2.1/../../../arm-none-eabi/lib/thumb/v7e-m+dp/hard/libc_nano.a(libc_a-fwalk.o)
 .debug_str     0x00000000      0x4cf /usr/lib/gcc/arm-none-eabi/13.2.1/../../../arm-none-eabi/lib/thumb/v7e-m+dp/hard/libc_nano.a(libc_a-fwalk.o)
 .comment       0x00000000       0x27 /usr/lib/gcc/arm-none-eabi/13.2.1/../../../arm-none-eabi/lib/thumb/v7e-m+dp/hard/libc_nano.a(libc_a-fwalk.o)
 .debug_frame   0x00000000       0x34 /usr/lib/gcc/arm-none-eabi/13.2.1/../../../arm-none-eabi/lib/thumb/v7e-m+dp/hard/libc_nano.a(libc_a-fwalk.o)
 .ARM.attributes
                0x00000000       0x32 /usr/lib/gcc/arm-none-eabi/13.2.1/../../../arm-none-eabi/lib/thumb/v7e-m+dp/hard/libc_nano.a(libc_a-fwalk.o)
 .text          0x00000000       0xac /usr/lib/gcc/arm-none-eabi/13.2.1/../../../arm-none-eabi/lib/thumb/v7e-m+dp/hard/libc_nano.a(libc_a-__atexit.o)
 .data          0x00000000        0x4 /usr/lib/gcc/arm-none-eabi/13.2.1/../../../arm-none-eabi/lib/thumb/v7e-m+dp/hard/libc_nano.a(libc_a-__atexit.o)
 .bss           0x00000000       0x8c /usr/lib/gcc/arm-none-eabi/13.2.1/../../../arm-none-eabi/lib/thumb/v7e-m+dp/hard/libc_nano.a(libc_a-__atexit.o)
 .debug_info    0x00000000      0x284 /usr/lib/gcc/arm-none-eabi/13.2.1/../../../arm-none-eabi/lib/thumb/v7e-m+dp/hard/libc_nano.a(libc_a-__atexit.o)
 .debug_abbrev  0x00000000      0x1d4 /usr/lib/gcc/arm-none-eabi/13.2.1/../../../arm-none-eabi/lib/thumb/v7e-m+dp/hard/libc_nano.a(libc_a-__atexit.o)
 .debug_loclists
                0x00000000      0x127 /usr/lib/gcc/arm-none-eabi/13.2.1/../../../arm-none-eabi/lib/thumb/v7e-m+dp/hard/libc_nano.a(libc_a-__atexit.o)
 .debug_aranges
                0x00000000       0x20 /usr/lib/gcc/arm-none-eabi/13.2.1/../../../arm-none-eabi/lib/thumb/v7e-m+dp/hard/libc_nano.a(libc_a-__atexit.o)
 .debug_line    0x00000000      0x230 /usr/lib/gcc/arm-none-eabi/13.2.1/../../../arm-none-eabi/lib/thumb/v7e-m+dp/hard/libc_nano.a(libc_a-__atexit.o)
 .debug_str     0x00000000      0x293 /usr/lib/gcc/arm-none-eabi/13.2.1/../../../arm-none-eabi/lib/thumb/v7e-m+dp/hard/libc_nano.a(libc_a-__atexit.o)
 .comment       0x00000000       0x27 /usr/lib/gcc/arm-none-eabi/13.2.1/../../../arm-none-eabi/lib/thumb/v7e-m+dp/hard/libc_nano.a(libc_a-__atexit.o)
 .debug_frame   0x00000000       0x38 /usr/lib/gcc/arm-none-eabi/13.2.1/../../../arm-none-eabi/lib/thumb/v7e-m+dp/hard/libc_nano.a(libc_a-__atexit.o)
 .ARM.attributes
                0x00000000       0x32 /usr/lib/gcc/arm-none-eabi/13.2.1/../../../arm-none-eabi/lib/thumb/v7e-m+dp/hard/libc_nano.a(libc_a-__atexit.o)
 .text          0x00000000       0xd4 /usr/lib/gcc/arm-none-eabi/13.2.1/../../../arm-none-eabi/lib/thumb/v7e-m+dp/hard/libc_nano.a(libc_a-reent.o)
 .data          0x00000000        0x0 /usr/lib/gcc/arm-none-eabi/13.2.1/../../../arm-none-eabi/lib/thumb/v7e-m+dp/hard/libc_nano.a(libc_a-reent.o)
 .text          0x00000000       0x94 /usr/lib/gcc/arm-none-eabi/13.2.1/../../../arm-none-eabi/lib/thumb/v7e-m+dp/hard/libc_nano.a(libc_a-stdio.o)
 .data          0x00000000        0x0 /usr/lib/gcc/arm-none-eabi/13.2.1/../../../arm-none-eabi/lib/thumb/v7e-m+dp/hard/libc_nano.a(libc_a-stdio.o)
 .bss           0x00000000        0x0 /usr/lib/gcc/arm-none-eabi/13.2.1/../../../arm-none-eabi/lib/thumb/v7e-m+dp/hard/libc_nano.a(libc_a-stdio.o)
 .debug_info    0x00000000      0xa80 /usr/lib/gcc/arm-none-eabi/13.2.1/../../../arm-none-eabi/lib/thumb/v7e-m+dp/hard/libc_nano.a(libc_a-stdio.o)
 .debug_abbrev  0x00000000      0x224 /usr/lib/gcc/arm-none-eabi/13.2.1/../../../arm-none-eabi/lib/thumb/v7e-m+dp/hard/libc_nano.a(libc_a-stdio.o)
 .debug_loclists
                0x00000000      0x23b /usr/lib/gcc/arm-none-eabi/13.2.1/../../../arm-none-eabi/lib/thumb/v7e-m+dp/hard/libc_nano.a(libc_a-stdio.o)
 .debug_aranges
                0x00000000       0x20 /usr/lib/gcc/arm-none-eabi/13.2.1/../../../arm-none-eabi/lib/thumb/v7e-m+dp/hard/libc_nano.a(libc_a-stdio.o)
 .debug_line    0x00000000      0x22b /usr/lib/gcc/arm-none-eabi/13.2.1/../../../arm-none-eabi/lib/thumb/v7e-m+dp/hard/libc_nano.a(libc_a-stdio.o)
 .debug_str     0x00000000      0x52c /usr/lib/gcc/arm-none-eabi/13.2.1/../../../arm-none-eabi/lib/thumb/v7e-m+dp/hard/libc_nano.a(libc_a-stdio.o)
 .comment       0x00000000       0x27 /usr/lib/gcc/arm-none-eabi/13.2.1/../../../arm-none-eabi/lib/thumb/v7e-m+dp/hard/libc_nano.a(libc_a-stdio.o)
 .debug_frame   0x00000000       0x8c /usr/lib/gcc/arm-none-eabi/13.2.1/../../../arm-none-eabi/lib/thumb/v7e-m+dp/hard/libc_nano.a(libc_a-stdio.o)
 .ARM.attributes
                0x00000000       0x32 /usr/lib/gcc/arm-none-eabi/13.2.1/../../../arm-none-eabi/lib/thumb/v7e-m+dp/hard/libc_nano.a(libc_a-stdio.o)
 .text          0x00000000       0x24 /usr/lib/gcc/arm-none-eabi/13.2.1/../../../arm-none-eabi/lib/thumb/v7e-m+dp/hard/libc_nano.a(libc_a-closer.o)
 .data          0x00000000        0x0 /usr/lib/gcc/arm-none-eabi/13.2.1/../../../arm-none-eabi/lib/thumb/v7e-m+dp/hard/libc_nano.a(libc_a-closer.o)
 .bss           0x00000000        0x0 /usr/lib/gcc/arm-none-eabi/13.2.1/../../../arm-none-eabi/lib/thumb/v7e-m+dp/hard/libc_nano.a(libc_a-closer.o)
 .debug_info    0x00000000      0x752 /usr/lib/gcc/arm-none-eabi/13.2.1/../../../arm-none-eabi/lib/thumb/v7e-m+dp/hard/libc_nano.a(libc_a-closer.o)
 .debug_abbrev  0x00000000      0x1b0 /usr/lib/gcc/arm-none-eabi/13.2.1/../../../arm-none-eabi/lib/thumb/v7e-m+dp/hard/libc_nano.a(libc_a-closer.o)
 .debug_loclists
                0x00000000       0x4b /usr/lib/gcc/arm-none-eabi/13.2.1/../../../arm-none-eabi/lib/thumb/v7e-m+dp/hard/libc_nano.a(libc_a-closer.o)
 .debug_aranges
                0x00000000       0x20 /usr/lib/gcc/arm-none-eabi/13.2.1/../../../arm-none-eabi/lib/thumb/v7e-m+dp/hard/libc_nano.a(libc_a-closer.o)
 .debug_line    0x00000000      0x193 /usr/lib/gcc/arm-none-eabi/13.2.1/../../../arm-none-eabi/lib/thumb/v7e-m+dp/hard/libc_nano.a(libc_a-closer.o)
 .debug_str     0x00000000      0x4b5 /usr/lib/gcc/arm-none-eabi/13.2.1/../../../arm-none-eabi/lib/thumb/v7e-m+dp/hard/libc_nano.a(libc_a-closer.o)
 .comment       0x00000000       0x27 /usr/lib/gcc/arm-none-eabi/13.2.1/../../../arm-none-eabi/lib/thumb/v7e-m+dp/hard/libc_nano.a(libc_a-closer.o)
 .debug_frame   0x00000000       0x2c /usr/lib/gcc/arm-none-eabi/13.2.1/../../../arm-none-eabi/lib/thumb/v7e-m+dp/hard/libc_nano.a(libc_a-closer.o)
 .ARM.attributes
                0x00000000       0x32 /usr/lib/gcc/arm-none-eabi/13.2.1/../../../arm-none-eabi/lib/thumb/v7e-m+dp/hard/libc_nano.a(libc_a-closer.o)
 .text          0x00000000       0xc4 /usr/lib/gcc/arm-none-eabi/13.2.1/../../../arm-none-eabi/lib/thumb/v7e-m+dp/hard/libc_nano.a(libc_a-__call_atexit.o)
 .data          0x00000000        0x0 /usr/lib/gcc/arm-none-eabi/13.2.1/../../../arm-none-eabi/lib/thumb/v7e-m+dp/hard/libc_nano.a(libc_a-__call_atexit.o)
 .bss           0x00000000        0x4 /usr/lib/gcc/arm-none-eabi/13.2.1/../../../arm-none-eabi/lib/thumb/v7e-m+dp/hard/libc_nano.a(libc_a-__call_atexit.o)
 .debug_info    0x00000000      0x235 /usr/lib/gcc/arm-none-eabi/13.2.1/../../../arm-none-eabi/lib/thumb/v7e-m+dp/hard/libc_nano.a(libc_a-__call_atexit.o)
 .debug_abbrev  0x00000000      0x179 /usr/lib/gcc/arm-none-eabi/13.2.1/../../../arm-none-eabi/lib/thumb/v7e-m+dp/hard/libc_nano.a(libc_a-__call_atexit.o)
 .debug_loclists
                0x00000000       0xff /usr/lib/gcc/arm-none-eabi/13.2.1/../../../arm-none-eabi/lib/thumb/v7e-m+dp/hard/libc_nano.a(libc_a-__call_atexit.o)
 .debug_aranges
                0x00000000       0x20 /usr/lib/gcc/arm-none-eabi/13.2.1/../../../arm-none-eabi/lib/thumb/v7e-m+dp/hard/libc_nano.a(libc_a-__call_atexit.o)
 .debug_rnglists
                0x00000000       0x2c /usr/lib/gcc/arm-none-eabi/13.2.1/../../../arm-none-eabi/lib/thumb/v7e-m+dp/hard/libc_nano.a(libc_a-__call_atexit.o)
 .debug_line    0x00000000      0x246 /usr/lib/gcc/arm-none-eabi/13.2.1/../../../arm-none-eabi/lib/thumb/v7e-m+dp/hard/libc_nano.a(libc_a-__call_atexit.o)
 .debug_str     0x00000000      0x245 /usr/lib/gcc/arm-none-eabi/13.2.1/../../../arm-none-eabi/lib/thumb/v7e-m+dp/hard/libc_nano.a(libc_a-__call_atexit.o)
 .comment       0x00000000       0x27 /usr/lib/gcc/arm-none-eabi/13.2.1/../../../arm-none-eabi/lib/thumb/v7e-m+dp/hard/libc_nano.a(libc_a-__call_atexit.o)
 .debug_frame   0x00000000       0x40 /usr/lib/gcc/arm-none-eabi/13.2.1/../../../arm-none-eabi/lib/thumb/v7e-m+dp/hard/libc_nano.a(libc_a-__call_atexit.o)
 .ARM.attributes
                0x00000000       0x32 /usr/lib/gcc/arm-none-eabi/13.2.1/../../../arm-none-eabi/lib/thumb/v7e-m+dp/hard/libc_nano.a(libc_a-__call_atexit.o)
 .text          0x00000000       0x2c /usr/lib/gcc/arm-none-eabi/13.2.1/../../../arm-none-eabi/lib/thumb/v7e-m+dp/hard/libc_nano.a(libc_a-readr.o)
 .data          0x00000000        0x0 /usr/lib/gcc/arm-none-eabi/13.2.1/../../../arm-none-eabi/lib/thumb/v7e-m+dp/hard/libc_nano.a(libc_a-readr.o)
 .bss           0x00000000        0x0 /usr/lib/gcc/arm-none-eabi/13.2.1/../../../arm-none-eabi/lib/thumb/v7e-m+dp/hard/libc_nano.a(libc_a-readr.o)
 .debug_info    0x00000000      0x7b5 /usr/lib/gcc/arm-none-eabi/13.2.1/../../../arm-none-eabi/lib/thumb/v7e-m+dp/hard/libc_nano.a(libc_a-readr.o)
 .debug_abbrev  0x00000000      0x1b0 /usr/lib/gcc/arm-none-eabi/13.2.1/../../../arm-none-eabi/lib/thumb/v7e-m+dp/hard/libc_nano.a(libc_a-readr.o)
 .debug_loclists
                0x00000000       0x9e /usr/lib/gcc/arm-none-eabi/13.2.1/../../../arm-none-eabi/lib/thumb/v7e-m+dp/hard/libc_nano.a(libc_a-readr.o)
 .debug_aranges
                0x00000000       0x20 /usr/lib/gcc/arm-none-eabi/13.2.1/../../../arm-none-eabi/lib/thumb/v7e-m+dp/hard/libc_nano.a(libc_a-readr.o)
 .debug_line    0x00000000      0x198 /usr/lib/gcc/arm-none-eabi/13.2.1/../../../arm-none-eabi/lib/thumb/v7e-m+dp/hard/libc_nano.a(libc_a-readr.o)
 .debug_str     0x00000000      0x4c3 /usr/lib/gcc/arm-none-eabi/13.2.1/../../../arm-none-eabi/lib/thumb/v7e-m+dp/hard/libc_nano.a(libc_a-readr.o)
 .comment       0x00000000       0x27 /usr/lib/gcc/arm-none-eabi/13.2.1/../../../arm-none-eabi/lib/thumb/v7e-m+dp/hard/libc_nano.a(libc_a-readr.o)
 .debug_frame   0x00000000       0x2c /usr/lib/gcc/arm-none-eabi/13.2.1/../../../arm-none-eabi/lib/thumb/v7e-m+dp/hard/libc_nano.a(libc_a-readr.o)
 .ARM.attributes
                0x00000000       0x32 /usr/lib/gcc/arm-none-eabi/13.2.1/../../../arm-none-eabi/lib/thumb/v7e-m+dp/hard/libc_nano.a(libc_a-readr.o)
 .text          0x00000000       0x2c /usr/lib/gcc/arm-none-eabi/13.2.1/../../../arm-none-eabi/lib/thumb/v7e-m+dp/hard/libc_nano.a(libc_a-lseekr.o)
 .data          0x00000000        0x0 /usr/lib/gcc/arm-none-eabi/13.2.1/../../../arm-none-eabi/lib/thumb/v7e-m+dp/hard/libc_nano.a(libc_a-lseekr.o)
 .bss           0x00000000        0x0 /usr/lib/gcc/arm-none-eabi/13.2.1/../../../arm-none-eabi/lib/thumb/v7e-m+dp/hard/libc_nano.a(libc_a-lseekr.o)
 .debug_info    0x00000000      0x79e /usr/lib/gcc/arm-none-eabi/13.2.1/../../../arm-none-eabi/lib/thumb/v7e-m+dp/hard/libc_nano.a(libc_a-lseekr.o)
 .debug_abbrev  0x00000000      0x1c4 /usr/lib/gcc/arm-none-eabi/13.2.1/../../../arm-none-eabi/lib/thumb/v7e-m+dp/hard/libc_nano.a(libc_a-lseekr.o)
 .debug_loclists
                0x00000000       0x9e /usr/lib/gcc/arm-none-eabi/13.2.1/../../../arm-none-eabi/lib/thumb/v7e-m+dp/hard/libc_nano.a(libc_a-lseekr.o)
 .debug_aranges
                0x00000000       0x20 /usr/lib/gcc/arm-none-eabi/13.2.1/../../../arm-none-eabi/lib/thumb/v7e-m+dp/hard/libc_nano.a(libc_a-lseekr.o)
 .debug_line    0x00000000      0x199 /usr/lib/gcc/arm-none-eabi/13.2.1/../../../arm-none-eabi/lib/thumb/v7e-m+dp/hard/libc_nano.a(libc_a-lseekr.o)
 .debug_str     0x00000000      0x4c3 /usr/lib/gcc/arm-none-eabi/13.2.1/../../../arm-none-eabi/lib/thumb/v7e-m+dp/hard/libc_nano.a(libc_a-lseekr.o)
 .comment       0x00000000       0x27 /usr/lib/gcc/arm-none-eabi/13.2.1/../../../arm-none-eabi/lib/thumb/v7e-m+dp/hard/libc_nano.a(libc_a-lseekr.o)
 .debug_frame   0x00000000       0x2c /usr/lib/gcc/arm-none-eabi/13.2.1/../../../arm-none-eabi/lib/thumb/v7e-m+dp/hard/libc_nano.a(libc_a-lseekr.o)
 .ARM.attributes
                0x00000000       0x32 /usr/lib/gcc/arm-none-eabi/13.2.1/../../../arm-none-eabi/lib/thumb/v7e-m+dp/hard/libc_nano.a(libc_a-lseekr.o)
 .text          0x00000000       0x2c /usr/lib/gcc/arm-none-eabi/13.2.1/../../../arm-none-eabi/lib/thumb/v7e-m+dp/hard/libc_nano.a(libc_a-writer.o)
 .data          0x00000000        0x0 /usr/lib/gcc/arm-none-eabi/13.2.1/../../../arm-none-eabi/lib/thumb/v7e-m+dp/hard/libc_nano.a(libc_a-writer.o)
 .bss           0x00000000        0x0 /usr/lib/gcc/arm-none-eabi/13.2.1/../../../arm-none-eabi/lib/thumb/v7e-m+dp/hard/libc_nano.a(libc_a-writer.o)
 .debug_info    0x00000000      0x7bb /usr/lib/gcc/arm-none-eabi/13.2.1/../../../arm-none-eabi/lib/thumb/v7e-m+dp/hard/libc_nano.a(libc_a-writer.o)
 .debug_abbrev  0x00000000      0x1b5 /usr/lib/gcc/arm-none-eabi/13.2.1/../../../arm-none-eabi/lib/thumb/v7e-m+dp/hard/libc_nano.a(libc_a-writer.o)
 .debug_loclists
                0x00000000       0x9e /usr/lib/gcc/arm-none-eabi/13.2.1/../../../arm-none-eabi/lib/thumb/v7e-m+dp/hard/libc_nano.a(libc_a-writer.o)
 .debug_aranges
                0x00000000       0x20 /usr/lib/gcc/arm-none-eabi/13.2.1/../../../arm-none-eabi/lib/thumb/v7e-m+dp/hard/libc_nano.a(libc_a-writer.o)
 .debug_line    0x00000000      0x199 /usr/lib/gcc/arm-none-eabi/13.2.1/../../../arm-none-eabi/lib/thumb/v7e-m+dp/hard/libc_nano.a(libc_a-writer.o)
 .debug_str     0x00000000      0x4c5 /usr/lib/gcc/arm-none-eabi/13.2.1/../../../arm-none-eabi/lib/thumb/v7e-m+dp/hard/libc_nano.a(libc_a-writer.o)
 .comment       0x00000000       0x27 /usr/lib/gcc/arm-none-eabi/13.2.1/../../../arm-none-eabi/lib/thumb/v7e-m+dp/hard/libc_nano.a(libc_a-writer.o)
 .debug_frame   0x00000000       0x2c /usr/lib/gcc/arm-none-eabi/13.2.1/../../../arm-none-eabi/lib/thumb/v7e-m+dp/hard/libc_nano.a(libc_a-writer.o)
 .ARM.attributes
                0x00000000       0x32 /usr/lib/gcc/arm-none-eabi/13.2.1/../../../arm-none-eabi/lib/thumb/v7e-m+dp/hard/libc_nano.a(libc_a-writer.o)
 .data          0x00000000        0x0 /usr/lib/gcc/arm-none-eabi/13.2.1/thumb/v7e-m+dp/hard/libgcc.a(_aeabi_uldivmod.o)
 .bss           0x00000000        0x0 /usr/lib/gcc/arm-none-eabi/13.2.1/thumb/v7e-m+dp/hard/libgcc.a(_aeabi_uldivmod.o)
 .data          0x00000000        0x0 /usr/lib/gcc/arm-none-eabi/13.2.1/thumb/v7e-m+dp/hard/libgcc.a(_udivmoddi4.o)
 .bss           0x00000000        0x0 /usr/lib/gcc/arm-none-eabi/13.2.1/thumb/v7e-m+dp/hard/libgcc.a(_udivmoddi4.o)
 .ARM.extab     0x00000000        0x0 /usr/lib/gcc/arm-none-eabi/13.2.1/thumb/v7e-m+dp/hard/libgcc.a(_udivmoddi4.o)
 .data          0x00000000        0x0 /usr/lib/gcc/arm-none-eabi/13.2.1/thumb/v7e-m+dp/hard/libgcc.a(_dvmd_tls.o)
 .bss           0x00000000        0x0 /usr/lib/gcc/arm-none-eabi/13.2.1/thumb/v7e-m+dp/hard/libgcc.a(_dvmd_tls.o)
 .text          0x00000000        0x0 /usr/lib/gcc/arm-none-eabi/13.2.1/thumb/v7e-m+dp/hard/crtend.o
 .data          0x00000000        0x0 /usr/lib/gcc/arm-none-eabi/13.2.1/thumb/v7e-m+dp/hard/crtend.o
 .bss           0x00000000        0x0 /usr/lib/gcc/arm-none-eabi/13.2.1/thumb/v7e-m+dp/hard/crtend.o
 .rodata        0x00000000       0x24 /usr/lib/gcc/arm-none-eabi/13.2.1/thumb/v7e-m+dp/hard/crtend.o
 .eh_frame      0x00000000        0x4 /usr/lib/gcc/arm-none-eabi/13.2.1/thumb/v7e-m+dp/hard/crtend.o
 .text          0x00000000        0x0 /usr/lib/gcc/arm-none-eabi/13.2.1/thumb/v7e-m+dp/hard/crtn.o
 .data          0x00000000        0x0 /usr/lib/gcc/arm-none-eabi/13.2.1/thumb/v7e-m+dp/hard/crtn.o
 .bss           0x00000000        0x0 /usr/lib/gcc/arm-none-eabi/13.2.1/thumb/v7e-m+dp/hard/crtn.o

Memory Configuration

Name             Origin             Length             Attributes
RAM              0x20000000         0x00080000         xrw
FLASH            0x08000000         0x00200000         xr
*default*        0x00000000         0xffffffff

Linker script and memory map

LOAD /usr/lib/gcc/arm-none-eabi/13.2.1/thumb/v7e-m+dp/hard/crti.o
LOAD /usr/lib/gcc/arm-none-eabi/13.2.1/thumb/v7e-m+dp/hard/crtbegin.o
LOAD /usr/lib/gcc/arm-none-eabi/13.2.1/../../../arm-none-eabi/lib/thumb/v7e-m+dp/hard/crt0.o
LOAD build/main.o
LOAD build/bsp_driver_sd.o
LOAD build/sd_diskio.o
LOAD build/fatfs.o
LOAD build/fatfs_platform.o
LOAD build/stm32f7xx_it.o
LOAD build/stm32f7xx_hal_msp.o
LOAD build/stm32f7xx_hal_adc.o
LOAD build/stm32f7xx_hal_adc_ex.o
LOAD build/stm32f7xx_hal_rcc.o
LOAD build/stm32f7xx_hal_rcc_ex.o
LOAD build/stm32f7xx_hal_flash.o
LOAD build/stm32f7xx_hal_flash_ex.o
LOAD build/stm32f7xx_hal_gpio.o
LOAD build/stm32f7xx_hal_dma.o
LOAD build/stm32f7xx_hal_dma_ex.o
LOAD build/stm32f7xx_hal_pwr.o
LOAD build/stm32f7xx_hal_pwr_ex.o
LOAD build/stm32f7xx_hal_cortex.o
LOAD build/stm32f7xx_hal.o
LOAD build/stm32f7xx_hal_i2c.o
LOAD build/stm32f7xx_hal_i2c_ex.o
LOAD build/stm32f7xx_hal_exti.o
LOAD build/stm32f7xx_ll_rcc.o
LOAD build/stm32f7xx_ll_utils.o
LOAD build/stm32f7xx_ll_exti.o
LOAD build/stm32f7xx_ll_gpio.o
LOAD build/stm32f7xx_ll_dma.o
LOAD build/stm32f7xx_ll_sdmmc.o
LOAD build/stm32f7xx_hal_sd.o
LOAD build/stm32f7xx_ll_spi.o
LOAD build/stm32f7xx_hal_tim.o
LOAD build/stm32f7xx_hal_tim_ex.o
LOAD build/stm32f7xx_ll_tim.o
LOAD build/stm32f7xx_ll_usart.o
LOAD build/system_stm32f7xx.o
LOAD build/File_Handling.o
LOAD build/diskio.o
LOAD build/ff.o
LOAD build/ff_gen_drv.o
LOAD build/syscall.o
LOAD build/sysmem.o
LOAD build/syscalls.o
LOAD build/stm32f7xx_hal_uart.o
LOAD build/stm32f7xx_hal_uart_ex.o
LOAD build/startup_stm32f767xx.o
LOAD /usr/lib/gcc/arm-none-eabi/13.2.1/../../../arm-none-eabi/lib/thumb/v7e-m+dp/hard/libc_nano.a
LOAD /usr/lib/gcc/arm-none-eabi/13.2.1/../../../arm-none-eabi/lib/thumb/v7e-m+dp/hard/libm.a
LOAD /usr/lib/gcc/arm-none-eabi/13.2.1/../../../arm-none-eabi/lib/thumb/v7e-m+dp/hard/libnosys.a
START GROUP
LOAD /usr/lib/gcc/arm-none-eabi/13.2.1/thumb/v7e-m+dp/hard/libgcc.a
LOAD /usr/lib/gcc/arm-none-eabi/13.2.1/../../../arm-none-eabi/lib/thumb/v7e-m+dp/hard/libc_nano.a
END GROUP
START GROUP
LOAD /usr/lib/gcc/arm-none-eabi/13.2.1/thumb/v7e-m+dp/hard/libgcc.a
LOAD /usr/lib/gcc/arm-none-eabi/13.2.1/../../../arm-none-eabi/lib/thumb/v7e-m+dp/hard/libc_nano.a
END GROUP
LOAD /usr/lib/gcc/arm-none-eabi/13.2.1/thumb/v7e-m+dp/hard/crtend.o
LOAD /usr/lib/gcc/arm-none-eabi/13.2.1/thumb/v7e-m+dp/hard/crtn.o
                0x20080000                        _estack = (ORIGIN (RAM) + LENGTH (RAM))
                0x00002000                        _Min_Heap_Size = 0x2000
                0x00004000                        _Min_Stack_Size = 0x4000

.isr_vector     0x08000000      0x1f8
                0x08000000                        . = ALIGN (0x4)
 *(.isr_vector)
 .isr_vector    0x08000000      0x1f8 build/startup_stm32f767xx.o
                0x08000000                g_pfnVectors
                0x080001f8                        . = ALIGN (0x4)

.text           0x08000200     0xa924
                0x08000200                        . = ALIGN (0x4)
 *(.text)
 .text          0x08000200       0x88 /usr/lib/gcc/arm-none-eabi/13.2.1/thumb/v7e-m+dp/hard/crtbegin.o
 .text          0x08000288       0x80 /usr/lib/gcc/arm-none-eabi/13.2.1/../../../arm-none-eabi/lib/thumb/v7e-m+dp/hard/libc_nano.a(libc_a-sprintf.o)
                0x08000288                _siprintf_r
                0x08000288                _sprintf_r
                0x080002c4                sprintf
                0x080002c4                siprintf
 .text          0x08000308      0x400 /usr/lib/gcc/arm-none-eabi/13.2.1/../../../arm-none-eabi/lib/thumb/v7e-m+dp/hard/libc_nano.a(libc_a-nano-svfprintf.o)
                0x08000308                __ssputs_r
                0x080003c8                __ssprint_r
                0x080004d0                _svfprintf_r
                0x080004d0                _svfiprintf_r
 .text          0x08000708       0x50 /usr/lib/gcc/arm-none-eabi/13.2.1/../../../arm-none-eabi/lib/thumb/v7e-m+dp/hard/libc_nano.a(libc_a-init.o)
                0x08000708                __libc_init_array
 .text          0x08000758       0xa4 /usr/lib/gcc/arm-none-eabi/13.2.1/../../../arm-none-eabi/lib/thumb/v7e-m+dp/hard/libc_nano.a(libc_a-memset.o)
                0x08000758                memset
 .text          0x080007fc        0xc /usr/lib/gcc/arm-none-eabi/13.2.1/../../../arm-none-eabi/lib/thumb/v7e-m+dp/hard/libc_nano.a(libc_a-errno.o)
                0x080007fc                __errno
 .text          0x08000808      0x148 /usr/lib/gcc/arm-none-eabi/13.2.1/../../../arm-none-eabi/lib/thumb/v7e-m+dp/hard/libc_nano.a(libc_a-mallocr.o)
                0x08000850                _malloc_r
 .text          0x08000950       0xbc /usr/lib/gcc/arm-none-eabi/13.2.1/../../../arm-none-eabi/lib/thumb/v7e-m+dp/hard/libc_nano.a(libc_a-freer.o)
                0x08000950                _free_r
 .text          0x08000a0c      0x100 /usr/lib/gcc/arm-none-eabi/13.2.1/../../../arm-none-eabi/lib/thumb/v7e-m+dp/hard/libc_nano.a(libc_a-memmove.o)
                0x08000a0c                memmove
 *fill*         0x08000b0c        0x4 
 .text          0x08000b10       0xa0 /usr/lib/gcc/arm-none-eabi/13.2.1/../../../arm-none-eabi/lib/thumb/v7e-m+dp/hard/libc_nano.a(libc_a-memchr.o)
                0x08000b10                memchr
 .text          0x08000bb0      0x134 /usr/lib/gcc/arm-none-eabi/13.2.1/../../../arm-none-eabi/lib/thumb/v7e-m+dp/hard/libc_nano.a(libc_a-memcpy.o)
                0x08000bb0                memcpy
 .text          0x08000ce4       0x20 /usr/lib/gcc/arm-none-eabi/13.2.1/../../../arm-none-eabi/lib/thumb/v7e-m+dp/hard/libc_nano.a(libc_a-malloc.o)
                0x08000ce4                malloc
                0x08000cf4                free
 .text          0x08000d04       0x64 /usr/lib/gcc/arm-none-eabi/13.2.1/../../../arm-none-eabi/lib/thumb/v7e-m+dp/hard/libc_nano.a(libc_a-reallocr.o)
                0x08000d04                _realloc_r
 .text          0x08000d68      0x3a8 /usr/lib/gcc/arm-none-eabi/13.2.1/../../../arm-none-eabi/lib/thumb/v7e-m+dp/hard/libc_nano.a(libc_a-nano-vfprintf_i.o)
                0x08000d68                _printf_common
                0x08000e8c                _printf_i
 .text          0x08001110        0x8 /usr/lib/gcc/arm-none-eabi/13.2.1/../../../arm-none-eabi/lib/thumb/v7e-m+dp/hard/libc_nano.a(libc_a-mlock.o)
                0x08001110                __malloc_lock
                0x08001114                __malloc_unlock
 .text          0x08001118       0x24 /usr/lib/gcc/arm-none-eabi/13.2.1/../../../arm-none-eabi/lib/thumb/v7e-m+dp/hard/libc_nano.a(libc_a-sbrkr.o)
                0x08001118                _sbrk_r
 .text          0x0800113c       0x10 /usr/lib/gcc/arm-none-eabi/13.2.1/../../../arm-none-eabi/lib/thumb/v7e-m+dp/hard/libc_nano.a(libc_a-msizer.o)
                0x0800113c                _malloc_usable_size_r
 .text          0x0800114c       0x30 /usr/lib/gcc/arm-none-eabi/13.2.1/thumb/v7e-m+dp/hard/libgcc.a(_aeabi_uldivmod.o)
                0x0800114c                __aeabi_uldivmod
 .text          0x0800117c      0x2bc /usr/lib/gcc/arm-none-eabi/13.2.1/thumb/v7e-m+dp/hard/libgcc.a(_udivmoddi4.o)
                0x0800117c                __udivmoddi4
 .text          0x08001438        0x4 /usr/lib/gcc/arm-none-eabi/13.2.1/thumb/v7e-m+dp/hard/libgcc.a(_dvmd_tls.o)
                0x08001438                __aeabi_ldiv0
                0x08001438                __aeabi_idiv0
 *(.text*)
 .text.NVIC_EncodePriority
                0x0800143c       0x3e build/main.o
 *fill*         0x0800147a        0x2 
 .text.MX_SDMMC1_SD_Init
                0x0800147c       0x24 build/main.o
 .text.MX_DMA_Init
                0x080014a0       0x48 build/main.o
 .text.Decode_task
                0x080014e8      0x168 build/main.o
 .text.PID_Controller_Temp
                0x08001650       0xe4 build/main.o
 .text.OUT_trigger
                0x08001734      0x124 build/main.o
 .text.MPhD_T   0x08001858      0x220 build/main.o
 .text.Stop_TIM10
                0x08001a78       0x20 build/main.o
 .text.MX_GPIO_Init
                0x08001a98      0x248 build/main.o
 .text.MX_SPI4_Init
                0x08001ce0       0xd4 build/main.o
 .text.MX_SPI2_Init
                0x08001db4       0xd0 build/main.o
 .text.MX_SPI5_Init
                0x08001e84       0xd0 build/main.o
 .text.MX_SPI6_Init
                0x08001f54       0xd0 build/main.o
 .text.MX_TIM2_Init
                0x08002024       0x9c build/main.o
 .text.MX_TIM5_Init
                0x080020c0       0x98 build/main.o
 .text.MX_TIM7_Init
                0x08002158       0x8c build/main.o
 .text.MX_TIM6_Init
                0x080021e4       0x8c build/main.o
 .text.Init_params
                0x08002270      0x30c build/main.o
 .text.Get_ADC  0x0800257c       0x70 build/main.o
 .text.Set_LTEC
                0x080025ec      0x158 build/main.o
                0x080025ec                Set_LTEC
 .text.Decode_uart
                0x08002744      0x2f8 build/main.o
 .text.CalculateChecksum
                0x08002a3c       0x18 build/main.o
                0x08002a3c                CalculateChecksum
 .text.CheckChecksum
                0x08002a54       0x48 build/main.o
                0x08002a54                CheckChecksum
 .text.SD_SAVE  0x08002a9c       0x3c build/main.o
                0x08002a9c                SD_SAVE
 .text.SD_READ  0x08002ad8       0x4c build/main.o
                0x08002ad8                SD_READ
 .text.SD_REMOVE
                0x08002b24       0x40 build/main.o
                0x08002b24                SD_REMOVE
 .text.USART_TX
                0x08002b64       0x2c build/main.o
                0x08002b64                USART_TX
 .text.USART_TX_DMA
                0x08002b90       0x40 build/main.o
                0x08002b90                USART_TX_DMA
 .text.Error_Handler
                0x08002bd0        0x4 build/main.o
                0x08002bd0                Error_Handler
 .text.MX_ADC1_Init
                0x08002bd4       0xc8 build/main.o
 .text.MX_ADC3_Init
                0x08002c9c       0x6c build/main.o
 .text.MX_USART1_UART_Init
                0x08002d08      0x190 build/main.o
 .text.MX_TIM10_Init
                0x08002e98       0x2c build/main.o
 .text.MX_UART8_Init
                0x08002ec4       0x38 build/main.o
 .text.MX_TIM8_Init
                0x08002efc       0x6c build/main.o
 .text.MX_TIM11_Init
                0x08002f68       0x70 build/main.o
 .text.MX_TIM4_Init
                0x08002fd8       0xa4 build/main.o
 .text.SystemClock_Config
                0x0800307c       0xb4 build/main.o
                0x0800307c                SystemClock_Config
 .text.main     0x08003130      0xa9c build/main.o
                0x08003130                main
 .text.BSP_SD_ReadBlocks
                0x08003bcc       0x20 build/bsp_driver_sd.o
                0x08003bcc                BSP_SD_ReadBlocks
 .text.BSP_SD_WriteBlocks
                0x08003bec       0x20 build/bsp_driver_sd.o
                0x08003bec                BSP_SD_WriteBlocks
 .text.BSP_SD_GetCardState
                0x08003c0c       0x14 build/bsp_driver_sd.o
                0x08003c0c                BSP_SD_GetCardState
 .text.BSP_SD_GetCardInfo
                0x08003c20       0x10 build/bsp_driver_sd.o
                0x08003c20                BSP_SD_GetCardInfo
 .text.BSP_SD_IsDetected
                0x08003c30       0x20 build/bsp_driver_sd.o
                0x08003c30                BSP_SD_IsDetected
 .text.BSP_SD_Init
                0x08003c50       0x34 build/bsp_driver_sd.o
                0x08003c50                BSP_SD_Init
 .text.SD_CheckStatus
                0x08003c84       0x24 build/sd_diskio.o
 .text.SD_initialize
                0x08003ca8       0x28 build/sd_diskio.o
                0x08003ca8                SD_initialize
 .text.SD_status
                0x08003cd0        0x8 build/sd_diskio.o
                0x08003cd0                SD_status
 .text.SD_read  0x08003cd8       0x24 build/sd_diskio.o
                0x08003cd8                SD_read
 .text.SD_write
                0x08003cfc       0x24 build/sd_diskio.o
                0x08003cfc                SD_write
 .text.SD_ioctl
                0x08003d20       0x58 build/sd_diskio.o
                0x08003d20                SD_ioctl
 .text.MX_FATFS_Init
                0x08003d78       0x1c build/fatfs.o
                0x08003d78                MX_FATFS_Init
 .text.get_fattime
                0x08003d94        0x4 build/fatfs.o
                0x08003d94                get_fattime
 .text.BSP_PlatformIsDetected
                0x08003d98       0x18 build/fatfs_platform.o
                0x08003d98                BSP_PlatformIsDetected
 .text.NMI_Handler
                0x08003db0        0x2 build/stm32f7xx_it.o
                0x08003db0                NMI_Handler
 .text.HardFault_Handler
                0x08003db2        0x2 build/stm32f7xx_it.o
                0x08003db2                HardFault_Handler
 .text.MemManage_Handler
                0x08003db4        0x2 build/stm32f7xx_it.o
                0x08003db4                MemManage_Handler
 .text.BusFault_Handler
                0x08003db6        0x2 build/stm32f7xx_it.o
                0x08003db6                BusFault_Handler
 .text.UsageFault_Handler
                0x08003db8        0x2 build/stm32f7xx_it.o
                0x08003db8                UsageFault_Handler
 .text.SVC_Handler
                0x08003dba        0x2 build/stm32f7xx_it.o
                0x08003dba                SVC_Handler
 .text.DebugMon_Handler
                0x08003dbc        0x2 build/stm32f7xx_it.o
                0x08003dbc                DebugMon_Handler
 .text.PendSV_Handler
                0x08003dbe        0x2 build/stm32f7xx_it.o
                0x08003dbe                PendSV_Handler
 .text.SysTick_Handler
                0x08003dc0        0x8 build/stm32f7xx_it.o
                0x08003dc0                SysTick_Handler
 .text.ADC_IRQHandler
                0x08003dc8       0x18 build/stm32f7xx_it.o
                0x08003dc8                ADC_IRQHandler
 .text.TIM1_UP_TIM10_IRQHandler
                0x08003de0       0x34 build/stm32f7xx_it.o
                0x08003de0                TIM1_UP_TIM10_IRQHandler
 .text.TIM1_TRG_COM_TIM11_IRQHandler
                0x08003e14       0x34 build/stm32f7xx_it.o
                0x08003e14                TIM1_TRG_COM_TIM11_IRQHandler
 .text.TIM2_IRQHandler
                0x08003e48        0x2 build/stm32f7xx_it.o
                0x08003e48                TIM2_IRQHandler
 *fill*         0x08003e4a        0x2 
 .text.TIM8_UP_TIM13_IRQHandler
                0x08003e4c       0x50 build/stm32f7xx_it.o
                0x08003e4c                TIM8_UP_TIM13_IRQHandler
 .text.TIM5_IRQHandler
                0x08003e9c        0x2 build/stm32f7xx_it.o
                0x08003e9c                TIM5_IRQHandler
 *fill*         0x08003e9e        0x2 
 .text.TIM6_DAC_IRQHandler
                0x08003ea0       0x34 build/stm32f7xx_it.o
                0x08003ea0                TIM6_DAC_IRQHandler
 .text.TIM7_IRQHandler
                0x08003ed4       0x24 build/stm32f7xx_it.o
                0x08003ed4                TIM7_IRQHandler
 .text.UART_RxCpltCallback
                0x08003ef8      0x28c build/stm32f7xx_it.o
                0x08003ef8                UART_RxCpltCallback
 .text.USART1_IRQHandler
                0x08004184       0xd0 build/stm32f7xx_it.o
                0x08004184                USART1_IRQHandler
 .text.DMA2_Stream7_TransferComplete
                0x08004254       0x10 build/stm32f7xx_it.o
                0x08004254                DMA2_Stream7_TransferComplete
 .text.DMA2_Stream7_IRQHandler
                0x08004264       0x34 build/stm32f7xx_it.o
                0x08004264                DMA2_Stream7_IRQHandler
 .text.HAL_MspInit
                0x08004298       0x30 build/stm32f7xx_hal_msp.o
                0x08004298                HAL_MspInit
 .text.HAL_ADC_MspInit
                0x080042c8      0x110 build/stm32f7xx_hal_msp.o
                0x080042c8                HAL_ADC_MspInit
 .text.HAL_SD_MspInit
                0x080043d8       0xb8 build/stm32f7xx_hal_msp.o
                0x080043d8                HAL_SD_MspInit
 .text.HAL_TIM_Base_MspInit
                0x08004490       0xc0 build/stm32f7xx_hal_msp.o
                0x08004490                HAL_TIM_Base_MspInit
 .text.HAL_TIM_MspPostInit
                0x08004550       0x8c build/stm32f7xx_hal_msp.o
                0x08004550                HAL_TIM_MspPostInit
 .text.HAL_UART_MspInit
                0x080045dc       0x88 build/stm32f7xx_hal_msp.o
                0x080045dc                HAL_UART_MspInit
 .text.ADC_Init
                0x08004664      0x134 build/stm32f7xx_hal_adc.o
 .text.HAL_ADC_Init
                0x08004798       0x58 build/stm32f7xx_hal_adc.o
                0x08004798                HAL_ADC_Init
 .text.HAL_ADC_Start
                0x080047f0      0x134 build/stm32f7xx_hal_adc.o
                0x080047f0                HAL_ADC_Start
 .text.HAL_ADC_Stop
                0x08004924       0x40 build/stm32f7xx_hal_adc.o
                0x08004924                HAL_ADC_Stop
 .text.HAL_ADC_PollForConversion
                0x08004964       0xc2 build/stm32f7xx_hal_adc.o
                0x08004964                HAL_ADC_PollForConversion
 .text.HAL_ADC_GetValue
                0x08004a26        0x6 build/stm32f7xx_hal_adc.o
                0x08004a26                HAL_ADC_GetValue
 .text.HAL_ADC_ConvCpltCallback
                0x08004a2c        0x2 build/stm32f7xx_hal_adc.o
                0x08004a2c                HAL_ADC_ConvCpltCallback
 .text.HAL_ADC_LevelOutOfWindowCallback
                0x08004a2e        0x2 build/stm32f7xx_hal_adc.o
                0x08004a2e                HAL_ADC_LevelOutOfWindowCallback
 .text.HAL_ADC_ErrorCallback
                0x08004a30        0x2 build/stm32f7xx_hal_adc.o
                0x08004a30                HAL_ADC_ErrorCallback
 .text.HAL_ADC_IRQHandler
                0x08004a32      0x136 build/stm32f7xx_hal_adc.o
                0x08004a32                HAL_ADC_IRQHandler
 .text.HAL_ADC_ConfigChannel
                0x08004b68      0x1e4 build/stm32f7xx_hal_adc.o
                0x08004b68                HAL_ADC_ConfigChannel
 .text.HAL_ADCEx_InjectedConvCpltCallback
                0x08004d4c        0x2 build/stm32f7xx_hal_adc_ex.o
                0x08004d4c                HAL_ADCEx_InjectedConvCpltCallback
 *fill*         0x08004d4e        0x2 
 .text.HAL_RCC_OscConfig
                0x08004d50      0x444 build/stm32f7xx_hal_rcc.o
                0x08004d50                HAL_RCC_OscConfig
 .text.HAL_RCC_GetSysClockFreq
                0x08005194       0xa8 build/stm32f7xx_hal_rcc.o
                0x08005194                HAL_RCC_GetSysClockFreq
 .text.HAL_RCC_ClockConfig
                0x0800523c      0x16c build/stm32f7xx_hal_rcc.o
                0x0800523c                HAL_RCC_ClockConfig
 .text.HAL_RCC_GetHCLKFreq
                0x080053a8        0xc build/stm32f7xx_hal_rcc.o
                0x080053a8                HAL_RCC_GetHCLKFreq
 .text.HAL_RCC_GetPCLK1Freq
                0x080053b4       0x20 build/stm32f7xx_hal_rcc.o
                0x080053b4                HAL_RCC_GetPCLK1Freq
 .text.HAL_RCC_GetPCLK2Freq
                0x080053d4       0x20 build/stm32f7xx_hal_rcc.o
                0x080053d4                HAL_RCC_GetPCLK2Freq
 .text.HAL_RCCEx_PeriphCLKConfig
                0x080053f4      0x600 build/stm32f7xx_hal_rcc_ex.o
                0x080053f4                HAL_RCCEx_PeriphCLKConfig
 .text.HAL_GPIO_Init
                0x080059f4      0x204 build/stm32f7xx_hal_gpio.o
                0x080059f4                HAL_GPIO_Init
 .text.HAL_GPIO_ReadPin
                0x08005bf8        0xe build/stm32f7xx_hal_gpio.o
                0x08005bf8                HAL_GPIO_ReadPin
 .text.HAL_GPIO_WritePin
                0x08005c06        0xc build/stm32f7xx_hal_gpio.o
                0x08005c06                HAL_GPIO_WritePin
 .text.HAL_GPIO_TogglePin
                0x08005c12       0x12 build/stm32f7xx_hal_gpio.o
                0x08005c12                HAL_GPIO_TogglePin
 .text.HAL_PWREx_EnableOverDrive
                0x08005c24       0x7c build/stm32f7xx_hal_pwr_ex.o
                0x08005c24                HAL_PWREx_EnableOverDrive
 .text.__NVIC_SetPriority
                0x08005ca0       0x24 build/stm32f7xx_hal_cortex.o
 .text.NVIC_EncodePriority
                0x08005cc4       0x3e build/stm32f7xx_hal_cortex.o
 *fill*         0x08005d02        0x2 
 .text.HAL_NVIC_SetPriorityGrouping
                0x08005d04       0x24 build/stm32f7xx_hal_cortex.o
                0x08005d04                HAL_NVIC_SetPriorityGrouping
 .text.HAL_NVIC_SetPriority
                0x08005d28       0x20 build/stm32f7xx_hal_cortex.o
                0x08005d28                HAL_NVIC_SetPriority
 .text.HAL_NVIC_EnableIRQ
                0x08005d48       0x1c build/stm32f7xx_hal_cortex.o
                0x08005d48                HAL_NVIC_EnableIRQ
 .text.HAL_SYSTICK_Config
                0x08005d64       0x28 build/stm32f7xx_hal_cortex.o
                0x08005d64                HAL_SYSTICK_Config
 .text.HAL_InitTick
                0x08005d8c       0x4c build/stm32f7xx_hal.o
                0x08005d8c                HAL_InitTick
 .text.HAL_Init
                0x08005dd8       0x16 build/stm32f7xx_hal.o
                0x08005dd8                HAL_Init
 *fill*         0x08005dee        0x2 
 .text.HAL_IncTick
                0x08005df0       0x18 build/stm32f7xx_hal.o
                0x08005df0                HAL_IncTick
 .text.HAL_GetTick
                0x08005e08        0xc build/stm32f7xx_hal.o
                0x08005e08                HAL_GetTick
 .text.HAL_Delay
                0x08005e14       0x28 build/stm32f7xx_hal.o
                0x08005e14                HAL_Delay
 .text.RCC_GetHCLKClockFreq
                0x08005e3c       0x18 build/stm32f7xx_ll_rcc.o
                0x08005e3c                RCC_GetHCLKClockFreq
 .text.RCC_GetPCLK1ClockFreq
                0x08005e54       0x18 build/stm32f7xx_ll_rcc.o
                0x08005e54                RCC_GetPCLK1ClockFreq
 .text.RCC_GetPCLK2ClockFreq
                0x08005e6c       0x18 build/stm32f7xx_ll_rcc.o
                0x08005e6c                RCC_GetPCLK2ClockFreq
 .text.RCC_PLL_GetFreqDomain_SYS
                0x08005e84       0x44 build/stm32f7xx_ll_rcc.o
                0x08005e84                RCC_PLL_GetFreqDomain_SYS
 .text.RCC_GetSystemClockFreq
                0x08005ec8       0x2c build/stm32f7xx_ll_rcc.o
                0x08005ec8                RCC_GetSystemClockFreq
 .text.LL_RCC_GetUSARTClockFreq
                0x08005ef4      0x178 build/stm32f7xx_ll_rcc.o
                0x08005ef4                LL_RCC_GetUSARTClockFreq
 .text.LL_RCC_GetUARTClockFreq
                0x0800606c      0x180 build/stm32f7xx_ll_rcc.o
                0x0800606c                LL_RCC_GetUARTClockFreq
 .text.LL_GPIO_SetPinSpeed
                0x080061ec       0x30 build/stm32f7xx_ll_gpio.o
 .text.LL_GPIO_SetPinPull
                0x0800621c       0x30 build/stm32f7xx_ll_gpio.o
 .text.LL_GPIO_SetAFPin_0_7
                0x0800624c       0x30 build/stm32f7xx_ll_gpio.o
 .text.LL_GPIO_SetAFPin_8_15
                0x0800627c       0x32 build/stm32f7xx_ll_gpio.o
 .text.LL_GPIO_SetPinMode
                0x080062ae       0x30 build/stm32f7xx_ll_gpio.o
 .text.LL_GPIO_Init
                0x080062de       0x8a build/stm32f7xx_ll_gpio.o
                0x080062de                LL_GPIO_Init
 .text.SDMMC_GetCmdError
                0x08006368       0x38 build/stm32f7xx_ll_sdmmc.o
 .text.SDMMC_Init
                0x080063a0       0x34 build/stm32f7xx_ll_sdmmc.o
                0x080063a0                SDMMC_Init
 .text.SDMMC_ReadFIFO
                0x080063d4        0x6 build/stm32f7xx_ll_sdmmc.o
                0x080063d4                SDMMC_ReadFIFO
 .text.SDMMC_WriteFIFO
                0x080063da        0xa build/stm32f7xx_ll_sdmmc.o
                0x080063da                SDMMC_WriteFIFO
 .text.SDMMC_PowerState_ON
                0x080063e4        0x8 build/stm32f7xx_ll_sdmmc.o
                0x080063e4                SDMMC_PowerState_ON
 .text.SDMMC_GetPowerState
                0x080063ec        0x8 build/stm32f7xx_ll_sdmmc.o
                0x080063ec                SDMMC_GetPowerState
 .text.SDMMC_SendCommand
                0x080063f4       0x20 build/stm32f7xx_ll_sdmmc.o
                0x080063f4                SDMMC_SendCommand
 .text.SDMMC_GetCommandResponse
                0x08006414        0x6 build/stm32f7xx_ll_sdmmc.o
                0x08006414                SDMMC_GetCommandResponse
 .text.SDMMC_GetResponse
                0x0800641a        0x6 build/stm32f7xx_ll_sdmmc.o
                0x0800641a                SDMMC_GetResponse
 .text.SDMMC_ConfigData
                0x08006420       0x24 build/stm32f7xx_ll_sdmmc.o
                0x08006420                SDMMC_ConfigData
 .text.SDMMC_CmdGoIdleState
                0x08006444       0x26 build/stm32f7xx_ll_sdmmc.o
                0x08006444                SDMMC_CmdGoIdleState
 *fill*         0x0800646a        0x2 
 .text.SDMMC_GetCmdResp1
                0x0800646c      0x154 build/stm32f7xx_ll_sdmmc.o
                0x0800646c                SDMMC_GetCmdResp1
 .text.SDMMC_CmdBlockLength
                0x080065c0       0x30 build/stm32f7xx_ll_sdmmc.o
                0x080065c0                SDMMC_CmdBlockLength
 .text.SDMMC_CmdReadSingleBlock
                0x080065f0       0x30 build/stm32f7xx_ll_sdmmc.o
                0x080065f0                SDMMC_CmdReadSingleBlock
 .text.SDMMC_CmdReadMultiBlock
                0x08006620       0x30 build/stm32f7xx_ll_sdmmc.o
                0x08006620                SDMMC_CmdReadMultiBlock
 .text.SDMMC_CmdWriteSingleBlock
                0x08006650       0x30 build/stm32f7xx_ll_sdmmc.o
                0x08006650                SDMMC_CmdWriteSingleBlock
 .text.SDMMC_CmdWriteMultiBlock
                0x08006680       0x30 build/stm32f7xx_ll_sdmmc.o
                0x08006680                SDMMC_CmdWriteMultiBlock
 .text.SDMMC_CmdStopTransfer
                0x080066b0       0x34 build/stm32f7xx_ll_sdmmc.o
                0x080066b0                SDMMC_CmdStopTransfer
 .text.SDMMC_CmdSelDesel
                0x080066e4       0x30 build/stm32f7xx_ll_sdmmc.o
                0x080066e4                SDMMC_CmdSelDesel
 .text.SDMMC_CmdAppCommand
                0x08006714       0x30 build/stm32f7xx_ll_sdmmc.o
                0x08006714                SDMMC_CmdAppCommand
 .text.SDMMC_CmdBusWidth
                0x08006744       0x30 build/stm32f7xx_ll_sdmmc.o
                0x08006744                SDMMC_CmdBusWidth
 .text.SDMMC_CmdSendSCR
                0x08006774       0x30 build/stm32f7xx_ll_sdmmc.o
                0x08006774                SDMMC_CmdSendSCR
 .text.SDMMC_CmdSendStatus
                0x080067a4       0x30 build/stm32f7xx_ll_sdmmc.o
                0x080067a4                SDMMC_CmdSendStatus
 .text.SDMMC_GetCmdResp2
                0x080067d4       0x5c build/stm32f7xx_ll_sdmmc.o
                0x080067d4                SDMMC_GetCmdResp2
 .text.SDMMC_CmdSendCID
                0x08006830       0x2a build/stm32f7xx_ll_sdmmc.o
                0x08006830                SDMMC_CmdSendCID
 .text.SDMMC_CmdSendCSD
                0x0800685a       0x2a build/stm32f7xx_ll_sdmmc.o
                0x0800685a                SDMMC_CmdSendCSD
 .text.SDMMC_GetCmdResp3
                0x08006884       0x4c build/stm32f7xx_ll_sdmmc.o
                0x08006884                SDMMC_GetCmdResp3
 .text.SDMMC_CmdAppOperCommand
                0x080068d0       0x34 build/stm32f7xx_ll_sdmmc.o
                0x080068d0                SDMMC_CmdAppOperCommand
 .text.SDMMC_GetCmdResp6
                0x08006904       0xa0 build/stm32f7xx_ll_sdmmc.o
                0x08006904                SDMMC_GetCmdResp6
 .text.SDMMC_CmdSetRelAdd
                0x080069a4       0x30 build/stm32f7xx_ll_sdmmc.o
                0x080069a4                SDMMC_CmdSetRelAdd
 .text.SDMMC_GetCmdResp7
                0x080069d4       0x64 build/stm32f7xx_ll_sdmmc.o
                0x080069d4                SDMMC_GetCmdResp7
 .text.SDMMC_CmdOperCond
                0x08006a38       0x2e build/stm32f7xx_ll_sdmmc.o
                0x08006a38                SDMMC_CmdOperCond
 *fill*         0x08006a66        0x2 
 .text.SD_PowerON
                0x08006a68       0xc0 build/stm32f7xx_hal_sd.o
 .text.SD_FindSCR
                0x08006b28      0x100 build/stm32f7xx_hal_sd.o
 .text.SD_WideBus_Enable
                0x08006c28       0x4e build/stm32f7xx_hal_sd.o
 .text.SD_WideBus_Disable
                0x08006c76       0x4e build/stm32f7xx_hal_sd.o
 .text.SD_SendStatus
                0x08006cc4       0x2c build/stm32f7xx_hal_sd.o
 .text.HAL_SD_ReadBlocks
                0x08006cf0      0x248 build/stm32f7xx_hal_sd.o
                0x08006cf0                HAL_SD_ReadBlocks
 .text.HAL_SD_WriteBlocks
                0x08006f38      0x200 build/stm32f7xx_hal_sd.o
                0x08006f38                HAL_SD_WriteBlocks
 .text.HAL_SD_GetCardCSD
                0x08007138      0x1b8 build/stm32f7xx_hal_sd.o
                0x08007138                HAL_SD_GetCardCSD
 .text.SD_InitCard
                0x080072f0      0x100 build/stm32f7xx_hal_sd.o
 .text.HAL_SD_InitCard
                0x080073f0       0xa8 build/stm32f7xx_hal_sd.o
                0x080073f0                HAL_SD_InitCard
 .text.HAL_SD_Init
                0x08007498       0x36 build/stm32f7xx_hal_sd.o
                0x08007498                HAL_SD_Init
 .text.HAL_SD_GetCardInfo
                0x080074ce       0x24 build/stm32f7xx_hal_sd.o
                0x080074ce                HAL_SD_GetCardInfo
 *fill*         0x080074f2        0x2 
 .text.HAL_SD_ConfigWideBusOperation
                0x080074f4       0xc0 build/stm32f7xx_hal_sd.o
                0x080074f4                HAL_SD_ConfigWideBusOperation
 .text.HAL_SD_GetCardState
                0x080075b4       0x22 build/stm32f7xx_hal_sd.o
                0x080075b4                HAL_SD_GetCardState
 *fill*         0x080075d6        0x2 
 .text.LL_SPI_Init
                0x080075d8       0x8c build/stm32f7xx_ll_spi.o
                0x080075d8                LL_SPI_Init
 .text.TIM_OC1_SetConfig
                0x08007664       0x68 build/stm32f7xx_hal_tim.o
 .text.TIM_OC3_SetConfig
                0x080076cc       0x70 build/stm32f7xx_hal_tim.o
 .text.TIM_OC4_SetConfig
                0x0800773c       0x54 build/stm32f7xx_hal_tim.o
 .text.TIM_OC5_SetConfig
                0x08007790       0x54 build/stm32f7xx_hal_tim.o
 .text.TIM_OC6_SetConfig
                0x080077e4       0x54 build/stm32f7xx_hal_tim.o
 .text.TIM_TI1_ConfigInputStage
                0x08007838       0x26 build/stm32f7xx_hal_tim.o
 .text.TIM_TI2_ConfigInputStage
                0x0800785e       0x28 build/stm32f7xx_hal_tim.o
 .text.TIM_ITRx_SetConfig
                0x08007886       0x10 build/stm32f7xx_hal_tim.o
 .text.HAL_TIM_Base_Stop
                0x08007896       0x28 build/stm32f7xx_hal_tim.o
                0x08007896                HAL_TIM_Base_Stop
 *fill*         0x080078be        0x2 
 .text.HAL_TIM_Base_Start_IT
                0x080078c0       0x90 build/stm32f7xx_hal_tim.o
                0x080078c0                HAL_TIM_Base_Start_IT
 .text.HAL_TIM_Base_Stop_IT
                0x08007950       0x32 build/stm32f7xx_hal_tim.o
                0x08007950                HAL_TIM_Base_Stop_IT
 .text.HAL_TIM_PWM_MspInit
                0x08007982        0x2 build/stm32f7xx_hal_tim.o
                0x08007982                HAL_TIM_PWM_MspInit
 .text.HAL_TIM_PeriodElapsedCallback
                0x08007984        0x2 build/stm32f7xx_hal_tim.o
                0x08007984                HAL_TIM_PeriodElapsedCallback
 .text.HAL_TIM_OC_DelayElapsedCallback
                0x08007986        0x2 build/stm32f7xx_hal_tim.o
                0x08007986                HAL_TIM_OC_DelayElapsedCallback
 .text.HAL_TIM_IC_CaptureCallback
                0x08007988        0x2 build/stm32f7xx_hal_tim.o
                0x08007988                HAL_TIM_IC_CaptureCallback
 .text.HAL_TIM_PWM_PulseFinishedCallback
                0x0800798a        0x2 build/stm32f7xx_hal_tim.o
                0x0800798a                HAL_TIM_PWM_PulseFinishedCallback
 .text.HAL_TIM_TriggerCallback
                0x0800798c        0x2 build/stm32f7xx_hal_tim.o
                0x0800798c                HAL_TIM_TriggerCallback
 .text.HAL_TIM_IRQHandler
                0x0800798e      0x17a build/stm32f7xx_hal_tim.o
                0x0800798e                HAL_TIM_IRQHandler
 .text.TIM_Base_SetConfig
                0x08007b08      0x120 build/stm32f7xx_hal_tim.o
                0x08007b08                TIM_Base_SetConfig
 .text.HAL_TIM_Base_Init
                0x08007c28       0x60 build/stm32f7xx_hal_tim.o
                0x08007c28                HAL_TIM_Base_Init
 .text.HAL_TIM_PWM_Init
                0x08007c88       0x60 build/stm32f7xx_hal_tim.o
                0x08007c88                HAL_TIM_PWM_Init
 .text.TIM_OC2_SetConfig
                0x08007ce8       0x70 build/stm32f7xx_hal_tim.o
                0x08007ce8                TIM_OC2_SetConfig
 .text.HAL_TIM_PWM_ConfigChannel
                0x08007d58      0x13a build/stm32f7xx_hal_tim.o
                0x08007d58                HAL_TIM_PWM_ConfigChannel
 .text.TIM_ETR_SetConfig
                0x08007e92       0x1a build/stm32f7xx_hal_tim.o
                0x08007e92                TIM_ETR_SetConfig
 .text.HAL_TIM_ConfigClockSource
                0x08007eac      0x100 build/stm32f7xx_hal_tim.o
                0x08007eac                HAL_TIM_ConfigClockSource
 .text.TIM_CCxChannelCmd
                0x08007fac       0x1e build/stm32f7xx_hal_tim.o
                0x08007fac                TIM_CCxChannelCmd
 *fill*         0x08007fca        0x2 
 .text.HAL_TIM_PWM_Start
                0x08007fcc      0x158 build/stm32f7xx_hal_tim.o
                0x08007fcc                HAL_TIM_PWM_Start
 .text.HAL_TIM_PWM_Stop
                0x08008124       0xac build/stm32f7xx_hal_tim.o
                0x08008124                HAL_TIM_PWM_Stop
 .text.HAL_TIMEx_MasterConfigSynchronization
                0x080081d0       0xa0 build/stm32f7xx_hal_tim_ex.o
                0x080081d0                HAL_TIMEx_MasterConfigSynchronization
 .text.HAL_TIMEx_CommutCallback
                0x08008270        0x2 build/stm32f7xx_hal_tim_ex.o
                0x08008270                HAL_TIMEx_CommutCallback
 .text.HAL_TIMEx_BreakCallback
                0x08008272        0x2 build/stm32f7xx_hal_tim_ex.o
                0x08008272                HAL_TIMEx_BreakCallback
 .text.HAL_TIMEx_Break2Callback
                0x08008274        0x2 build/stm32f7xx_hal_tim_ex.o
                0x08008274                HAL_TIMEx_Break2Callback
 *fill*         0x08008276        0x2 
 .text.LL_TIM_Init
                0x08008278      0x110 build/stm32f7xx_ll_tim.o
                0x08008278                LL_TIM_Init
 .text.LL_USART_SetBaudRate
                0x08008388       0x2e build/stm32f7xx_ll_usart.o
 *fill*         0x080083b6        0x2 
 .text.LL_USART_Init
                0x080083b8       0xfc build/stm32f7xx_ll_usart.o
                0x080083b8                LL_USART_Init
 .text.SystemInit
                0x080084b4       0x14 build/system_stm32f7xx.o
                0x080084b4                SystemInit
 .text.Mount_SD
                0x080084c8       0x24 build/File_Handling.o
                0x080084c8                Mount_SD
 .text.Unmount_SD
                0x080084ec       0x20 build/File_Handling.o
                0x080084ec                Unmount_SD
 .text.Write_File_byte
                0x0800850c       0x5c build/File_Handling.o
                0x0800850c                Write_File_byte
 .text.Seek_Read_File
                0x08008568      0x148 build/File_Handling.o
                0x08008568                Seek_Read_File
 .text.Create_File
                0x080086b0       0x44 build/File_Handling.o
                0x080086b0                Create_File
 .text.Remove_File
                0x080086f4       0x84 build/File_Handling.o
                0x080086f4                Remove_File
 .text.Update_File_byte
                0x08008778       0x5c build/File_Handling.o
                0x08008778                Update_File_byte
 .text.disk_status
                0x080087d4       0x18 build/diskio.o
                0x080087d4                disk_status
 .text.disk_initialize
                0x080087ec       0x28 build/diskio.o
                0x080087ec                disk_initialize
 .text.disk_read
                0x08008814       0x18 build/diskio.o
                0x08008814                disk_read
 .text.disk_write
                0x0800882c       0x18 build/diskio.o
                0x0800882c                disk_write
 .text.disk_ioctl
                0x08008844       0x18 build/diskio.o
                0x08008844                disk_ioctl
 .text.ld_word  0x0800885c        0xa build/ff.o
 .text.ld_dword
                0x08008866       0x16 build/ff.o
 .text.st_word  0x0800887c        0x8 build/ff.o
 .text.st_dword
                0x08008884       0x14 build/ff.o
 .text.mem_cpy  0x08008898       0x14 build/ff.o
 .text.mem_set  0x080088ac        0xa build/ff.o
 .text.mem_cmp  0x080088b6       0x1a build/ff.o
 .text.chk_chr  0x080088d0       0x10 build/ff.o
 .text.chk_lock
                0x080088e0       0x7c build/ff.o
 .text.enq_lock
                0x0800895c       0x20 build/ff.o
 .text.inc_lock
                0x0800897c       0xa0 build/ff.o
 .text.dec_lock
                0x08008a1c       0x40 build/ff.o
 .text.clear_lock
                0x08008a5c       0x3c build/ff.o
 .text.clust2sect
                0x08008a98       0x18 build/ff.o
 .text.clmt_clust
                0x08008ab0       0x26 build/ff.o
 .text.ld_clust
                0x08008ad6       0x26 build/ff.o
 .text.st_clust
                0x08008afc       0x26 build/ff.o
 .text.get_fileinfo
                0x08008b22       0x6a build/ff.o
 .text.create_name
                0x08008b8c       0xd0 build/ff.o
 .text.get_ldnumber
                0x08008c5c       0x48 build/ff.o
 .text.validate
                0x08008ca4       0x46 build/ff.o
 .text.sync_window
                0x08008cea       0x54 build/ff.o
 .text.move_window
                0x08008d3e       0x36 build/ff.o
 .text.check_fs
                0x08008d74       0x78 build/ff.o
 .text.find_volume
                0x08008dec      0x34c build/ff.o
 .text.put_fat  0x08009138      0x136 build/ff.o
 .text.get_fat  0x0800926e       0xfc build/ff.o
 .text.dir_sdi  0x0800936a       0xc0 build/ff.o
 .text.create_chain
                0x0800942a       0xd6 build/ff.o
 .text.remove_chain
                0x08009500       0x7e build/ff.o
 .text.dir_remove
                0x0800957e       0x1c build/ff.o
 .text.dir_next
                0x0800959a      0x118 build/ff.o
 .text.dir_find
                0x080096b2       0x5a build/ff.o
 .text.follow_path
                0x0800970c       0x92 build/ff.o
 .text.dir_alloc
                0x0800979e       0x4e build/ff.o
 .text.dir_register
                0x080097ec       0x3e build/ff.o
 .text.dir_read
                0x0800982a       0x5e build/ff.o
 .text.sync_fs  0x08009888       0x88 build/ff.o
 .text.f_mount  0x08009910       0x60 build/ff.o
                0x08009910                f_mount
 .text.f_open   0x08009970      0x232 build/ff.o
                0x08009970                f_open
 .text.f_read   0x08009ba2      0x1d8 build/ff.o
                0x08009ba2                f_read
 .text.f_write  0x08009d7a      0x210 build/ff.o
                0x08009d7a                f_write
 .text.f_sync   0x08009f8a       0x98 build/ff.o
                0x08009f8a                f_sync
 .text.f_close  0x0800a022       0x2a build/ff.o
                0x0800a022                f_close
 .text.f_lseek  0x0800a04c      0x2a6 build/ff.o
                0x0800a04c                f_lseek
 .text.f_stat   0x0800a2f2       0x44 build/ff.o
                0x0800a2f2                f_stat
 .text.f_unlink
                0x0800a336       0xc4 build/ff.o
                0x0800a336                f_unlink
 *fill*         0x0800a3fa        0x2 
 .text.FATFS_LinkDriverEx
                0x0800a3fc       0x54 build/ff_gen_drv.o
                0x0800a3fc                FATFS_LinkDriverEx
 .text.FATFS_LinkDriver
                0x0800a450        0xa build/ff_gen_drv.o
                0x0800a450                FATFS_LinkDriver
 *fill*         0x0800a45a        0x2 
 .text._sbrk    0x0800a45c       0x48 build/sysmem.o
                0x0800a45c                _sbrk
 .text.UART_EndRxTransfer
                0x0800a4a4       0x52 build/stm32f7xx_hal_uart.o
 *fill*         0x0800a4f6        0x2 
 .text.UART_SetConfig
                0x0800a4f8      0x328 build/stm32f7xx_hal_uart.o
                0x0800a4f8                UART_SetConfig
 .text.UART_AdvFeatureConfig
                0x0800a820       0xca build/stm32f7xx_hal_uart.o
                0x0800a820                UART_AdvFeatureConfig
 .text.UART_WaitOnFlagUntilTimeout
                0x0800a8ea       0xa6 build/stm32f7xx_hal_uart.o
                0x0800a8ea                UART_WaitOnFlagUntilTimeout
 .text.UART_CheckIdleState
                0x0800a990       0xc6 build/stm32f7xx_hal_uart.o
                0x0800a990                UART_CheckIdleState
 .text.HAL_UART_Init
                0x0800aa56       0x62 build/stm32f7xx_hal_uart.o
                0x0800aa56                HAL_UART_Init
 .text.Reset_Handler
                0x0800aab8       0x50 build/startup_stm32f767xx.o
                0x0800aab8                Reset_Handler
 .text.Default_Handler
                0x0800ab08        0x2 build/startup_stm32f767xx.o
                0x0800ab08                RTC_Alarm_IRQHandler
                0x0800ab08                EXTI2_IRQHandler
                0x0800ab08                TIM8_CC_IRQHandler
                0x0800ab08                UART8_IRQHandler
                0x0800ab08                SPI4_IRQHandler
                0x0800ab08                TIM1_CC_IRQHandler
                0x0800ab08                DMA2_Stream5_IRQHandler
                0x0800ab08                JPEG_IRQHandler
                0x0800ab08                DMA1_Stream5_IRQHandler
                0x0800ab08                CAN3_RX1_IRQHandler
                0x0800ab08                PVD_IRQHandler
                0x0800ab08                TAMP_STAMP_IRQHandler
                0x0800ab08                CAN2_RX1_IRQHandler
                0x0800ab08                EXTI3_IRQHandler
                0x0800ab08                TIM8_TRG_COM_TIM14_IRQHandler
                0x0800ab08                DFSDM1_FLT1_IRQHandler
                0x0800ab08                I2C3_ER_IRQHandler
                0x0800ab08                DFSDM1_FLT2_IRQHandler
                0x0800ab08                EXTI0_IRQHandler
                0x0800ab08                I2C2_EV_IRQHandler
                0x0800ab08                DMA1_Stream2_IRQHandler
                0x0800ab08                CAN1_RX0_IRQHandler
                0x0800ab08                FPU_IRQHandler
                0x0800ab08                OTG_HS_WKUP_IRQHandler
                0x0800ab08                CAN3_SCE_IRQHandler
                0x0800ab08                LTDC_ER_IRQHandler
                0x0800ab08                CAN2_SCE_IRQHandler
                0x0800ab08                DMA2_Stream2_IRQHandler
                0x0800ab08                SPI1_IRQHandler
                0x0800ab08                TIM1_BRK_TIM9_IRQHandler
                0x0800ab08                DCMI_IRQHandler
                0x0800ab08                CAN2_RX0_IRQHandler
                0x0800ab08                DMA2_Stream3_IRQHandler
                0x0800ab08                SAI2_IRQHandler
                0x0800ab08                DFSDM1_FLT3_IRQHandler
                0x0800ab08                USART6_IRQHandler
                0x0800ab08                CAN3_RX0_IRQHandler
                0x0800ab08                USART3_IRQHandler
                0x0800ab08                CAN1_RX1_IRQHandler
                0x0800ab08                UART5_IRQHandler
                0x0800ab08                DMA2_Stream0_IRQHandler
                0x0800ab08                TIM4_IRQHandler
                0x0800ab08                QUADSPI_IRQHandler
                0x0800ab08                I2C1_EV_IRQHandler
                0x0800ab08                DMA1_Stream6_IRQHandler
                0x0800ab08                DMA1_Stream1_IRQHandler
                0x0800ab08                UART4_IRQHandler
                0x0800ab08                TIM3_IRQHandler
                0x0800ab08                RCC_IRQHandler
                0x0800ab08                TIM8_BRK_TIM12_IRQHandler
                0x0800ab08                Default_Handler
                0x0800ab08                CEC_IRQHandler
                0x0800ab08                EXTI15_10_IRQHandler
                0x0800ab08                DMA1_Stream7_IRQHandler
                0x0800ab08                SPI5_IRQHandler
                0x0800ab08                SDMMC1_IRQHandler
                0x0800ab08                CAN2_TX_IRQHandler
                0x0800ab08                I2C3_EV_IRQHandler
                0x0800ab08                EXTI9_5_IRQHandler
                0x0800ab08                RTC_WKUP_IRQHandler
                0x0800ab08                LTDC_IRQHandler
                0x0800ab08                ETH_WKUP_IRQHandler
                0x0800ab08                SPDIF_RX_IRQHandler
                0x0800ab08                SPI2_IRQHandler
                0x0800ab08                OTG_HS_EP1_IN_IRQHandler
                0x0800ab08                DMA1_Stream0_IRQHandler
                0x0800ab08                CAN1_TX_IRQHandler
                0x0800ab08                EXTI4_IRQHandler
                0x0800ab08                RNG_IRQHandler
                0x0800ab08                ETH_IRQHandler
                0x0800ab08                OTG_HS_EP1_OUT_IRQHandler
                0x0800ab08                WWDG_IRQHandler
                0x0800ab08                SPI6_IRQHandler
                0x0800ab08                MDIOS_IRQHandler
                0x0800ab08                I2C4_EV_IRQHandler
                0x0800ab08                CAN3_TX_IRQHandler
                0x0800ab08                OTG_FS_WKUP_IRQHandler
                0x0800ab08                OTG_HS_IRQHandler
                0x0800ab08                DMA2D_IRQHandler
                0x0800ab08                EXTI1_IRQHandler
                0x0800ab08                SDMMC2_IRQHandler
                0x0800ab08                UART7_IRQHandler
                0x0800ab08                USART2_IRQHandler
                0x0800ab08                DFSDM1_FLT0_IRQHandler
                0x0800ab08                I2C2_ER_IRQHandler
                0x0800ab08                DMA2_Stream1_IRQHandler
                0x0800ab08                CAN1_SCE_IRQHandler
                0x0800ab08                FLASH_IRQHandler
                0x0800ab08                DMA2_Stream4_IRQHandler
                0x0800ab08                OTG_FS_IRQHandler
                0x0800ab08                SPI3_IRQHandler
                0x0800ab08                DMA1_Stream4_IRQHandler
                0x0800ab08                I2C1_ER_IRQHandler
                0x0800ab08                FMC_IRQHandler
                0x0800ab08                LPTIM1_IRQHandler
                0x0800ab08                I2C4_ER_IRQHandler
                0x0800ab08                DMA2_Stream6_IRQHandler
                0x0800ab08                SAI1_IRQHandler
                0x0800ab08                DMA1_Stream3_IRQHandler
 *(.glue_7)
 .glue_7        0x0800ab0a        0x0 linker stubs
 *(.glue_7t)
 .glue_7t       0x0800ab0a        0x0 linker stubs
 *(.eh_frame)
 *fill*         0x0800ab0a        0x2 
 .eh_frame      0x0800ab0c        0x0 /usr/lib/gcc/arm-none-eabi/13.2.1/thumb/v7e-m+dp/hard/crtbegin.o
 *(.init)
 .init          0x0800ab0c        0x4 /usr/lib/gcc/arm-none-eabi/13.2.1/thumb/v7e-m+dp/hard/crti.o
                0x0800ab0c                _init
 .init          0x0800ab10        0x8 /usr/lib/gcc/arm-none-eabi/13.2.1/thumb/v7e-m+dp/hard/crtn.o
 *(.fini)
 .fini          0x0800ab18        0x4 /usr/lib/gcc/arm-none-eabi/13.2.1/thumb/v7e-m+dp/hard/crti.o
                0x0800ab18                _fini
 .fini          0x0800ab1c        0x8 /usr/lib/gcc/arm-none-eabi/13.2.1/thumb/v7e-m+dp/hard/crtn.o
                0x0800ab24                        . = ALIGN (0x4)
                0x0800ab24                        _etext = .

.vfp11_veneer   0x0800ab24        0x0
 .vfp11_veneer  0x0800ab24        0x0 linker stubs

.v4_bx          0x0800ab24        0x0
 .v4_bx         0x0800ab24        0x0 linker stubs

.iplt           0x0800ab24        0x0
 .iplt          0x0800ab24        0x0 /usr/lib/gcc/arm-none-eabi/13.2.1/thumb/v7e-m+dp/hard/crtbegin.o

.rodata         0x0800ab24      0x25c
                0x0800ab24                        . = ALIGN (0x4)
 *(.rodata)
 *(.rodata*)
 .rodata.Init_params.str1.4
                0x0800ab24      0x1ad build/main.o
                                 0x10 (size before relaxing)
 .rodata.SD_SAVE.str1.4
                0x0800acd1        0xa build/main.o
 *fill*         0x0800acd1        0x3 
 .rodata.SD_Driver
                0x0800acd4       0x14 build/sd_diskio.o
                0x0800acd4                SD_Driver
 .rodata.APBPrescTable
                0x0800ace8        0x8 build/system_stm32f7xx.o
                0x0800ace8                APBPrescTable
 .rodata.AHBPrescTable
                0x0800acf0       0x10 build/system_stm32f7xx.o
                0x0800acf0                AHBPrescTable
 .rodata.Read_File.str1.4
                0x0800ad00       0xbb build/File_Handling.o
 .rodata.Seek_Read_File.str1.4
                0x0800ad00       0x27 build/File_Handling.o
 .rodata.Remove_File.str1.4
                0x0800ad00       0x64 build/File_Handling.o
 .rodata.create_name.str1.4
                0x0800ad00        0xf build/ff.o
 .rodata.ExCvt  0x0800ad00       0x80 build/ff.o
 .rodata.str1.4
                0x0800ad80       0x13 /usr/lib/gcc/arm-none-eabi/13.2.1/../../../arm-none-eabi/lib/thumb/v7e-m+dp/hard/libc_nano.a(libc_a-nano-svfprintf.o)
 .rodata.str1.4
                0x0800ad80       0x25 /usr/lib/gcc/arm-none-eabi/13.2.1/../../../arm-none-eabi/lib/thumb/v7e-m+dp/hard/libc_nano.a(libc_a-nano-vfprintf_i.o)
                0x0800adbc                        . = ALIGN (0x4)

.ARM.extab
 *(.ARM.extab* .gnu.linkonce.armextab.*)

.ARM            0x0800ad80        0x8
                0x0800ad80                        __exidx_start = .
 *(.ARM.exidx*)
 .ARM.exidx     0x0800ad80        0x8 /usr/lib/gcc/arm-none-eabi/13.2.1/../../../arm-none-eabi/lib/thumb/v7e-m+dp/hard/libc_nano.a(libc_a-memchr.o)
 .ARM.exidx     0x0800ad88        0x0 /usr/lib/gcc/arm-none-eabi/13.2.1/../../../arm-none-eabi/lib/thumb/v7e-m+dp/hard/libc_nano.a(libc_a-memcpy.o)
                                  0x8 (size before relaxing)
 .ARM.exidx     0x0800ad88        0x0 /usr/lib/gcc/arm-none-eabi/13.2.1/thumb/v7e-m+dp/hard/libgcc.a(_udivmoddi4.o)
                                  0x8 (size before relaxing)
                0x0800ad88                        __exidx_end = .

.rel.dyn        0x0800ad88        0x0
 .rel.iplt      0x0800ad88        0x0 /usr/lib/gcc/arm-none-eabi/13.2.1/thumb/v7e-m+dp/hard/crtbegin.o

.preinit_array  0x0800ad88        0x0
                0x0800ad88                        PROVIDE (__preinit_array_start = .)
 *(.preinit_array*)
                0x0800ad88                        PROVIDE (__preinit_array_end = .)

.init_array     0x0800ad88        0x4
                0x0800ad88                        PROVIDE (__init_array_start = .)
 *(SORT_BY_NAME(.init_array.*))
 *(.init_array*)
 .init_array    0x0800ad88        0x4 /usr/lib/gcc/arm-none-eabi/13.2.1/thumb/v7e-m+dp/hard/crtbegin.o
                0x0800ad8c                        PROVIDE (__init_array_end = .)

.fini_array     0x0800ad8c        0x4
                0x0800ad8c                        PROVIDE (__fini_array_start = .)
 *(SORT_BY_NAME(.fini_array.*))
 *(.fini_array*)
 .fini_array    0x0800ad8c        0x4 /usr/lib/gcc/arm-none-eabi/13.2.1/thumb/v7e-m+dp/hard/crtbegin.o
                0x0800ad90                        PROVIDE (__fini_array_end = .)
                0x0800ad90                        _sidata = LOADADDR (.data)

.data           0x20000000       0x5c load address 0x0800ad90
                0x20000000                        . = ALIGN (0x4)
                0x20000000                        _sdata = .
 *(.data)
 .data          0x20000000       0x50 /usr/lib/gcc/arm-none-eabi/13.2.1/../../../arm-none-eabi/lib/thumb/v7e-m+dp/hard/libc_nano.a(libc_a-impure.o)
                0x20000000                _impure_ptr
                0x20000004                _impure_data
 *(.data*)
 .data.Stat     0x20000050        0x1 build/sd_diskio.o
 .data.uwTickFreq
                0x20000051        0x1 build/stm32f7xx_hal.o
                0x20000051                uwTickFreq
 *fill*         0x20000052        0x2 
 .data.uwTickPrio
                0x20000054        0x4 build/stm32f7xx_hal.o
                0x20000054                uwTickPrio
 .data.SystemCoreClock
                0x20000058        0x4 build/system_stm32f7xx.o
                0x20000058                SystemCoreClock
                0x2000005c                        . = ALIGN (0x4)
                0x2000005c                        _edata = .

.tm_clone_table
                0x2000005c        0x0 load address 0x0800adec
 .tm_clone_table
                0x2000005c        0x0 /usr/lib/gcc/arm-none-eabi/13.2.1/thumb/v7e-m+dp/hard/crtbegin.o
 .tm_clone_table
                0x2000005c        0x0 /usr/lib/gcc/arm-none-eabi/13.2.1/thumb/v7e-m+dp/hard/crtend.o

.igot.plt       0x2000005c        0x0 load address 0x0800adec
 .igot.plt      0x2000005c        0x0 /usr/lib/gcc/arm-none-eabi/13.2.1/thumb/v7e-m+dp/hard/crtbegin.o
                0x2000005c                        . = ALIGN (0x4)

.bss            0x2000005c     0x266c load address 0x0800adec
                0x2000005c                        _sbss = .
                0x2000005c                        __bss_start__ = _sbss
 *(.bss)
 .bss           0x2000005c       0x1c /usr/lib/gcc/arm-none-eabi/13.2.1/thumb/v7e-m+dp/hard/crtbegin.o
 .bss           0x20000078        0x8 /usr/lib/gcc/arm-none-eabi/13.2.1/../../../arm-none-eabi/lib/thumb/v7e-m+dp/hard/libc_nano.a(libc_a-mallocr.o)
                0x20000078                __malloc_sbrk_start
                0x2000007c                __malloc_free_list
 .bss           0x20000080      0x13c /usr/lib/gcc/arm-none-eabi/13.2.1/../../../arm-none-eabi/lib/thumb/v7e-m+dp/hard/libc_nano.a(libc_a-findfp.o)
                0x20000080                __sf
                0x200001b8                __stdio_exit_handler
 .bss           0x200001bc        0x4 /usr/lib/gcc/arm-none-eabi/13.2.1/../../../arm-none-eabi/lib/thumb/v7e-m+dp/hard/libc_nano.a(libc_a-reent.o)
                0x200001bc                errno
 *(.bss*)
 .bss.task      0x200001c0       0x34 build/main.o
                0x200001c0                task
 .bss.LD_blinker
                0x200001f4        0xc build/main.o
                0x200001f4                LD_blinker
 .bss.LD2_param
                0x20000200        0xc build/main.o
                0x20000200                LD2_param
 .bss.LD1_param
                0x2000020c        0xc build/main.o
                0x2000020c                LD1_param
 .bss.Def_setup
                0x20000218       0x12 build/main.o
                0x20000218                Def_setup
 *fill*         0x2000022a        0x2 
 .bss.Curr_setup
                0x2000022c       0x12 build/main.o
                0x2000022c                Curr_setup
 *fill*         0x2000023e        0x2 
 .bss.LD2_def_setup
                0x20000240       0x10 build/main.o
                0x20000240                LD2_def_setup
 .bss.LD1_def_setup
                0x20000250       0x10 build/main.o
                0x20000250                LD1_def_setup
 .bss.LD2_curr_setup
                0x20000260       0x10 build/main.o
                0x20000260                LD2_curr_setup
 .bss.LD1_curr_setup
                0x20000270       0x10 build/main.o
                0x20000270                LD1_curr_setup
 .bss.sizeoffile
                0x20000280        0x4 build/main.o
                0x20000280                sizeoffile
 .bss.fgoto     0x20000284        0x4 build/main.o
                0x20000284                fgoto
 .bss.test      0x20000288        0x4 build/main.o
                0x20000288                test
 .bss.fresult   0x2000028c        0x1 build/main.o
                0x2000028c                fresult
 *fill*         0x2000028d        0x3 
 .bss.COMMAND   0x20000290       0x1e build/main.o
                0x20000290                COMMAND
 *fill*         0x200002ae        0x2 
 .bss.Long_Data
                0x200002b0       0x1e build/main.o
                0x200002b0                Long_Data
 .bss.temp16    0x200002ce        0x2 build/main.o
                0x200002ce                temp16
 .bss.CS_result
                0x200002d0        0x2 build/main.o
                0x200002d0                CS_result
 .bss.UART_header
                0x200002d2        0x2 build/main.o
                0x200002d2                UART_header
 .bss.UART_rec_incr
                0x200002d4        0x2 build/main.o
                0x200002d4                UART_rec_incr
 .bss.TIM10_coflag
                0x200002d6        0x1 build/main.o
                0x200002d6                TIM10_coflag
 .bss.u_rx_flg  0x200002d7        0x1 build/main.o
                0x200002d7                u_rx_flg
 .bss.u_tx_flg  0x200002d8        0x1 build/main.o
                0x200002d8                u_tx_flg
 .bss.flg_tmt   0x200002d9        0x1 build/main.o
                0x200002d9                flg_tmt
 *fill*         0x200002da        0x2 
 .bss.UART_DATA
                0x200002dc       0x1e build/main.o
                0x200002dc                UART_DATA
 *fill*         0x200002fa        0x2 
 .bss.State_Data
                0x200002fc        0x2 build/main.o
                0x200002fc                State_Data
 .bss.UART_transmission_request
                0x200002fe        0x1 build/main.o
                0x200002fe                UART_transmission_request
 .bss.CPU_state_old
                0x200002ff        0x1 build/main.o
                0x200002ff                CPU_state_old
 .bss.CPU_state
                0x20000300        0x1 build/main.o
                0x20000300                CPU_state
 .bss.uart_buf  0x20000301        0x1 build/main.o
                0x20000301                uart_buf
 *fill*         0x20000302        0x2 
 .bss.TIM10_period
                0x20000304        0x4 build/main.o
                0x20000304                TIM10_period
 .bss.TO10_counter
                0x20000308        0x4 build/main.o
                0x20000308                TO10_counter
 .bss.TO10      0x2000030c        0x4 build/main.o
                0x2000030c                TO10
 .bss.TO7_PID   0x20000310        0x4 build/main.o
                0x20000310                TO7_PID
 .bss.TO7_before
                0x20000314        0x4 build/main.o
                0x20000314                TO7_before
 .bss.TO7       0x20000318        0x4 build/main.o
                0x20000318                TO7
 .bss.SD_SLIDE  0x2000031c        0x4 build/main.o
                0x2000031c                SD_SLIDE
 .bss.SD_SEEK   0x20000320        0x4 build/main.o
                0x20000320                SD_SEEK
 .bss.TO6_uart  0x20000324        0x4 build/main.o
                0x20000324                TO6_uart
 .bss.TO6_stop  0x20000328        0x4 build/main.o
                0x20000328                TO6_stop
 .bss.TO6_before
                0x2000032c        0x4 build/main.o
                0x2000032c                TO6_before
 .bss.TO6       0x20000330        0x4 build/main.o
                0x20000330                TO6
 .bss.huart8    0x20000334       0x88 build/main.o
                0x20000334                huart8
 .bss.htim11    0x200003bc       0x4c build/main.o
                0x200003bc                htim11
 .bss.htim10    0x20000408       0x4c build/main.o
                0x20000408                htim10
 .bss.htim8     0x20000454       0x4c build/main.o
                0x20000454                htim8
 .bss.htim4     0x200004a0       0x4c build/main.o
                0x200004a0                htim4
 .bss.hsd1      0x200004ec       0x84 build/main.o
                0x200004ec                hsd1
 .bss.hadc3     0x20000570       0x48 build/main.o
                0x20000570                hadc3
 .bss.hadc1     0x200005b8       0x48 build/main.o
                0x200005b8                hadc1
 .bss.SDPath    0x20000600        0x4 build/fatfs.o
                0x20000600                SDPath
 .bss.retSD     0x20000604        0x1 build/fatfs.o
                0x20000604                retSD
 *fill*         0x20000605        0x3 
 .bss.uwTick    0x20000608        0x4 build/stm32f7xx_hal.o
                0x20000608                uwTick
 .bss.bw        0x2000060c        0x4 build/File_Handling.o
                0x2000060c                bw
 .bss.br        0x20000610        0x4 build/File_Handling.o
                0x20000610                br
 .bss.fno       0x20000614       0x18 build/File_Handling.o
                0x20000614                fno
 .bss.fil       0x2000062c     0x1030 build/File_Handling.o
                0x2000062c                fil
 .bss.fs        0x2000165c     0x1034 build/File_Handling.o
                0x2000165c                fs
 .bss.Files     0x20002690       0x20 build/ff.o
 .bss.Fsid      0x200026b0        0x2 build/ff.o
 *fill*         0x200026b2        0x2 
 .bss.FatFs     0x200026b4        0x4 build/ff.o
 .bss.disk      0x200026b8        0xc build/ff_gen_drv.o
                0x200026b8                disk
 .bss.__sbrk_heap_end
                0x200026c4        0x4 build/sysmem.o
 *(COMMON)
                0x200026c8                        . = ALIGN (0x4)
                0x200026c8                        _ebss = .
                0x200026c8                        __bss_end__ = _ebss

._user_heap_stack
                0x200026c8     0x6000 load address 0x0800adec
                0x200026c8                        . = ALIGN (0x8)
                [!provide]                        PROVIDE (end = .)
                0x200026c8                        PROVIDE (_end = .)
                0x200046c8                        . = (. + _Min_Heap_Size)
 *fill*         0x200026c8     0x2000 
                0x200086c8                        . = (. + _Min_Stack_Size)
 *fill*         0x200046c8     0x4000 
                0x200086c8                        . = ALIGN (0x8)

/DISCARD/
 libc.a(*)
 libm.a(*)
 libgcc.a(*)
OUTPUT(build/For_stm32.elf elf32-littlearm)
LOAD linker stubs
LOAD /usr/lib/gcc/arm-none-eabi/13.2.1/../../../arm-none-eabi/lib/thumb/v7e-m+dp/hard/libc.a
LOAD /usr/lib/gcc/arm-none-eabi/13.2.1/../../../arm-none-eabi/lib/thumb/v7e-m+dp/hard/libm.a
LOAD /usr/lib/gcc/arm-none-eabi/13.2.1/thumb/v7e-m+dp/hard/libgcc.a

.ARM.attributes
                0x00000000       0x2e
 .ARM.attributes
                0x00000000       0x20 /usr/lib/gcc/arm-none-eabi/13.2.1/thumb/v7e-m+dp/hard/crti.o
 .ARM.attributes
                0x00000020       0x32 /usr/lib/gcc/arm-none-eabi/13.2.1/thumb/v7e-m+dp/hard/crtbegin.o
 .ARM.attributes
                0x00000052       0x32 build/main.o
 .ARM.attributes
                0x00000084       0x32 build/bsp_driver_sd.o
 .ARM.attributes
                0x000000b6       0x32 build/sd_diskio.o
 .ARM.attributes
                0x000000e8       0x32 build/fatfs.o
 .ARM.attributes
                0x0000011a       0x32 build/fatfs_platform.o
 .ARM.attributes
                0x0000014c       0x32 build/stm32f7xx_it.o
 .ARM.attributes
                0x0000017e       0x32 build/stm32f7xx_hal_msp.o
 .ARM.attributes
                0x000001b0       0x32 build/stm32f7xx_hal_adc.o
 .ARM.attributes
                0x000001e2       0x32 build/stm32f7xx_hal_adc_ex.o
 .ARM.attributes
                0x00000214       0x32 build/stm32f7xx_hal_rcc.o
 .ARM.attributes
                0x00000246       0x32 build/stm32f7xx_hal_rcc_ex.o
 .ARM.attributes
                0x00000278       0x32 build/stm32f7xx_hal_gpio.o
 .ARM.attributes
                0x000002aa       0x32 build/stm32f7xx_hal_pwr_ex.o
 .ARM.attributes
                0x000002dc       0x32 build/stm32f7xx_hal_cortex.o
 .ARM.attributes
                0x0000030e       0x32 build/stm32f7xx_hal.o
 .ARM.attributes
                0x00000340       0x32 build/stm32f7xx_ll_rcc.o
 .ARM.attributes
                0x00000372       0x32 build/stm32f7xx_ll_gpio.o
 .ARM.attributes
                0x000003a4       0x32 build/stm32f7xx_ll_sdmmc.o
 .ARM.attributes
                0x000003d6       0x32 build/stm32f7xx_hal_sd.o
 .ARM.attributes
                0x00000408       0x32 build/stm32f7xx_ll_spi.o
 .ARM.attributes
                0x0000043a       0x32 build/stm32f7xx_hal_tim.o
 .ARM.attributes
                0x0000046c       0x32 build/stm32f7xx_hal_tim_ex.o
 .ARM.attributes
                0x0000049e       0x32 build/stm32f7xx_ll_tim.o
 .ARM.attributes
                0x000004d0       0x32 build/stm32f7xx_ll_usart.o
 .ARM.attributes
                0x00000502       0x32 build/system_stm32f7xx.o
 .ARM.attributes
                0x00000534       0x32 build/File_Handling.o
 .ARM.attributes
                0x00000566       0x32 build/diskio.o
 .ARM.attributes
                0x00000598       0x32 build/ff.o
 .ARM.attributes
                0x000005ca       0x32 build/ff_gen_drv.o
 .ARM.attributes
                0x000005fc       0x32 build/sysmem.o
 .ARM.attributes
                0x0000062e       0x32 build/stm32f7xx_hal_uart.o
 .ARM.attributes
                0x00000660       0x21 build/startup_stm32f767xx.o
 .ARM.attributes
                0x00000681       0x32 /usr/lib/gcc/arm-none-eabi/13.2.1/../../../arm-none-eabi/lib/thumb/v7e-m+dp/hard/libc_nano.a(libc_a-sprintf.o)
 .ARM.attributes
                0x000006b3       0x32 /usr/lib/gcc/arm-none-eabi/13.2.1/../../../arm-none-eabi/lib/thumb/v7e-m+dp/hard/libc_nano.a(libc_a-impure.o)
 .ARM.attributes
                0x000006e5       0x32 /usr/lib/gcc/arm-none-eabi/13.2.1/../../../arm-none-eabi/lib/thumb/v7e-m+dp/hard/libc_nano.a(libc_a-nano-svfprintf.o)
 .ARM.attributes
                0x00000717       0x32 /usr/lib/gcc/arm-none-eabi/13.2.1/../../../arm-none-eabi/lib/thumb/v7e-m+dp/hard/libc_nano.a(libc_a-init.o)
 .ARM.attributes
                0x00000749       0x32 /usr/lib/gcc/arm-none-eabi/13.2.1/../../../arm-none-eabi/lib/thumb/v7e-m+dp/hard/libc_nano.a(libc_a-memset.o)
 .ARM.attributes
                0x0000077b       0x32 /usr/lib/gcc/arm-none-eabi/13.2.1/../../../arm-none-eabi/lib/thumb/v7e-m+dp/hard/libc_nano.a(libc_a-errno.o)
 .ARM.attributes
                0x000007ad       0x32 /usr/lib/gcc/arm-none-eabi/13.2.1/../../../arm-none-eabi/lib/thumb/v7e-m+dp/hard/libc_nano.a(libc_a-mallocr.o)
 .ARM.attributes
                0x000007df       0x32 /usr/lib/gcc/arm-none-eabi/13.2.1/../../../arm-none-eabi/lib/thumb/v7e-m+dp/hard/libc_nano.a(libc_a-freer.o)
 .ARM.attributes
                0x00000811       0x32 /usr/lib/gcc/arm-none-eabi/13.2.1/../../../arm-none-eabi/lib/thumb/v7e-m+dp/hard/libc_nano.a(libc_a-memmove.o)
 .ARM.attributes
                0x00000843       0x1c /usr/lib/gcc/arm-none-eabi/13.2.1/../../../arm-none-eabi/lib/thumb/v7e-m+dp/hard/libc_nano.a(libc_a-memchr.o)
 .ARM.attributes
                0x0000085f       0x1e /usr/lib/gcc/arm-none-eabi/13.2.1/../../../arm-none-eabi/lib/thumb/v7e-m+dp/hard/libc_nano.a(libc_a-memcpy.o)
 .ARM.attributes
                0x0000087d       0x32 /usr/lib/gcc/arm-none-eabi/13.2.1/../../../arm-none-eabi/lib/thumb/v7e-m+dp/hard/libc_nano.a(libc_a-malloc.o)
 .ARM.attributes
                0x000008af       0x32 /usr/lib/gcc/arm-none-eabi/13.2.1/../../../arm-none-eabi/lib/thumb/v7e-m+dp/hard/libc_nano.a(libc_a-reallocr.o)
 .ARM.attributes
                0x000008e1       0x32 /usr/lib/gcc/arm-none-eabi/13.2.1/../../../arm-none-eabi/lib/thumb/v7e-m+dp/hard/libc_nano.a(libc_a-nano-vfprintf_i.o)
 .ARM.attributes
                0x00000913       0x32 /usr/lib/gcc/arm-none-eabi/13.2.1/../../../arm-none-eabi/lib/thumb/v7e-m+dp/hard/libc_nano.a(libc_a-mlock.o)
 .ARM.attributes
                0x00000945       0x32 /usr/lib/gcc/arm-none-eabi/13.2.1/../../../arm-none-eabi/lib/thumb/v7e-m+dp/hard/libc_nano.a(libc_a-sbrkr.o)
 .ARM.attributes
                0x00000977       0x32 /usr/lib/gcc/arm-none-eabi/13.2.1/../../../arm-none-eabi/lib/thumb/v7e-m+dp/hard/libc_nano.a(libc_a-msizer.o)
 .ARM.attributes
                0x000009a9       0x32 /usr/lib/gcc/arm-none-eabi/13.2.1/../../../arm-none-eabi/lib/thumb/v7e-m+dp/hard/libc_nano.a(libc_a-findfp.o)
 .ARM.attributes
                0x000009db       0x32 /usr/lib/gcc/arm-none-eabi/13.2.1/../../../arm-none-eabi/lib/thumb/v7e-m+dp/hard/libc_nano.a(libc_a-reent.o)
 .ARM.attributes
                0x00000a0d       0x20 /usr/lib/gcc/arm-none-eabi/13.2.1/thumb/v7e-m+dp/hard/libgcc.a(_aeabi_uldivmod.o)
 .ARM.attributes
                0x00000a2d       0x32 /usr/lib/gcc/arm-none-eabi/13.2.1/thumb/v7e-m+dp/hard/libgcc.a(_udivmoddi4.o)
 .ARM.attributes
                0x00000a5f       0x20 /usr/lib/gcc/arm-none-eabi/13.2.1/thumb/v7e-m+dp/hard/libgcc.a(_dvmd_tls.o)
 .ARM.attributes
                0x00000a7f       0x32 /usr/lib/gcc/arm-none-eabi/13.2.1/thumb/v7e-m+dp/hard/crtend.o
 .ARM.attributes
                0x00000ab1       0x20 /usr/lib/gcc/arm-none-eabi/13.2.1/thumb/v7e-m+dp/hard/crtn.o

.comment        0x00000000       0x26
 .comment       0x00000000       0x26 /usr/lib/gcc/arm-none-eabi/13.2.1/thumb/v7e-m+dp/hard/crtbegin.o
                                 0x27 (size before relaxing)
 .comment       0x00000026       0x27 build/main.o
 .comment       0x00000026       0x27 build/bsp_driver_sd.o
 .comment       0x00000026       0x27 build/sd_diskio.o
 .comment       0x00000026       0x27 build/fatfs.o
 .comment       0x00000026       0x27 build/fatfs_platform.o
 .comment       0x00000026       0x27 build/stm32f7xx_it.o
 .comment       0x00000026       0x27 build/stm32f7xx_hal_msp.o
 .comment       0x00000026       0x27 build/stm32f7xx_hal_adc.o
 .comment       0x00000026       0x27 build/stm32f7xx_hal_adc_ex.o
 .comment       0x00000026       0x27 build/stm32f7xx_hal_rcc.o
 .comment       0x00000026       0x27 build/stm32f7xx_hal_rcc_ex.o
 .comment       0x00000026       0x27 build/stm32f7xx_hal_gpio.o
 .comment       0x00000026       0x27 build/stm32f7xx_hal_pwr_ex.o
 .comment       0x00000026       0x27 build/stm32f7xx_hal_cortex.o
 .comment       0x00000026       0x27 build/stm32f7xx_hal.o
 .comment       0x00000026       0x27 build/stm32f7xx_ll_rcc.o
 .comment       0x00000026       0x27 build/stm32f7xx_ll_gpio.o
 .comment       0x00000026       0x27 build/stm32f7xx_ll_sdmmc.o
 .comment       0x00000026       0x27 build/stm32f7xx_hal_sd.o
 .comment       0x00000026       0x27 build/stm32f7xx_ll_spi.o
 .comment       0x00000026       0x27 build/stm32f7xx_hal_tim.o
 .comment       0x00000026       0x27 build/stm32f7xx_hal_tim_ex.o
 .comment       0x00000026       0x27 build/stm32f7xx_ll_tim.o
 .comment       0x00000026       0x27 build/stm32f7xx_ll_usart.o
 .comment       0x00000026       0x27 build/system_stm32f7xx.o
 .comment       0x00000026       0x27 build/File_Handling.o
 .comment       0x00000026       0x27 build/diskio.o
 .comment       0x00000026       0x27 build/ff.o
 .comment       0x00000026       0x27 build/ff_gen_drv.o
 .comment       0x00000026       0x27 build/sysmem.o
 .comment       0x00000026       0x27 build/stm32f7xx_hal_uart.o
 .comment       0x00000026       0x27 /usr/lib/gcc/arm-none-eabi/13.2.1/../../../arm-none-eabi/lib/thumb/v7e-m+dp/hard/libc_nano.a(libc_a-sprintf.o)
 .comment       0x00000026       0x27 /usr/lib/gcc/arm-none-eabi/13.2.1/../../../arm-none-eabi/lib/thumb/v7e-m+dp/hard/libc_nano.a(libc_a-impure.o)
 .comment       0x00000026       0x27 /usr/lib/gcc/arm-none-eabi/13.2.1/../../../arm-none-eabi/lib/thumb/v7e-m+dp/hard/libc_nano.a(libc_a-nano-svfprintf.o)
 .comment       0x00000026       0x27 /usr/lib/gcc/arm-none-eabi/13.2.1/../../../arm-none-eabi/lib/thumb/v7e-m+dp/hard/libc_nano.a(libc_a-init.o)
 .comment       0x00000026       0x27 /usr/lib/gcc/arm-none-eabi/13.2.1/../../../arm-none-eabi/lib/thumb/v7e-m+dp/hard/libc_nano.a(libc_a-memset.o)
 .comment       0x00000026       0x27 /usr/lib/gcc/arm-none-eabi/13.2.1/../../../arm-none-eabi/lib/thumb/v7e-m+dp/hard/libc_nano.a(libc_a-errno.o)
 .comment       0x00000026       0x27 /usr/lib/gcc/arm-none-eabi/13.2.1/../../../arm-none-eabi/lib/thumb/v7e-m+dp/hard/libc_nano.a(libc_a-mallocr.o)
 .comment       0x00000026       0x27 /usr/lib/gcc/arm-none-eabi/13.2.1/../../../arm-none-eabi/lib/thumb/v7e-m+dp/hard/libc_nano.a(libc_a-freer.o)
 .comment       0x00000026       0x27 /usr/lib/gcc/arm-none-eabi/13.2.1/../../../arm-none-eabi/lib/thumb/v7e-m+dp/hard/libc_nano.a(libc_a-memmove.o)
 .comment       0x00000026       0x27 /usr/lib/gcc/arm-none-eabi/13.2.1/../../../arm-none-eabi/lib/thumb/v7e-m+dp/hard/libc_nano.a(libc_a-malloc.o)
 .comment       0x00000026       0x27 /usr/lib/gcc/arm-none-eabi/13.2.1/../../../arm-none-eabi/lib/thumb/v7e-m+dp/hard/libc_nano.a(libc_a-reallocr.o)
 .comment       0x00000026       0x27 /usr/lib/gcc/arm-none-eabi/13.2.1/../../../arm-none-eabi/lib/thumb/v7e-m+dp/hard/libc_nano.a(libc_a-nano-vfprintf_i.o)
 .comment       0x00000026       0x27 /usr/lib/gcc/arm-none-eabi/13.2.1/../../../arm-none-eabi/lib/thumb/v7e-m+dp/hard/libc_nano.a(libc_a-mlock.o)
 .comment       0x00000026       0x27 /usr/lib/gcc/arm-none-eabi/13.2.1/../../../arm-none-eabi/lib/thumb/v7e-m+dp/hard/libc_nano.a(libc_a-sbrkr.o)
 .comment       0x00000026       0x27 /usr/lib/gcc/arm-none-eabi/13.2.1/../../../arm-none-eabi/lib/thumb/v7e-m+dp/hard/libc_nano.a(libc_a-msizer.o)
 .comment       0x00000026       0x27 /usr/lib/gcc/arm-none-eabi/13.2.1/../../../arm-none-eabi/lib/thumb/v7e-m+dp/hard/libc_nano.a(libc_a-findfp.o)
 .comment       0x00000026       0x27 /usr/lib/gcc/arm-none-eabi/13.2.1/../../../arm-none-eabi/lib/thumb/v7e-m+dp/hard/libc_nano.a(libc_a-reent.o)
 .comment       0x00000026       0x27 /usr/lib/gcc/arm-none-eabi/13.2.1/thumb/v7e-m+dp/hard/libgcc.a(_udivmoddi4.o)
 .comment       0x00000026       0x27 /usr/lib/gcc/arm-none-eabi/13.2.1/thumb/v7e-m+dp/hard/crtend.o

.debug_info     0x00000000    0x3a851
 .debug_info    0x00000000     0x824c build/main.o
 .debug_info    0x0000824c      0xe39 build/bsp_driver_sd.o
 .debug_info    0x00009085      0x74a build/sd_diskio.o
 .debug_info    0x000097cf      0x65a build/fatfs.o
 .debug_info    0x00009e29      0x1f0 build/fatfs_platform.o
 .debug_info    0x0000a019     0x1925 build/stm32f7xx_it.o
 .debug_info    0x0000b93e     0x23e6 build/stm32f7xx_hal_msp.o
 .debug_info    0x0000dd24      0xfb5 build/stm32f7xx_hal_adc.o
 .debug_info    0x0000ecd9      0xd39 build/stm32f7xx_hal_adc_ex.o
 .debug_info    0x0000fa12      0xd0b build/stm32f7xx_hal_rcc.o
 .debug_info    0x0001071d      0x96b build/stm32f7xx_hal_rcc_ex.o
 .debug_info    0x00011088      0x867 build/stm32f7xx_hal_gpio.o
 .debug_info    0x000118ef      0xb00 build/stm32f7xx_hal_pwr_ex.o
 .debug_info    0x000123ef     0x145b build/stm32f7xx_hal_cortex.o
 .debug_info    0x0001384a      0xc0b build/stm32f7xx_hal.o
 .debug_info    0x00014455     0x1d6b build/stm32f7xx_ll_rcc.o
 .debug_info    0x000161c0      0xda5 build/stm32f7xx_ll_gpio.o
 .debug_info    0x00016f65     0x1ad6 build/stm32f7xx_ll_sdmmc.o
 .debug_info    0x00018a3b     0x2a28 build/stm32f7xx_hal_sd.o
 .debug_info    0x0001b463      0xb14 build/stm32f7xx_ll_spi.o
 .debug_info    0x0001bf77     0x42a3 build/stm32f7xx_hal_tim.o
 .debug_info    0x0002021a     0x2009 build/stm32f7xx_hal_tim_ex.o
 .debug_info    0x00022223     0x19f0 build/stm32f7xx_ll_tim.o
 .debug_info    0x00023c13      0xc07 build/stm32f7xx_ll_usart.o
 .debug_info    0x0002481a      0x7ea build/system_stm32f7xx.o
 .debug_info    0x00025004     0x1ef6 build/File_Handling.o
 .debug_info    0x00026efa      0x5f7 build/diskio.o
 .debug_info    0x000274f1     0x47f5 build/ff.o
 .debug_info    0x0002bce6      0x525 build/ff_gen_drv.o
 .debug_info    0x0002c20b      0x174 build/sysmem.o
 .debug_info    0x0002c37f     0x54ac build/stm32f7xx_hal_uart.o
 .debug_info    0x0003182b       0x30 build/startup_stm32f767xx.o
 .debug_info    0x0003185b      0x87b /usr/lib/gcc/arm-none-eabi/13.2.1/../../../arm-none-eabi/lib/thumb/v7e-m+dp/hard/libc_nano.a(libc_a-sprintf.o)
 .debug_info    0x000320d6      0x70b /usr/lib/gcc/arm-none-eabi/13.2.1/../../../arm-none-eabi/lib/thumb/v7e-m+dp/hard/libc_nano.a(libc_a-impure.o)
 .debug_info    0x000327e1     0x1092 /usr/lib/gcc/arm-none-eabi/13.2.1/../../../arm-none-eabi/lib/thumb/v7e-m+dp/hard/libc_nano.a(libc_a-nano-svfprintf.o)
 .debug_info    0x00033873      0x10b /usr/lib/gcc/arm-none-eabi/13.2.1/../../../arm-none-eabi/lib/thumb/v7e-m+dp/hard/libc_nano.a(libc_a-init.o)
 .debug_info    0x0003397e      0x135 /usr/lib/gcc/arm-none-eabi/13.2.1/../../../arm-none-eabi/lib/thumb/v7e-m+dp/hard/libc_nano.a(libc_a-memset.o)
 .debug_info    0x00033ab3      0x6f1 /usr/lib/gcc/arm-none-eabi/13.2.1/../../../arm-none-eabi/lib/thumb/v7e-m+dp/hard/libc_nano.a(libc_a-errno.o)
 .debug_info    0x000341a4      0x9b6 /usr/lib/gcc/arm-none-eabi/13.2.1/../../../arm-none-eabi/lib/thumb/v7e-m+dp/hard/libc_nano.a(libc_a-mallocr.o)
 .debug_info    0x00034b5a      0x87f /usr/lib/gcc/arm-none-eabi/13.2.1/../../../arm-none-eabi/lib/thumb/v7e-m+dp/hard/libc_nano.a(libc_a-freer.o)
 .debug_info    0x000353d9      0x148 /usr/lib/gcc/arm-none-eabi/13.2.1/../../../arm-none-eabi/lib/thumb/v7e-m+dp/hard/libc_nano.a(libc_a-memmove.o)
 .debug_info    0x00035521       0x25 /usr/lib/gcc/arm-none-eabi/13.2.1/../../../arm-none-eabi/lib/thumb/v7e-m+dp/hard/libc_nano.a(libc_a-memchr.o)
 .debug_info    0x00035546       0x33 /usr/lib/gcc/arm-none-eabi/13.2.1/../../../arm-none-eabi/lib/thumb/v7e-m+dp/hard/libc_nano.a(libc_a-memcpy.o)
 .debug_info    0x00035579      0x796 /usr/lib/gcc/arm-none-eabi/13.2.1/../../../arm-none-eabi/lib/thumb/v7e-m+dp/hard/libc_nano.a(libc_a-malloc.o)
 .debug_info    0x00035d0f      0x8cd /usr/lib/gcc/arm-none-eabi/13.2.1/../../../arm-none-eabi/lib/thumb/v7e-m+dp/hard/libc_nano.a(libc_a-reallocr.o)
 .debug_info    0x000365dc      0xdd7 /usr/lib/gcc/arm-none-eabi/13.2.1/../../../arm-none-eabi/lib/thumb/v7e-m+dp/hard/libc_nano.a(libc_a-nano-vfprintf_i.o)
 .debug_info    0x000373b3      0x71c /usr/lib/gcc/arm-none-eabi/13.2.1/../../../arm-none-eabi/lib/thumb/v7e-m+dp/hard/libc_nano.a(libc_a-mlock.o)
 .debug_info    0x00037acf      0x778 /usr/lib/gcc/arm-none-eabi/13.2.1/../../../arm-none-eabi/lib/thumb/v7e-m+dp/hard/libc_nano.a(libc_a-sbrkr.o)
 .debug_info    0x00038247      0x78a /usr/lib/gcc/arm-none-eabi/13.2.1/../../../arm-none-eabi/lib/thumb/v7e-m+dp/hard/libc_nano.a(libc_a-msizer.o)
 .debug_info    0x000389d1      0xe8c /usr/lib/gcc/arm-none-eabi/13.2.1/../../../arm-none-eabi/lib/thumb/v7e-m+dp/hard/libc_nano.a(libc_a-findfp.o)
 .debug_info    0x0003985d      0x89f /usr/lib/gcc/arm-none-eabi/13.2.1/../../../arm-none-eabi/lib/thumb/v7e-m+dp/hard/libc_nano.a(libc_a-reent.o)
 .debug_info    0x0003a0fc       0x24 /usr/lib/gcc/arm-none-eabi/13.2.1/thumb/v7e-m+dp/hard/libgcc.a(_aeabi_uldivmod.o)
 .debug_info    0x0003a120      0x6f5 /usr/lib/gcc/arm-none-eabi/13.2.1/thumb/v7e-m+dp/hard/libgcc.a(_udivmoddi4.o)
 .debug_info    0x0003a815       0x3c /usr/lib/gcc/arm-none-eabi/13.2.1/thumb/v7e-m+dp/hard/libgcc.a(_dvmd_tls.o)

.debug_abbrev   0x00000000     0x7012
 .debug_abbrev  0x00000000      0x506 build/main.o
 .debug_abbrev  0x00000506      0x2a1 build/bsp_driver_sd.o
 .debug_abbrev  0x000007a7      0x1e1 build/sd_diskio.o
 .debug_abbrev  0x00000988      0x181 build/fatfs.o
 .debug_abbrev  0x00000b09      0x11e build/fatfs_platform.o
 .debug_abbrev  0x00000c27      0x33b build/stm32f7xx_it.o
 .debug_abbrev  0x00000f62      0x299 build/stm32f7xx_hal_msp.o
 .debug_abbrev  0x000011fb      0x2b6 build/stm32f7xx_hal_adc.o
 .debug_abbrev  0x000014b1      0x2d9 build/stm32f7xx_hal_adc_ex.o
 .debug_abbrev  0x0000178a      0x306 build/stm32f7xx_hal_rcc.o
 .debug_abbrev  0x00001a90      0x1f3 build/stm32f7xx_hal_rcc_ex.o
 .debug_abbrev  0x00001c83      0x22b build/stm32f7xx_hal_gpio.o
 .debug_abbrev  0x00001eae      0x1d5 build/stm32f7xx_hal_pwr_ex.o
 .debug_abbrev  0x00002083      0x3ca build/stm32f7xx_hal_cortex.o
 .debug_abbrev  0x0000244d      0x244 build/stm32f7xx_hal.o
 .debug_abbrev  0x00002691      0x294 build/stm32f7xx_ll_rcc.o
 .debug_abbrev  0x00002925      0x2ad build/stm32f7xx_ll_gpio.o
 .debug_abbrev  0x00002bd2      0x236 build/stm32f7xx_ll_sdmmc.o
 .debug_abbrev  0x00002e08      0x306 build/stm32f7xx_hal_sd.o
 .debug_abbrev  0x0000310e      0x2e3 build/stm32f7xx_ll_spi.o
 .debug_abbrev  0x000033f1      0x2bd build/stm32f7xx_hal_tim.o
 .debug_abbrev  0x000036ae      0x2b7 build/stm32f7xx_hal_tim_ex.o
 .debug_abbrev  0x00003965      0x2af build/stm32f7xx_ll_tim.o
 .debug_abbrev  0x00003c14      0x2d3 build/stm32f7xx_ll_usart.o
 .debug_abbrev  0x00003ee7      0x12a build/system_stm32f7xx.o
 .debug_abbrev  0x00004011      0x307 build/File_Handling.o
 .debug_abbrev  0x00004318      0x1ca build/diskio.o
 .debug_abbrev  0x000044e2      0x309 build/ff.o
 .debug_abbrev  0x000047eb      0x1da build/ff_gen_drv.o
 .debug_abbrev  0x000049c5       0xeb build/sysmem.o
 .debug_abbrev  0x00004ab0      0x346 build/stm32f7xx_hal_uart.o
 .debug_abbrev  0x00004df6       0x1d build/startup_stm32f767xx.o
 .debug_abbrev  0x00004e13      0x21c /usr/lib/gcc/arm-none-eabi/13.2.1/../../../arm-none-eabi/lib/thumb/v7e-m+dp/hard/libc_nano.a(libc_a-sprintf.o)
 .debug_abbrev  0x0000502f      0x149 /usr/lib/gcc/arm-none-eabi/13.2.1/../../../arm-none-eabi/lib/thumb/v7e-m+dp/hard/libc_nano.a(libc_a-impure.o)
 .debug_abbrev  0x00005178      0x32f /usr/lib/gcc/arm-none-eabi/13.2.1/../../../arm-none-eabi/lib/thumb/v7e-m+dp/hard/libc_nano.a(libc_a-nano-svfprintf.o)
 .debug_abbrev  0x000054a7       0xc9 /usr/lib/gcc/arm-none-eabi/13.2.1/../../../arm-none-eabi/lib/thumb/v7e-m+dp/hard/libc_nano.a(libc_a-init.o)
 .debug_abbrev  0x00005570       0xb7 /usr/lib/gcc/arm-none-eabi/13.2.1/../../../arm-none-eabi/lib/thumb/v7e-m+dp/hard/libc_nano.a(libc_a-memset.o)
 .debug_abbrev  0x00005627      0x15e /usr/lib/gcc/arm-none-eabi/13.2.1/../../../arm-none-eabi/lib/thumb/v7e-m+dp/hard/libc_nano.a(libc_a-errno.o)
 .debug_abbrev  0x00005785      0x24a /usr/lib/gcc/arm-none-eabi/13.2.1/../../../arm-none-eabi/lib/thumb/v7e-m+dp/hard/libc_nano.a(libc_a-mallocr.o)
 .debug_abbrev  0x000059cf      0x249 /usr/lib/gcc/arm-none-eabi/13.2.1/../../../arm-none-eabi/lib/thumb/v7e-m+dp/hard/libc_nano.a(libc_a-freer.o)
 .debug_abbrev  0x00005c18       0xc3 /usr/lib/gcc/arm-none-eabi/13.2.1/../../../arm-none-eabi/lib/thumb/v7e-m+dp/hard/libc_nano.a(libc_a-memmove.o)
 .debug_abbrev  0x00005cdb       0x14 /usr/lib/gcc/arm-none-eabi/13.2.1/../../../arm-none-eabi/lib/thumb/v7e-m+dp/hard/libc_nano.a(libc_a-memchr.o)
 .debug_abbrev  0x00005cef       0x28 /usr/lib/gcc/arm-none-eabi/13.2.1/../../../arm-none-eabi/lib/thumb/v7e-m+dp/hard/libc_nano.a(libc_a-memcpy.o)
 .debug_abbrev  0x00005d17      0x1cf /usr/lib/gcc/arm-none-eabi/13.2.1/../../../arm-none-eabi/lib/thumb/v7e-m+dp/hard/libc_nano.a(libc_a-malloc.o)
 .debug_abbrev  0x00005ee6      0x20c /usr/lib/gcc/arm-none-eabi/13.2.1/../../../arm-none-eabi/lib/thumb/v7e-m+dp/hard/libc_nano.a(libc_a-reallocr.o)
 .debug_abbrev  0x000060f2      0x284 /usr/lib/gcc/arm-none-eabi/13.2.1/../../../arm-none-eabi/lib/thumb/v7e-m+dp/hard/libc_nano.a(libc_a-nano-vfprintf_i.o)
 .debug_abbrev  0x00006376      0x192 /usr/lib/gcc/arm-none-eabi/13.2.1/../../../arm-none-eabi/lib/thumb/v7e-m+dp/hard/libc_nano.a(libc_a-mlock.o)
 .debug_abbrev  0x00006508      0x1da /usr/lib/gcc/arm-none-eabi/13.2.1/../../../arm-none-eabi/lib/thumb/v7e-m+dp/hard/libc_nano.a(libc_a-sbrkr.o)
 .debug_abbrev  0x000066e2      0x196 /usr/lib/gcc/arm-none-eabi/13.2.1/../../../arm-none-eabi/lib/thumb/v7e-m+dp/hard/libc_nano.a(libc_a-msizer.o)
 .debug_abbrev  0x00006878      0x408 /usr/lib/gcc/arm-none-eabi/13.2.1/../../../arm-none-eabi/lib/thumb/v7e-m+dp/hard/libc_nano.a(libc_a-findfp.o)
 .debug_abbrev  0x00006c80      0x1ee /usr/lib/gcc/arm-none-eabi/13.2.1/../../../arm-none-eabi/lib/thumb/v7e-m+dp/hard/libc_nano.a(libc_a-reent.o)
 .debug_abbrev  0x00006e6e       0x14 /usr/lib/gcc/arm-none-eabi/13.2.1/thumb/v7e-m+dp/hard/libgcc.a(_aeabi_uldivmod.o)
 .debug_abbrev  0x00006e82      0x16a /usr/lib/gcc/arm-none-eabi/13.2.1/thumb/v7e-m+dp/hard/libgcc.a(_udivmoddi4.o)
 .debug_abbrev  0x00006fec       0x26 /usr/lib/gcc/arm-none-eabi/13.2.1/thumb/v7e-m+dp/hard/libgcc.a(_dvmd_tls.o)

.debug_loc      0x00000000    0x2625b
 .debug_loc     0x00000000     0x2a18 build/main.o
 .debug_loc     0x00002a18      0x6f0 build/bsp_driver_sd.o
 .debug_loc     0x00003108      0x544 build/sd_diskio.o
 .debug_loc     0x0000364c       0x20 build/fatfs.o
 .debug_loc     0x0000366c       0x51 build/fatfs_platform.o
 .debug_loc     0x000036bd      0x43a build/stm32f7xx_it.o
 .debug_loc     0x00003af7      0x5a7 build/stm32f7xx_hal_msp.o
 .debug_loc     0x0000409e      0xe7b build/stm32f7xx_hal_adc.o
 .debug_loc     0x00004f19      0xc11 build/stm32f7xx_hal_adc_ex.o
 .debug_loc     0x00005b2a      0x849 build/stm32f7xx_hal_rcc.o
 .debug_loc     0x00006373      0x924 build/stm32f7xx_hal_rcc_ex.o
 .debug_loc     0x00006c97      0x60b build/stm32f7xx_hal_gpio.o
 .debug_loc     0x000072a2      0x3e6 build/stm32f7xx_hal_pwr_ex.o
 .debug_loc     0x00007688      0x886 build/stm32f7xx_hal_cortex.o
 .debug_loc     0x00007f0e      0x1f9 build/stm32f7xx_hal.o
 .debug_loc     0x00008107     0x1806 build/stm32f7xx_ll_rcc.o
 .debug_loc     0x0000990d      0x9ad build/stm32f7xx_ll_gpio.o
 .debug_loc     0x0000a2ba     0x1873 build/stm32f7xx_ll_sdmmc.o
 .debug_loc     0x0000bb2d     0x29f6 build/stm32f7xx_hal_sd.o
 .debug_loc     0x0000e523      0x6d7 build/stm32f7xx_ll_spi.o
 .debug_loc     0x0000ebfa     0x6372 build/stm32f7xx_hal_tim.o
 .debug_loc     0x00014f6c     0x291a build/stm32f7xx_hal_tim_ex.o
 .debug_loc     0x00017886     0x1b79 build/stm32f7xx_ll_tim.o
 .debug_loc     0x000193ff      0x8b1 build/stm32f7xx_ll_usart.o
 .debug_loc     0x00019cb0      0x181 build/system_stm32f7xx.o
 .debug_loc     0x00019e31      0xa9c build/File_Handling.o
 .debug_loc     0x0001a8cd      0x377 build/diskio.o
 .debug_loc     0x0001ac44     0x6040 build/ff.o
 .debug_loc     0x00020c84      0x37c build/ff_gen_drv.o
 .debug_loc     0x00021000       0x90 build/sysmem.o
 .debug_loc     0x00021090     0x51cb build/stm32f7xx_hal_uart.o

.debug_aranges  0x00000000     0x1c50
 .debug_aranges
                0x00000000      0x158 build/main.o
 .debug_aranges
                0x00000158       0x98 build/bsp_driver_sd.o
 .debug_aranges
                0x000001f0       0x48 build/sd_diskio.o
 .debug_aranges
                0x00000238       0x28 build/fatfs.o
 .debug_aranges
                0x00000260       0x20 build/fatfs_platform.o
 .debug_aranges
                0x00000280       0xc0 build/stm32f7xx_it.o
 .debug_aranges
                0x00000340       0x68 build/stm32f7xx_hal_msp.o
 .debug_aranges
                0x000003a8       0xe8 build/stm32f7xx_hal_adc.o
 .debug_aranges
                0x00000490       0x90 build/stm32f7xx_hal_adc_ex.o
 .debug_aranges
                0x00000520       0x88 build/stm32f7xx_hal_rcc.o
 .debug_aranges
                0x000005a8       0x50 build/stm32f7xx_hal_rcc_ex.o
 .debug_aranges
                0x000005f8       0x58 build/stm32f7xx_hal_gpio.o
 .debug_aranges
                0x00000650       0x80 build/stm32f7xx_hal_pwr_ex.o
 .debug_aranges
                0x000006d0       0xe8 build/stm32f7xx_hal_cortex.o
 .debug_aranges
                0x000007b8      0x110 build/stm32f7xx_hal.o
 .debug_aranges
                0x000008c8       0xf8 build/stm32f7xx_ll_rcc.o
 .debug_aranges
                0x000009c0       0x58 build/stm32f7xx_ll_gpio.o
 .debug_aranges
                0x00000a18      0x188 build/stm32f7xx_ll_sdmmc.o
 .debug_aranges
                0x00000ba0      0x168 build/stm32f7xx_hal_sd.o
 .debug_aranges
                0x00000d08       0x50 build/stm32f7xx_ll_spi.o
 .debug_aranges
                0x00000d58      0x3e0 build/stm32f7xx_hal_tim.o
 .debug_aranges
                0x00001138      0x180 build/stm32f7xx_hal_tim_ex.o
 .debug_aranges
                0x000012b8       0xd0 build/stm32f7xx_ll_tim.o
 .debug_aranges
                0x00001388       0x48 build/stm32f7xx_ll_usart.o
 .debug_aranges
                0x000013d0       0x28 build/system_stm32f7xx.o
 .debug_aranges
                0x000013f8       0x98 build/File_Handling.o
 .debug_aranges
                0x00001490       0x48 build/diskio.o
 .debug_aranges
                0x000014d8      0x208 build/ff.o
 .debug_aranges
                0x000016e0       0x40 build/ff_gen_drv.o
 .debug_aranges
                0x00001720       0x20 build/sysmem.o
 .debug_aranges
                0x00001740      0x230 build/stm32f7xx_hal_uart.o
 .debug_aranges
                0x00001970       0x28 build/startup_stm32f767xx.o
 .debug_aranges
                0x00001998       0x20 /usr/lib/gcc/arm-none-eabi/13.2.1/../../../arm-none-eabi/lib/thumb/v7e-m+dp/hard/libc_nano.a(libc_a-sprintf.o)
 .debug_aranges
                0x000019b8       0x18 /usr/lib/gcc/arm-none-eabi/13.2.1/../../../arm-none-eabi/lib/thumb/v7e-m+dp/hard/libc_nano.a(libc_a-impure.o)
 .debug_aranges
                0x000019d0       0x20 /usr/lib/gcc/arm-none-eabi/13.2.1/../../../arm-none-eabi/lib/thumb/v7e-m+dp/hard/libc_nano.a(libc_a-nano-svfprintf.o)
 .debug_aranges
                0x000019f0       0x20 /usr/lib/gcc/arm-none-eabi/13.2.1/../../../arm-none-eabi/lib/thumb/v7e-m+dp/hard/libc_nano.a(libc_a-init.o)
 .debug_aranges
                0x00001a10       0x20 /usr/lib/gcc/arm-none-eabi/13.2.1/../../../arm-none-eabi/lib/thumb/v7e-m+dp/hard/libc_nano.a(libc_a-memset.o)
 .debug_aranges
                0x00001a30       0x20 /usr/lib/gcc/arm-none-eabi/13.2.1/../../../arm-none-eabi/lib/thumb/v7e-m+dp/hard/libc_nano.a(libc_a-errno.o)
 .debug_aranges
                0x00001a50       0x20 /usr/lib/gcc/arm-none-eabi/13.2.1/../../../arm-none-eabi/lib/thumb/v7e-m+dp/hard/libc_nano.a(libc_a-mallocr.o)
 .debug_aranges
                0x00001a70       0x20 /usr/lib/gcc/arm-none-eabi/13.2.1/../../../arm-none-eabi/lib/thumb/v7e-m+dp/hard/libc_nano.a(libc_a-freer.o)
 .debug_aranges
                0x00001a90       0x20 /usr/lib/gcc/arm-none-eabi/13.2.1/../../../arm-none-eabi/lib/thumb/v7e-m+dp/hard/libc_nano.a(libc_a-memmove.o)
 .debug_aranges
                0x00001ab0       0x20 /usr/lib/gcc/arm-none-eabi/13.2.1/../../../arm-none-eabi/lib/thumb/v7e-m+dp/hard/libc_nano.a(libc_a-memchr.o)
 .debug_aranges
                0x00001ad0       0x20 /usr/lib/gcc/arm-none-eabi/13.2.1/../../../arm-none-eabi/lib/thumb/v7e-m+dp/hard/libc_nano.a(libc_a-memcpy.o)
 .debug_aranges
                0x00001af0       0x20 /usr/lib/gcc/arm-none-eabi/13.2.1/../../../arm-none-eabi/lib/thumb/v7e-m+dp/hard/libc_nano.a(libc_a-malloc.o)
 .debug_aranges
                0x00001b10       0x20 /usr/lib/gcc/arm-none-eabi/13.2.1/../../../arm-none-eabi/lib/thumb/v7e-m+dp/hard/libc_nano.a(libc_a-reallocr.o)
 .debug_aranges
                0x00001b30       0x20 /usr/lib/gcc/arm-none-eabi/13.2.1/../../../arm-none-eabi/lib/thumb/v7e-m+dp/hard/libc_nano.a(libc_a-nano-vfprintf_i.o)
 .debug_aranges
                0x00001b50       0x20 /usr/lib/gcc/arm-none-eabi/13.2.1/../../../arm-none-eabi/lib/thumb/v7e-m+dp/hard/libc_nano.a(libc_a-mlock.o)
 .debug_aranges
                0x00001b70       0x20 /usr/lib/gcc/arm-none-eabi/13.2.1/../../../arm-none-eabi/lib/thumb/v7e-m+dp/hard/libc_nano.a(libc_a-sbrkr.o)
 .debug_aranges
                0x00001b90       0x20 /usr/lib/gcc/arm-none-eabi/13.2.1/../../../arm-none-eabi/lib/thumb/v7e-m+dp/hard/libc_nano.a(libc_a-msizer.o)
 .debug_aranges
                0x00001bb0       0x20 /usr/lib/gcc/arm-none-eabi/13.2.1/../../../arm-none-eabi/lib/thumb/v7e-m+dp/hard/libc_nano.a(libc_a-findfp.o)
 .debug_aranges
                0x00001bd0       0x20 /usr/lib/gcc/arm-none-eabi/13.2.1/../../../arm-none-eabi/lib/thumb/v7e-m+dp/hard/libc_nano.a(libc_a-reent.o)
 .debug_aranges
                0x00001bf0       0x20 /usr/lib/gcc/arm-none-eabi/13.2.1/thumb/v7e-m+dp/hard/libgcc.a(_aeabi_uldivmod.o)
 .debug_aranges
                0x00001c10       0x20 /usr/lib/gcc/arm-none-eabi/13.2.1/thumb/v7e-m+dp/hard/libgcc.a(_udivmoddi4.o)
 .debug_aranges
                0x00001c30       0x20 /usr/lib/gcc/arm-none-eabi/13.2.1/thumb/v7e-m+dp/hard/libgcc.a(_dvmd_tls.o)

.debug_ranges   0x00000000     0x1b90
 .debug_ranges  0x00000000      0x1c0 build/main.o
 .debug_ranges  0x000001c0       0x88 build/bsp_driver_sd.o
 .debug_ranges  0x00000248       0x38 build/sd_diskio.o
 .debug_ranges  0x00000280       0x18 build/fatfs.o
 .debug_ranges  0x00000298       0x10 build/fatfs_platform.o
 .debug_ranges  0x000002a8       0xb0 build/stm32f7xx_it.o
 .debug_ranges  0x00000358       0x58 build/stm32f7xx_hal_msp.o
 .debug_ranges  0x000003b0       0xd8 build/stm32f7xx_hal_adc.o
 .debug_ranges  0x00000488       0x80 build/stm32f7xx_hal_adc_ex.o
 .debug_ranges  0x00000508       0x78 build/stm32f7xx_hal_rcc.o
 .debug_ranges  0x00000580       0x40 build/stm32f7xx_hal_rcc_ex.o
 .debug_ranges  0x000005c0       0x48 build/stm32f7xx_hal_gpio.o
 .debug_ranges  0x00000608       0x70 build/stm32f7xx_hal_pwr_ex.o
 .debug_ranges  0x00000678       0xd8 build/stm32f7xx_hal_cortex.o
 .debug_ranges  0x00000750      0x100 build/stm32f7xx_hal.o
 .debug_ranges  0x00000850       0xe8 build/stm32f7xx_ll_rcc.o
 .debug_ranges  0x00000938      0x150 build/stm32f7xx_ll_gpio.o
 .debug_ranges  0x00000a88      0x178 build/stm32f7xx_ll_sdmmc.o
 .debug_ranges  0x00000c00      0x158 build/stm32f7xx_hal_sd.o
 .debug_ranges  0x00000d58       0x58 build/stm32f7xx_ll_spi.o
 .debug_ranges  0x00000db0      0x3d0 build/stm32f7xx_hal_tim.o
 .debug_ranges  0x00001180      0x170 build/stm32f7xx_hal_tim_ex.o
 .debug_ranges  0x000012f0      0x210 build/stm32f7xx_ll_tim.o
 .debug_ranges  0x00001500      0x110 build/stm32f7xx_ll_usart.o
 .debug_ranges  0x00001610       0x18 build/system_stm32f7xx.o
 .debug_ranges  0x00001628       0xa0 build/File_Handling.o
 .debug_ranges  0x000016c8       0x38 build/diskio.o
 .debug_ranges  0x00001700      0x1f8 build/ff.o
 .debug_ranges  0x000018f8       0x30 build/ff_gen_drv.o
 .debug_ranges  0x00001928       0x10 build/sysmem.o
 .debug_ranges  0x00001938      0x238 build/stm32f7xx_hal_uart.o
 .debug_ranges  0x00001b70       0x20 build/startup_stm32f767xx.o

.debug_line     0x00000000    0x239e9
 .debug_line    0x00000000     0x37a2 build/main.o
 .debug_line    0x000037a2      0x39e build/bsp_driver_sd.o
 .debug_line    0x00003b40      0x2f2 build/sd_diskio.o
 .debug_line    0x00003e32      0x170 build/fatfs.o
 .debug_line    0x00003fa2      0x111 build/fatfs_platform.o
 .debug_line    0x000040b3      0x934 build/stm32f7xx_it.o
 .debug_line    0x000049e7      0x66d build/stm32f7xx_hal_msp.o
 .debug_line    0x00005054      0xfc7 build/stm32f7xx_hal_adc.o
 .debug_line    0x0000601b      0xb34 build/stm32f7xx_hal_adc_ex.o
 .debug_line    0x00006b4f      0xd15 build/stm32f7xx_hal_rcc.o
 .debug_line    0x00007864      0xbd9 build/stm32f7xx_hal_rcc_ex.o
 .debug_line    0x0000843d      0x6aa build/stm32f7xx_hal_gpio.o
 .debug_line    0x00008ae7      0x52c build/stm32f7xx_hal_pwr_ex.o
 .debug_line    0x00009013      0x77a build/stm32f7xx_hal_cortex.o
 .debug_line    0x0000978d      0x548 build/stm32f7xx_hal.o
 .debug_line    0x00009cd5     0x1721 build/stm32f7xx_ll_rcc.o
 .debug_line    0x0000b3f6      0x76d build/stm32f7xx_ll_gpio.o
 .debug_line    0x0000bb63     0x104d build/stm32f7xx_ll_sdmmc.o
 .debug_line    0x0000cbb0     0x263f build/stm32f7xx_hal_sd.o
 .debug_line    0x0000f1ef      0x56b build/stm32f7xx_ll_spi.o
 .debug_line    0x0000f75a     0x4839 build/stm32f7xx_hal_tim.o
 .debug_line    0x00013f93     0x1bb4 build/stm32f7xx_hal_tim_ex.o
 .debug_line    0x00015b47      0xe26 build/stm32f7xx_ll_tim.o
 .debug_line    0x0001696d      0x62f build/stm32f7xx_ll_usart.o
 .debug_line    0x00016f9c      0x1c2 build/system_stm32f7xx.o
 .debug_line    0x0001715e      0xa76 build/File_Handling.o
 .debug_line    0x00017bd4      0x217 build/diskio.o
 .debug_line    0x00017deb     0x42e1 build/ff.o
 .debug_line    0x0001c0cc      0x25a build/ff_gen_drv.o
 .debug_line    0x0001c326       0xf8 build/sysmem.o
 .debug_line    0x0001c41e     0x3f43 build/stm32f7xx_hal_uart.o
 .debug_line    0x00020361       0x73 build/startup_stm32f767xx.o
 .debug_line    0x000203d4      0x224 /usr/lib/gcc/arm-none-eabi/13.2.1/../../../arm-none-eabi/lib/thumb/v7e-m+dp/hard/libc_nano.a(libc_a-sprintf.o)
 .debug_line    0x000205f8       0xe7 /usr/lib/gcc/arm-none-eabi/13.2.1/../../../arm-none-eabi/lib/thumb/v7e-m+dp/hard/libc_nano.a(libc_a-impure.o)
 .debug_line    0x000206df      0x854 /usr/lib/gcc/arm-none-eabi/13.2.1/../../../arm-none-eabi/lib/thumb/v7e-m+dp/hard/libc_nano.a(libc_a-nano-svfprintf.o)
 .debug_line    0x00020f33      0x11e /usr/lib/gcc/arm-none-eabi/13.2.1/../../../arm-none-eabi/lib/thumb/v7e-m+dp/hard/libc_nano.a(libc_a-init.o)
 .debug_line    0x00021051      0x1b6 /usr/lib/gcc/arm-none-eabi/13.2.1/../../../arm-none-eabi/lib/thumb/v7e-m+dp/hard/libc_nano.a(libc_a-memset.o)
 .debug_line    0x00021207      0x10c /usr/lib/gcc/arm-none-eabi/13.2.1/../../../arm-none-eabi/lib/thumb/v7e-m+dp/hard/libc_nano.a(libc_a-errno.o)
 .debug_line    0x00021313      0x446 /usr/lib/gcc/arm-none-eabi/13.2.1/../../../arm-none-eabi/lib/thumb/v7e-m+dp/hard/libc_nano.a(libc_a-mallocr.o)
 .debug_line    0x00021759      0x2c3 /usr/lib/gcc/arm-none-eabi/13.2.1/../../../arm-none-eabi/lib/thumb/v7e-m+dp/hard/libc_nano.a(libc_a-freer.o)
 .debug_line    0x00021a1c      0x1f1 /usr/lib/gcc/arm-none-eabi/13.2.1/../../../arm-none-eabi/lib/thumb/v7e-m+dp/hard/libc_nano.a(libc_a-memmove.o)
 .debug_line    0x00021c0d       0x84 /usr/lib/gcc/arm-none-eabi/13.2.1/../../../arm-none-eabi/lib/thumb/v7e-m+dp/hard/libc_nano.a(libc_a-memchr.o)
 .debug_line    0x00021c91       0xb9 /usr/lib/gcc/arm-none-eabi/13.2.1/../../../arm-none-eabi/lib/thumb/v7e-m+dp/hard/libc_nano.a(libc_a-memcpy.o)
 .debug_line    0x00021d4a      0x16b /usr/lib/gcc/arm-none-eabi/13.2.1/../../../arm-none-eabi/lib/thumb/v7e-m+dp/hard/libc_nano.a(libc_a-malloc.o)
 .debug_line    0x00021eb5      0x1f8 /usr/lib/gcc/arm-none-eabi/13.2.1/../../../arm-none-eabi/lib/thumb/v7e-m+dp/hard/libc_nano.a(libc_a-reallocr.o)
 .debug_line    0x000220ad      0x75d /usr/lib/gcc/arm-none-eabi/13.2.1/../../../arm-none-eabi/lib/thumb/v7e-m+dp/hard/libc_nano.a(libc_a-nano-vfprintf_i.o)
 .debug_line    0x0002280a      0x153 /usr/lib/gcc/arm-none-eabi/13.2.1/../../../arm-none-eabi/lib/thumb/v7e-m+dp/hard/libc_nano.a(libc_a-mlock.o)
 .debug_line    0x0002295d      0x193 /usr/lib/gcc/arm-none-eabi/13.2.1/../../../arm-none-eabi/lib/thumb/v7e-m+dp/hard/libc_nano.a(libc_a-sbrkr.o)
 .debug_line    0x00022af0      0x176 /usr/lib/gcc/arm-none-eabi/13.2.1/../../../arm-none-eabi/lib/thumb/v7e-m+dp/hard/libc_nano.a(libc_a-msizer.o)
 .debug_line    0x00022c66      0x4fc /usr/lib/gcc/arm-none-eabi/13.2.1/../../../arm-none-eabi/lib/thumb/v7e-m+dp/hard/libc_nano.a(libc_a-findfp.o)
 .debug_line    0x00023162      0x27b /usr/lib/gcc/arm-none-eabi/13.2.1/../../../arm-none-eabi/lib/thumb/v7e-m+dp/hard/libc_nano.a(libc_a-reent.o)
 .debug_line    0x000233dd       0x4e /usr/lib/gcc/arm-none-eabi/13.2.1/thumb/v7e-m+dp/hard/libgcc.a(_aeabi_uldivmod.o)
 .debug_line    0x0002342b      0x574 /usr/lib/gcc/arm-none-eabi/13.2.1/thumb/v7e-m+dp/hard/libgcc.a(_udivmoddi4.o)
 .debug_line    0x0002399f       0x4a /usr/lib/gcc/arm-none-eabi/13.2.1/thumb/v7e-m+dp/hard/libgcc.a(_dvmd_tls.o)

.debug_str      0x00000000     0x96d0
 .debug_str     0x00000000     0x96d0 build/main.o
                               0x2d59 (size before relaxing)
 .debug_str     0x000096d0      0x8f5 build/bsp_driver_sd.o
 .debug_str     0x000096d0      0x3f8 build/sd_diskio.o
 .debug_str     0x000096d0      0x3f0 build/fatfs.o
 .debug_str     0x000096d0      0x23d build/fatfs_platform.o
 .debug_str     0x000096d0      0xed1 build/stm32f7xx_it.o
 .debug_str     0x000096d0     0x1975 build/stm32f7xx_hal_msp.o
 .debug_str     0x000096d0      0x93c build/stm32f7xx_hal_adc.o
 .debug_str     0x000096d0      0x990 build/stm32f7xx_hal_adc_ex.o
 .debug_str     0x000096d0      0x714 build/stm32f7xx_hal_rcc.o
 .debug_str     0x000096d0      0x72c build/stm32f7xx_hal_rcc_ex.o
 .debug_str     0x000096d0      0x4e5 build/stm32f7xx_hal_gpio.o
 .debug_str     0x000096d0      0x63f build/stm32f7xx_hal_pwr_ex.o
 .debug_str     0x000096d0      0xe66 build/stm32f7xx_hal_cortex.o
 .debug_str     0x000096d0      0xd38 build/stm32f7xx_hal.o
 .debug_str     0x000096d0      0xbce build/stm32f7xx_ll_rcc.o
 .debug_str     0x000096d0      0x499 build/stm32f7xx_ll_gpio.o
 .debug_str     0x000096d0      0x7ec build/stm32f7xx_ll_sdmmc.o
 .debug_str     0x000096d0     0x10c7 build/stm32f7xx_hal_sd.o
 .debug_str     0x000096d0      0x5bf build/stm32f7xx_ll_spi.o
 .debug_str     0x000096d0     0x1770 build/stm32f7xx_hal_tim.o
 .debug_str     0x000096d0     0x1076 build/stm32f7xx_hal_tim_ex.o
 .debug_str     0x000096d0      0x9cb build/stm32f7xx_ll_tim.o
 .debug_str     0x000096d0      0x5be build/stm32f7xx_ll_usart.o
 .debug_str     0x000096d0      0x449 build/system_stm32f7xx.o
 .debug_str     0x000096d0      0x647 build/File_Handling.o
 .debug_str     0x000096d0      0x325 build/diskio.o
 .debug_str     0x000096d0      0x8bb build/ff.o
 .debug_str     0x000096d0      0x376 build/ff_gen_drv.o
 .debug_str     0x000096d0      0x213 build/sysmem.o
 .debug_str     0x000096d0     0x1014 build/stm32f7xx_hal_uart.o
 .debug_str     0x000096d0       0x88 build/startup_stm32f767xx.o
 .debug_str     0x000096d0      0x4fe /usr/lib/gcc/arm-none-eabi/13.2.1/../../../arm-none-eabi/lib/thumb/v7e-m+dp/hard/libc_nano.a(libc_a-sprintf.o)
 .debug_str     0x000096d0      0x4bf /usr/lib/gcc/arm-none-eabi/13.2.1/../../../arm-none-eabi/lib/thumb/v7e-m+dp/hard/libc_nano.a(libc_a-impure.o)
 .debug_str     0x000096d0      0x808 /usr/lib/gcc/arm-none-eabi/13.2.1/../../../arm-none-eabi/lib/thumb/v7e-m+dp/hard/libc_nano.a(libc_a-nano-svfprintf.o)
 .debug_str     0x000096d0      0x1fd /usr/lib/gcc/arm-none-eabi/13.2.1/../../../arm-none-eabi/lib/thumb/v7e-m+dp/hard/libc_nano.a(libc_a-init.o)
 .debug_str     0x000096d0      0x1b0 /usr/lib/gcc/arm-none-eabi/13.2.1/../../../arm-none-eabi/lib/thumb/v7e-m+dp/hard/libc_nano.a(libc_a-memset.o)
 .debug_str     0x000096d0      0x4b9 /usr/lib/gcc/arm-none-eabi/13.2.1/../../../arm-none-eabi/lib/thumb/v7e-m+dp/hard/libc_nano.a(libc_a-errno.o)
 .debug_str     0x000096d0      0x5a0 /usr/lib/gcc/arm-none-eabi/13.2.1/../../../arm-none-eabi/lib/thumb/v7e-m+dp/hard/libc_nano.a(libc_a-mallocr.o)
 .debug_str     0x000096d0      0x53f /usr/lib/gcc/arm-none-eabi/13.2.1/../../../arm-none-eabi/lib/thumb/v7e-m+dp/hard/libc_nano.a(libc_a-freer.o)
 .debug_str     0x000096d0      0x1cf /usr/lib/gcc/arm-none-eabi/13.2.1/../../../arm-none-eabi/lib/thumb/v7e-m+dp/hard/libc_nano.a(libc_a-memmove.o)
 .debug_str     0x000096d0       0x9e /usr/lib/gcc/arm-none-eabi/13.2.1/../../../arm-none-eabi/lib/thumb/v7e-m+dp/hard/libc_nano.a(libc_a-memchr.o)
 .debug_str     0x000096d0       0xac /usr/lib/gcc/arm-none-eabi/13.2.1/../../../arm-none-eabi/lib/thumb/v7e-m+dp/hard/libc_nano.a(libc_a-memcpy.o)
 .debug_str     0x000096d0      0x4e4 /usr/lib/gcc/arm-none-eabi/13.2.1/../../../arm-none-eabi/lib/thumb/v7e-m+dp/hard/libc_nano.a(libc_a-malloc.o)
 .debug_str     0x000096d0      0x535 /usr/lib/gcc/arm-none-eabi/13.2.1/../../../arm-none-eabi/lib/thumb/v7e-m+dp/hard/libc_nano.a(libc_a-reallocr.o)
 .debug_str     0x000096d0      0x79e /usr/lib/gcc/arm-none-eabi/13.2.1/../../../arm-none-eabi/lib/thumb/v7e-m+dp/hard/libc_nano.a(libc_a-nano-vfprintf_i.o)
 .debug_str     0x000096d0      0x4dd /usr/lib/gcc/arm-none-eabi/13.2.1/../../../arm-none-eabi/lib/thumb/v7e-m+dp/hard/libc_nano.a(libc_a-mlock.o)
 .debug_str     0x000096d0      0x4c8 /usr/lib/gcc/arm-none-eabi/13.2.1/../../../arm-none-eabi/lib/thumb/v7e-m+dp/hard/libc_nano.a(libc_a-sbrkr.o)
 .debug_str     0x000096d0      0x508 /usr/lib/gcc/arm-none-eabi/13.2.1/../../../arm-none-eabi/lib/thumb/v7e-m+dp/hard/libc_nano.a(libc_a-msizer.o)
 .debug_str     0x000096d0      0x6c2 /usr/lib/gcc/arm-none-eabi/13.2.1/../../../arm-none-eabi/lib/thumb/v7e-m+dp/hard/libc_nano.a(libc_a-findfp.o)
 .debug_str     0x000096d0      0x4de /usr/lib/gcc/arm-none-eabi/13.2.1/../../../arm-none-eabi/lib/thumb/v7e-m+dp/hard/libc_nano.a(libc_a-reent.o)
 .debug_str     0x000096d0       0xa3 /usr/lib/gcc/arm-none-eabi/13.2.1/thumb/v7e-m+dp/hard/libgcc.a(_aeabi_uldivmod.o)
 .debug_str     0x000096d0      0x688 /usr/lib/gcc/arm-none-eabi/13.2.1/thumb/v7e-m+dp/hard/libgcc.a(_udivmoddi4.o)
 .debug_str     0x000096d0       0xc3 /usr/lib/gcc/arm-none-eabi/13.2.1/thumb/v7e-m+dp/hard/libgcc.a(_dvmd_tls.o)

.debug_frame    0x00000000     0x4ce4
 .debug_frame   0x00000000      0x4b0 build/main.o
 .debug_frame   0x000004b0      0x180 build/bsp_driver_sd.o
 .debug_frame   0x00000630       0xac build/sd_diskio.o
 .debug_frame   0x000006dc       0x38 build/fatfs.o
 .debug_frame   0x00000714       0x28 build/fatfs_platform.o
 .debug_frame   0x0000073c      0x1b4 build/stm32f7xx_it.o
 .debug_frame   0x000008f0      0x138 build/stm32f7xx_hal_msp.o
 .debug_frame   0x00000a28      0x268 build/stm32f7xx_hal_adc.o
 .debug_frame   0x00000c90      0x18c build/stm32f7xx_hal_adc_ex.o
 .debug_frame   0x00000e1c      0x178 build/stm32f7xx_hal_rcc.o
 .debug_frame   0x00000f94       0xc0 build/stm32f7xx_hal_rcc_ex.o
 .debug_frame   0x00001054       0xd8 build/stm32f7xx_hal_gpio.o
 .debug_frame   0x0000112c      0x134 build/stm32f7xx_hal_pwr_ex.o
 .debug_frame   0x00001260      0x1ec build/stm32f7xx_hal_cortex.o
 .debug_frame   0x0000144c      0x22c build/stm32f7xx_hal.o
 .debug_frame   0x00001678      0x250 build/stm32f7xx_ll_rcc.o
 .debug_frame   0x000018c8       0xc8 build/stm32f7xx_ll_gpio.o
 .debug_frame   0x00001990      0x4c8 build/stm32f7xx_ll_sdmmc.o
 .debug_frame   0x00001e58      0x4b8 build/stm32f7xx_hal_sd.o
 .debug_frame   0x00002310       0xa8 build/stm32f7xx_ll_spi.o
 .debug_frame   0x000023b8      0xb6c build/stm32f7xx_hal_tim.o
 .debug_frame   0x00002f24      0x478 build/stm32f7xx_hal_tim_ex.o
 .debug_frame   0x0000339c      0x24c build/stm32f7xx_ll_tim.o
 .debug_frame   0x000035e8       0x88 build/stm32f7xx_ll_usart.o
 .debug_frame   0x00003670       0x30 build/system_stm32f7xx.o
 .debug_frame   0x000036a0      0x1e8 build/File_Handling.o
 .debug_frame   0x00003888       0xa0 build/diskio.o
 .debug_frame   0x00003928      0x7bc build/ff.o
 .debug_frame   0x000040e4       0x7c build/ff_gen_drv.o
 .debug_frame   0x00004160       0x28 build/sysmem.o
 .debug_frame   0x00004188      0x608 build/stm32f7xx_hal_uart.o
 .debug_frame   0x00004790       0x78 /usr/lib/gcc/arm-none-eabi/13.2.1/../../../arm-none-eabi/lib/thumb/v7e-m+dp/hard/libc_nano.a(libc_a-sprintf.o)
 .debug_frame   0x00004808       0x98 /usr/lib/gcc/arm-none-eabi/13.2.1/../../../arm-none-eabi/lib/thumb/v7e-m+dp/hard/libc_nano.a(libc_a-nano-svfprintf.o)
 .debug_frame   0x000048a0       0x2c /usr/lib/gcc/arm-none-eabi/13.2.1/../../../arm-none-eabi/lib/thumb/v7e-m+dp/hard/libc_nano.a(libc_a-init.o)
 .debug_frame   0x000048cc       0x2c /usr/lib/gcc/arm-none-eabi/13.2.1/../../../arm-none-eabi/lib/thumb/v7e-m+dp/hard/libc_nano.a(libc_a-memset.o)
 .debug_frame   0x000048f8       0x20 /usr/lib/gcc/arm-none-eabi/13.2.1/../../../arm-none-eabi/lib/thumb/v7e-m+dp/hard/libc_nano.a(libc_a-errno.o)
 .debug_frame   0x00004918       0x50 /usr/lib/gcc/arm-none-eabi/13.2.1/../../../arm-none-eabi/lib/thumb/v7e-m+dp/hard/libc_nano.a(libc_a-mallocr.o)
 .debug_frame   0x00004968       0x58 /usr/lib/gcc/arm-none-eabi/13.2.1/../../../arm-none-eabi/lib/thumb/v7e-m+dp/hard/libc_nano.a(libc_a-freer.o)
 .debug_frame   0x000049c0       0x40 /usr/lib/gcc/arm-none-eabi/13.2.1/../../../arm-none-eabi/lib/thumb/v7e-m+dp/hard/libc_nano.a(libc_a-memmove.o)
 .debug_frame   0x00004a00       0x30 /usr/lib/gcc/arm-none-eabi/13.2.1/../../../arm-none-eabi/lib/thumb/v7e-m+dp/hard/libc_nano.a(libc_a-malloc.o)
 .debug_frame   0x00004a30       0x38 /usr/lib/gcc/arm-none-eabi/13.2.1/../../../arm-none-eabi/lib/thumb/v7e-m+dp/hard/libc_nano.a(libc_a-reallocr.o)
 .debug_frame   0x00004a68       0x6c /usr/lib/gcc/arm-none-eabi/13.2.1/../../../arm-none-eabi/lib/thumb/v7e-m+dp/hard/libc_nano.a(libc_a-nano-vfprintf_i.o)
 .debug_frame   0x00004ad4       0x30 /usr/lib/gcc/arm-none-eabi/13.2.1/../../../arm-none-eabi/lib/thumb/v7e-m+dp/hard/libc_nano.a(libc_a-mlock.o)
 .debug_frame   0x00004b04       0x2c /usr/lib/gcc/arm-none-eabi/13.2.1/../../../arm-none-eabi/lib/thumb/v7e-m+dp/hard/libc_nano.a(libc_a-sbrkr.o)
 .debug_frame   0x00004b30       0x20 /usr/lib/gcc/arm-none-eabi/13.2.1/../../../arm-none-eabi/lib/thumb/v7e-m+dp/hard/libc_nano.a(libc_a-msizer.o)
 .debug_frame   0x00004b50       0xf4 /usr/lib/gcc/arm-none-eabi/13.2.1/../../../arm-none-eabi/lib/thumb/v7e-m+dp/hard/libc_nano.a(libc_a-findfp.o)
 .debug_frame   0x00004c44       0x40 /usr/lib/gcc/arm-none-eabi/13.2.1/../../../arm-none-eabi/lib/thumb/v7e-m+dp/hard/libc_nano.a(libc_a-reent.o)
 .debug_frame   0x00004c84       0x2c /usr/lib/gcc/arm-none-eabi/13.2.1/thumb/v7e-m+dp/hard/libgcc.a(_aeabi_uldivmod.o)
 .debug_frame   0x00004cb0       0x34 /usr/lib/gcc/arm-none-eabi/13.2.1/thumb/v7e-m+dp/hard/libgcc.a(_udivmoddi4.o)

.debug_loclists
                0x00000000     0x2087
 .debug_loclists
                0x00000000       0x88 /usr/lib/gcc/arm-none-eabi/13.2.1/../../../arm-none-eabi/lib/thumb/v7e-m+dp/hard/libc_nano.a(libc_a-sprintf.o)
 .debug_loclists
                0x00000088      0x56b /usr/lib/gcc/arm-none-eabi/13.2.1/../../../arm-none-eabi/lib/thumb/v7e-m+dp/hard/libc_nano.a(libc_a-nano-svfprintf.o)
 .debug_loclists
                0x000005f3       0x65 /usr/lib/gcc/arm-none-eabi/13.2.1/../../../arm-none-eabi/lib/thumb/v7e-m+dp/hard/libc_nano.a(libc_a-init.o)
 .debug_loclists
                0x00000658      0x1c2 /usr/lib/gcc/arm-none-eabi/13.2.1/../../../arm-none-eabi/lib/thumb/v7e-m+dp/hard/libc_nano.a(libc_a-memset.o)
 .debug_loclists
                0x0000081a      0x263 /usr/lib/gcc/arm-none-eabi/13.2.1/../../../arm-none-eabi/lib/thumb/v7e-m+dp/hard/libc_nano.a(libc_a-mallocr.o)
 .debug_loclists
                0x00000a7d      0x164 /usr/lib/gcc/arm-none-eabi/13.2.1/../../../arm-none-eabi/lib/thumb/v7e-m+dp/hard/libc_nano.a(libc_a-freer.o)
 .debug_loclists
                0x00000be1      0x233 /usr/lib/gcc/arm-none-eabi/13.2.1/../../../arm-none-eabi/lib/thumb/v7e-m+dp/hard/libc_nano.a(libc_a-memmove.o)
 .debug_loclists
                0x00000e14       0x4a /usr/lib/gcc/arm-none-eabi/13.2.1/../../../arm-none-eabi/lib/thumb/v7e-m+dp/hard/libc_nano.a(libc_a-malloc.o)
 .debug_loclists
                0x00000e5e      0x102 /usr/lib/gcc/arm-none-eabi/13.2.1/../../../arm-none-eabi/lib/thumb/v7e-m+dp/hard/libc_nano.a(libc_a-reallocr.o)
 .debug_loclists
                0x00000f60      0x44f /usr/lib/gcc/arm-none-eabi/13.2.1/../../../arm-none-eabi/lib/thumb/v7e-m+dp/hard/libc_nano.a(libc_a-nano-vfprintf_i.o)
 .debug_loclists
                0x000013af       0x4b /usr/lib/gcc/arm-none-eabi/13.2.1/../../../arm-none-eabi/lib/thumb/v7e-m+dp/hard/libc_nano.a(libc_a-sbrkr.o)
 .debug_loclists
                0x000013fa       0x59 /usr/lib/gcc/arm-none-eabi/13.2.1/../../../arm-none-eabi/lib/thumb/v7e-m+dp/hard/libc_nano.a(libc_a-msizer.o)
 .debug_loclists
                0x00001453      0x1d0 /usr/lib/gcc/arm-none-eabi/13.2.1/../../../arm-none-eabi/lib/thumb/v7e-m+dp/hard/libc_nano.a(libc_a-findfp.o)
 .debug_loclists
                0x00001623       0x80 /usr/lib/gcc/arm-none-eabi/13.2.1/../../../arm-none-eabi/lib/thumb/v7e-m+dp/hard/libc_nano.a(libc_a-reent.o)
 .debug_loclists
                0x000016a3      0x9e4 /usr/lib/gcc/arm-none-eabi/13.2.1/thumb/v7e-m+dp/hard/libgcc.a(_udivmoddi4.o)

.debug_rnglists
                0x00000000      0x1d4
 .debug_rnglists
                0x00000000       0x42 /usr/lib/gcc/arm-none-eabi/13.2.1/../../../arm-none-eabi/lib/thumb/v7e-m+dp/hard/libc_nano.a(libc_a-nano-svfprintf.o)
 .debug_rnglists
                0x00000042       0x1e /usr/lib/gcc/arm-none-eabi/13.2.1/../../../arm-none-eabi/lib/thumb/v7e-m+dp/hard/libc_nano.a(libc_a-mallocr.o)
 .debug_rnglists
                0x00000060       0x13 /usr/lib/gcc/arm-none-eabi/13.2.1/../../../arm-none-eabi/lib/thumb/v7e-m+dp/hard/libc_nano.a(libc_a-freer.o)
 .debug_rnglists
                0x00000073       0x66 /usr/lib/gcc/arm-none-eabi/13.2.1/../../../arm-none-eabi/lib/thumb/v7e-m+dp/hard/libc_nano.a(libc_a-nano-vfprintf_i.o)
 .debug_rnglists
                0x000000d9       0x77 /usr/lib/gcc/arm-none-eabi/13.2.1/../../../arm-none-eabi/lib/thumb/v7e-m+dp/hard/libc_nano.a(libc_a-findfp.o)
 .debug_rnglists
                0x00000150       0x84 /usr/lib/gcc/arm-none-eabi/13.2.1/thumb/v7e-m+dp/hard/libgcc.a(_udivmoddi4.o)

.debug_line_str
                0x00000000      0x145
 .debug_line_str
                0x00000000      0x145 /usr/lib/gcc/arm-none-eabi/13.2.1/../../../arm-none-eabi/lib/thumb/v7e-m+dp/hard/libc_nano.a(libc_a-memchr.o)
                                 0x92 (size before relaxing)
 .debug_line_str
                0x00000145       0x99 /usr/lib/gcc/arm-none-eabi/13.2.1/../../../arm-none-eabi/lib/thumb/v7e-m+dp/hard/libc_nano.a(libc_a-memcpy.o)
 .debug_line_str
                0x00000145       0x97 /usr/lib/gcc/arm-none-eabi/13.2.1/thumb/v7e-m+dp/hard/libgcc.a(_aeabi_uldivmod.o)
 .debug_line_str
                0x00000145       0x9b /usr/lib/gcc/arm-none-eabi/13.2.1/thumb/v7e-m+dp/hard/libgcc.a(_dvmd_tls.o)

Cross Reference Table

Symbol                                            File
ADC_IRQHandler                                    build/stm32f7xx_it.o
AHBPrescTable                                     build/system_stm32f7xx.o
                                                  build/stm32f7xx_ll_utils.o
                                                  build/stm32f7xx_ll_rcc.o
                                                  build/stm32f7xx_hal_rcc.o
APBPrescTable                                     build/system_stm32f7xx.o
                                                  build/stm32f7xx_ll_rcc.o
                                                  build/stm32f7xx_hal_rcc.o
Advanced_Controller_Temp                          build/main.o
BSP_PlatformIsDetected                            build/fatfs_platform.o
                                                  build/bsp_driver_sd.o
BSP_SD_AbortCallback                              build/bsp_driver_sd.o
BSP_SD_Erase                                      build/bsp_driver_sd.o
BSP_SD_GetCardInfo                                build/bsp_driver_sd.o
                                                  build/sd_diskio.o
BSP_SD_GetCardState                               build/bsp_driver_sd.o
                                                  build/sd_diskio.o
BSP_SD_ITConfig                                   build/bsp_driver_sd.o
BSP_SD_Init                                       build/bsp_driver_sd.o
                                                  build/sd_diskio.o
BSP_SD_IsDetected                                 build/bsp_driver_sd.o
BSP_SD_ReadBlocks                                 build/bsp_driver_sd.o
                                                  build/sd_diskio.o
BSP_SD_ReadBlocks_DMA                             build/bsp_driver_sd.o
BSP_SD_ReadCpltCallback                           build/bsp_driver_sd.o
BSP_SD_WriteBlocks                                build/bsp_driver_sd.o
                                                  build/sd_diskio.o
BSP_SD_WriteBlocks_DMA                            build/bsp_driver_sd.o
BSP_SD_WriteCpltCallback                          build/bsp_driver_sd.o
BusFault_Handler                                  build/stm32f7xx_it.o
CAN1_RX0_IRQHandler                               build/startup_stm32f767xx.o
CAN1_RX1_IRQHandler                               build/startup_stm32f767xx.o
CAN1_SCE_IRQHandler                               build/startup_stm32f767xx.o
CAN1_TX_IRQHandler                                build/startup_stm32f767xx.o
CAN2_RX0_IRQHandler                               build/startup_stm32f767xx.o
CAN2_RX1_IRQHandler                               build/startup_stm32f767xx.o
CAN2_SCE_IRQHandler                               build/startup_stm32f767xx.o
CAN2_TX_IRQHandler                                build/startup_stm32f767xx.o
CAN3_RX0_IRQHandler                               build/startup_stm32f767xx.o
CAN3_RX1_IRQHandler                               build/startup_stm32f767xx.o
CAN3_SCE_IRQHandler                               build/startup_stm32f767xx.o
CAN3_TX_IRQHandler                                build/startup_stm32f767xx.o
CEC_IRQHandler                                    build/startup_stm32f767xx.o
COMMAND                                           build/main.o
                                                  build/stm32f7xx_it.o
CPU_state                                         build/main.o
                                                  build/stm32f7xx_it.o
CPU_state_old                                     build/main.o
CS_result                                         build/main.o
CalculateChecksum                                 build/main.o
CheckChecksum                                     build/main.o
Check_SD_Space                                    build/File_Handling.o
Create_Dir                                        build/File_Handling.o
Create_File                                       build/File_Handling.o
                                                  build/main.o
Curr_setup                                        build/main.o
DCMI_IRQHandler                                   build/startup_stm32f767xx.o
DFSDM1_FLT0_IRQHandler                            build/startup_stm32f767xx.o
DFSDM1_FLT1_IRQHandler                            build/startup_stm32f767xx.o
DFSDM1_FLT2_IRQHandler                            build/startup_stm32f767xx.o
DFSDM1_FLT3_IRQHandler                            build/startup_stm32f767xx.o
DMA1_Stream0_IRQHandler                           build/startup_stm32f767xx.o
DMA1_Stream1_IRQHandler                           build/startup_stm32f767xx.o
DMA1_Stream2_IRQHandler                           build/startup_stm32f767xx.o
DMA1_Stream3_IRQHandler                           build/startup_stm32f767xx.o
DMA1_Stream4_IRQHandler                           build/startup_stm32f767xx.o
DMA1_Stream5_IRQHandler                           build/startup_stm32f767xx.o
DMA1_Stream6_IRQHandler                           build/startup_stm32f767xx.o
DMA1_Stream7_IRQHandler                           build/startup_stm32f767xx.o
DMA2D_IRQHandler                                  build/startup_stm32f767xx.o
DMA2_Stream0_IRQHandler                           build/startup_stm32f767xx.o
DMA2_Stream1_IRQHandler                           build/startup_stm32f767xx.o
DMA2_Stream2_IRQHandler                           build/startup_stm32f767xx.o
DMA2_Stream3_IRQHandler                           build/startup_stm32f767xx.o
DMA2_Stream4_IRQHandler                           build/startup_stm32f767xx.o
DMA2_Stream5_IRQHandler                           build/startup_stm32f767xx.o
DMA2_Stream6_IRQHandler                           build/startup_stm32f767xx.o
DMA2_Stream7_IRQHandler                           build/stm32f7xx_it.o
DMA2_Stream7_TransferComplete                     build/stm32f7xx_it.o
DebugMon_Handler                                  build/stm32f7xx_it.o
Def_setup                                         build/main.o
Default_Handler                                   build/startup_stm32f767xx.o
ETH_IRQHandler                                    build/startup_stm32f767xx.o
ETH_WKUP_IRQHandler                               build/startup_stm32f767xx.o
EXTI0_IRQHandler                                  build/startup_stm32f767xx.o
EXTI15_10_IRQHandler                              build/startup_stm32f767xx.o
EXTI1_IRQHandler                                  build/startup_stm32f767xx.o
EXTI2_IRQHandler                                  build/startup_stm32f767xx.o
EXTI3_IRQHandler                                  build/startup_stm32f767xx.o
EXTI4_IRQHandler                                  build/startup_stm32f767xx.o
EXTI9_5_IRQHandler                                build/startup_stm32f767xx.o
Error_Handler                                     build/main.o
                                                  build/stm32f7xx_hal_msp.o
FATFS_GetAttachedDriversNbr                       build/ff_gen_drv.o
FATFS_LinkDriver                                  build/ff_gen_drv.o
                                                  build/fatfs.o
FATFS_LinkDriverEx                                build/ff_gen_drv.o
FATFS_UnLinkDriver                                build/ff_gen_drv.o
FATFS_UnLinkDriverEx                              build/ff_gen_drv.o
FLASH_Erase_Sector                                build/stm32f7xx_hal_flash_ex.o
                                                  build/stm32f7xx_hal_flash.o
FLASH_IRQHandler                                  build/startup_stm32f767xx.o
FLASH_WaitForLastOperation                        build/stm32f7xx_hal_flash.o
                                                  build/stm32f7xx_hal_flash_ex.o
FMC_IRQHandler                                    build/startup_stm32f767xx.o
FPU_IRQHandler                                    build/startup_stm32f767xx.o
Format_SD                                         build/File_Handling.o
HAL_ADCEx_InjectedConfigChannel                   build/stm32f7xx_hal_adc_ex.o
HAL_ADCEx_InjectedConvCpltCallback                build/stm32f7xx_hal_adc_ex.o
                                                  build/stm32f7xx_hal_adc.o
HAL_ADCEx_InjectedGetValue                        build/stm32f7xx_hal_adc_ex.o
HAL_ADCEx_InjectedPollForConversion               build/stm32f7xx_hal_adc_ex.o
HAL_ADCEx_InjectedStart                           build/stm32f7xx_hal_adc_ex.o
HAL_ADCEx_InjectedStart_IT                        build/stm32f7xx_hal_adc_ex.o
HAL_ADCEx_InjectedStop                            build/stm32f7xx_hal_adc_ex.o
HAL_ADCEx_InjectedStop_IT                         build/stm32f7xx_hal_adc_ex.o
HAL_ADCEx_MultiModeConfigChannel                  build/stm32f7xx_hal_adc_ex.o
HAL_ADCEx_MultiModeGetValue                       build/stm32f7xx_hal_adc_ex.o
HAL_ADCEx_MultiModeStart_DMA                      build/stm32f7xx_hal_adc_ex.o
HAL_ADCEx_MultiModeStop_DMA                       build/stm32f7xx_hal_adc_ex.o
HAL_ADC_AnalogWDGConfig                           build/stm32f7xx_hal_adc.o
HAL_ADC_ConfigChannel                             build/stm32f7xx_hal_adc.o
                                                  build/main.o
HAL_ADC_ConvCpltCallback                          build/stm32f7xx_hal_adc.o
                                                  build/stm32f7xx_hal_adc_ex.o
HAL_ADC_ConvHalfCpltCallback                      build/stm32f7xx_hal_adc.o
                                                  build/stm32f7xx_hal_adc_ex.o
HAL_ADC_DeInit                                    build/stm32f7xx_hal_adc.o
HAL_ADC_ErrorCallback                             build/stm32f7xx_hal_adc.o
                                                  build/stm32f7xx_hal_adc_ex.o
HAL_ADC_GetError                                  build/stm32f7xx_hal_adc.o
HAL_ADC_GetState                                  build/stm32f7xx_hal_adc.o
HAL_ADC_GetValue                                  build/stm32f7xx_hal_adc.o
                                                  build/main.o
HAL_ADC_IRQHandler                                build/stm32f7xx_hal_adc.o
                                                  build/stm32f7xx_it.o
HAL_ADC_Init                                      build/stm32f7xx_hal_adc.o
                                                  build/main.o
HAL_ADC_LevelOutOfWindowCallback                  build/stm32f7xx_hal_adc.o
HAL_ADC_MspDeInit                                 build/stm32f7xx_hal_msp.o
HAL_ADC_MspInit                                   build/stm32f7xx_hal_msp.o
HAL_ADC_PollForConversion                         build/stm32f7xx_hal_adc.o
                                                  build/main.o
HAL_ADC_PollForEvent                              build/stm32f7xx_hal_adc.o
HAL_ADC_Start                                     build/stm32f7xx_hal_adc.o
                                                  build/main.o
HAL_ADC_Start_DMA                                 build/stm32f7xx_hal_adc.o
HAL_ADC_Start_IT                                  build/stm32f7xx_hal_adc.o
HAL_ADC_Stop                                      build/stm32f7xx_hal_adc.o
                                                  build/main.o
HAL_ADC_Stop_DMA                                  build/stm32f7xx_hal_adc.o
HAL_ADC_Stop_IT                                   build/stm32f7xx_hal_adc.o
HAL_DBGMCU_DisableDBGSleepMode                    build/stm32f7xx_hal.o
HAL_DBGMCU_DisableDBGStandbyMode                  build/stm32f7xx_hal.o
HAL_DBGMCU_DisableDBGStopMode                     build/stm32f7xx_hal.o
HAL_DBGMCU_EnableDBGSleepMode                     build/stm32f7xx_hal.o
HAL_DBGMCU_EnableDBGStandbyMode                   build/stm32f7xx_hal.o
HAL_DBGMCU_EnableDBGStopMode                      build/stm32f7xx_hal.o
HAL_DMAEx_ChangeMemory                            build/stm32f7xx_hal_dma_ex.o
HAL_DMAEx_MultiBufferStart                        build/stm32f7xx_hal_dma_ex.o
HAL_DMAEx_MultiBufferStart_IT                     build/stm32f7xx_hal_dma_ex.o
HAL_DMA_Abort                                     build/stm32f7xx_hal_dma.o
                                                  build/stm32f7xx_hal_uart.o
                                                  build/stm32f7xx_hal_sd.o
                                                  build/stm32f7xx_hal_adc_ex.o
                                                  build/stm32f7xx_hal_adc.o
HAL_DMA_Abort_IT                                  build/stm32f7xx_hal_dma.o
                                                  build/stm32f7xx_hal_uart.o
                                                  build/stm32f7xx_hal_tim_ex.o
                                                  build/stm32f7xx_hal_tim.o
                                                  build/stm32f7xx_hal_sd.o
                                                  build/stm32f7xx_hal_i2c.o
HAL_DMA_DeInit                                    build/stm32f7xx_hal_dma.o
HAL_DMA_GetError                                  build/stm32f7xx_hal_dma.o
                                                  build/stm32f7xx_hal_uart.o
                                                  build/stm32f7xx_hal_sd.o
                                                  build/stm32f7xx_hal_i2c.o
HAL_DMA_GetState                                  build/stm32f7xx_hal_dma.o
                                                  build/stm32f7xx_hal_i2c.o
HAL_DMA_IRQHandler                                build/stm32f7xx_hal_dma.o
HAL_DMA_Init                                      build/stm32f7xx_hal_dma.o
HAL_DMA_PollForTransfer                           build/stm32f7xx_hal_dma.o
HAL_DMA_RegisterCallback                          build/stm32f7xx_hal_dma.o
HAL_DMA_Start                                     build/stm32f7xx_hal_dma.o
HAL_DMA_Start_IT                                  build/stm32f7xx_hal_dma.o
                                                  build/stm32f7xx_hal_uart.o
                                                  build/stm32f7xx_hal_tim_ex.o
                                                  build/stm32f7xx_hal_tim.o
                                                  build/stm32f7xx_hal_sd.o
                                                  build/stm32f7xx_hal_i2c.o
                                                  build/stm32f7xx_hal_adc_ex.o
                                                  build/stm32f7xx_hal_adc.o
HAL_DMA_UnRegisterCallback                        build/stm32f7xx_hal_dma.o
HAL_DeInit                                        build/stm32f7xx_hal.o
HAL_Delay                                         build/stm32f7xx_hal.o
                                                  build/stm32f7xx_hal_sd.o
HAL_DisableCompensationCell                       build/stm32f7xx_hal.o
HAL_DisableFMCMemorySwapping                      build/stm32f7xx_hal.o
HAL_DisableMemorySwappingBank                     build/stm32f7xx_hal.o
HAL_EXTI_ClearConfigLine                          build/stm32f7xx_hal_exti.o
HAL_EXTI_ClearPending                             build/stm32f7xx_hal_exti.o
HAL_EXTI_GenerateSWI                              build/stm32f7xx_hal_exti.o
HAL_EXTI_GetConfigLine                            build/stm32f7xx_hal_exti.o
HAL_EXTI_GetHandle                                build/stm32f7xx_hal_exti.o
HAL_EXTI_GetPending                               build/stm32f7xx_hal_exti.o
HAL_EXTI_IRQHandler                               build/stm32f7xx_hal_exti.o
HAL_EXTI_RegisterCallback                         build/stm32f7xx_hal_exti.o
HAL_EXTI_SetConfigLine                            build/stm32f7xx_hal_exti.o
HAL_EnableCompensationCell                        build/stm32f7xx_hal.o
HAL_EnableFMCMemorySwapping                       build/stm32f7xx_hal.o
HAL_EnableMemorySwappingBank                      build/stm32f7xx_hal.o
HAL_FLASHEx_Erase                                 build/stm32f7xx_hal_flash_ex.o
HAL_FLASHEx_Erase_IT                              build/stm32f7xx_hal_flash_ex.o
HAL_FLASHEx_OBGetConfig                           build/stm32f7xx_hal_flash_ex.o
HAL_FLASHEx_OBProgram                             build/stm32f7xx_hal_flash_ex.o
HAL_FLASH_EndOfOperationCallback                  build/stm32f7xx_hal_flash.o
HAL_FLASH_GetError                                build/stm32f7xx_hal_flash.o
HAL_FLASH_IRQHandler                              build/stm32f7xx_hal_flash.o
HAL_FLASH_Lock                                    build/stm32f7xx_hal_flash.o
HAL_FLASH_OB_Launch                               build/stm32f7xx_hal_flash.o
HAL_FLASH_OB_Lock                                 build/stm32f7xx_hal_flash.o
HAL_FLASH_OB_Unlock                               build/stm32f7xx_hal_flash.o
HAL_FLASH_OperationErrorCallback                  build/stm32f7xx_hal_flash.o
HAL_FLASH_Program                                 build/stm32f7xx_hal_flash.o
HAL_FLASH_Program_IT                              build/stm32f7xx_hal_flash.o
HAL_FLASH_Unlock                                  build/stm32f7xx_hal_flash.o
HAL_GPIO_DeInit                                   build/stm32f7xx_hal_gpio.o
                                                  build/stm32f7xx_hal_msp.o
HAL_GPIO_EXTI_Callback                            build/stm32f7xx_hal_gpio.o
HAL_GPIO_EXTI_IRQHandler                          build/stm32f7xx_hal_gpio.o
HAL_GPIO_Init                                     build/stm32f7xx_hal_gpio.o
                                                  build/stm32f7xx_hal_rcc.o
                                                  build/stm32f7xx_hal_msp.o
                                                  build/main.o
HAL_GPIO_LockPin                                  build/stm32f7xx_hal_gpio.o
HAL_GPIO_ReadPin                                  build/stm32f7xx_hal_gpio.o
                                                  build/fatfs_platform.o
                                                  build/main.o
HAL_GPIO_TogglePin                                build/stm32f7xx_hal_gpio.o
                                                  build/stm32f7xx_it.o
                                                  build/main.o
HAL_GPIO_WritePin                                 build/stm32f7xx_hal_gpio.o
                                                  build/stm32f7xx_it.o
                                                  build/main.o
HAL_GetDEVID                                      build/stm32f7xx_hal.o
HAL_GetHalVersion                                 build/stm32f7xx_hal.o
HAL_GetREVID                                      build/stm32f7xx_hal.o
HAL_GetTick                                       build/stm32f7xx_hal.o
                                                  build/stm32f7xx_hal_uart_ex.o
                                                  build/stm32f7xx_hal_uart.o
                                                  build/stm32f7xx_hal_sd.o
                                                  build/stm32f7xx_hal_i2c.o
                                                  build/stm32f7xx_hal_pwr_ex.o
                                                  build/stm32f7xx_hal_dma.o
                                                  build/stm32f7xx_hal_flash.o
                                                  build/stm32f7xx_hal_rcc_ex.o
                                                  build/stm32f7xx_hal_rcc.o
                                                  build/stm32f7xx_hal_adc_ex.o
                                                  build/stm32f7xx_hal_adc.o
HAL_GetTickFreq                                   build/stm32f7xx_hal.o
HAL_GetTickPrio                                   build/stm32f7xx_hal.o
HAL_GetUIDw0                                      build/stm32f7xx_hal.o
HAL_GetUIDw1                                      build/stm32f7xx_hal.o
HAL_GetUIDw2                                      build/stm32f7xx_hal.o
HAL_HalfDuplex_EnableReceiver                     build/stm32f7xx_hal_uart.o
HAL_HalfDuplex_EnableTransmitter                  build/stm32f7xx_hal_uart.o
HAL_HalfDuplex_Init                               build/stm32f7xx_hal_uart.o
HAL_I2CEx_ConfigAnalogFilter                      build/stm32f7xx_hal_i2c_ex.o
HAL_I2CEx_ConfigDigitalFilter                     build/stm32f7xx_hal_i2c_ex.o
HAL_I2CEx_DisableFastModePlus                     build/stm32f7xx_hal_i2c_ex.o
HAL_I2CEx_EnableFastModePlus                      build/stm32f7xx_hal_i2c_ex.o
HAL_I2C_AbortCpltCallback                         build/stm32f7xx_hal_i2c.o
HAL_I2C_AddrCallback                              build/stm32f7xx_hal_i2c.o
HAL_I2C_DeInit                                    build/stm32f7xx_hal_i2c.o
HAL_I2C_DisableListen_IT                          build/stm32f7xx_hal_i2c.o
HAL_I2C_ER_IRQHandler                             build/stm32f7xx_hal_i2c.o
HAL_I2C_EV_IRQHandler                             build/stm32f7xx_hal_i2c.o
HAL_I2C_EnableListen_IT                           build/stm32f7xx_hal_i2c.o
HAL_I2C_ErrorCallback                             build/stm32f7xx_hal_i2c.o
HAL_I2C_GetError                                  build/stm32f7xx_hal_i2c.o
HAL_I2C_GetMode                                   build/stm32f7xx_hal_i2c.o
HAL_I2C_GetState                                  build/stm32f7xx_hal_i2c.o
HAL_I2C_Init                                      build/stm32f7xx_hal_i2c.o
HAL_I2C_IsDeviceReady                             build/stm32f7xx_hal_i2c.o
HAL_I2C_ListenCpltCallback                        build/stm32f7xx_hal_i2c.o
HAL_I2C_MasterRxCpltCallback                      build/stm32f7xx_hal_i2c.o
HAL_I2C_MasterTxCpltCallback                      build/stm32f7xx_hal_i2c.o
HAL_I2C_Master_Abort_IT                           build/stm32f7xx_hal_i2c.o
HAL_I2C_Master_Receive                            build/stm32f7xx_hal_i2c.o
HAL_I2C_Master_Receive_DMA                        build/stm32f7xx_hal_i2c.o
HAL_I2C_Master_Receive_IT                         build/stm32f7xx_hal_i2c.o
HAL_I2C_Master_Seq_Receive_DMA                    build/stm32f7xx_hal_i2c.o
HAL_I2C_Master_Seq_Receive_IT                     build/stm32f7xx_hal_i2c.o
HAL_I2C_Master_Seq_Transmit_DMA                   build/stm32f7xx_hal_i2c.o
HAL_I2C_Master_Seq_Transmit_IT                    build/stm32f7xx_hal_i2c.o
HAL_I2C_Master_Transmit                           build/stm32f7xx_hal_i2c.o
HAL_I2C_Master_Transmit_DMA                       build/stm32f7xx_hal_i2c.o
HAL_I2C_Master_Transmit_IT                        build/stm32f7xx_hal_i2c.o
HAL_I2C_MemRxCpltCallback                         build/stm32f7xx_hal_i2c.o
HAL_I2C_MemTxCpltCallback                         build/stm32f7xx_hal_i2c.o
HAL_I2C_Mem_Read                                  build/stm32f7xx_hal_i2c.o
HAL_I2C_Mem_Read_DMA                              build/stm32f7xx_hal_i2c.o
HAL_I2C_Mem_Read_IT                               build/stm32f7xx_hal_i2c.o
HAL_I2C_Mem_Write                                 build/stm32f7xx_hal_i2c.o
HAL_I2C_Mem_Write_DMA                             build/stm32f7xx_hal_i2c.o
HAL_I2C_Mem_Write_IT                              build/stm32f7xx_hal_i2c.o
HAL_I2C_MspDeInit                                 build/stm32f7xx_hal_i2c.o
HAL_I2C_MspInit                                   build/stm32f7xx_hal_i2c.o
HAL_I2C_SlaveRxCpltCallback                       build/stm32f7xx_hal_i2c.o
HAL_I2C_SlaveTxCpltCallback                       build/stm32f7xx_hal_i2c.o
HAL_I2C_Slave_Receive                             build/stm32f7xx_hal_i2c.o
HAL_I2C_Slave_Receive_DMA                         build/stm32f7xx_hal_i2c.o
HAL_I2C_Slave_Receive_IT                          build/stm32f7xx_hal_i2c.o
HAL_I2C_Slave_Seq_Receive_DMA                     build/stm32f7xx_hal_i2c.o
HAL_I2C_Slave_Seq_Receive_IT                      build/stm32f7xx_hal_i2c.o
HAL_I2C_Slave_Seq_Transmit_DMA                    build/stm32f7xx_hal_i2c.o
HAL_I2C_Slave_Seq_Transmit_IT                     build/stm32f7xx_hal_i2c.o
HAL_I2C_Slave_Transmit                            build/stm32f7xx_hal_i2c.o
HAL_I2C_Slave_Transmit_DMA                        build/stm32f7xx_hal_i2c.o
HAL_I2C_Slave_Transmit_IT                         build/stm32f7xx_hal_i2c.o
HAL_IncTick                                       build/stm32f7xx_hal.o
                                                  build/stm32f7xx_it.o
HAL_Init                                          build/stm32f7xx_hal.o
                                                  build/main.o
HAL_InitTick                                      build/stm32f7xx_hal.o
                                                  build/stm32f7xx_hal_rcc.o
HAL_LIN_Init                                      build/stm32f7xx_hal_uart.o
HAL_LIN_SendBreak                                 build/stm32f7xx_hal_uart.o
HAL_MPU_ConfigRegion                              build/stm32f7xx_hal_cortex.o
HAL_MPU_Disable                                   build/stm32f7xx_hal_cortex.o
HAL_MPU_DisableRegion                             build/stm32f7xx_hal_cortex.o
HAL_MPU_Enable                                    build/stm32f7xx_hal_cortex.o
HAL_MPU_EnableRegion                              build/stm32f7xx_hal_cortex.o
HAL_MspDeInit                                     build/stm32f7xx_hal.o
HAL_MspInit                                       build/stm32f7xx_hal_msp.o
HAL_MultiProcessorEx_AddressLength_Set            build/stm32f7xx_hal_uart_ex.o
HAL_MultiProcessor_DisableMuteMode                build/stm32f7xx_hal_uart.o
HAL_MultiProcessor_EnableMuteMode                 build/stm32f7xx_hal_uart.o
HAL_MultiProcessor_EnterMuteMode                  build/stm32f7xx_hal_uart.o
HAL_MultiProcessor_Init                           build/stm32f7xx_hal_uart.o
HAL_NVIC_ClearPendingIRQ                          build/stm32f7xx_hal_cortex.o
HAL_NVIC_DisableIRQ                               build/stm32f7xx_hal_cortex.o
                                                  build/stm32f7xx_hal_msp.o
HAL_NVIC_EnableIRQ                                build/stm32f7xx_hal_cortex.o
                                                  build/stm32f7xx_hal_msp.o
HAL_NVIC_GetActive                                build/stm32f7xx_hal_cortex.o
HAL_NVIC_GetPendingIRQ                            build/stm32f7xx_hal_cortex.o
HAL_NVIC_GetPriority                              build/stm32f7xx_hal_cortex.o
HAL_NVIC_GetPriorityGrouping                      build/stm32f7xx_hal_cortex.o
HAL_NVIC_SetPendingIRQ                            build/stm32f7xx_hal_cortex.o
HAL_NVIC_SetPriority                              build/stm32f7xx_hal_cortex.o
                                                  build/stm32f7xx_hal.o
                                                  build/stm32f7xx_hal_msp.o
HAL_NVIC_SetPriorityGrouping                      build/stm32f7xx_hal_cortex.o
                                                  build/stm32f7xx_hal.o
HAL_NVIC_SystemReset                              build/stm32f7xx_hal_cortex.o
HAL_PWREx_ControlVoltageScaling                   build/stm32f7xx_hal_pwr_ex.o
HAL_PWREx_DisableBkUpReg                          build/stm32f7xx_hal_pwr_ex.o
HAL_PWREx_DisableFlashPowerDown                   build/stm32f7xx_hal_pwr_ex.o
HAL_PWREx_DisableLowRegulatorLowVoltage           build/stm32f7xx_hal_pwr_ex.o
HAL_PWREx_DisableMainRegulatorLowVoltage          build/stm32f7xx_hal_pwr_ex.o
HAL_PWREx_DisableOverDrive                        build/stm32f7xx_hal_pwr_ex.o
HAL_PWREx_EnableBkUpReg                           build/stm32f7xx_hal_pwr_ex.o
HAL_PWREx_EnableFlashPowerDown                    build/stm32f7xx_hal_pwr_ex.o
HAL_PWREx_EnableLowRegulatorLowVoltage            build/stm32f7xx_hal_pwr_ex.o
HAL_PWREx_EnableMainRegulatorLowVoltage           build/stm32f7xx_hal_pwr_ex.o
HAL_PWREx_EnableOverDrive                         build/stm32f7xx_hal_pwr_ex.o
                                                  build/main.o
HAL_PWREx_EnterUnderDriveSTOPMode                 build/stm32f7xx_hal_pwr_ex.o
HAL_PWREx_GetVoltageRange                         build/stm32f7xx_hal_pwr_ex.o
HAL_PWR_ConfigPVD                                 build/stm32f7xx_hal_pwr.o
HAL_PWR_DeInit                                    build/stm32f7xx_hal_pwr.o
HAL_PWR_DisableBkUpAccess                         build/stm32f7xx_hal_pwr.o
HAL_PWR_DisablePVD                                build/stm32f7xx_hal_pwr.o
HAL_PWR_DisableSEVOnPend                          build/stm32f7xx_hal_pwr.o
HAL_PWR_DisableSleepOnExit                        build/stm32f7xx_hal_pwr.o
HAL_PWR_DisableWakeUpPin                          build/stm32f7xx_hal_pwr.o
HAL_PWR_EnableBkUpAccess                          build/stm32f7xx_hal_pwr.o
HAL_PWR_EnablePVD                                 build/stm32f7xx_hal_pwr.o
HAL_PWR_EnableSEVOnPend                           build/stm32f7xx_hal_pwr.o
HAL_PWR_EnableSleepOnExit                         build/stm32f7xx_hal_pwr.o
HAL_PWR_EnableWakeUpPin                           build/stm32f7xx_hal_pwr.o
HAL_PWR_EnterSLEEPMode                            build/stm32f7xx_hal_pwr.o
HAL_PWR_EnterSTANDBYMode                          build/stm32f7xx_hal_pwr.o
HAL_PWR_EnterSTOPMode                             build/stm32f7xx_hal_pwr.o
HAL_PWR_PVDCallback                               build/stm32f7xx_hal_pwr.o
HAL_PWR_PVD_IRQHandler                            build/stm32f7xx_hal_pwr.o
HAL_RCCEx_DisablePLLI2S                           build/stm32f7xx_hal_rcc_ex.o
HAL_RCCEx_DisablePLLSAI                           build/stm32f7xx_hal_rcc_ex.o
HAL_RCCEx_EnablePLLI2S                            build/stm32f7xx_hal_rcc_ex.o
HAL_RCCEx_EnablePLLSAI                            build/stm32f7xx_hal_rcc_ex.o
HAL_RCCEx_GetPeriphCLKConfig                      build/stm32f7xx_hal_rcc_ex.o
HAL_RCCEx_GetPeriphCLKFreq                        build/stm32f7xx_hal_rcc_ex.o
HAL_RCCEx_PeriphCLKConfig                         build/stm32f7xx_hal_rcc_ex.o
                                                  build/stm32f7xx_hal_msp.o
                                                  build/main.o
HAL_RCC_CSSCallback                               build/stm32f7xx_hal_rcc.o
HAL_RCC_ClockConfig                               build/stm32f7xx_hal_rcc.o
                                                  build/main.o
HAL_RCC_DeInit                                    build/stm32f7xx_hal_rcc.o
HAL_RCC_DisableCSS                                build/stm32f7xx_hal_rcc.o
HAL_RCC_EnableCSS                                 build/stm32f7xx_hal_rcc.o
HAL_RCC_GetClockConfig                            build/stm32f7xx_hal_rcc.o
HAL_RCC_GetHCLKFreq                               build/stm32f7xx_hal_rcc.o
HAL_RCC_GetOscConfig                              build/stm32f7xx_hal_rcc.o
HAL_RCC_GetPCLK1Freq                              build/stm32f7xx_hal_rcc.o
                                                  build/stm32f7xx_hal_uart.o
HAL_RCC_GetPCLK2Freq                              build/stm32f7xx_hal_rcc.o
                                                  build/stm32f7xx_hal_uart.o
HAL_RCC_GetSysClockFreq                           build/stm32f7xx_hal_rcc.o
                                                  build/stm32f7xx_hal_uart.o
HAL_RCC_MCOConfig                                 build/stm32f7xx_hal_rcc.o
HAL_RCC_NMI_IRQHandler                            build/stm32f7xx_hal_rcc.o
HAL_RCC_OscConfig                                 build/stm32f7xx_hal_rcc.o
                                                  build/main.o
HAL_RS485Ex_Init                                  build/stm32f7xx_hal_uart_ex.o
HAL_ResumeTick                                    build/stm32f7xx_hal.o
HAL_SD_Abort                                      build/stm32f7xx_hal_sd.o
HAL_SD_AbortCallback                              build/bsp_driver_sd.o
HAL_SD_Abort_IT                                   build/stm32f7xx_hal_sd.o
HAL_SD_ConfigWideBusOperation                     build/stm32f7xx_hal_sd.o
                                                  build/bsp_driver_sd.o
HAL_SD_DeInit                                     build/stm32f7xx_hal_sd.o
HAL_SD_Erase                                      build/stm32f7xx_hal_sd.o
                                                  build/bsp_driver_sd.o
HAL_SD_ErrorCallback                              build/stm32f7xx_hal_sd.o
HAL_SD_GetCardCID                                 build/stm32f7xx_hal_sd.o
HAL_SD_GetCardCSD                                 build/stm32f7xx_hal_sd.o
HAL_SD_GetCardInfo                                build/stm32f7xx_hal_sd.o
                                                  build/bsp_driver_sd.o
HAL_SD_GetCardState                               build/stm32f7xx_hal_sd.o
                                                  build/bsp_driver_sd.o
HAL_SD_GetCardStatus                              build/stm32f7xx_hal_sd.o
HAL_SD_GetError                                   build/stm32f7xx_hal_sd.o
HAL_SD_GetState                                   build/stm32f7xx_hal_sd.o
HAL_SD_IRQHandler                                 build/stm32f7xx_hal_sd.o
HAL_SD_Init                                       build/stm32f7xx_hal_sd.o
                                                  build/bsp_driver_sd.o
HAL_SD_InitCard                                   build/stm32f7xx_hal_sd.o
HAL_SD_MspDeInit                                  build/stm32f7xx_hal_msp.o
HAL_SD_MspInit                                    build/stm32f7xx_hal_msp.o
HAL_SD_ReadBlocks                                 build/stm32f7xx_hal_sd.o
                                                  build/bsp_driver_sd.o
HAL_SD_ReadBlocks_DMA                             build/stm32f7xx_hal_sd.o
                                                  build/bsp_driver_sd.o
HAL_SD_ReadBlocks_IT                              build/stm32f7xx_hal_sd.o
HAL_SD_RxCpltCallback                             build/bsp_driver_sd.o
HAL_SD_TxCpltCallback                             build/bsp_driver_sd.o
HAL_SD_WriteBlocks                                build/stm32f7xx_hal_sd.o
                                                  build/bsp_driver_sd.o
HAL_SD_WriteBlocks_DMA                            build/stm32f7xx_hal_sd.o
                                                  build/bsp_driver_sd.o
HAL_SD_WriteBlocks_IT                             build/stm32f7xx_hal_sd.o
HAL_SYSTICK_CLKSourceConfig                       build/stm32f7xx_hal_cortex.o
HAL_SYSTICK_Callback                              build/stm32f7xx_hal_cortex.o
HAL_SYSTICK_Config                                build/stm32f7xx_hal_cortex.o
                                                  build/stm32f7xx_hal.o
HAL_SYSTICK_IRQHandler                            build/stm32f7xx_hal_cortex.o
HAL_SetTickFreq                                   build/stm32f7xx_hal.o
HAL_SuspendTick                                   build/stm32f7xx_hal.o
HAL_TIMEx_Break2Callback                          build/stm32f7xx_hal_tim_ex.o
                                                  build/stm32f7xx_hal_tim.o
HAL_TIMEx_BreakCallback                           build/stm32f7xx_hal_tim_ex.o
                                                  build/stm32f7xx_hal_tim.o
HAL_TIMEx_CommutCallback                          build/stm32f7xx_hal_tim_ex.o
                                                  build/stm32f7xx_hal_tim.o
HAL_TIMEx_CommutHalfCpltCallback                  build/stm32f7xx_hal_tim_ex.o
HAL_TIMEx_ConfigBreakDeadTime                     build/stm32f7xx_hal_tim_ex.o
HAL_TIMEx_ConfigBreakInput                        build/stm32f7xx_hal_tim_ex.o
HAL_TIMEx_ConfigCommutEvent                       build/stm32f7xx_hal_tim_ex.o
HAL_TIMEx_ConfigCommutEvent_DMA                   build/stm32f7xx_hal_tim_ex.o
HAL_TIMEx_ConfigCommutEvent_IT                    build/stm32f7xx_hal_tim_ex.o
HAL_TIMEx_GetChannelNState                        build/stm32f7xx_hal_tim_ex.o
HAL_TIMEx_GroupChannel5                           build/stm32f7xx_hal_tim_ex.o
HAL_TIMEx_HallSensor_DeInit                       build/stm32f7xx_hal_tim_ex.o
HAL_TIMEx_HallSensor_GetState                     build/stm32f7xx_hal_tim_ex.o
HAL_TIMEx_HallSensor_Init                         build/stm32f7xx_hal_tim_ex.o
HAL_TIMEx_HallSensor_MspDeInit                    build/stm32f7xx_hal_tim_ex.o
HAL_TIMEx_HallSensor_MspInit                      build/stm32f7xx_hal_tim_ex.o
HAL_TIMEx_HallSensor_Start                        build/stm32f7xx_hal_tim_ex.o
HAL_TIMEx_HallSensor_Start_DMA                    build/stm32f7xx_hal_tim_ex.o
HAL_TIMEx_HallSensor_Start_IT                     build/stm32f7xx_hal_tim_ex.o
HAL_TIMEx_HallSensor_Stop                         build/stm32f7xx_hal_tim_ex.o
HAL_TIMEx_HallSensor_Stop_DMA                     build/stm32f7xx_hal_tim_ex.o
HAL_TIMEx_HallSensor_Stop_IT                      build/stm32f7xx_hal_tim_ex.o
HAL_TIMEx_MasterConfigSynchronization             build/stm32f7xx_hal_tim_ex.o
                                                  build/main.o
HAL_TIMEx_OCN_Start                               build/stm32f7xx_hal_tim_ex.o
HAL_TIMEx_OCN_Start_DMA                           build/stm32f7xx_hal_tim_ex.o
HAL_TIMEx_OCN_Start_IT                            build/stm32f7xx_hal_tim_ex.o
HAL_TIMEx_OCN_Stop                                build/stm32f7xx_hal_tim_ex.o
HAL_TIMEx_OCN_Stop_DMA                            build/stm32f7xx_hal_tim_ex.o
HAL_TIMEx_OCN_Stop_IT                             build/stm32f7xx_hal_tim_ex.o
HAL_TIMEx_OnePulseN_Start                         build/stm32f7xx_hal_tim_ex.o
HAL_TIMEx_OnePulseN_Start_IT                      build/stm32f7xx_hal_tim_ex.o
HAL_TIMEx_OnePulseN_Stop                          build/stm32f7xx_hal_tim_ex.o
HAL_TIMEx_OnePulseN_Stop_IT                       build/stm32f7xx_hal_tim_ex.o
HAL_TIMEx_PWMN_Start                              build/stm32f7xx_hal_tim_ex.o
HAL_TIMEx_PWMN_Start_DMA                          build/stm32f7xx_hal_tim_ex.o
HAL_TIMEx_PWMN_Start_IT                           build/stm32f7xx_hal_tim_ex.o
HAL_TIMEx_PWMN_Stop                               build/stm32f7xx_hal_tim_ex.o
HAL_TIMEx_PWMN_Stop_DMA                           build/stm32f7xx_hal_tim_ex.o
HAL_TIMEx_PWMN_Stop_IT                            build/stm32f7xx_hal_tim_ex.o
HAL_TIMEx_RemapConfig                             build/stm32f7xx_hal_tim_ex.o
HAL_TIM_Base_DeInit                               build/stm32f7xx_hal_tim.o
HAL_TIM_Base_GetState                             build/stm32f7xx_hal_tim.o
HAL_TIM_Base_Init                                 build/stm32f7xx_hal_tim.o
                                                  build/main.o
HAL_TIM_Base_MspDeInit                            build/stm32f7xx_hal_msp.o
HAL_TIM_Base_MspInit                              build/stm32f7xx_hal_msp.o
HAL_TIM_Base_Start                                build/stm32f7xx_hal_tim.o
HAL_TIM_Base_Start_DMA                            build/stm32f7xx_hal_tim.o
HAL_TIM_Base_Start_IT                             build/stm32f7xx_hal_tim.o
                                                  build/main.o
HAL_TIM_Base_Stop                                 build/stm32f7xx_hal_tim.o
                                                  build/main.o
HAL_TIM_Base_Stop_DMA                             build/stm32f7xx_hal_tim.o
HAL_TIM_Base_Stop_IT                              build/stm32f7xx_hal_tim.o
                                                  build/main.o
HAL_TIM_ConfigClockSource                         build/stm32f7xx_hal_tim.o
                                                  build/main.o
HAL_TIM_ConfigOCrefClear                          build/stm32f7xx_hal_tim.o
HAL_TIM_ConfigTI1Input                            build/stm32f7xx_hal_tim.o
HAL_TIM_DMABurstState                             build/stm32f7xx_hal_tim.o
HAL_TIM_DMABurst_MultiReadStart                   build/stm32f7xx_hal_tim.o
HAL_TIM_DMABurst_MultiWriteStart                  build/stm32f7xx_hal_tim.o
HAL_TIM_DMABurst_ReadStart                        build/stm32f7xx_hal_tim.o
HAL_TIM_DMABurst_ReadStop                         build/stm32f7xx_hal_tim.o
HAL_TIM_DMABurst_WriteStart                       build/stm32f7xx_hal_tim.o
HAL_TIM_DMABurst_WriteStop                        build/stm32f7xx_hal_tim.o
HAL_TIM_Encoder_DeInit                            build/stm32f7xx_hal_tim.o
HAL_TIM_Encoder_GetState                          build/stm32f7xx_hal_tim.o
HAL_TIM_Encoder_Init                              build/stm32f7xx_hal_tim.o
HAL_TIM_Encoder_MspDeInit                         build/stm32f7xx_hal_tim.o
HAL_TIM_Encoder_MspInit                           build/stm32f7xx_hal_tim.o
HAL_TIM_Encoder_Start                             build/stm32f7xx_hal_tim.o
HAL_TIM_Encoder_Start_DMA                         build/stm32f7xx_hal_tim.o
HAL_TIM_Encoder_Start_IT                          build/stm32f7xx_hal_tim.o
HAL_TIM_Encoder_Stop                              build/stm32f7xx_hal_tim.o
HAL_TIM_Encoder_Stop_DMA                          build/stm32f7xx_hal_tim.o
HAL_TIM_Encoder_Stop_IT                           build/stm32f7xx_hal_tim.o
HAL_TIM_ErrorCallback                             build/stm32f7xx_hal_tim.o
                                                  build/stm32f7xx_hal_tim_ex.o
HAL_TIM_GenerateEvent                             build/stm32f7xx_hal_tim.o
HAL_TIM_GetActiveChannel                          build/stm32f7xx_hal_tim.o
HAL_TIM_GetChannelState                           build/stm32f7xx_hal_tim.o
HAL_TIM_IC_CaptureCallback                        build/stm32f7xx_hal_tim.o
HAL_TIM_IC_CaptureHalfCpltCallback                build/stm32f7xx_hal_tim.o
HAL_TIM_IC_ConfigChannel                          build/stm32f7xx_hal_tim.o
HAL_TIM_IC_DeInit                                 build/stm32f7xx_hal_tim.o
HAL_TIM_IC_GetState                               build/stm32f7xx_hal_tim.o
HAL_TIM_IC_Init                                   build/stm32f7xx_hal_tim.o
HAL_TIM_IC_MspDeInit                              build/stm32f7xx_hal_tim.o
HAL_TIM_IC_MspInit                                build/stm32f7xx_hal_tim.o
HAL_TIM_IC_Start                                  build/stm32f7xx_hal_tim.o
HAL_TIM_IC_Start_DMA                              build/stm32f7xx_hal_tim.o
HAL_TIM_IC_Start_IT                               build/stm32f7xx_hal_tim.o
HAL_TIM_IC_Stop                                   build/stm32f7xx_hal_tim.o
HAL_TIM_IC_Stop_DMA                               build/stm32f7xx_hal_tim.o
HAL_TIM_IC_Stop_IT                                build/stm32f7xx_hal_tim.o
HAL_TIM_IRQHandler                                build/stm32f7xx_hal_tim.o
                                                  build/stm32f7xx_it.o
HAL_TIM_MspPostInit                               build/stm32f7xx_hal_msp.o
                                                  build/main.o
HAL_TIM_OC_ConfigChannel                          build/stm32f7xx_hal_tim.o
HAL_TIM_OC_DeInit                                 build/stm32f7xx_hal_tim.o
HAL_TIM_OC_DelayElapsedCallback                   build/stm32f7xx_hal_tim.o
HAL_TIM_OC_GetState                               build/stm32f7xx_hal_tim.o
HAL_TIM_OC_Init                                   build/stm32f7xx_hal_tim.o
HAL_TIM_OC_MspDeInit                              build/stm32f7xx_hal_tim.o
HAL_TIM_OC_MspInit                                build/stm32f7xx_hal_tim.o
HAL_TIM_OC_Start                                  build/stm32f7xx_hal_tim.o
HAL_TIM_OC_Start_DMA                              build/stm32f7xx_hal_tim.o
HAL_TIM_OC_Start_IT                               build/stm32f7xx_hal_tim.o
HAL_TIM_OC_Stop                                   build/stm32f7xx_hal_tim.o
HAL_TIM_OC_Stop_DMA                               build/stm32f7xx_hal_tim.o
HAL_TIM_OC_Stop_IT                                build/stm32f7xx_hal_tim.o
HAL_TIM_OnePulse_ConfigChannel                    build/stm32f7xx_hal_tim.o
HAL_TIM_OnePulse_DeInit                           build/stm32f7xx_hal_tim.o
HAL_TIM_OnePulse_GetState                         build/stm32f7xx_hal_tim.o
HAL_TIM_OnePulse_Init                             build/stm32f7xx_hal_tim.o
HAL_TIM_OnePulse_MspDeInit                        build/stm32f7xx_hal_tim.o
HAL_TIM_OnePulse_MspInit                          build/stm32f7xx_hal_tim.o
HAL_TIM_OnePulse_Start                            build/stm32f7xx_hal_tim.o
HAL_TIM_OnePulse_Start_IT                         build/stm32f7xx_hal_tim.o
HAL_TIM_OnePulse_Stop                             build/stm32f7xx_hal_tim.o
HAL_TIM_OnePulse_Stop_IT                          build/stm32f7xx_hal_tim.o
HAL_TIM_PWM_ConfigChannel                         build/stm32f7xx_hal_tim.o
                                                  build/main.o
HAL_TIM_PWM_DeInit                                build/stm32f7xx_hal_tim.o
HAL_TIM_PWM_GetState                              build/stm32f7xx_hal_tim.o
HAL_TIM_PWM_Init                                  build/stm32f7xx_hal_tim.o
                                                  build/main.o
HAL_TIM_PWM_MspDeInit                             build/stm32f7xx_hal_tim.o
HAL_TIM_PWM_MspInit                               build/stm32f7xx_hal_tim.o
HAL_TIM_PWM_PulseFinishedCallback                 build/stm32f7xx_hal_tim.o
                                                  build/stm32f7xx_hal_tim_ex.o
HAL_TIM_PWM_PulseFinishedHalfCpltCallback         build/stm32f7xx_hal_tim.o
HAL_TIM_PWM_Start                                 build/stm32f7xx_hal_tim.o
                                                  build/main.o
HAL_TIM_PWM_Start_DMA                             build/stm32f7xx_hal_tim.o
HAL_TIM_PWM_Start_IT                              build/stm32f7xx_hal_tim.o
HAL_TIM_PWM_Stop                                  build/stm32f7xx_hal_tim.o
                                                  build/main.o
HAL_TIM_PWM_Stop_DMA                              build/stm32f7xx_hal_tim.o
HAL_TIM_PWM_Stop_IT                               build/stm32f7xx_hal_tim.o
HAL_TIM_PeriodElapsedCallback                     build/stm32f7xx_hal_tim.o
HAL_TIM_PeriodElapsedHalfCpltCallback             build/stm32f7xx_hal_tim.o
HAL_TIM_ReadCapturedValue                         build/stm32f7xx_hal_tim.o
HAL_TIM_SlaveConfigSynchro                        build/stm32f7xx_hal_tim.o
HAL_TIM_SlaveConfigSynchro_IT                     build/stm32f7xx_hal_tim.o
HAL_TIM_TriggerCallback                           build/stm32f7xx_hal_tim.o
HAL_TIM_TriggerHalfCpltCallback                   build/stm32f7xx_hal_tim.o
HAL_UARTEx_DisableClockStopMode                   build/stm32f7xx_hal_uart_ex.o
HAL_UARTEx_DisableStopMode                        build/stm32f7xx_hal_uart_ex.o
HAL_UARTEx_EnableClockStopMode                    build/stm32f7xx_hal_uart_ex.o
HAL_UARTEx_EnableStopMode                         build/stm32f7xx_hal_uart_ex.o
HAL_UARTEx_GetRxEventType                         build/stm32f7xx_hal_uart_ex.o
HAL_UARTEx_ReceiveToIdle                          build/stm32f7xx_hal_uart_ex.o
HAL_UARTEx_ReceiveToIdle_DMA                      build/stm32f7xx_hal_uart_ex.o
HAL_UARTEx_ReceiveToIdle_IT                       build/stm32f7xx_hal_uart_ex.o
HAL_UARTEx_RxEventCallback                        build/stm32f7xx_hal_uart.o
HAL_UARTEx_StopModeWakeUpSourceConfig             build/stm32f7xx_hal_uart_ex.o
HAL_UARTEx_WakeupCallback                         build/stm32f7xx_hal_uart.o
HAL_UART_Abort                                    build/stm32f7xx_hal_uart.o
HAL_UART_AbortCpltCallback                        build/stm32f7xx_hal_uart.o
HAL_UART_AbortReceive                             build/stm32f7xx_hal_uart.o
HAL_UART_AbortReceiveCpltCallback                 build/stm32f7xx_hal_uart.o
HAL_UART_AbortReceive_IT                          build/stm32f7xx_hal_uart.o
HAL_UART_AbortTransmit                            build/stm32f7xx_hal_uart.o
HAL_UART_AbortTransmitCpltCallback                build/stm32f7xx_hal_uart.o
HAL_UART_AbortTransmit_IT                         build/stm32f7xx_hal_uart.o
HAL_UART_Abort_IT                                 build/stm32f7xx_hal_uart.o
HAL_UART_DMAPause                                 build/stm32f7xx_hal_uart.o
HAL_UART_DMAResume                                build/stm32f7xx_hal_uart.o
HAL_UART_DMAStop                                  build/stm32f7xx_hal_uart.o
HAL_UART_DeInit                                   build/stm32f7xx_hal_uart.o
HAL_UART_DisableReceiverTimeout                   build/stm32f7xx_hal_uart.o
HAL_UART_EnableReceiverTimeout                    build/stm32f7xx_hal_uart.o
HAL_UART_ErrorCallback                            build/stm32f7xx_hal_uart.o
HAL_UART_GetError                                 build/stm32f7xx_hal_uart.o
HAL_UART_GetState                                 build/stm32f7xx_hal_uart.o
HAL_UART_IRQHandler                               build/stm32f7xx_hal_uart.o
HAL_UART_Init                                     build/stm32f7xx_hal_uart.o
                                                  build/main.o
HAL_UART_MspDeInit                                build/stm32f7xx_hal_msp.o
HAL_UART_MspInit                                  build/stm32f7xx_hal_msp.o
                                                  build/stm32f7xx_hal_uart_ex.o
HAL_UART_Receive                                  build/stm32f7xx_hal_uart.o
HAL_UART_Receive_DMA                              build/stm32f7xx_hal_uart.o
HAL_UART_Receive_IT                               build/stm32f7xx_hal_uart.o
HAL_UART_ReceiverTimeout_Config                   build/stm32f7xx_hal_uart.o
HAL_UART_RxCpltCallback                           build/stm32f7xx_hal_uart.o
HAL_UART_RxHalfCpltCallback                       build/stm32f7xx_hal_uart.o
HAL_UART_Transmit                                 build/stm32f7xx_hal_uart.o
HAL_UART_Transmit_DMA                             build/stm32f7xx_hal_uart.o
HAL_UART_Transmit_IT                              build/stm32f7xx_hal_uart.o
HAL_UART_TxCpltCallback                           build/stm32f7xx_hal_uart.o
HAL_UART_TxHalfCpltCallback                       build/stm32f7xx_hal_uart.o
HardFault_Handler                                 build/stm32f7xx_it.o
I2C1_ER_IRQHandler                                build/startup_stm32f767xx.o
I2C1_EV_IRQHandler                                build/startup_stm32f767xx.o
I2C2_ER_IRQHandler                                build/startup_stm32f767xx.o
I2C2_EV_IRQHandler                                build/startup_stm32f767xx.o
I2C3_ER_IRQHandler                                build/startup_stm32f767xx.o
I2C3_EV_IRQHandler                                build/startup_stm32f767xx.o
I2C4_ER_IRQHandler                                build/startup_stm32f767xx.o
I2C4_EV_IRQHandler                                build/startup_stm32f767xx.o
JPEG_IRQHandler                                   build/startup_stm32f767xx.o
LD1_curr_setup                                    build/main.o
LD1_def_setup                                     build/main.o
LD1_param                                         build/main.o
LD2_curr_setup                                    build/main.o
LD2_def_setup                                     build/main.o
LD2_param                                         build/main.o
LD_blinker                                        build/main.o
                                                  build/stm32f7xx_it.o
LL_DMA_DeInit                                     build/stm32f7xx_ll_dma.o
LL_DMA_Init                                       build/stm32f7xx_ll_dma.o
LL_DMA_StructInit                                 build/stm32f7xx_ll_dma.o
LL_EXTI_DeInit                                    build/stm32f7xx_ll_exti.o
LL_EXTI_Init                                      build/stm32f7xx_ll_exti.o
LL_EXTI_StructInit                                build/stm32f7xx_ll_exti.o
LL_GPIO_DeInit                                    build/stm32f7xx_ll_gpio.o
LL_GPIO_Init                                      build/stm32f7xx_ll_gpio.o
                                                  build/main.o
LL_GPIO_StructInit                                build/stm32f7xx_ll_gpio.o
LL_I2S_ConfigPrescaler                            build/stm32f7xx_ll_spi.o
LL_I2S_DeInit                                     build/stm32f7xx_ll_spi.o
LL_I2S_Init                                       build/stm32f7xx_ll_spi.o
LL_I2S_StructInit                                 build/stm32f7xx_ll_spi.o
LL_Init1msTick                                    build/stm32f7xx_ll_utils.o
LL_PLL_ConfigSystemClock_HSE                      build/stm32f7xx_ll_utils.o
LL_PLL_ConfigSystemClock_HSI                      build/stm32f7xx_ll_utils.o
LL_RCC_DeInit                                     build/stm32f7xx_ll_rcc.o
LL_RCC_GetCECClockFreq                            build/stm32f7xx_ll_rcc.o
LL_RCC_GetDFSDMAudioClockFreq                     build/stm32f7xx_ll_rcc.o
LL_RCC_GetDFSDMClockFreq                          build/stm32f7xx_ll_rcc.o
LL_RCC_GetI2CClockFreq                            build/stm32f7xx_ll_rcc.o
LL_RCC_GetI2SClockFreq                            build/stm32f7xx_ll_rcc.o
                                                  build/stm32f7xx_ll_spi.o
LL_RCC_GetLPTIMClockFreq                          build/stm32f7xx_ll_rcc.o
LL_RCC_GetLTDCClockFreq                           build/stm32f7xx_ll_rcc.o
LL_RCC_GetRNGClockFreq                            build/stm32f7xx_ll_rcc.o
LL_RCC_GetSAIClockFreq                            build/stm32f7xx_ll_rcc.o
LL_RCC_GetSDMMCClockFreq                          build/stm32f7xx_ll_rcc.o
LL_RCC_GetSPDIFRXClockFreq                        build/stm32f7xx_ll_rcc.o
LL_RCC_GetSystemClocksFreq                        build/stm32f7xx_ll_rcc.o
LL_RCC_GetUARTClockFreq                           build/stm32f7xx_ll_rcc.o
                                                  build/stm32f7xx_ll_usart.o
LL_RCC_GetUSARTClockFreq                          build/stm32f7xx_ll_rcc.o
                                                  build/stm32f7xx_ll_usart.o
LL_RCC_GetUSBClockFreq                            build/stm32f7xx_ll_rcc.o
LL_SPI_DeInit                                     build/stm32f7xx_ll_spi.o
LL_SPI_Init                                       build/stm32f7xx_ll_spi.o
                                                  build/main.o
LL_SPI_StructInit                                 build/stm32f7xx_ll_spi.o
LL_SetFlashLatency                                build/stm32f7xx_ll_utils.o
LL_SetSystemCoreClock                             build/stm32f7xx_ll_utils.o
LL_TIM_BDTR_Init                                  build/stm32f7xx_ll_tim.o
LL_TIM_BDTR_StructInit                            build/stm32f7xx_ll_tim.o
LL_TIM_DeInit                                     build/stm32f7xx_ll_tim.o
LL_TIM_ENCODER_Init                               build/stm32f7xx_ll_tim.o
LL_TIM_ENCODER_StructInit                         build/stm32f7xx_ll_tim.o
LL_TIM_HALLSENSOR_Init                            build/stm32f7xx_ll_tim.o
LL_TIM_HALLSENSOR_StructInit                      build/stm32f7xx_ll_tim.o
LL_TIM_IC_Init                                    build/stm32f7xx_ll_tim.o
LL_TIM_IC_StructInit                              build/stm32f7xx_ll_tim.o
LL_TIM_Init                                       build/stm32f7xx_ll_tim.o
                                                  build/main.o
LL_TIM_OC_Init                                    build/stm32f7xx_ll_tim.o
LL_TIM_OC_StructInit                              build/stm32f7xx_ll_tim.o
LL_TIM_StructInit                                 build/stm32f7xx_ll_tim.o
LL_USART_ClockInit                                build/stm32f7xx_ll_usart.o
LL_USART_ClockStructInit                          build/stm32f7xx_ll_usart.o
LL_USART_DeInit                                   build/stm32f7xx_ll_usart.o
LL_USART_Init                                     build/stm32f7xx_ll_usart.o
                                                  build/main.o
LL_USART_StructInit                               build/stm32f7xx_ll_usart.o
LL_mDelay                                         build/stm32f7xx_ll_utils.o
LPTIM1_IRQHandler                                 build/startup_stm32f767xx.o
LTDC_ER_IRQHandler                                build/startup_stm32f767xx.o
LTDC_IRQHandler                                   build/startup_stm32f767xx.o
Long_Data                                         build/main.o
MDIOS_IRQHandler                                  build/startup_stm32f767xx.o
MX_FATFS_Init                                     build/fatfs.o
                                                  build/main.o
MemManage_Handler                                 build/stm32f7xx_it.o
Mount_SD                                          build/File_Handling.o
                                                  build/main.o
NMI_Handler                                       build/stm32f7xx_it.o
OTG_FS_IRQHandler                                 build/startup_stm32f767xx.o
OTG_FS_WKUP_IRQHandler                            build/startup_stm32f767xx.o
OTG_HS_EP1_IN_IRQHandler                          build/startup_stm32f767xx.o
OTG_HS_EP1_OUT_IRQHandler                         build/startup_stm32f767xx.o
OTG_HS_IRQHandler                                 build/startup_stm32f767xx.o
OTG_HS_WKUP_IRQHandler                            build/startup_stm32f767xx.o
PVD_IRQHandler                                    build/startup_stm32f767xx.o
PendSV_Handler                                    build/stm32f7xx_it.o
QUADSPI_IRQHandler                                build/startup_stm32f767xx.o
RCC_GetHCLKClockFreq                              build/stm32f7xx_ll_rcc.o
RCC_GetPCLK1ClockFreq                             build/stm32f7xx_ll_rcc.o
RCC_GetPCLK2ClockFreq                             build/stm32f7xx_ll_rcc.o
RCC_GetSystemClockFreq                            build/stm32f7xx_ll_rcc.o
RCC_IRQHandler                                    build/startup_stm32f767xx.o
RCC_PLLI2S_GetFreqDomain_I2S                      build/stm32f7xx_ll_rcc.o
RCC_PLLI2S_GetFreqDomain_SAI                      build/stm32f7xx_ll_rcc.o
RCC_PLLI2S_GetFreqDomain_SPDIFRX                  build/stm32f7xx_ll_rcc.o
RCC_PLLSAI_GetFreqDomain_48M                      build/stm32f7xx_ll_rcc.o
RCC_PLLSAI_GetFreqDomain_LTDC                     build/stm32f7xx_ll_rcc.o
RCC_PLLSAI_GetFreqDomain_SAI                      build/stm32f7xx_ll_rcc.o
RCC_PLL_GetFreqDomain_48M                         build/stm32f7xx_ll_rcc.o
RCC_PLL_GetFreqDomain_SYS                         build/stm32f7xx_ll_rcc.o
RNG_IRQHandler                                    build/startup_stm32f767xx.o
RTC_Alarm_IRQHandler                              build/startup_stm32f767xx.o
RTC_WKUP_IRQHandler                               build/startup_stm32f767xx.o
Read_File                                         build/File_Handling.o
Remove_File                                       build/File_Handling.o
                                                  build/main.o
Reset_Handler                                     build/startup_stm32f767xx.o
SAI1_IRQHandler                                   build/startup_stm32f767xx.o
SAI2_IRQHandler                                   build/startup_stm32f767xx.o
SDFatFS                                           build/fatfs.o
SDFile                                            build/fatfs.o
SDMMC1_IRQHandler                                 build/startup_stm32f767xx.o
SDMMC2_IRQHandler                                 build/startup_stm32f767xx.o
SDMMC_CmdAppCommand                               build/stm32f7xx_ll_sdmmc.o
                                                  build/stm32f7xx_hal_sd.o
SDMMC_CmdAppOperCommand                           build/stm32f7xx_ll_sdmmc.o
                                                  build/stm32f7xx_hal_sd.o
SDMMC_CmdBlockLength                              build/stm32f7xx_ll_sdmmc.o
                                                  build/stm32f7xx_hal_sd.o
SDMMC_CmdBusWidth                                 build/stm32f7xx_ll_sdmmc.o
                                                  build/stm32f7xx_hal_sd.o
SDMMC_CmdErase                                    build/stm32f7xx_ll_sdmmc.o
                                                  build/stm32f7xx_hal_sd.o
SDMMC_CmdEraseEndAdd                              build/stm32f7xx_ll_sdmmc.o
SDMMC_CmdEraseStartAdd                            build/stm32f7xx_ll_sdmmc.o
SDMMC_CmdGoIdleState                              build/stm32f7xx_ll_sdmmc.o
                                                  build/stm32f7xx_hal_sd.o
SDMMC_CmdOpCondition                              build/stm32f7xx_ll_sdmmc.o
SDMMC_CmdOperCond                                 build/stm32f7xx_ll_sdmmc.o
                                                  build/stm32f7xx_hal_sd.o
SDMMC_CmdReadMultiBlock                           build/stm32f7xx_ll_sdmmc.o
                                                  build/stm32f7xx_hal_sd.o
SDMMC_CmdReadSingleBlock                          build/stm32f7xx_ll_sdmmc.o
                                                  build/stm32f7xx_hal_sd.o
SDMMC_CmdSDEraseEndAdd                            build/stm32f7xx_ll_sdmmc.o
                                                  build/stm32f7xx_hal_sd.o
SDMMC_CmdSDEraseStartAdd                          build/stm32f7xx_ll_sdmmc.o
                                                  build/stm32f7xx_hal_sd.o
SDMMC_CmdSelDesel                                 build/stm32f7xx_ll_sdmmc.o
                                                  build/stm32f7xx_hal_sd.o
SDMMC_CmdSendCID                                  build/stm32f7xx_ll_sdmmc.o
                                                  build/stm32f7xx_hal_sd.o
SDMMC_CmdSendCSD                                  build/stm32f7xx_ll_sdmmc.o
                                                  build/stm32f7xx_hal_sd.o
SDMMC_CmdSendEXTCSD                               build/stm32f7xx_ll_sdmmc.o
SDMMC_CmdSendSCR                                  build/stm32f7xx_ll_sdmmc.o
                                                  build/stm32f7xx_hal_sd.o
SDMMC_CmdSendStatus                               build/stm32f7xx_ll_sdmmc.o
                                                  build/stm32f7xx_hal_sd.o
SDMMC_CmdSetRelAdd                                build/stm32f7xx_ll_sdmmc.o
                                                  build/stm32f7xx_hal_sd.o
SDMMC_CmdSetRelAddMmc                             build/stm32f7xx_ll_sdmmc.o
SDMMC_CmdStatusRegister                           build/stm32f7xx_ll_sdmmc.o
                                                  build/stm32f7xx_hal_sd.o
SDMMC_CmdStopTransfer                             build/stm32f7xx_ll_sdmmc.o
                                                  build/stm32f7xx_hal_sd.o
SDMMC_CmdSwitch                                   build/stm32f7xx_ll_sdmmc.o
SDMMC_CmdWriteMultiBlock                          build/stm32f7xx_ll_sdmmc.o
                                                  build/stm32f7xx_hal_sd.o
SDMMC_CmdWriteSingleBlock                         build/stm32f7xx_ll_sdmmc.o
                                                  build/stm32f7xx_hal_sd.o
SDMMC_ConfigData                                  build/stm32f7xx_ll_sdmmc.o
                                                  build/stm32f7xx_hal_sd.o
SDMMC_GetCmdResp1                                 build/stm32f7xx_ll_sdmmc.o
SDMMC_GetCmdResp2                                 build/stm32f7xx_ll_sdmmc.o
SDMMC_GetCmdResp3                                 build/stm32f7xx_ll_sdmmc.o
SDMMC_GetCmdResp6                                 build/stm32f7xx_ll_sdmmc.o
SDMMC_GetCmdResp7                                 build/stm32f7xx_ll_sdmmc.o
SDMMC_GetCommandResponse                          build/stm32f7xx_ll_sdmmc.o
SDMMC_GetDataCounter                              build/stm32f7xx_ll_sdmmc.o
SDMMC_GetFIFOCount                                build/stm32f7xx_ll_sdmmc.o
SDMMC_GetPowerState                               build/stm32f7xx_ll_sdmmc.o
                                                  build/stm32f7xx_hal_sd.o
SDMMC_GetResponse                                 build/stm32f7xx_ll_sdmmc.o
                                                  build/stm32f7xx_hal_sd.o
SDMMC_Init                                        build/stm32f7xx_ll_sdmmc.o
                                                  build/stm32f7xx_hal_sd.o
SDMMC_PowerState_OFF                              build/stm32f7xx_ll_sdmmc.o
                                                  build/stm32f7xx_hal_sd.o
SDMMC_PowerState_ON                               build/stm32f7xx_ll_sdmmc.o
                                                  build/stm32f7xx_hal_sd.o
SDMMC_ReadFIFO                                    build/stm32f7xx_ll_sdmmc.o
                                                  build/stm32f7xx_hal_sd.o
SDMMC_SendCommand                                 build/stm32f7xx_ll_sdmmc.o
SDMMC_SetSDMMCReadWaitMode                        build/stm32f7xx_ll_sdmmc.o
SDMMC_WriteFIFO                                   build/stm32f7xx_ll_sdmmc.o
                                                  build/stm32f7xx_hal_sd.o
SDPath                                            build/fatfs.o
SD_Driver                                         build/sd_diskio.o
                                                  build/fatfs.o
SD_READ                                           build/main.o
SD_REMOVE                                         build/main.o
SD_SAVE                                           build/main.o
SD_SEEK                                           build/main.o
SD_SLIDE                                          build/main.o
SD_initialize                                     build/sd_diskio.o
SD_ioctl                                          build/sd_diskio.o
SD_read                                           build/sd_diskio.o
SD_status                                         build/sd_diskio.o
SD_write                                          build/sd_diskio.o
SPDIF_RX_IRQHandler                               build/startup_stm32f767xx.o
SPI1_IRQHandler                                   build/startup_stm32f767xx.o
SPI2_IRQHandler                                   build/startup_stm32f767xx.o
SPI3_IRQHandler                                   build/startup_stm32f767xx.o
SPI4_IRQHandler                                   build/startup_stm32f767xx.o
SPI5_IRQHandler                                   build/startup_stm32f767xx.o
SPI6_IRQHandler                                   build/startup_stm32f767xx.o
SVC_Handler                                       build/stm32f7xx_it.o
Scan_SD                                           build/File_Handling.o
Seek_Read_File                                    build/File_Handling.o
                                                  build/main.o
Send_Uart                                         build/File_Handling.o
Set_LTEC                                          build/main.o
                                                  build/stm32f7xx_it.o
State_Data                                        build/main.o
                                                  build/stm32f7xx_it.o
SysTick_Handler                                   build/stm32f7xx_it.o
SystemClock_Config                                build/main.o
SystemCoreClock                                   build/system_stm32f7xx.o
                                                  build/stm32f7xx_ll_sdmmc.o
                                                  build/stm32f7xx_ll_utils.o
                                                  build/stm32f7xx_hal.o
                                                  build/stm32f7xx_hal_dma.o
                                                  build/stm32f7xx_hal_rcc.o
                                                  build/stm32f7xx_hal_adc_ex.o
                                                  build/stm32f7xx_hal_adc.o
SystemCoreClockUpdate                             build/system_stm32f7xx.o
SystemInit                                        build/system_stm32f7xx.o
                                                  build/startup_stm32f767xx.o
TAMP_STAMP_IRQHandler                             build/startup_stm32f767xx.o
TIM10_coflag                                      build/main.o
                                                  build/stm32f7xx_it.o
TIM10_period                                      build/main.o
TIM1_BRK_TIM9_IRQHandler                          build/startup_stm32f767xx.o
TIM1_CC_IRQHandler                                build/startup_stm32f767xx.o
TIM1_TRG_COM_TIM11_IRQHandler                     build/stm32f7xx_it.o
TIM1_UP_TIM10_IRQHandler                          build/stm32f7xx_it.o
TIM2_IRQHandler                                   build/stm32f7xx_it.o
TIM3_IRQHandler                                   build/startup_stm32f767xx.o
TIM4_IRQHandler                                   build/startup_stm32f767xx.o
TIM5_IRQHandler                                   build/stm32f7xx_it.o
TIM6_DAC_IRQHandler                               build/stm32f7xx_it.o
TIM7_IRQHandler                                   build/stm32f7xx_it.o
TIM8_BRK_TIM12_IRQHandler                         build/startup_stm32f767xx.o
TIM8_CC_IRQHandler                                build/startup_stm32f767xx.o
TIM8_TRG_COM_TIM14_IRQHandler                     build/startup_stm32f767xx.o
TIM8_UP_TIM13_IRQHandler                          build/stm32f7xx_it.o
TIMEx_DMACommutationCplt                          build/stm32f7xx_hal_tim_ex.o
                                                  build/stm32f7xx_hal_tim.o
TIMEx_DMACommutationHalfCplt                      build/stm32f7xx_hal_tim_ex.o
                                                  build/stm32f7xx_hal_tim.o
TIM_Base_SetConfig                                build/stm32f7xx_hal_tim.o
                                                  build/stm32f7xx_hal_tim_ex.o
TIM_CCxChannelCmd                                 build/stm32f7xx_hal_tim.o
                                                  build/stm32f7xx_hal_tim_ex.o
TIM_DMACaptureCplt                                build/stm32f7xx_hal_tim.o
                                                  build/stm32f7xx_hal_tim_ex.o
TIM_DMACaptureHalfCplt                            build/stm32f7xx_hal_tim.o
                                                  build/stm32f7xx_hal_tim_ex.o
TIM_DMADelayPulseHalfCplt                         build/stm32f7xx_hal_tim.o
                                                  build/stm32f7xx_hal_tim_ex.o
TIM_DMAError                                      build/stm32f7xx_hal_tim.o
                                                  build/stm32f7xx_hal_tim_ex.o
TIM_ETR_SetConfig                                 build/stm32f7xx_hal_tim.o
TIM_OC2_SetConfig                                 build/stm32f7xx_hal_tim.o
                                                  build/stm32f7xx_hal_tim_ex.o
TIM_TI1_SetConfig                                 build/stm32f7xx_hal_tim.o
                                                  build/stm32f7xx_hal_tim_ex.o
TO10                                              build/main.o
                                                  build/stm32f7xx_it.o
TO10_counter                                      build/main.o
                                                  build/stm32f7xx_it.o
TO6                                               build/main.o
                                                  build/stm32f7xx_it.o
TO6_before                                        build/main.o
TO6_stop                                          build/main.o
TO6_uart                                          build/main.o
                                                  build/stm32f7xx_it.o
TO7                                               build/main.o
                                                  build/stm32f7xx_it.o
TO7_PID                                           build/main.o
TO7_before                                        build/main.o
UART4_IRQHandler                                  build/startup_stm32f767xx.o
UART5_IRQHandler                                  build/startup_stm32f767xx.o
UART7_IRQHandler                                  build/startup_stm32f767xx.o
UART8_IRQHandler                                  build/startup_stm32f767xx.o
UART_AdvFeatureConfig                             build/stm32f7xx_hal_uart.o
                                                  build/stm32f7xx_hal_uart_ex.o
UART_CheckIdleState                               build/stm32f7xx_hal_uart.o
                                                  build/stm32f7xx_hal_uart_ex.o
UART_DATA                                         build/main.o
UART_RxCpltCallback                               build/stm32f7xx_it.o
UART_SetConfig                                    build/stm32f7xx_hal_uart.o
                                                  build/stm32f7xx_hal_uart_ex.o
UART_Start_Receive_DMA                            build/stm32f7xx_hal_uart.o
                                                  build/stm32f7xx_hal_uart_ex.o
UART_Start_Receive_IT                             build/stm32f7xx_hal_uart.o
                                                  build/stm32f7xx_hal_uart_ex.o
UART_WaitOnFlagUntilTimeout                       build/stm32f7xx_hal_uart.o
                                                  build/stm32f7xx_hal_uart_ex.o
UART_header                                       build/main.o
                                                  build/stm32f7xx_it.o
UART_rec_incr                                     build/main.o
                                                  build/stm32f7xx_it.o
UART_transmission_request                         build/main.o
                                                  build/stm32f7xx_it.o
USART1_IRQHandler                                 build/stm32f7xx_it.o
USART2_IRQHandler                                 build/startup_stm32f767xx.o
USART3_IRQHandler                                 build/startup_stm32f767xx.o
USART6_IRQHandler                                 build/startup_stm32f767xx.o
USART_TX                                          build/main.o
USART_TX_DMA                                      build/main.o
Unmount_SD                                        build/File_Handling.o
                                                  build/main.o
Update_File                                       build/File_Handling.o
Update_File_byte                                  build/File_Handling.o
                                                  build/main.o
Update_File_float                                 build/File_Handling.o
UsageFault_Handler                                build/stm32f7xx_it.o
WWDG_IRQHandler                                   build/startup_stm32f767xx.o
Write_File                                        build/File_Handling.o
Write_File_byte                                   build/File_Handling.o
                                                  build/main.o
_ITM_deregisterTMCloneTable                       /usr/lib/gcc/arm-none-eabi/13.2.1/thumb/v7e-m+dp/hard/crtbegin.o
_ITM_registerTMCloneTable                         /usr/lib/gcc/arm-none-eabi/13.2.1/thumb/v7e-m+dp/hard/crtbegin.o
_Min_Stack_Size                                   build/sysmem.o
__TMC_END__                                       /usr/lib/gcc/arm-none-eabi/13.2.1/thumb/v7e-m+dp/hard/crtend.o
                                                  /usr/lib/gcc/arm-none-eabi/13.2.1/thumb/v7e-m+dp/hard/crtbegin.o
__aeabi_idiv0                                     /usr/lib/gcc/arm-none-eabi/13.2.1/thumb/v7e-m+dp/hard/libgcc.a(_dvmd_tls.o)
__aeabi_ldiv0                                     /usr/lib/gcc/arm-none-eabi/13.2.1/thumb/v7e-m+dp/hard/libgcc.a(_dvmd_tls.o)
                                                  /usr/lib/gcc/arm-none-eabi/13.2.1/thumb/v7e-m+dp/hard/libgcc.a(_aeabi_uldivmod.o)
__aeabi_uldivmod                                  /usr/lib/gcc/arm-none-eabi/13.2.1/thumb/v7e-m+dp/hard/libgcc.a(_aeabi_uldivmod.o)
                                                  build/stm32f7xx_hal_rcc.o
__atexit                                          /usr/lib/gcc/arm-none-eabi/13.2.1/../../../arm-none-eabi/lib/thumb/v7e-m+dp/hard/libc_nano.a(libc_a-__call_atexit.o)
                                                  /usr/lib/gcc/arm-none-eabi/13.2.1/../../../arm-none-eabi/lib/thumb/v7e-m+dp/hard/libc_nano.a(libc_a-__atexit.o)
__atexit0                                         /usr/lib/gcc/arm-none-eabi/13.2.1/../../../arm-none-eabi/lib/thumb/v7e-m+dp/hard/libc_nano.a(libc_a-__atexit.o)
__atexit_dummy                                    /usr/lib/gcc/arm-none-eabi/13.2.1/../../../arm-none-eabi/lib/thumb/v7e-m+dp/hard/libc_nano.a(libc_a-__atexit.o)
__bss_end__                                       /usr/lib/gcc/arm-none-eabi/13.2.1/../../../arm-none-eabi/lib/thumb/v7e-m+dp/hard/crt0.o
__bss_start__                                     /usr/lib/gcc/arm-none-eabi/13.2.1/../../../arm-none-eabi/lib/thumb/v7e-m+dp/hard/crt0.o
__call_exitprocs                                  /usr/lib/gcc/arm-none-eabi/13.2.1/../../../arm-none-eabi/lib/thumb/v7e-m+dp/hard/libc_nano.a(libc_a-__call_atexit.o)
                                                  /usr/lib/gcc/arm-none-eabi/13.2.1/../../../arm-none-eabi/lib/thumb/v7e-m+dp/hard/libc_nano.a(libc_a-__atexit.o)
                                                  /usr/lib/gcc/arm-none-eabi/13.2.1/../../../arm-none-eabi/lib/thumb/v7e-m+dp/hard/libc_nano.a(libc_a-exit.o)
__deregister_frame_info                           /usr/lib/gcc/arm-none-eabi/13.2.1/thumb/v7e-m+dp/hard/crtbegin.o
__dso_handle                                      /usr/lib/gcc/arm-none-eabi/13.2.1/thumb/v7e-m+dp/hard/crtbegin.o
__env                                             build/syscalls.o
__errno                                           /usr/lib/gcc/arm-none-eabi/13.2.1/../../../arm-none-eabi/lib/thumb/v7e-m+dp/hard/libc_nano.a(libc_a-errno.o)
                                                  build/syscalls.o
                                                  build/sysmem.o
__fini_array_end                                  /usr/lib/gcc/arm-none-eabi/13.2.1/../../../arm-none-eabi/lib/thumb/v7e-m+dp/hard/libc_nano.a(libc_a-fini.o)
__fini_array_start                                /usr/lib/gcc/arm-none-eabi/13.2.1/../../../arm-none-eabi/lib/thumb/v7e-m+dp/hard/libc_nano.a(libc_a-fini.o)
__fp_lock_all                                     /usr/lib/gcc/arm-none-eabi/13.2.1/../../../arm-none-eabi/lib/thumb/v7e-m+dp/hard/libc_nano.a(libc_a-findfp.o)
__fp_unlock_all                                   /usr/lib/gcc/arm-none-eabi/13.2.1/../../../arm-none-eabi/lib/thumb/v7e-m+dp/hard/libc_nano.a(libc_a-findfp.o)
__init_array_end                                  /usr/lib/gcc/arm-none-eabi/13.2.1/../../../arm-none-eabi/lib/thumb/v7e-m+dp/hard/libc_nano.a(libc_a-init.o)
__init_array_start                                /usr/lib/gcc/arm-none-eabi/13.2.1/../../../arm-none-eabi/lib/thumb/v7e-m+dp/hard/libc_nano.a(libc_a-init.o)
__io_getchar                                      build/syscalls.o
__io_putchar                                      build/syscalls.o
__libc_fini_array                                 /usr/lib/gcc/arm-none-eabi/13.2.1/../../../arm-none-eabi/lib/thumb/v7e-m+dp/hard/libc_nano.a(libc_a-fini.o)
                                                  /usr/lib/gcc/arm-none-eabi/13.2.1/../../../arm-none-eabi/lib/thumb/v7e-m+dp/hard/crt0.o
__libc_init_array                                 /usr/lib/gcc/arm-none-eabi/13.2.1/../../../arm-none-eabi/lib/thumb/v7e-m+dp/hard/libc_nano.a(libc_a-init.o)
                                                  build/startup_stm32f767xx.o
                                                  /usr/lib/gcc/arm-none-eabi/13.2.1/../../../arm-none-eabi/lib/thumb/v7e-m+dp/hard/crt0.o
__malloc_free_list                                /usr/lib/gcc/arm-none-eabi/13.2.1/../../../arm-none-eabi/lib/thumb/v7e-m+dp/hard/libc_nano.a(libc_a-mallocr.o)
                                                  /usr/lib/gcc/arm-none-eabi/13.2.1/../../../arm-none-eabi/lib/thumb/v7e-m+dp/hard/libc_nano.a(libc_a-freer.o)
__malloc_lock                                     /usr/lib/gcc/arm-none-eabi/13.2.1/../../../arm-none-eabi/lib/thumb/v7e-m+dp/hard/libc_nano.a(libc_a-mlock.o)
                                                  /usr/lib/gcc/arm-none-eabi/13.2.1/../../../arm-none-eabi/lib/thumb/v7e-m+dp/hard/libc_nano.a(libc_a-freer.o)
                                                  /usr/lib/gcc/arm-none-eabi/13.2.1/../../../arm-none-eabi/lib/thumb/v7e-m+dp/hard/libc_nano.a(libc_a-mallocr.o)
__malloc_sbrk_start                               /usr/lib/gcc/arm-none-eabi/13.2.1/../../../arm-none-eabi/lib/thumb/v7e-m+dp/hard/libc_nano.a(libc_a-mallocr.o)
__malloc_unlock                                   /usr/lib/gcc/arm-none-eabi/13.2.1/../../../arm-none-eabi/lib/thumb/v7e-m+dp/hard/libc_nano.a(libc_a-mlock.o)
                                                  /usr/lib/gcc/arm-none-eabi/13.2.1/../../../arm-none-eabi/lib/thumb/v7e-m+dp/hard/libc_nano.a(libc_a-freer.o)
                                                  /usr/lib/gcc/arm-none-eabi/13.2.1/../../../arm-none-eabi/lib/thumb/v7e-m+dp/hard/libc_nano.a(libc_a-mallocr.o)
__on_exit_args                                    /usr/lib/gcc/arm-none-eabi/13.2.1/../../../arm-none-eabi/lib/thumb/v7e-m+dp/hard/libc_nano.a(libc_a-__atexit.o)
__preinit_array_end                               /usr/lib/gcc/arm-none-eabi/13.2.1/../../../arm-none-eabi/lib/thumb/v7e-m+dp/hard/libc_nano.a(libc_a-init.o)
__preinit_array_start                             /usr/lib/gcc/arm-none-eabi/13.2.1/../../../arm-none-eabi/lib/thumb/v7e-m+dp/hard/libc_nano.a(libc_a-init.o)
__register_exitproc                               /usr/lib/gcc/arm-none-eabi/13.2.1/../../../arm-none-eabi/lib/thumb/v7e-m+dp/hard/libc_nano.a(libc_a-__atexit.o)
                                                  /usr/lib/gcc/arm-none-eabi/13.2.1/../../../arm-none-eabi/lib/thumb/v7e-m+dp/hard/libc_nano.a(libc_a-atexit.o)
__register_frame_info                             /usr/lib/gcc/arm-none-eabi/13.2.1/thumb/v7e-m+dp/hard/crtbegin.o
__sclose                                          /usr/lib/gcc/arm-none-eabi/13.2.1/../../../arm-none-eabi/lib/thumb/v7e-m+dp/hard/libc_nano.a(libc_a-stdio.o)
                                                  /usr/lib/gcc/arm-none-eabi/13.2.1/../../../arm-none-eabi/lib/thumb/v7e-m+dp/hard/libc_nano.a(libc_a-findfp.o)
__seofread                                        /usr/lib/gcc/arm-none-eabi/13.2.1/../../../arm-none-eabi/lib/thumb/v7e-m+dp/hard/libc_nano.a(libc_a-stdio.o)
__sf                                              /usr/lib/gcc/arm-none-eabi/13.2.1/../../../arm-none-eabi/lib/thumb/v7e-m+dp/hard/libc_nano.a(libc_a-findfp.o)
                                                  /usr/lib/gcc/arm-none-eabi/13.2.1/../../../arm-none-eabi/lib/thumb/v7e-m+dp/hard/libc_nano.a(libc_a-impure.o)
__sflush_r                                        /usr/lib/gcc/arm-none-eabi/13.2.1/../../../arm-none-eabi/lib/thumb/v7e-m+dp/hard/libc_nano.a(libc_a-fflush.o)
__sfp                                             /usr/lib/gcc/arm-none-eabi/13.2.1/../../../arm-none-eabi/lib/thumb/v7e-m+dp/hard/libc_nano.a(libc_a-findfp.o)
__sfp_lock_acquire                                /usr/lib/gcc/arm-none-eabi/13.2.1/../../../arm-none-eabi/lib/thumb/v7e-m+dp/hard/libc_nano.a(libc_a-findfp.o)
__sfp_lock_release                                /usr/lib/gcc/arm-none-eabi/13.2.1/../../../arm-none-eabi/lib/thumb/v7e-m+dp/hard/libc_nano.a(libc_a-findfp.o)
__sglue                                           /usr/lib/gcc/arm-none-eabi/13.2.1/../../../arm-none-eabi/lib/thumb/v7e-m+dp/hard/libc_nano.a(libc_a-findfp.o)
                                                  /usr/lib/gcc/arm-none-eabi/13.2.1/../../../arm-none-eabi/lib/thumb/v7e-m+dp/hard/libc_nano.a(libc_a-fflush.o)
__sinit                                           /usr/lib/gcc/arm-none-eabi/13.2.1/../../../arm-none-eabi/lib/thumb/v7e-m+dp/hard/libc_nano.a(libc_a-findfp.o)
                                                  /usr/lib/gcc/arm-none-eabi/13.2.1/../../../arm-none-eabi/lib/thumb/v7e-m+dp/hard/libc_nano.a(libc_a-fflush.o)
__sread                                           /usr/lib/gcc/arm-none-eabi/13.2.1/../../../arm-none-eabi/lib/thumb/v7e-m+dp/hard/libc_nano.a(libc_a-stdio.o)
                                                  /usr/lib/gcc/arm-none-eabi/13.2.1/../../../arm-none-eabi/lib/thumb/v7e-m+dp/hard/libc_nano.a(libc_a-findfp.o)
__sseek                                           /usr/lib/gcc/arm-none-eabi/13.2.1/../../../arm-none-eabi/lib/thumb/v7e-m+dp/hard/libc_nano.a(libc_a-stdio.o)
                                                  /usr/lib/gcc/arm-none-eabi/13.2.1/../../../arm-none-eabi/lib/thumb/v7e-m+dp/hard/libc_nano.a(libc_a-findfp.o)
__ssprint_r                                       /usr/lib/gcc/arm-none-eabi/13.2.1/../../../arm-none-eabi/lib/thumb/v7e-m+dp/hard/libc_nano.a(libc_a-nano-svfprintf.o)
__ssputs_r                                        /usr/lib/gcc/arm-none-eabi/13.2.1/../../../arm-none-eabi/lib/thumb/v7e-m+dp/hard/libc_nano.a(libc_a-nano-svfprintf.o)
__stack                                           /usr/lib/gcc/arm-none-eabi/13.2.1/../../../arm-none-eabi/lib/thumb/v7e-m+dp/hard/crt0.o
__stdio_exit_handler                              /usr/lib/gcc/arm-none-eabi/13.2.1/../../../arm-none-eabi/lib/thumb/v7e-m+dp/hard/libc_nano.a(libc_a-findfp.o)
                                                  /usr/lib/gcc/arm-none-eabi/13.2.1/../../../arm-none-eabi/lib/thumb/v7e-m+dp/hard/libc_nano.a(libc_a-exit.o)
__swrite                                          /usr/lib/gcc/arm-none-eabi/13.2.1/../../../arm-none-eabi/lib/thumb/v7e-m+dp/hard/libc_nano.a(libc_a-stdio.o)
                                                  /usr/lib/gcc/arm-none-eabi/13.2.1/../../../arm-none-eabi/lib/thumb/v7e-m+dp/hard/libc_nano.a(libc_a-findfp.o)
__udivmoddi4                                      /usr/lib/gcc/arm-none-eabi/13.2.1/thumb/v7e-m+dp/hard/libgcc.a(_udivmoddi4.o)
                                                  /usr/lib/gcc/arm-none-eabi/13.2.1/thumb/v7e-m+dp/hard/libgcc.a(_aeabi_uldivmod.o)
_close                                            build/syscalls.o
                                                  /usr/lib/gcc/arm-none-eabi/13.2.1/../../../arm-none-eabi/lib/thumb/v7e-m+dp/hard/libc_nano.a(libc_a-closer.o)
_close_r                                          /usr/lib/gcc/arm-none-eabi/13.2.1/../../../arm-none-eabi/lib/thumb/v7e-m+dp/hard/libc_nano.a(libc_a-closer.o)
                                                  /usr/lib/gcc/arm-none-eabi/13.2.1/../../../arm-none-eabi/lib/thumb/v7e-m+dp/hard/libc_nano.a(libc_a-stdio.o)
_ebss                                             build/startup_stm32f767xx.o
_edata                                            build/startup_stm32f767xx.o
_end                                              build/sysmem.o
_estack                                           build/startup_stm32f767xx.o
                                                  build/sysmem.o
_execve                                           build/syscalls.o
_exit                                             build/syscalls.o
                                                  /usr/lib/gcc/arm-none-eabi/13.2.1/../../../arm-none-eabi/lib/thumb/v7e-m+dp/hard/libc_nano.a(libc_a-exit.o)
_fflush_r                                         /usr/lib/gcc/arm-none-eabi/13.2.1/../../../arm-none-eabi/lib/thumb/v7e-m+dp/hard/libc_nano.a(libc_a-fflush.o)
                                                  /usr/lib/gcc/arm-none-eabi/13.2.1/../../../arm-none-eabi/lib/thumb/v7e-m+dp/hard/libc_nano.a(libc_a-findfp.o)
_fini                                             /usr/lib/gcc/arm-none-eabi/13.2.1/thumb/v7e-m+dp/hard/crti.o
                                                  /usr/lib/gcc/arm-none-eabi/13.2.1/../../../arm-none-eabi/lib/thumb/v7e-m+dp/hard/libc_nano.a(libc_a-fini.o)
_fork                                             build/syscalls.o
_free_r                                           /usr/lib/gcc/arm-none-eabi/13.2.1/../../../arm-none-eabi/lib/thumb/v7e-m+dp/hard/libc_nano.a(libc_a-freer.o)
                                                  /usr/lib/gcc/arm-none-eabi/13.2.1/../../../arm-none-eabi/lib/thumb/v7e-m+dp/hard/libc_nano.a(libc_a-reent.o)
                                                  /usr/lib/gcc/arm-none-eabi/13.2.1/../../../arm-none-eabi/lib/thumb/v7e-m+dp/hard/libc_nano.a(libc_a-fflush.o)
                                                  /usr/lib/gcc/arm-none-eabi/13.2.1/../../../arm-none-eabi/lib/thumb/v7e-m+dp/hard/libc_nano.a(libc_a-reallocr.o)
                                                  /usr/lib/gcc/arm-none-eabi/13.2.1/../../../arm-none-eabi/lib/thumb/v7e-m+dp/hard/libc_nano.a(libc_a-malloc.o)
                                                  /usr/lib/gcc/arm-none-eabi/13.2.1/../../../arm-none-eabi/lib/thumb/v7e-m+dp/hard/libc_nano.a(libc_a-nano-svfprintf.o)
_fstat                                            build/syscalls.o
_fwalk_sglue                                      /usr/lib/gcc/arm-none-eabi/13.2.1/../../../arm-none-eabi/lib/thumb/v7e-m+dp/hard/libc_nano.a(libc_a-fwalk.o)
                                                  /usr/lib/gcc/arm-none-eabi/13.2.1/../../../arm-none-eabi/lib/thumb/v7e-m+dp/hard/libc_nano.a(libc_a-fflush.o)
                                                  /usr/lib/gcc/arm-none-eabi/13.2.1/../../../arm-none-eabi/lib/thumb/v7e-m+dp/hard/libc_nano.a(libc_a-findfp.o)
_getpid                                           build/syscalls.o
_impure_data                                      /usr/lib/gcc/arm-none-eabi/13.2.1/../../../arm-none-eabi/lib/thumb/v7e-m+dp/hard/libc_nano.a(libc_a-impure.o)
                                                  /usr/lib/gcc/arm-none-eabi/13.2.1/../../../arm-none-eabi/lib/thumb/v7e-m+dp/hard/libc_nano.a(libc_a-fflush.o)
                                                  /usr/lib/gcc/arm-none-eabi/13.2.1/../../../arm-none-eabi/lib/thumb/v7e-m+dp/hard/libc_nano.a(libc_a-findfp.o)
_impure_ptr                                       /usr/lib/gcc/arm-none-eabi/13.2.1/../../../arm-none-eabi/lib/thumb/v7e-m+dp/hard/libc_nano.a(libc_a-impure.o)
                                                  /usr/lib/gcc/arm-none-eabi/13.2.1/../../../arm-none-eabi/lib/thumb/v7e-m+dp/hard/libc_nano.a(libc_a-reent.o)
                                                  /usr/lib/gcc/arm-none-eabi/13.2.1/../../../arm-none-eabi/lib/thumb/v7e-m+dp/hard/libc_nano.a(libc_a-fflush.o)
                                                  /usr/lib/gcc/arm-none-eabi/13.2.1/../../../arm-none-eabi/lib/thumb/v7e-m+dp/hard/libc_nano.a(libc_a-malloc.o)
                                                  /usr/lib/gcc/arm-none-eabi/13.2.1/../../../arm-none-eabi/lib/thumb/v7e-m+dp/hard/libc_nano.a(libc_a-errno.o)
                                                  /usr/lib/gcc/arm-none-eabi/13.2.1/../../../arm-none-eabi/lib/thumb/v7e-m+dp/hard/libc_nano.a(libc_a-sprintf.o)
_init                                             /usr/lib/gcc/arm-none-eabi/13.2.1/thumb/v7e-m+dp/hard/crti.o
                                                  /usr/lib/gcc/arm-none-eabi/13.2.1/../../../arm-none-eabi/lib/thumb/v7e-m+dp/hard/libc_nano.a(libc_a-init.o)
_isatty                                           build/syscalls.o
_kill                                             build/syscalls.o
_link                                             build/syscalls.o
_lseek                                            build/syscalls.o
                                                  /usr/lib/gcc/arm-none-eabi/13.2.1/../../../arm-none-eabi/lib/thumb/v7e-m+dp/hard/libc_nano.a(libc_a-lseekr.o)
_lseek_r                                          /usr/lib/gcc/arm-none-eabi/13.2.1/../../../arm-none-eabi/lib/thumb/v7e-m+dp/hard/libc_nano.a(libc_a-lseekr.o)
                                                  /usr/lib/gcc/arm-none-eabi/13.2.1/../../../arm-none-eabi/lib/thumb/v7e-m+dp/hard/libc_nano.a(libc_a-stdio.o)
_mainCRTStartup                                   /usr/lib/gcc/arm-none-eabi/13.2.1/../../../arm-none-eabi/lib/thumb/v7e-m+dp/hard/crt0.o
_malloc_r                                         /usr/lib/gcc/arm-none-eabi/13.2.1/../../../arm-none-eabi/lib/thumb/v7e-m+dp/hard/libc_nano.a(libc_a-mallocr.o)
                                                  /usr/lib/gcc/arm-none-eabi/13.2.1/../../../arm-none-eabi/lib/thumb/v7e-m+dp/hard/libc_nano.a(libc_a-findfp.o)
                                                  /usr/lib/gcc/arm-none-eabi/13.2.1/../../../arm-none-eabi/lib/thumb/v7e-m+dp/hard/libc_nano.a(libc_a-reallocr.o)
                                                  /usr/lib/gcc/arm-none-eabi/13.2.1/../../../arm-none-eabi/lib/thumb/v7e-m+dp/hard/libc_nano.a(libc_a-malloc.o)
                                                  /usr/lib/gcc/arm-none-eabi/13.2.1/../../../arm-none-eabi/lib/thumb/v7e-m+dp/hard/libc_nano.a(libc_a-nano-svfprintf.o)
_malloc_usable_size_r                             /usr/lib/gcc/arm-none-eabi/13.2.1/../../../arm-none-eabi/lib/thumb/v7e-m+dp/hard/libc_nano.a(libc_a-msizer.o)
                                                  /usr/lib/gcc/arm-none-eabi/13.2.1/../../../arm-none-eabi/lib/thumb/v7e-m+dp/hard/libc_nano.a(libc_a-reallocr.o)
_open                                             build/syscalls.o
_printf_common                                    /usr/lib/gcc/arm-none-eabi/13.2.1/../../../arm-none-eabi/lib/thumb/v7e-m+dp/hard/libc_nano.a(libc_a-nano-vfprintf_i.o)
_printf_float                                     /usr/lib/gcc/arm-none-eabi/13.2.1/../../../arm-none-eabi/lib/thumb/v7e-m+dp/hard/libc_nano.a(libc_a-nano-svfprintf.o)
_printf_i                                         /usr/lib/gcc/arm-none-eabi/13.2.1/../../../arm-none-eabi/lib/thumb/v7e-m+dp/hard/libc_nano.a(libc_a-nano-vfprintf_i.o)
                                                  /usr/lib/gcc/arm-none-eabi/13.2.1/../../../arm-none-eabi/lib/thumb/v7e-m+dp/hard/libc_nano.a(libc_a-nano-svfprintf.o)
_read                                             build/syscalls.o
                                                  /usr/lib/gcc/arm-none-eabi/13.2.1/../../../arm-none-eabi/lib/thumb/v7e-m+dp/hard/libc_nano.a(libc_a-readr.o)
_read_r                                           /usr/lib/gcc/arm-none-eabi/13.2.1/../../../arm-none-eabi/lib/thumb/v7e-m+dp/hard/libc_nano.a(libc_a-readr.o)
                                                  /usr/lib/gcc/arm-none-eabi/13.2.1/../../../arm-none-eabi/lib/thumb/v7e-m+dp/hard/libc_nano.a(libc_a-stdio.o)
_realloc_r                                        /usr/lib/gcc/arm-none-eabi/13.2.1/../../../arm-none-eabi/lib/thumb/v7e-m+dp/hard/libc_nano.a(libc_a-reallocr.o)
                                                  /usr/lib/gcc/arm-none-eabi/13.2.1/../../../arm-none-eabi/lib/thumb/v7e-m+dp/hard/libc_nano.a(libc_a-nano-svfprintf.o)
_reclaim_reent                                    /usr/lib/gcc/arm-none-eabi/13.2.1/../../../arm-none-eabi/lib/thumb/v7e-m+dp/hard/libc_nano.a(libc_a-reent.o)
_sbrk                                             build/sysmem.o
                                                  /usr/lib/gcc/arm-none-eabi/13.2.1/../../../arm-none-eabi/lib/thumb/v7e-m+dp/hard/libc_nano.a(libc_a-sbrkr.o)
_sbrk_r                                           /usr/lib/gcc/arm-none-eabi/13.2.1/../../../arm-none-eabi/lib/thumb/v7e-m+dp/hard/libc_nano.a(libc_a-sbrkr.o)
                                                  /usr/lib/gcc/arm-none-eabi/13.2.1/../../../arm-none-eabi/lib/thumb/v7e-m+dp/hard/libc_nano.a(libc_a-mallocr.o)
_sbss                                             build/startup_stm32f767xx.o
_sdata                                            build/startup_stm32f767xx.o
_sidata                                           build/startup_stm32f767xx.o
_siprintf_r                                       /usr/lib/gcc/arm-none-eabi/13.2.1/../../../arm-none-eabi/lib/thumb/v7e-m+dp/hard/libc_nano.a(libc_a-sprintf.o)
_sprintf_r                                        /usr/lib/gcc/arm-none-eabi/13.2.1/../../../arm-none-eabi/lib/thumb/v7e-m+dp/hard/libc_nano.a(libc_a-sprintf.o)
_stack_init                                       /usr/lib/gcc/arm-none-eabi/13.2.1/../../../arm-none-eabi/lib/thumb/v7e-m+dp/hard/crt0.o
_start                                            /usr/lib/gcc/arm-none-eabi/13.2.1/../../../arm-none-eabi/lib/thumb/v7e-m+dp/hard/crt0.o
_stat                                             build/syscalls.o
_svfiprintf_r                                     /usr/lib/gcc/arm-none-eabi/13.2.1/../../../arm-none-eabi/lib/thumb/v7e-m+dp/hard/libc_nano.a(libc_a-nano-svfprintf.o)
_svfprintf_r                                      /usr/lib/gcc/arm-none-eabi/13.2.1/../../../arm-none-eabi/lib/thumb/v7e-m+dp/hard/libc_nano.a(libc_a-nano-svfprintf.o)
                                                  /usr/lib/gcc/arm-none-eabi/13.2.1/../../../arm-none-eabi/lib/thumb/v7e-m+dp/hard/libc_nano.a(libc_a-sprintf.o)
_times                                            build/syscalls.o
_unlink                                           build/syscalls.o
_wait                                             build/syscalls.o
_write                                            build/syscalls.o
                                                  /usr/lib/gcc/arm-none-eabi/13.2.1/../../../arm-none-eabi/lib/thumb/v7e-m+dp/hard/libc_nano.a(libc_a-writer.o)
_write_r                                          /usr/lib/gcc/arm-none-eabi/13.2.1/../../../arm-none-eabi/lib/thumb/v7e-m+dp/hard/libc_nano.a(libc_a-writer.o)
                                                  /usr/lib/gcc/arm-none-eabi/13.2.1/../../../arm-none-eabi/lib/thumb/v7e-m+dp/hard/libc_nano.a(libc_a-stdio.o)
atexit                                            /usr/lib/gcc/arm-none-eabi/13.2.1/../../../arm-none-eabi/lib/thumb/v7e-m+dp/hard/libc_nano.a(libc_a-atexit.o)
                                                  /usr/lib/gcc/arm-none-eabi/13.2.1/../../../arm-none-eabi/lib/thumb/v7e-m+dp/hard/crt0.o
br                                                build/File_Handling.o
bw                                                build/File_Handling.o
disk                                              build/ff_gen_drv.o
                                                  build/diskio.o
disk_initialize                                   build/diskio.o
                                                  build/ff.o
disk_ioctl                                        build/diskio.o
                                                  build/ff.o
disk_read                                         build/diskio.o
                                                  build/ff.o
disk_status                                       build/diskio.o
                                                  build/ff.o
disk_write                                        build/diskio.o
                                                  build/ff.o
environ                                           build/syscalls.o
errno                                             /usr/lib/gcc/arm-none-eabi/13.2.1/../../../arm-none-eabi/lib/thumb/v7e-m+dp/hard/libc_nano.a(libc_a-reent.o)
                                                  /usr/lib/gcc/arm-none-eabi/13.2.1/../../../arm-none-eabi/lib/thumb/v7e-m+dp/hard/libc_nano.a(libc_a-writer.o)
                                                  /usr/lib/gcc/arm-none-eabi/13.2.1/../../../arm-none-eabi/lib/thumb/v7e-m+dp/hard/libc_nano.a(libc_a-lseekr.o)
                                                  /usr/lib/gcc/arm-none-eabi/13.2.1/../../../arm-none-eabi/lib/thumb/v7e-m+dp/hard/libc_nano.a(libc_a-readr.o)
                                                  /usr/lib/gcc/arm-none-eabi/13.2.1/../../../arm-none-eabi/lib/thumb/v7e-m+dp/hard/libc_nano.a(libc_a-closer.o)
                                                  /usr/lib/gcc/arm-none-eabi/13.2.1/../../../arm-none-eabi/lib/thumb/v7e-m+dp/hard/libc_nano.a(libc_a-sbrkr.o)
exit                                              /usr/lib/gcc/arm-none-eabi/13.2.1/../../../arm-none-eabi/lib/thumb/v7e-m+dp/hard/libc_nano.a(libc_a-exit.o)
                                                  /usr/lib/gcc/arm-none-eabi/13.2.1/../../../arm-none-eabi/lib/thumb/v7e-m+dp/hard/crt0.o
f_close                                           build/ff.o
                                                  build/File_Handling.o
f_closedir                                        build/ff.o
                                                  build/File_Handling.o
f_getfree                                         build/ff.o
                                                  build/File_Handling.o
f_gets                                            build/ff.o
f_lseek                                           build/ff.o
                                                  build/File_Handling.o
f_mkdir                                           build/ff.o
                                                  build/File_Handling.o
f_mkfs                                            build/ff.o
f_mount                                           build/ff.o
                                                  build/File_Handling.o
f_open                                            build/ff.o
                                                  build/File_Handling.o
f_opendir                                         build/ff.o
                                                  build/File_Handling.o
f_printf                                          build/ff.o
f_putc                                            build/ff.o
f_puts                                            build/ff.o
f_read                                            build/ff.o
                                                  build/File_Handling.o
f_readdir                                         build/ff.o
                                                  build/File_Handling.o
f_rename                                          build/ff.o
f_stat                                            build/ff.o
                                                  build/File_Handling.o
f_sync                                            build/ff.o
f_truncate                                        build/ff.o
f_unlink                                          build/ff.o
                                                  build/File_Handling.o
f_write                                           build/ff.o
                                                  build/File_Handling.o
fflush                                            /usr/lib/gcc/arm-none-eabi/13.2.1/../../../arm-none-eabi/lib/thumb/v7e-m+dp/hard/libc_nano.a(libc_a-fflush.o)
fgoto                                             build/main.o
fil                                               build/File_Handling.o
flg_tmt                                           build/main.o
                                                  build/stm32f7xx_it.o
fno                                               build/File_Handling.o
fre_clust                                         build/File_Handling.o
free                                              /usr/lib/gcc/arm-none-eabi/13.2.1/../../../arm-none-eabi/lib/thumb/v7e-m+dp/hard/libc_nano.a(libc_a-malloc.o)
                                                  build/File_Handling.o
free_space                                        build/File_Handling.o
fresult                                           build/main.o
                                                  build/File_Handling.o
fs                                                build/File_Handling.o
g_pfnVectors                                      build/startup_stm32f767xx.o
get_fattime                                       build/fatfs.o
                                                  build/ff.o
hadc1                                             build/main.o
                                                  build/stm32f7xx_it.o
hadc3                                             build/main.o
                                                  build/stm32f7xx_it.o
hardware_init_hook                                /usr/lib/gcc/arm-none-eabi/13.2.1/../../../arm-none-eabi/lib/thumb/v7e-m+dp/hard/crt0.o
hsd1                                              build/main.o
                                                  build/bsp_driver_sd.o
htim10                                            build/main.o
                                                  build/stm32f7xx_it.o
htim11                                            build/main.o
                                                  build/stm32f7xx_it.o
htim4                                             build/main.o
htim8                                             build/main.o
                                                  build/stm32f7xx_it.o
huart8                                            build/main.o
initialise_monitor_handles                        build/syscalls.o
main                                              build/main.o
                                                  build/startup_stm32f767xx.o
                                                  /usr/lib/gcc/arm-none-eabi/13.2.1/../../../arm-none-eabi/lib/thumb/v7e-m+dp/hard/crt0.o
malloc                                            /usr/lib/gcc/arm-none-eabi/13.2.1/../../../arm-none-eabi/lib/thumb/v7e-m+dp/hard/libc_nano.a(libc_a-malloc.o)
                                                  /usr/lib/gcc/arm-none-eabi/13.2.1/../../../arm-none-eabi/lib/thumb/v7e-m+dp/hard/libc_nano.a(libc_a-__atexit.o)
                                                  build/File_Handling.o
memchr                                            /usr/lib/gcc/arm-none-eabi/13.2.1/../../../arm-none-eabi/lib/thumb/v7e-m+dp/hard/libc_nano.a(libc_a-memchr.o)
                                                  /usr/lib/gcc/arm-none-eabi/13.2.1/../../../arm-none-eabi/lib/thumb/v7e-m+dp/hard/libc_nano.a(libc_a-nano-vfprintf_i.o)
                                                  /usr/lib/gcc/arm-none-eabi/13.2.1/../../../arm-none-eabi/lib/thumb/v7e-m+dp/hard/libc_nano.a(libc_a-nano-svfprintf.o)
memcpy                                            /usr/lib/gcc/arm-none-eabi/13.2.1/../../../arm-none-eabi/lib/thumb/v7e-m+dp/hard/libc_nano.a(libc_a-memcpy.o)
                                                  /usr/lib/gcc/arm-none-eabi/13.2.1/../../../arm-none-eabi/lib/thumb/v7e-m+dp/hard/libc_nano.a(libc_a-reallocr.o)
                                                  /usr/lib/gcc/arm-none-eabi/13.2.1/../../../arm-none-eabi/lib/thumb/v7e-m+dp/hard/libc_nano.a(libc_a-nano-svfprintf.o)
memmove                                           /usr/lib/gcc/arm-none-eabi/13.2.1/../../../arm-none-eabi/lib/thumb/v7e-m+dp/hard/libc_nano.a(libc_a-memmove.o)
                                                  /usr/lib/gcc/arm-none-eabi/13.2.1/../../../arm-none-eabi/lib/thumb/v7e-m+dp/hard/libc_nano.a(libc_a-nano-svfprintf.o)
memset                                            /usr/lib/gcc/arm-none-eabi/13.2.1/../../../arm-none-eabi/lib/thumb/v7e-m+dp/hard/libc_nano.a(libc_a-memset.o)
                                                  /usr/lib/gcc/arm-none-eabi/13.2.1/../../../arm-none-eabi/lib/thumb/v7e-m+dp/hard/libc_nano.a(libc_a-findfp.o)
                                                  build/stm32f7xx_hal_msp.o
                                                  build/main.o
                                                  /usr/lib/gcc/arm-none-eabi/13.2.1/../../../arm-none-eabi/lib/thumb/v7e-m+dp/hard/crt0.o
pFlash                                            build/stm32f7xx_hal_flash.o
                                                  build/stm32f7xx_hal_flash_ex.o
pfs                                               build/File_Handling.o
retSD                                             build/fatfs.o
siprintf                                          /usr/lib/gcc/arm-none-eabi/13.2.1/../../../arm-none-eabi/lib/thumb/v7e-m+dp/hard/libc_nano.a(libc_a-sprintf.o)
sizeoffile                                        build/main.o
                                                  build/File_Handling.o
software_init_hook                                /usr/lib/gcc/arm-none-eabi/13.2.1/../../../arm-none-eabi/lib/thumb/v7e-m+dp/hard/crt0.o
sprintf                                           /usr/lib/gcc/arm-none-eabi/13.2.1/../../../arm-none-eabi/lib/thumb/v7e-m+dp/hard/libc_nano.a(libc_a-sprintf.o)
                                                  build/File_Handling.o
strcmp                                            /usr/lib/gcc/arm-none-eabi/13.2.1/../../../arm-none-eabi/lib/thumb/v7e-m+dp/hard/libc_nano.a(libc_a-strcmp.o)
                                                  build/File_Handling.o
strcpy                                            /usr/lib/gcc/arm-none-eabi/13.2.1/../../../arm-none-eabi/lib/thumb/v7e-m+dp/hard/libc_nano.a(libc_a-strcpy.o)
                                                  build/File_Handling.o
strlen                                            /usr/lib/gcc/arm-none-eabi/13.2.1/../../../arm-none-eabi/lib/thumb/v7e-m+dp/hard/libc_nano.a(libc_a-strlen.o)
                                                  build/File_Handling.o
task                                              build/main.o
temp16                                            build/main.o
temp32                                            build/main.o
test                                              build/main.o
total                                             build/File_Handling.o
u_rx_flg                                          build/main.o
u_tx_flg                                          build/main.o
                                                  build/stm32f7xx_it.o
uart_buf                                          build/main.o
                                                  build/stm32f7xx_it.o
uwTick                                            build/stm32f7xx_hal.o
uwTickFreq                                        build/stm32f7xx_hal.o
uwTickPrio                                        build/stm32f7xx_hal.o
                                                  build/stm32f7xx_hal_rcc.o
